 npUnity3D32

 Timestamp is 514f15f7 (Sun Mar 24 16:04:23 2013)

 Preferred load address is 10000000

 Start         Length     Name                   Class
 0001:00000000 00038f2eH .text                   CODE
 0001:00038f2e 000000feH .text$x                 CODE
 0001:0003902c 00000103H .text$yc                CODE
 0001:0003912f 000000bbH .text$yd                CODE
 0002:00000000 00000410H .idata$5                DATA
 0002:00000410 00000004H .CRT$XCA                DATA
 0002:00000414 00000028H .CRT$XCU                DATA
 0002:0000043c 00000004H .CRT$XCZ                DATA
 0002:00000440 00000004H .CRT$XIA                DATA
 0002:00000444 00000014H .CRT$XIC                DATA
 0002:00000458 00000004H .CRT$XIZ                DATA
 0002:0000045c 00000004H .CRT$XPA                DATA
 0002:00000460 00000004H .CRT$XPX                DATA
 0002:00000464 00000004H .CRT$XPXA               DATA
 0002:00000468 00000004H .CRT$XPZ                DATA
 0002:0000046c 00000004H .CRT$XTA                DATA
 0002:00000470 00000004H .CRT$XTZ                DATA
 0002:00000480 0000d4f8H .rdata                  DATA
 0002:0000d978 0000006aH .rdata$debug            DATA
 0002:0000d9e4 00000214H .rdata$r                DATA
 0002:0000dc00 00000070H .rdata$sxdata           DATA
 0002:0000dc70 00000004H .rtc$IAA                DATA
 0002:0000dc74 00000004H .rtc$IZZ                DATA
 0002:0000dc78 00000004H .rtc$TAA                DATA
 0002:0000dc7c 00000004H .rtc$TZZ                DATA
 0002:0000dc80 00000fc8H .xdata$x                DATA
 0002:0000ec48 000000c8H .idata$2                DATA
 0002:0000ed10 00000014H .idata$3                DATA
 0002:0000ed24 00000410H .idata$4                DATA
 0002:0000f134 0000119aH .idata$6                DATA
 0002:000102d0 00000099H .edata                  DATA
 0003:00000000 00001614H .data                   DATA
 0003:00001620 00004160H .bss                    DATA
 0004:00000000 00000380H .rsrc$01                DATA
 0004:00000380 000235c8H .rsrc$02                DATA

  Address         Publics by Value              Rva+Base       Lib:Object

 0000:00000000       __except_list              00000000     <absolute>
 0000:0000001c       ___safe_se_handler_count   0000001c     <absolute>
 0000:00000000       ___ImageBase               10000000     <linker-defined>
 0001:00000000       ??1ContextMenu@@QAE@XZ     10001000 f   ContextMenu.obj
 0001:0000003e       ?WindowProc@ContextMenu@@CGJPAUHWND__@@IIJ@Z 1000103e f   ContextMenu.obj
 0001:00000326       ??_GContextSubmenu@@QAEPAXI@Z 10001326 f i ContextMenu.obj
 0001:00000367       ??0ContextMenuWindowClass@@QAE@XZ 10001367 f   ContextMenuWindowClass.obj
 0001:000003d9       ??0ContextSubmenu@@QAE@PBVContextMenu@@PAUHWND__@@@Z 100013d9 f   ContextSubmenu.obj
 0001:00000418       ??1ContextSubmenu@@QAE@XZ  10001418 f   ContextSubmenu.obj
 0001:00000454       ?ShowMenu@ContextSubmenu@@QBEXHH@Z 10001454 f   ContextSubmenu.obj
 0001:0000047d       ?HideChildren@ContextSubmenu@@QAEXXZ 1000147d f   ContextSubmenu.obj
 0001:000004b3       ?RedrawMenu@ContextSubmenu@@QBEXXZ 100014b3 f   ContextSubmenu.obj
 0001:000004e5       ?Initialize@ContextSubmenu@@QAEXPAUHMENU__@@@Z 100014e5 f   ContextSubmenu.obj
 0001:000006c5       ?Update@ContextSubmenu@@AAEXXZ 100016c5 f   ContextSubmenu.obj
 0001:00000895       ?SelectAndRedraw@ContextSubmenu@@QAEXABUtagPOINT@@@Z 10001895 f   ContextSubmenu.obj
 0001:00000905       ?OnPaint@ContextSubmenu@@ABEXPAUHDC__@@@Z 10001905 f   ContextSubmenu.obj
 0001:00000bf5       ??0?$basic_string@_WU?$char_traits@_W@std@@V?$allocator@_W@2@@std@@QAE@ABV01@@Z 10001bf5 f i ContextSubmenu.obj
 0001:00000c1d       ??1?$vector@UItem@ContextSubmenu@@V?$allocator@UItem@ContextSubmenu@@@std@@@std@@QAE@XZ 10001c1d f i ContextSubmenu.obj
 0001:00000c52       ?reserve@?$vector@UItem@ContextSubmenu@@V?$allocator@UItem@ContextSubmenu@@@std@@@std@@QAEXI@Z 10001c52 f i ContextSubmenu.obj
 0001:00000d25       ?assign@?$basic_string@_WU?$char_traits@_W@std@@V?$allocator@_W@2@@std@@QAEAAV12@ABV12@II@Z 10001d25 f i ContextSubmenu.obj
 0001:00000dc0       ?_Tidy@?$basic_string@_WU?$char_traits@_W@std@@V?$allocator@_W@2@@std@@QAEX_NI@Z 10001dc0 f i ContextSubmenu.obj
 0001:00000e09       ?_Reserve@?$vector@UItem@ContextSubmenu@@V?$allocator@UItem@ContextSubmenu@@@std@@@std@@IAEXI@Z 10001e09 f i ContextSubmenu.obj
 0001:00000e60       ?allocate@?$allocator@UItem@ContextSubmenu@@@std@@QAEPAUItem@ContextSubmenu@@I@Z 10001e60 f i ContextSubmenu.obj
 0001:00000ea9       ?assign@?$basic_string@_WU?$char_traits@_W@std@@V?$allocator@_W@2@@std@@QAEAAV12@PB_WI@Z 10001ea9 f i ContextSubmenu.obj
 0001:00000f27       ?erase@?$basic_string@_WU?$char_traits@_W@std@@V?$allocator@_W@2@@std@@QAEAAV12@II@Z 10001f27 f i ContextSubmenu.obj
 0001:00000fa6       ?_Grow@?$basic_string@_WU?$char_traits@_W@std@@V?$allocator@_W@2@@std@@QAE_NI_N@Z 10001fa6 f i ContextSubmenu.obj
 0001:0000100f       ?_Copy@?$basic_string@_WU?$char_traits@_W@std@@V?$allocator@_W@2@@std@@QAEXII@Z 1000200f f i ContextSubmenu.obj
 0001:00001117       ?_Inside@?$basic_string@_WU?$char_traits@_W@std@@V?$allocator@_W@2@@std@@QAE_NPB_W@Z 10002117 f i ContextSubmenu.obj
 0001:00001153       ??$for_each@V?$_Vector_iterator@V?$_Vector_val@UItem@ContextSubmenu@@V?$allocator@UItem@ContextSubmenu@@@std@@@std@@@std@@Udelete_child_submenus@@@std@@YA?AUdelete_child_submenus@@V?$_Vector_iterator@V?$_Vector_val@UItem@ContextSubmenu@@V?$allocator@UItem@ContextSubmenu@@@std@@@std@@@0@0U1@@Z 10002153 f i ContextSubmenu.obj
 0001:00001196       ??$_Move@PAUItem@ContextSubmenu@@PAU12@@std@@YAPAUItem@ContextSubmenu@@PAU12@00@Z 10002196 f i ContextSubmenu.obj
 0001:000011fd       ??$_Allocate@_W@std@@YAPA_WIPA_W@Z 100021fd f i ContextSubmenu.obj
 0001:00001249       ??0bad_alloc@std@@QAE@ABV01@@Z 10002249 f i ContextSubmenu.obj
 0001:00001264       ??0Item@ContextSubmenu@@QAE@ABU01@@Z 10002264 f i ContextSubmenu.obj
 0001:0000129d       ??$_Uninit_move@PAUItem@ContextSubmenu@@PAU12@V?$allocator@UItem@ContextSubmenu@@@std@@U12@@std@@YAPAUItem@ContextSubmenu@@PAU12@00AAV?$allocator@UItem@ContextSubmenu@@@0@0U_Nonscalar_ptr_iterator_tag@0@@Z 1000229d f i ContextSubmenu.obj
 0001:0000130d       ??1bad_alloc@std@@UAE@XZ   1000230d f i ContextSubmenu.obj
 0001:00001318       ??_Ebad_alloc@std@@UAEPAXI@Z 10002318 f i  CIL library: CIL module
 0001:00001318       ??_Gbad_alloc@std@@UAEPAXI@Z 10002318 f i ContextSubmenu.obj
 0001:0000133d       ?UT_Uninstall@@YGXPAUHWND__@@PB_W11@Z 1000233d f   Uninstall.obj
 0001:00001340       ?StreamAsFile@nsPluginInstanceBase@@UAEXPAU_NPStream@@PBD@Z 10002340 f i UnityWebPlayerPlugin.obj
 0001:00001343       ?WriteReady@nsPluginInstanceBase@@UAEHPAU_NPStream@@@Z 10002343 f i UnityWebPlayerPlugin.obj
 0001:0000134b       ?Print@nsPluginInstanceBase@@UAEXPAU_NPPrint@@@Z 1000234b f i UnityWebPlayerPlugin.obj
 0001:0000134e       ?HandleEvent@nsPluginInstanceBase@@UAEGPAX@Z 1000234e f i UnityWebPlayerPlugin.obj
 0001:00001353       ?SetValue@nsPluginInstanceBase@@UAEFW4NPNVariable@@PAX@Z 10002353 f i UnityWebPlayerPlugin.obj
 0001:00001358       ?convert@multi_byte_to_wide@detail@@QBEXPBDIAAV?$basic_string@_WU?$char_traits@_W@std@@V?$allocator@_W@2@@std@@@Z 10002358 f i UnityWebPlayerPlugin.obj
 0001:00001382       ?ConvertUTF8ToWideString@@YAXABV?$basic_string@DU?$char_traits@D@std@@V?$allocator@D@2@@std@@AAV?$basic_string@_WU?$char_traits@_W@std@@V?$allocator@_W@2@@2@@Z 10002382 f i UnityWebPlayerPlugin.obj
 0001:000013b8       _DllMain@12                100023b8 f   UnityWebPlayerPlugin.obj
 0001:000013da       ?NS_PluginInitialize@@YAFXZ 100023da f   UnityWebPlayerPlugin.obj
 0001:0000149d       ?NS_PluginShutdown@@YAXXZ  1000249d f   UnityWebPlayerPlugin.obj
 0001:00001530       ?NS_NewPluginInstance@@YAPAVnsPluginInstanceBase@@PAUnsPluginCreateData@@@Z 10002530 f   UnityWebPlayerPlugin.obj
 0001:0000158e       ??0UnityWebPlayerPluginInstance@@QAE@PAUnsPluginCreateData@@@Z 1000258e f   UnityWebPlayerPlugin.obj
 0001:000017ec       ??1UnityWebPlayerPluginInstance@@QAE@XZ 100027ec f   UnityWebPlayerPlugin.obj
 0001:000018a8       ?GetValue@UnityWebPlayerPluginInstance@@UAEFW4NPPVariable@@PAX@Z 100028a8 f   UnityWebPlayerPlugin.obj
 0001:000018dd       ?InternalInitWindow@UnityWebPlayerPluginInstance@@AAEXPAUHWND__@@HH@Z 100028dd f   UnityWebPlayerPlugin.obj
 0001:00001974       ?InternalCleanupWindow@UnityWebPlayerPluginInstance@@AAEXXZ 10002974 f   UnityWebPlayerPlugin.obj
 0001:00001991       ?init@UnityWebPlayerPluginInstance@@UAEEPAU_NPWindow@@@Z 10002991 f   UnityWebPlayerPlugin.obj
 0001:000019e8       ?shut@UnityWebPlayerPluginInstance@@UAEXXZ 100029e8 f   UnityWebPlayerPlugin.obj
 0001:00001a10       ?isInitialized@UnityWebPlayerPluginInstance@@UAEEXZ 10002a10 f   UnityWebPlayerPlugin.obj
 0001:00001a17       ?SetWindow@UnityWebPlayerPluginInstance@@UAEFPAU_NPWindow@@@Z 10002a17 f   UnityWebPlayerPlugin.obj
 0001:00001aad       ?PluginParentWindowProc@UnityWebPlayerPluginInstance@@CGJPAUHWND__@@IIJ@Z 10002aad f   UnityWebPlayerPlugin.obj
 0001:00001e3a       ?NewStream@UnityWebPlayerPluginInstance@@UAEFPADPAU_NPStream@@EPAG@Z 10002e3a f   UnityWebPlayerPlugin.obj
 0001:00001e87       ?Write@UnityWebPlayerPluginInstance@@UAEHPAU_NPStream@@HHPAX@Z 10002e87 f   UnityWebPlayerPlugin.obj
 0001:00001eed       ?DestroyStream@UnityWebPlayerPluginInstance@@UAEFPAU_NPStream@@F@Z 10002eed f   UnityWebPlayerPlugin.obj
 0001:00001f13       ?URLNotify@UnityWebPlayerPluginInstance@@UAEXPBDFPAX@Z 10002f13 f   UnityWebPlayerPlugin.obj
 0001:00001f6a       ?Redraw@UnityWebPlayerPluginInstance@@AAEXXZ 10002f6a f   UnityWebPlayerPlugin.obj
 0001:00001fa3       ?PrepareDoubleBuffer@UnityWebPlayerPluginInstance@@AAEXPAUHDC__@@@Z 10002fa3 f   UnityWebPlayerPlugin.obj
 0001:00002096       ?OnDestroy@UnityWebPlayerPluginInstance@@QAEXXZ 10003096 f   UnityWebPlayerPlugin.obj
 0001:00002118       ?CheckError@UnityWebPlayerPluginInstance@@AAE_NXZ 10003118 f   UnityWebPlayerPlugin.obj
 0001:0000217f       ?CheckRuntimeError@UnityWebPlayerPluginInstance@@AAE_NXZ 1000317f f   UnityWebPlayerPlugin.obj
 0001:000021f8       ?Tick@UnityWebPlayerPluginInstance@@QAEXXZ 100031f8 f   UnityWebPlayerPlugin.obj
 0001:0000229d       ?TickWrap@UnityWebPlayerPluginInstance@@AAEXXZ 1000329d f   UnityWebPlayerPlugin.obj
 0001:0000255b       ?OnDraw@UnityWebPlayerPluginInstance@@QAEXPAUHWND__@@PAUHDC__@@ABUtagRECT@@@Z 1000355b f   UnityWebPlayerPlugin.obj
 0001:0000276e       ?OnContextMenu@UnityWebPlayerPluginInstance@@QAEXHH@Z 1000376e f   UnityWebPlayerPlugin.obj
 0001:00002a76       ??0?$basic_string@DU?$char_traits@D@std@@V?$allocator@D@2@@std@@QAE@ABV01@@Z 10003a76 f i UnityWebPlayerPlugin.obj
 0001:00002a9c       ??0?$basic_string@DU?$char_traits@D@std@@V?$allocator@D@2@@std@@QAE@PBDI@Z 10003a9c f i UnityWebPlayerPlugin.obj
 0001:00002ac0       ??0?$basic_string@DU?$char_traits@D@std@@V?$allocator@D@2@@std@@QAE@PBD@Z 10003ac0 f i UnityWebPlayerPlugin.obj
 0001:00002aef       ??0?$basic_string@DU?$char_traits@D@std@@V?$allocator@D@2@@std@@QAE@$$QAV01@@Z 10003aef f i UnityWebPlayerPlugin.obj
 0001:00002b12       ??0?$basic_string@_WU?$char_traits@_W@std@@V?$allocator@_W@2@@std@@QAE@PB_W@Z 10003b12 f i UnityWebPlayerPlugin.obj
 0001:00002b43       ??E?$_Tree_const_iterator@V?$_Tree_val@V?$_Tset_traits@V?$basic_string@DU?$char_traits@D@std@@V?$allocator@D@2@@std@@U?$less@V?$basic_string@DU?$char_traits@D@std@@V?$allocator@D@2@@std@@@2@V?$allocator@V?$basic_string@DU?$char_traits@D@std@@V?$allocator@D@2@@std@@@2@$0A@@std@@@std@@@std@@QAEAAV01@XZ 10003b43 f i UnityWebPlayerPlugin.obj
 0001:00002b79       ?assign@?$basic_string@DU?$char_traits@D@std@@V?$allocator@D@2@@std@@QAEAAV12@$$QAV12@@Z 10003b79 f i UnityWebPlayerPlugin.obj
 0001:00002bd0       ?assign@?$basic_string@DU?$char_traits@D@std@@V?$allocator@D@2@@std@@QAEAAV12@ABV12@II@Z 10003bd0 f i UnityWebPlayerPlugin.obj
 0001:00002c69       ?assign@?$basic_string@DU?$char_traits@D@std@@V?$allocator@D@2@@std@@QAEAAV12@PBDI@Z 10003c69 f i UnityWebPlayerPlugin.obj
 0001:00002cde       ?compare@?$basic_string@DU?$char_traits@D@std@@V?$allocator@D@2@@std@@QBEHIIPBDI@Z 10003cde f i UnityWebPlayerPlugin.obj
 0001:00002d40       ?_Tidy@?$basic_string@DU?$char_traits@D@std@@V?$allocator@D@2@@std@@QAEX_NI@Z 10003d40 f i UnityWebPlayerPlugin.obj
 0001:00002d84       ??0?$_Tree@V?$_Tset_traits@V?$basic_string@DU?$char_traits@D@std@@V?$allocator@D@2@@std@@U?$less@V?$basic_string@DU?$char_traits@D@std@@V?$allocator@D@2@@std@@@2@V?$allocator@V?$basic_string@DU?$char_traits@D@std@@V?$allocator@D@2@@std@@@2@$0A@@std@@@std@@QAE@ABV01@@Z 10003d84 f i UnityWebPlayerPlugin.obj
 0001:00002e2f       ?_Tidy@?$_Tree@V?$_Tset_traits@V?$basic_string@DU?$char_traits@D@std@@V?$allocator@D@2@@std@@U?$less@V?$basic_string@DU?$char_traits@D@std@@V?$allocator@D@2@@std@@@2@V?$allocator@V?$basic_string@DU?$char_traits@D@std@@V?$allocator@D@2@@std@@@2@$0A@@std@@@std@@IAEXXZ 10003e2f f i UnityWebPlayerPlugin.obj
 0001:00002e54       ?erase@?$basic_string@DU?$char_traits@D@std@@V?$allocator@D@2@@std@@QAEAAV12@II@Z 10003e54 f i UnityWebPlayerPlugin.obj
 0001:00002ecc       ?_Grow@?$basic_string@DU?$char_traits@D@std@@V?$allocator@D@2@@std@@QAE_NI_N@Z 10003ecc f i UnityWebPlayerPlugin.obj
 0001:00002f30       ?_Inside@?$basic_string@DU?$char_traits@D@std@@V?$allocator@D@2@@std@@QAE_NPBD@Z 10003f30 f i UnityWebPlayerPlugin.obj
 0001:00002f6b       ??0?$_Tree_val@V?$_Tset_traits@V?$basic_string@DU?$char_traits@D@std@@V?$allocator@D@2@@std@@U?$less@V?$basic_string@DU?$char_traits@D@std@@V?$allocator@D@2@@std@@@2@V?$allocator@V?$basic_string@DU?$char_traits@D@std@@V?$allocator@D@2@@std@@@2@$0A@@std@@@std@@QAE@ABU?$less@V?$basic_string@DU?$char_traits@D@std@@V?$allocator@D@2@@std@@@1@V?$allocator@V?$basic_string@DU?$char_traits@D@std@@V?$allocator@D@2@@std@@@1@@Z 10003f6b f i UnityWebPlayerPlugin.obj
 0001:00002f98       ?_Copy@?$basic_string@DU?$char_traits@D@std@@V?$allocator@D@2@@std@@QAEXII@Z 10003f98 f i UnityWebPlayerPlugin.obj
 0001:00003096       ?_Copy@?$_Tree@V?$_Tset_traits@V?$basic_string@DU?$char_traits@D@std@@V?$allocator@D@2@@std@@U?$less@V?$basic_string@DU?$char_traits@D@std@@V?$allocator@D@2@@std@@@2@V?$allocator@V?$basic_string@DU?$char_traits@D@std@@V?$allocator@D@2@@std@@@2@$0A@@std@@@std@@IAEPAU_Node@?$_Tree_nod@V?$_Tset_traits@V?$basic_string@DU?$char_traits@D@std@@V?$allocator@D@2@@std@@U?$less@V?$basic_string@DU?$char_traits@D@std@@V?$allocator@D@2@@std@@@2@V?$allocator@V?$basic_string@DU?$char_traits@D@std@@V?$allocator@D@2@@std@@@2@$0A@@std@@@2@PAU342@0@Z 10004096 f i UnityWebPlayerPlugin.obj
 0001:0000312b       ?allocate@?$allocator@U_Node@?$_Tree_nod@V?$_Tset_traits@V?$basic_string@DU?$char_traits@D@std@@V?$allocator@D@2@@std@@U?$less@V?$basic_string@DU?$char_traits@D@std@@V?$allocator@D@2@@std@@@2@V?$allocator@V?$basic_string@DU?$char_traits@D@std@@V?$allocator@D@2@@std@@@2@$0A@@std@@@std@@@std@@QAEPAU_Node@?$_Tree_nod@V?$_Tset_traits@V?$basic_string@DU?$char_traits@D@std@@V?$allocator@D@2@@std@@U?$less@V?$basic_string@DU?$char_traits@D@std@@V?$allocator@D@2@@std@@@2@V?$allocator@V?$basic_string@DU?$char_traits@D@std@@V?$allocator@D@2@@std@@@2@$0A@@std@@@2@I@Z 1000412b f i UnityWebPlayerPlugin.obj
 0001:00003163       ?_Erase@?$_Tree@V?$_Tset_traits@V?$basic_string@DU?$char_traits@D@std@@V?$allocator@D@2@@std@@U?$less@V?$basic_string@DU?$char_traits@D@std@@V?$allocator@D@2@@std@@@2@V?$allocator@V?$basic_string@DU?$char_traits@D@std@@V?$allocator@D@2@@std@@@2@$0A@@std@@@std@@IAEXPAU_Node@?$_Tree_nod@V?$_Tset_traits@V?$basic_string@DU?$char_traits@D@std@@V?$allocator@D@2@@std@@U?$less@V?$basic_string@DU?$char_traits@D@std@@V?$allocator@D@2@@std@@@2@V?$allocator@V?$basic_string@DU?$char_traits@D@std@@V?$allocator@D@2@@std@@@2@$0A@@std@@@2@@Z 10004163 f i UnityWebPlayerPlugin.obj
 0001:000031a5       ?_Lrotate@?$_Tree@V?$_Tset_traits@V?$basic_string@DU?$char_traits@D@std@@V?$allocator@D@2@@std@@U?$less@V?$basic_string@DU?$char_traits@D@std@@V?$allocator@D@2@@std@@@2@V?$allocator@V?$basic_string@DU?$char_traits@D@std@@V?$allocator@D@2@@std@@@2@$0A@@std@@@std@@IAEXPAU_Node@?$_Tree_nod@V?$_Tset_traits@V?$basic_string@DU?$char_traits@D@std@@V?$allocator@D@2@@std@@U?$less@V?$basic_string@DU?$char_traits@D@std@@V?$allocator@D@2@@std@@@2@V?$allocator@V?$basic_string@DU?$char_traits@D@std@@V?$allocator@D@2@@std@@@2@$0A@@std@@@2@@Z 100041a5 f i UnityWebPlayerPlugin.obj
 0001:000031e8       ?_Rrotate@?$_Tree@V?$_Tset_traits@V?$basic_string@DU?$char_traits@D@std@@V?$allocator@D@2@@std@@U?$less@V?$basic_string@DU?$char_traits@D@std@@V?$allocator@D@2@@std@@@2@V?$allocator@V?$basic_string@DU?$char_traits@D@std@@V?$allocator@D@2@@std@@@2@$0A@@std@@@std@@IAEXPAU_Node@?$_Tree_nod@V?$_Tset_traits@V?$basic_string@DU?$char_traits@D@std@@V?$allocator@D@2@@std@@U?$less@V?$basic_string@DU?$char_traits@D@std@@V?$allocator@D@2@@std@@@2@V?$allocator@V?$basic_string@DU?$char_traits@D@std@@V?$allocator@D@2@@std@@@2@$0A@@std@@@2@@Z 100041e8 f i UnityWebPlayerPlugin.obj
 0001:0000322d       ??$ChangeStringFormat@PBDV?$basic_string@_WU?$char_traits@_W@std@@V?$allocator@_W@2@@std@@Umulti_byte_to_wide@detail@@@detail@@YAXABQBDIAAV?$basic_string@_WU?$char_traits@_W@std@@V?$allocator@_W@2@@std@@Umulti_byte_to_wide@0@@Z 1000422d f i UnityWebPlayerPlugin.obj
 0001:0000329c       ??$?HDU?$char_traits@D@std@@V?$allocator@D@1@@std@@YA?AV?$basic_string@DU?$char_traits@D@std@@V?$allocator@D@2@@0@PBDABV10@@Z 1000429c f i UnityWebPlayerPlugin.obj
 0001:000032e7       ??$?8DU?$char_traits@D@std@@V?$allocator@D@1@@std@@YA_NABV?$basic_string@DU?$char_traits@D@std@@V?$allocator@D@2@@0@0@Z 100042e7 f i UnityWebPlayerPlugin.obj
 0001:00003304       ??$_Buynode@AAV?$basic_string@DU?$char_traits@D@std@@V?$allocator@D@2@@std@@@?$_Tree_val@V?$_Tset_traits@V?$basic_string@DU?$char_traits@D@std@@V?$allocator@D@2@@std@@U?$less@V?$basic_string@DU?$char_traits@D@std@@V?$allocator@D@2@@std@@@2@V?$allocator@V?$basic_string@DU?$char_traits@D@std@@V?$allocator@D@2@@std@@@2@$0A@@std@@@std@@QAEPAU_Node@?$_Tree_nod@V?$_Tset_traits@V?$basic_string@DU?$char_traits@D@std@@V?$allocator@D@2@@std@@U?$less@V?$basic_string@DU?$char_traits@D@std@@V?$allocator@D@2@@std@@@2@V?$allocator@V?$basic_string@DU?$char_traits@D@std@@V?$allocator@D@2@@std@@@2@$0A@@std@@@1@AAV?$basic_string@DU?$char_traits@D@std@@V?$allocator@D@2@@1@@Z 10004304 f i UnityWebPlayerPlugin.obj
 0001:00003375       ??$_Allocate@D@std@@YAPADIPAD@Z 10004375 f i UnityWebPlayerPlugin.obj
 0001:000033bc       ?reserve@?$basic_string@DU?$char_traits@D@std@@V?$allocator@D@2@@std@@QAEXI@Z 100043bc f i UnityWebPlayerPlugin.obj
 0001:000033f3       ?_Linsert@?$_Tree@V?$_Tset_traits@V?$basic_string@DU?$char_traits@D@std@@V?$allocator@D@2@@std@@U?$less@V?$basic_string@DU?$char_traits@D@std@@V?$allocator@D@2@@std@@@2@V?$allocator@V?$basic_string@DU?$char_traits@D@std@@V?$allocator@D@2@@std@@@2@$0A@@std@@@std@@QAE?AU?$pair@V?$_Tree_const_iterator@V?$_Tree_val@V?$_Tset_traits@V?$basic_string@DU?$char_traits@D@std@@V?$allocator@D@2@@std@@U?$less@V?$basic_string@DU?$char_traits@D@std@@V?$allocator@D@2@@std@@@2@V?$allocator@V?$basic_string@DU?$char_traits@D@std@@V?$allocator@D@2@@std@@@2@$0A@@std@@@std@@@std@@_N@2@PAU_Node@?$_Tree_nod@V?$_Tset_traits@V?$basic_string@DU?$char_traits@D@std@@V?$allocator@D@2@@std@@U?$less@V?$basic_string@DU?$char_traits@D@std@@V?$allocator@D@2@@std@@@2@V?$allocator@V?$basic_string@DU?$char_traits@D@std@@V?$allocator@D@2@@std@@@2@$0A@@std@@@2@_N@Z 100043f3 f i UnityWebPlayerPlugin.obj
 0001:000034d8       ?resize@?$basic_string@_WU?$char_traits@_W@std@@V?$allocator@_W@2@@std@@QAEXI_W@Z 100044d8 f i UnityWebPlayerPlugin.obj
 0001:000034fe       ?_Insert@?$_Tree@V?$_Tset_traits@V?$basic_string@DU?$char_traits@D@std@@V?$allocator@D@2@@std@@U?$less@V?$basic_string@DU?$char_traits@D@std@@V?$allocator@D@2@@std@@@2@V?$allocator@V?$basic_string@DU?$char_traits@D@std@@V?$allocator@D@2@@std@@@2@$0A@@std@@@std@@IAE?AV?$_Tree_const_iterator@V?$_Tree_val@V?$_Tset_traits@V?$basic_string@DU?$char_traits@D@std@@V?$allocator@D@2@@std@@U?$less@V?$basic_string@DU?$char_traits@D@std@@V?$allocator@D@2@@std@@@2@V?$allocator@V?$basic_string@DU?$char_traits@D@std@@V?$allocator@D@2@@std@@@2@$0A@@std@@@std@@@2@_NPAU_Node@?$_Tree_nod@V?$_Tset_traits@V?$basic_string@DU?$char_traits@D@std@@V?$allocator@D@2@@std@@U?$less@V?$basic_string@DU?$char_traits@D@std@@V?$allocator@D@2@@std@@@2@V?$allocator@V?$basic_string@DU?$char_traits@D@std@@V?$allocator@D@2@@std@@@2@$0A@@std@@@2@1@Z 100044fe f i UnityWebPlayerPlugin.obj
 0001:00003623       ??R?$less@V?$basic_string@DU?$char_traits@D@std@@V?$allocator@D@2@@std@@@std@@QBE_NABV?$basic_string@DU?$char_traits@D@std@@V?$allocator@D@2@@1@0@Z 10004623 f i UnityWebPlayerPlugin.obj
 0001:00003642       ?append@?$basic_string@DU?$char_traits@D@std@@V?$allocator@D@2@@std@@QAEAAV12@ABV12@II@Z 10004642 f i UnityWebPlayerPlugin.obj
 0001:000036dc       ?append@?$basic_string@DU?$char_traits@D@std@@V?$allocator@D@2@@std@@QAEAAV12@PBDI@Z 100046dc f i UnityWebPlayerPlugin.obj
 0001:00003775       ?append@?$basic_string@_WU?$char_traits@_W@std@@V?$allocator@_W@2@@std@@QAEAAV12@I_W@Z 10004775 f i UnityWebPlayerPlugin.obj
 0001:000037d7       ?_Chassign@?$basic_string@_WU?$char_traits@_W@std@@V?$allocator@_W@2@@std@@QAEXII_W@Z 100047d7 f i UnityWebPlayerPlugin.obj
 0001:00003816       _wmemset                   10004816 f i UnityWebPlayerPlugin.obj
 0001:00003840       _NP_Shutdown@0             10004840 f   np_entry.obj
 0001:000038d2       _NP_Initialize@4           100048d2 f   np_entry.obj
 0001:0000396a       _NP_GetEntryPoints@4       1000496a f   np_entry.obj
 0001:00003979       _NPP_New                   10004979 f   npp_gate.obj
 0001:000039dd       _NPP_Destroy               100049dd f   npp_gate.obj
 0001:00003a0d       _NPP_SetWindow             10004a0d f   npp_gate.obj
 0001:00003aa5       _NPP_NewStream             10004aa5 f   npp_gate.obj
 0001:00003ad2       _NPP_WriteReady            10004ad2 f   npp_gate.obj
 0001:00003af3       _NPP_Write                 10004af3 f   npp_gate.obj
 0001:00003b1b       _NPP_DestroyStream         10004b1b f   npp_gate.obj
 0001:00003b42       _NPP_StreamAsFile          10004b42 f   npp_gate.obj
 0001:00003b5f       _NPP_Print                 10004b5f f   npp_gate.obj
 0001:00003b79       _NPP_URLNotify             10004b79 f   npp_gate.obj
 0001:00003b99       _NPP_GetValue              10004b99 f   npp_gate.obj
 0001:00003bc0       _NPP_SetValue              10004bc0 f   npp_gate.obj
 0001:00003be7       _NPP_HandleEvent           10004be7 f   npp_gate.obj
 0001:00003c05       ??0DownloaderNetscape@@QAE@ABV?$basic_string@DU?$char_traits@D@std@@V?$allocator@D@2@@std@@AAVLogger@@PAX@Z 10004c05 f i DownloadNetscape.obj
 0001:00003ced       ?CancelDownload@@YAXPAVDownload@@@Z 10004ced f   DownloadNetscape.obj
 0001:00003d68       ?StartDownload@@YAPAVDownload@@ABV?$basic_string@DU?$char_traits@D@std@@V?$allocator@D@2@@std@@AAVLogger@@PAXPBXI3I@Z 10004d68 f   DownloadNetscape.obj
 0001:00003ea1       ?NetscapeStartNaturalDownload@@YAPAVDownload@@AAU_NPStream@@AAVLogger@@@Z 10004ea1 f   DownloadNetscape.obj
 0001:00003f33       ?OnNetscapeNewStream@@YAFPADPAU_NPStream@@EPAG@Z 10004f33 f   DownloadNetscape.obj
 0001:00003fae       ?OnNetscapeDestroyStream@@YAFPAU_NPStream@@F@Z 10004fae f   DownloadNetscape.obj
 0001:0000404d       ?NetscapeSetupProgressParams@@YAXAAVPluginInstance@@PAU_NPP@@FQAPAD2@Z 1000504d f   DownloadNetscape.obj
 0001:00004180       ?GetBoolValue@?A0x5b7c1c12@@YA_NPBD@Z 10005180 f i DownloadNetscape.obj
 0001:000041c1       ?NetscapeParseEmbedParameters@@YAXAAVPluginInstance@@FQAPAD1@Z 100051c1 f   DownloadNetscape.obj
 0001:0000436e       ?erase@?$_Tree@V?$_Tmap_traits@IPAVDownloaderNetscape@@U?$less@I@std@@V?$allocator@U?$pair@$$CBIPAVDownloaderNetscape@@@std@@@3@$0A@@std@@@std@@QAEIABI@Z 1000536e f i DownloadNetscape.obj
 0001:00004402       ?erase@?$_Tree@V?$_Tmap_traits@PAVDownload@@PAU_NPStream@@U?$less@PAVDownload@@@std@@V?$allocator@U?$pair@QAVDownload@@PAU_NPStream@@@std@@@4@$0A@@std@@@std@@QAEIABQAVDownload@@@Z 10005402 f i DownloadNetscape.obj
 0001:00004496       ?find@?$_Tree@V?$_Tmap_traits@PAVDownload@@PAU_NPStream@@U?$less@PAVDownload@@@std@@V?$allocator@U?$pair@QAVDownload@@PAU_NPStream@@@std@@@4@$0A@@std@@@std@@QAE?AV?$_Tree_iterator@V?$_Tree_val@V?$_Tmap_traits@PAVDownload@@PAU_NPStream@@U?$less@PAVDownload@@@std@@V?$allocator@U?$pair@QAVDownload@@PAU_NPStream@@@std@@@4@$0A@@std@@@std@@@2@ABQAVDownload@@@Z 10005496 f i DownloadNetscape.obj
 0001:000044e5       ?erase@?$_Tree@V?$_Tmap_traits@IPAVDownloaderNetscape@@U?$less@I@std@@V?$allocator@U?$pair@$$CBIPAVDownloaderNetscape@@@std@@@3@$0A@@std@@@std@@QAE?AV?$_Tree_iterator@V?$_Tree_val@V?$_Tmap_traits@IPAVDownloaderNetscape@@U?$less@I@std@@V?$allocator@U?$pair@$$CBIPAVDownloaderNetscape@@@std@@@3@$0A@@std@@@std@@@2@V?$_Tree_const_iterator@V?$_Tree_val@V?$_Tmap_traits@IPAVDownloaderNetscape@@U?$less@I@std@@V?$allocator@U?$pair@$$CBIPAVDownloaderNetscape@@@std@@@3@$0A@@std@@@std@@@2@0@Z 100054e5 f i DownloadNetscape.obj
 0001:0000455b       ?erase@?$_Tree@V?$_Tmap_traits@PAVDownload@@PAU_NPStream@@U?$less@PAVDownload@@@std@@V?$allocator@U?$pair@QAVDownload@@PAU_NPStream@@@std@@@4@$0A@@std@@@std@@QAE?AV?$_Tree_iterator@V?$_Tree_val@V?$_Tmap_traits@PAVDownload@@PAU_NPStream@@U?$less@PAVDownload@@@std@@V?$allocator@U?$pair@QAVDownload@@PAU_NPStream@@@std@@@4@$0A@@std@@@std@@@2@V?$_Tree_const_iterator@V?$_Tree_val@V?$_Tmap_traits@PAVDownload@@PAU_NPStream@@U?$less@PAVDownload@@@std@@V?$allocator@U?$pair@QAVDownload@@PAU_NPStream@@@std@@@4@$0A@@std@@@std@@@2@0@Z 1000555b f i DownloadNetscape.obj
 0001:000045d1       ?erase@?$_Tree@V?$_Tmap_traits@IPAVDownloaderNetscape@@U?$less@I@std@@V?$allocator@U?$pair@$$CBIPAVDownloaderNetscape@@@std@@@3@$0A@@std@@@std@@QAE?AV?$_Tree_iterator@V?$_Tree_val@V?$_Tmap_traits@IPAVDownloaderNetscape@@U?$less@I@std@@V?$allocator@U?$pair@$$CBIPAVDownloaderNetscape@@@std@@@3@$0A@@std@@@std@@@2@V?$_Tree_const_iterator@V?$_Tree_val@V?$_Tmap_traits@IPAVDownloaderNetscape@@U?$less@I@std@@V?$allocator@U?$pair@$$CBIPAVDownloaderNetscape@@@std@@@3@$0A@@std@@@std@@@2@@Z 100055d1 f i DownloadNetscape.obj
 0001:0000480f       ?erase@?$_Tree@V?$_Tmap_traits@PAVDownload@@PAU_NPStream@@U?$less@PAVDownload@@@std@@V?$allocator@U?$pair@QAVDownload@@PAU_NPStream@@@std@@@4@$0A@@std@@@std@@QAE?AV?$_Tree_iterator@V?$_Tree_val@V?$_Tmap_traits@PAVDownload@@PAU_NPStream@@U?$less@PAVDownload@@@std@@V?$allocator@U?$pair@QAVDownload@@PAU_NPStream@@@std@@@4@$0A@@std@@@std@@@2@V?$_Tree_const_iterator@V?$_Tree_val@V?$_Tmap_traits@PAVDownload@@PAU_NPStream@@U?$less@PAVDownload@@@std@@V?$allocator@U?$pair@QAVDownload@@PAU_NPStream@@@std@@@4@$0A@@std@@@std@@@2@@Z 1000580f f i DownloadNetscape.obj
 0001:00004a4d       ?_Erase@?$_Tree@V?$_Tmap_traits@PAVDownload@@PAU_NPStream@@U?$less@PAVDownload@@@std@@V?$allocator@U?$pair@QAVDownload@@PAU_NPStream@@@std@@@4@$0A@@std@@@std@@IAEXPAU_Node@?$_Tree_nod@V?$_Tmap_traits@PAVDownload@@PAU_NPStream@@U?$less@PAVDownload@@@std@@V?$allocator@U?$pair@QAVDownload@@PAU_NPStream@@@std@@@4@$0A@@std@@@2@@Z 10005a4d f i DownloadNetscape.obj
 0001:00004a4d       ?_Erase@?$_Tree@V?$_Tmap_traits@IPAVDownloaderNetscape@@U?$less@I@std@@V?$allocator@U?$pair@$$CBIPAVDownloaderNetscape@@@std@@@3@$0A@@std@@@std@@IAEXPAU_Node@?$_Tree_nod@V?$_Tmap_traits@IPAVDownloaderNetscape@@U?$less@I@std@@V?$allocator@U?$pair@$$CBIPAVDownloaderNetscape@@@std@@@3@$0A@@std@@@2@@Z 10005a4d f i DownloadNetscape.obj
 0001:00004a4d       ?_Erase@?$_Tree@V?$_Tmap_traits@KPAVTimer@?A0xa59a0aab@@U?$less@K@std@@V?$allocator@U?$pair@$$CBKPAVTimer@?A0xa59a0aab@@@std@@@4@$0A@@std@@@std@@IAEXPAU_Node@?$_Tree_nod@V?$_Tmap_traits@KPAVTimer@?A0xa59a0aab@@U?$less@K@std@@V?$allocator@U?$pair@$$CBKPAVTimer@?A0xa59a0aab@@@std@@@4@$0A@@std@@@2@@Z 10005a4d f i WebCommonLib:PluginManager.obj
 0001:00004a4d       ?_Erase@?$_Tree@V?$_Tmap_traits@IW4UpdateStatus@UpdaterProxy@@U?$less@I@std@@V?$allocator@U?$pair@$$CBIW4UpdateStatus@UpdaterProxy@@@std@@@4@$0A@@std@@@std@@IAEXPAU_Node@?$_Tree_nod@V?$_Tmap_traits@IW4UpdateStatus@UpdaterProxy@@U?$less@I@std@@V?$allocator@U?$pair@$$CBIW4UpdateStatus@UpdaterProxy@@@std@@@4@$0A@@std@@@2@@Z 10005a4d f i WebCommonLib:PluginManager.obj
 0001:00004a82       ?_Lrotate@?$_Tree@V?$_Tmap_traits@IPAVDownloaderNetscape@@U?$less@I@std@@V?$allocator@U?$pair@$$CBIPAVDownloaderNetscape@@@std@@@3@$0A@@std@@@std@@IAEXPAU_Node@?$_Tree_nod@V?$_Tmap_traits@IPAVDownloaderNetscape@@U?$less@I@std@@V?$allocator@U?$pair@$$CBIPAVDownloaderNetscape@@@std@@@3@$0A@@std@@@2@@Z 10005a82 f i DownloadNetscape.obj
 0001:00004abf       ?_Rrotate@?$_Tree@V?$_Tmap_traits@IPAVDownloaderNetscape@@U?$less@I@std@@V?$allocator@U?$pair@$$CBIPAVDownloaderNetscape@@@std@@@3@$0A@@std@@@std@@IAEXPAU_Node@?$_Tree_nod@V?$_Tmap_traits@IPAVDownloaderNetscape@@U?$less@I@std@@V?$allocator@U?$pair@$$CBIPAVDownloaderNetscape@@@std@@@3@$0A@@std@@@2@@Z 10005abf f i DownloadNetscape.obj
 0001:00004afe       ?_Lrotate@?$_Tree@V?$_Tmap_traits@PAVDownload@@PAU_NPStream@@U?$less@PAVDownload@@@std@@V?$allocator@U?$pair@QAVDownload@@PAU_NPStream@@@std@@@4@$0A@@std@@@std@@IAEXPAU_Node@?$_Tree_nod@V?$_Tmap_traits@PAVDownload@@PAU_NPStream@@U?$less@PAVDownload@@@std@@V?$allocator@U?$pair@QAVDownload@@PAU_NPStream@@@std@@@4@$0A@@std@@@2@@Z 10005afe f i DownloadNetscape.obj
 0001:00004b3b       ?_Rrotate@?$_Tree@V?$_Tmap_traits@PAVDownload@@PAU_NPStream@@U?$less@PAVDownload@@@std@@V?$allocator@U?$pair@QAVDownload@@PAU_NPStream@@@std@@@4@$0A@@std@@@std@@IAEXPAU_Node@?$_Tree_nod@V?$_Tmap_traits@PAVDownload@@PAU_NPStream@@U?$less@PAVDownload@@@std@@V?$allocator@U?$pair@QAVDownload@@PAU_NPStream@@@std@@@4@$0A@@std@@@2@@Z 10005b3b f i DownloadNetscape.obj
 0001:00004b7a       ?_Linsert@?$_Tree@V?$_Tmap_traits@IPAVDownloaderNetscape@@U?$less@I@std@@V?$allocator@U?$pair@$$CBIPAVDownloaderNetscape@@@std@@@3@$0A@@std@@@std@@QAE?AU?$pair@V?$_Tree_iterator@V?$_Tree_val@V?$_Tmap_traits@IPAVDownloaderNetscape@@U?$less@I@std@@V?$allocator@U?$pair@$$CBIPAVDownloaderNetscape@@@std@@@3@$0A@@std@@@std@@@std@@_N@2@PAU_Node@?$_Tree_nod@V?$_Tmap_traits@IPAVDownloaderNetscape@@U?$less@I@std@@V?$allocator@U?$pair@$$CBIPAVDownloaderNetscape@@@std@@@3@$0A@@std@@@2@_N@Z 10005b7a f i DownloadNetscape.obj
 0001:00004c3d       ?_Linsert@?$_Tree@V?$_Tmap_traits@PAVDownload@@PAU_NPStream@@U?$less@PAVDownload@@@std@@V?$allocator@U?$pair@QAVDownload@@PAU_NPStream@@@std@@@4@$0A@@std@@@std@@QAE?AU?$pair@V?$_Tree_iterator@V?$_Tree_val@V?$_Tmap_traits@PAVDownload@@PAU_NPStream@@U?$less@PAVDownload@@@std@@V?$allocator@U?$pair@QAVDownload@@PAU_NPStream@@@std@@@4@$0A@@std@@@std@@@std@@_N@2@PAU_Node@?$_Tree_nod@V?$_Tmap_traits@PAVDownload@@PAU_NPStream@@U?$less@PAVDownload@@@std@@V?$allocator@U?$pair@QAVDownload@@PAU_NPStream@@@std@@@4@$0A@@std@@@2@_N@Z 10005c3d f i DownloadNetscape.obj
 0001:00004d00       ?_Insert@?$_Tree@V?$_Tmap_traits@IPAVDownloaderNetscape@@U?$less@I@std@@V?$allocator@U?$pair@$$CBIPAVDownloaderNetscape@@@std@@@3@$0A@@std@@@std@@IAE?AV?$_Tree_iterator@V?$_Tree_val@V?$_Tmap_traits@IPAVDownloaderNetscape@@U?$less@I@std@@V?$allocator@U?$pair@$$CBIPAVDownloaderNetscape@@@std@@@3@$0A@@std@@@std@@@2@_NPAU_Node@?$_Tree_nod@V?$_Tmap_traits@IPAVDownloaderNetscape@@U?$less@I@std@@V?$allocator@U?$pair@$$CBIPAVDownloaderNetscape@@@std@@@3@$0A@@std@@@2@1@Z 10005d00 f i DownloadNetscape.obj
 0001:00004e24       ?_Insert@?$_Tree@V?$_Tmap_traits@PAVDownload@@PAU_NPStream@@U?$less@PAVDownload@@@std@@V?$allocator@U?$pair@QAVDownload@@PAU_NPStream@@@std@@@4@$0A@@std@@@std@@IAE?AV?$_Tree_iterator@V?$_Tree_val@V?$_Tmap_traits@PAVDownload@@PAU_NPStream@@U?$less@PAVDownload@@@std@@V?$allocator@U?$pair@QAVDownload@@PAU_NPStream@@@std@@@4@$0A@@std@@@std@@@2@_NPAU_Node@?$_Tree_nod@V?$_Tmap_traits@PAVDownload@@PAU_NPStream@@U?$less@PAVDownload@@@std@@V?$allocator@U?$pair@QAVDownload@@PAU_NPStream@@@std@@@4@$0A@@std@@@2@1@Z 10005e24 f i DownloadNetscape.obj
 0001:00004f48       ??$_Buynode@U?$pair@IPAVDownloaderNetscape@@@std@@@?$_Tree_val@V?$_Tmap_traits@IPAVDownloaderNetscape@@U?$less@I@std@@V?$allocator@U?$pair@$$CBIPAVDownloaderNetscape@@@std@@@3@$0A@@std@@@std@@QAEPAU_Node@?$_Tree_nod@V?$_Tmap_traits@IPAVDownloaderNetscape@@U?$less@I@std@@V?$allocator@U?$pair@$$CBIPAVDownloaderNetscape@@@std@@@3@$0A@@std@@@1@$$QAU?$pair@IPAVDownloaderNetscape@@@1@@Z 10005f48 f i DownloadNetscape.obj
 0001:00004fbe       ??$_Buynode@U?$pair@PAVDownloaderNetscape@@PAU_NPStream@@@std@@@?$_Tree_val@V?$_Tmap_traits@PAVDownload@@PAU_NPStream@@U?$less@PAVDownload@@@std@@V?$allocator@U?$pair@QAVDownload@@PAU_NPStream@@@std@@@4@$0A@@std@@@std@@QAEPAU_Node@?$_Tree_nod@V?$_Tmap_traits@PAVDownload@@PAU_NPStream@@U?$less@PAVDownload@@@std@@V?$allocator@U?$pair@QAVDownload@@PAU_NPStream@@@std@@@4@$0A@@std@@@1@$$QAU?$pair@PAVDownloaderNetscape@@PAU_NPStream@@@1@@Z 10005fbe f i DownloadNetscape.obj
 0001:00005034       ??0VariantValue@@QAE@XZ    10006034 f i NetscapeScriptablePlugin.obj
 0001:0000504b       ??0VariantValue@@QAE@ABU0@@Z 1000604b f i NetscapeScriptablePlugin.obj
 0001:00005085       ?pluginRemoveProperty@@YA_NPAUNPObject@@PAX@Z 10006085 f   NetscapeScriptablePlugin.obj
 0001:00005085       ?pluginHasProperty@@YA_NPAUNPObject@@PAX@Z 10006085 f   NetscapeScriptablePlugin.obj
 0001:00005088       ?pluginHasMethod@@YA_NPAUNPObject@@PAX@Z 10006088 f   NetscapeScriptablePlugin.obj
 0001:000050a9       ?pluginGetProperty@@YA_NPAUNPObject@@PAXPAU_NPVariant@@@Z 100060a9 f   NetscapeScriptablePlugin.obj
 0001:000050ba       ?pluginSetProperty@@YA_NPAUNPObject@@PAXPBU_NPVariant@@@Z 100060ba f   NetscapeScriptablePlugin.obj
 0001:00005371       ?pluginInvoke@@YA_NPAUNPObject@@PAXPBU_NPVariant@@IPAU2@@Z 10006371 f   NetscapeScriptablePlugin.obj
 0001:000055fe       ?pluginInvokeDefault@@YA_NPAUNPObject@@PBU_NPVariant@@IPAU2@@Z 100065fe f   NetscapeScriptablePlugin.obj
 0001:0000560b       ?Tick@Download@@UAEXXZ     1000660b f   DownloadNetscape.obj
 0001:0000560b       ?Cancel@Download@@UAEXXZ   1000660b f   DownloadNetscape.obj
 0001:0000560b       ?pluginInvalidate@@YAXPAUNPObject@@@Z 1000660b f   NetscapeScriptablePlugin.obj
 0001:0000560c       ?pluginAllocate@@YAPAUNPObject@@PAU_NPP@@PAUNPClass@@@Z 1000660c f   NetscapeScriptablePlugin.obj
 0001:00005658       ?pluginDeallocate@@YAXPAUNPObject@@@Z 10006658 f   NetscapeScriptablePlugin.obj
 0001:00005661       ?GetPluginPageURLFromDOM@NetscapeScriptablePlugin@@SA?AV?$basic_string@DU?$char_traits@D@std@@V?$allocator@D@2@@std@@PAU_NPP@@AAVLogger@@@Z 10006661 f   NetscapeScriptablePlugin.obj
 0001:000057ce       ?ProcessExternalCalls@NetscapeScriptablePlugin@@SAXPAU_NPP@@ABV?$basic_string@DU?$char_traits@D@std@@V?$allocator@D@2@@std@@@Z 100067ce f   NetscapeScriptablePlugin.obj
 0001:00005844       ?push_back@?$vector@UVariantValue@@V?$allocator@UVariantValue@@@std@@@std@@QAEX$$QAUVariantValue@@@Z 10006844 f i NetscapeScriptablePlugin.obj
 0001:00005899       ?replace@?$basic_string@DU?$char_traits@D@std@@V?$allocator@D@2@@std@@QAEAAV12@IIABV12@II@Z 10006899 f i NetscapeScriptablePlugin.obj
 0001:00005b22       ?find@?$basic_string@DU?$char_traits@D@std@@V?$allocator@D@2@@std@@QBEIPBDII@Z 10006b22 f i NetscapeScriptablePlugin.obj
 0001:00005bab       ?_Reserve@?$vector@UVariantValue@@V?$allocator@UVariantValue@@@std@@@std@@IAEXI@Z 10006bab f i NetscapeScriptablePlugin.obj
 0001:00005c02       ?reserve@?$vector@UVariantValue@@V?$allocator@UVariantValue@@@std@@@std@@QAEXI@Z 10006c02 f i NetscapeScriptablePlugin.obj
 0001:00005cbc       ?_Destroy@?$vector@UVariantValue@@V?$allocator@UVariantValue@@@std@@@std@@IAEXPAUVariantValue@@0@Z 10006cbc f i NetscapeScriptablePlugin.obj
 0001:00005ce7       ?allocate@?$allocator@UVariantValue@@@std@@QAEPAUVariantValue@@I@Z 10006ce7 f i NetscapeScriptablePlugin.obj
 0001:00005d30       ??$_Uninit_move@PAUVariantValue@@PAU1@V?$allocator@UVariantValue@@@std@@U1@@std@@YAPAUVariantValue@@PAU1@00AAV?$allocator@UVariantValue@@@0@0U_Nonscalar_ptr_iterator_tag@0@@Z 10006d30 f i NetscapeScriptablePlugin.obj
 0001:00005db2       ??0AutoLock@SystemWideMutex@@QAE@AAV1@M@Z 10006db2 f i WebCommonLib:PluginManager.obj
 0001:00005e02       ?convert@wide_to_multi_byte@detail@@QBEXPB_WIAAV?$basic_string@DU?$char_traits@D@std@@V?$allocator@D@2@@std@@@Z 10006e02 f i WebCommonLib:PluginManager.obj
 0001:00005e2e       ?ConvertSeparatorsToWindows@@YAXAAV?$basic_string@DU?$char_traits@D@std@@V?$allocator@D@2@@std@@@Z 10006e2e f i WebCommonLib:PluginManager.obj
 0001:00005e61       ?ConvertWindowsPathName@@YAXPB_WAAV?$basic_string@DU?$char_traits@D@std@@V?$allocator@D@2@@std@@@Z 10006e61 f i WebCommonLib:PluginManager.obj
 0001:00005fb9       ??0Timer@?A0xa59a0aab@@QAE@G@Z 10006fb9 f i WebCommonLib:PluginManager.obj
 0001:00006025       ?AddPlugin@Timer@?A0xa59a0aab@@QAEXPAVUnityWebPlayerPluginInstance@@@Z 10007025 f i WebCommonLib:PluginManager.obj
 0001:000060b3       ?RemovePlugin@Timer@?A0xa59a0aab@@QAE_NPAVUnityWebPlayerPluginInstance@@@Z 100070b3 f i WebCommonLib:PluginManager.obj
 0001:00006121       ?DestroyTimerWindow@Timer@?A0xa59a0aab@@QAEXXZ 10007121 f i WebCommonLib:PluginManager.obj
 0001:0000615b       ?Tick@Timer@?A0xa59a0aab@@CGXPAXE@Z 1000715b f i WebCommonLib:PluginManager.obj
 0001:0000618e       ?ComparePlugins@Timer@?A0xa59a0aab@@CA_NPAVUnityWebPlayerPluginInstance@@0@Z 1000718e f i WebCommonLib:PluginManager.obj
 0001:000061be       ?WindowProc@Timer@?A0xa59a0aab@@CGJPAUHWND__@@IIJ@Z 100071be f i WebCommonLib:PluginManager.obj
 0001:000062fc       ??0WindowsTimerManager@?A0xa59a0aab@@IAE@XZ 100072fc f i WebCommonLib:PluginManager.obj
 0001:00006376       ?CleanupPluginImpl@WindowsTimerManager@?A0xa59a0aab@@CAXAAU?$pair@$$CBKPAVTimer@?A0xa59a0aab@@@std@@@Z 10007376 f i WebCommonLib:PluginManager.obj
 0001:000063bb       ?AddPlugin@WindowsTimerManager@?A0xa59a0aab@@AAEXKPAVUnityWebPlayerPluginInstance@@@Z 100073bb f i WebCommonLib:PluginManager.obj
 0001:0000642f       ??_GWindowsTimerManager@?A0xa59a0aab@@IAEPAXI@Z 1000742f f i WebCommonLib:PluginManager.obj
 0001:00006498       ?RemovePlugin@WindowsTimerManager@?A0xa59a0aab@@SAXPAVUnityWebPlayerPluginInstance@@@Z 10007498 f   WebCommonLib:PluginManager.obj
 0001:000064f9       ?GetDefaultReleaseChannel@PluginManager@@QAE?AV?$basic_string@DU?$char_traits@D@std@@V?$allocator@D@2@@std@@XZ 100074f9 f   WebCommonLib:PluginManager.obj
 0001:0000654a       ?GetDevelopmentPlayer@PluginManager@@QBE_NXZ 1000754a f   WebCommonLib:PluginManager.obj
 0001:000065bc       ?OnCrashCallback@PluginManager@@SAXPBD@Z 100075bc f   WebCommonLib:PluginManager.obj
 0001:00006680       ?IsAdminPath@PluginManager@@AAE_NABV?$basic_string@DU?$char_traits@D@std@@V?$allocator@D@2@@std@@@Z 10007680 f   WebCommonLib:PluginManager.obj
 0001:0000674e       ??0PluginManager@@AAE@XZ   1000774e f   WebCommonLib:PluginManager.obj
 0001:00006e1c       ??1PluginManager@@AAE@XZ   10007e1c f   WebCommonLib:PluginManager.obj
 0001:00006f6a       ??_GLogger@@QAEPAXI@Z      10007f6a f i WebCommonLib:PluginManager.obj
 0001:00006f90       ?AddPlugin@PluginManager@@QAEXAAVPluginInstance@@@Z 10007f90 f   WebCommonLib:PluginManager.obj
 0001:00007072       ?RemovePlugin@PluginManager@@QAEXAAVPluginInstance@@@Z 10008072 f   WebCommonLib:PluginManager.obj
 0001:000071a0       ?DeleteTempFiles@PluginManager@@QAEX_N@Z 100081a0 f   WebCommonLib:PluginManager.obj
 0001:0000722c       ?GetInstalledRevision@PluginManager@@QAEHW4BundleID@@ABV?$basic_string@DU?$char_traits@D@std@@V?$allocator@D@2@@std@@1PAV34@@Z 1000822c f   WebCommonLib:PluginManager.obj
 0001:00007318       ?GetTemporaryPathRevision@PluginManager@@QAEHABV?$basic_string@DU?$char_traits@D@std@@V?$allocator@D@2@@std@@W4BundleID@@0@Z 10008318 f   WebCommonLib:PluginManager.obj
 0001:0000735d       ?GetRevisionFromPath@PluginManager@@CAHABV?$basic_string@DU?$char_traits@D@std@@V?$allocator@D@2@@std@@PAV23@@Z 1000835d f   WebCommonLib:PluginManager.obj
 0001:000074a9       ?ApplySelfUpdate@PluginManager@@AAE?AW4UpdateResult@1@PBEIAAUUpdateInfo@1@PAUHWND__@@@Z 100084a9 f   WebCommonLib:PluginManager.obj
 0001:000076d1       ?ApplyUpdate@PluginManager@@AAE?AW4UpdateResult@1@PBEIW4BundleID@@ABV?$basic_string@DU?$char_traits@D@std@@V?$allocator@D@2@@std@@AAUUpdateInfo@1@PAUHWND__@@@Z 100086d1 f   WebCommonLib:PluginManager.obj
 0001:00007934       ?DoneWithUpdates@PluginManager@@QAEXXZ 10008934 f   WebCommonLib:PluginManager.obj
 0001:00007975       ?GetHomePath@PluginManager@@CA?AV?$basic_string@DU?$char_traits@D@std@@V?$allocator@D@2@@std@@PAUHKEY__@@@Z 10008975 f   WebCommonLib:PluginManager.obj
 0001:000079ec       ?GetDefaultUserHomePath@PluginManager@@CA?AV?$basic_string@DU?$char_traits@D@std@@V?$allocator@D@2@@std@@XZ 100089ec f   WebCommonLib:PluginManager.obj
 0001:00007abf       ?GetDefaultOldUserHomePath@PluginManager@@CA?AV?$basic_string@DU?$char_traits@D@std@@V?$allocator@D@2@@std@@XZ 10008abf f   WebCommonLib:PluginManager.obj
 0001:00007b13       ?CheckBundleExistsInUserLocation@PluginManager@@ABE_NW4BundleID@@ABV?$basic_string@DU?$char_traits@D@std@@V?$allocator@D@2@@std@@_N1@Z 10008b13 f   WebCommonLib:PluginManager.obj
 0001:00007bdf       ?CreateUpdaterProxy@PluginManager@@AAE_NXZ 10008bdf f   WebCommonLib:PluginManager.obj
 0001:00007d5d       ?GetInstalledPath@PluginManager@@QBE?AV?$basic_string@DU?$char_traits@D@std@@V?$allocator@D@2@@std@@W4BundleID@@ABV23@1HPAW4LocationType@1@@Z 10008d5d f   WebCommonLib:PluginManager.obj
 0001:00007f10       ?OnUpdateDownloadProcessing@PluginManager@@AAEXAAUUpdateInfo@1@@Z 10008f10 f   WebCommonLib:PluginManager.obj
 0001:00007fa6       ?Tick@PluginManager@@QAEXPAUHWND__@@@Z 10008fa6 f   WebCommonLib:PluginManager.obj
 0001:0000815f       ?Log@PluginManager@@QAAXPBDZZ 1000915f f   WebCommonLib:PluginManager.obj
 0001:00008178       ?compare@?$basic_string@DU?$char_traits@D@std@@V?$allocator@D@2@@std@@QBEHPBD@Z 10009178 f i WebCommonLib:PluginManager.obj
 0001:0000819c       ?erase@?$_Tree@V?$_Tmap_traits@IW4UpdateStatus@UpdaterProxy@@U?$less@I@std@@V?$allocator@U?$pair@$$CBIW4UpdateStatus@UpdaterProxy@@@std@@@4@$0A@@std@@@std@@QAEIABI@Z 1000919c f i WebCommonLib:PluginManager.obj
 0001:0000823a       ?push_back@?$vector@PAVPluginInstance@@V?$allocator@PAVPluginInstance@@@std@@@std@@QAEX$$QAPAVPluginInstance@@@Z 1000923a f i WebCommonLib:PluginManager.obj
 0001:00008286       ??1?$vector@UUpdateInfo@PluginManager@@V?$allocator@UUpdateInfo@PluginManager@@@std@@@std@@QAE@XZ 10009286 f i WebCommonLib:PluginManager.obj
 0001:000082a8       ?push_back@?$vector@UUpdateInfo@PluginManager@@V?$allocator@UUpdateInfo@PluginManager@@@std@@@std@@QAEXABUUpdateInfo@PluginManager@@@Z 100092a8 f i WebCommonLib:PluginManager.obj
 0001:000082fc       ?erase@?$vector@UUpdateInfo@PluginManager@@V?$allocator@UUpdateInfo@PluginManager@@@std@@@std@@QAE?AV?$_Vector_iterator@V?$_Vector_val@UUpdateInfo@PluginManager@@V?$allocator@UUpdateInfo@PluginManager@@@std@@@std@@@2@V?$_Vector_const_iterator@V?$_Vector_val@UUpdateInfo@PluginManager@@V?$allocator@UUpdateInfo@PluginManager@@@std@@@std@@@2@@Z 100092fc f i WebCommonLib:PluginManager.obj
 0001:00008374       ?erase@?$_Tree@V?$_Tmap_traits@IW4UpdateStatus@UpdaterProxy@@U?$less@I@std@@V?$allocator@U?$pair@$$CBIW4UpdateStatus@UpdaterProxy@@@std@@@4@$0A@@std@@@std@@QAE?AV?$_Tree_iterator@V?$_Tree_val@V?$_Tmap_traits@IW4UpdateStatus@UpdaterProxy@@U?$less@I@std@@V?$allocator@U?$pair@$$CBIW4UpdateStatus@UpdaterProxy@@@std@@@4@$0A@@std@@@std@@@2@V?$_Tree_const_iterator@V?$_Tree_val@V?$_Tmap_traits@IW4UpdateStatus@UpdaterProxy@@U?$less@I@std@@V?$allocator@U?$pair@$$CBIW4UpdateStatus@UpdaterProxy@@@std@@@4@$0A@@std@@@std@@@2@@Z 10009374 f i WebCommonLib:PluginManager.obj
 0001:00008374       ?erase@?$_Tree@V?$_Tmap_traits@KPAVTimer@?A0xa59a0aab@@U?$less@K@std@@V?$allocator@U?$pair@$$CBKPAVTimer@?A0xa59a0aab@@@std@@@4@$0A@@std@@@std@@QAE?AV?$_Tree_iterator@V?$_Tree_val@V?$_Tmap_traits@KPAVTimer@?A0xa59a0aab@@U?$less@K@std@@V?$allocator@U?$pair@$$CBKPAVTimer@?A0xa59a0aab@@@std@@@4@$0A@@std@@@std@@@2@V?$_Tree_const_iterator@V?$_Tree_val@V?$_Tmap_traits@KPAVTimer@?A0xa59a0aab@@U?$less@K@std@@V?$allocator@U?$pair@$$CBKPAVTimer@?A0xa59a0aab@@@std@@@4@$0A@@std@@@std@@@2@@Z 10009374 f i WebCommonLib:PluginManager.obj
 0001:000085c9       ?clear@?$_Tree@V?$_Tmap_traits@IW4UpdateStatus@UpdaterProxy@@U?$less@I@std@@V?$allocator@U?$pair@$$CBIW4UpdateStatus@UpdaterProxy@@@std@@@4@$0A@@std@@@std@@QAEXXZ 100095c9 f i WebCommonLib:PluginManager.obj
 0001:000085c9       ?clear@?$_Tree@V?$_Tmap_traits@KPAVTimer@?A0xa59a0aab@@U?$less@K@std@@V?$allocator@U?$pair@$$CBKPAVTimer@?A0xa59a0aab@@@std@@@4@$0A@@std@@@std@@QAEXXZ 100095c9 f i WebCommonLib:PluginManager.obj
 0001:000085ee       ?find@?$_Tree@V?$_Tmap_traits@KPAVTimer@?A0xa59a0aab@@U?$less@K@std@@V?$allocator@U?$pair@$$CBKPAVTimer@?A0xa59a0aab@@@std@@@4@$0A@@std@@@std@@QAE?AV?$_Tree_iterator@V?$_Tree_val@V?$_Tmap_traits@KPAVTimer@?A0xa59a0aab@@U?$less@K@std@@V?$allocator@U?$pair@$$CBKPAVTimer@?A0xa59a0aab@@@std@@@4@$0A@@std@@@std@@@2@ABK@Z 100095ee f i WebCommonLib:PluginManager.obj
 0001:000085ee       ?find@?$_Tree@V?$_Tmap_traits@IW4UpdateStatus@UpdaterProxy@@U?$less@I@std@@V?$allocator@U?$pair@$$CBIW4UpdateStatus@UpdaterProxy@@@std@@@4@$0A@@std@@@std@@QAE?AV?$_Tree_iterator@V?$_Tree_val@V?$_Tmap_traits@IW4UpdateStatus@UpdaterProxy@@U?$less@I@std@@V?$allocator@U?$pair@$$CBIW4UpdateStatus@UpdaterProxy@@@std@@@4@$0A@@std@@@std@@@2@ABI@Z 100095ee f i WebCommonLib:UpdaterProxy.obj
 0001:0000863d       ?erase@?$_Tree@V?$_Tmap_traits@IW4UpdateStatus@UpdaterProxy@@U?$less@I@std@@V?$allocator@U?$pair@$$CBIW4UpdateStatus@UpdaterProxy@@@std@@@4@$0A@@std@@@std@@QAE?AV?$_Tree_iterator@V?$_Tree_val@V?$_Tmap_traits@IW4UpdateStatus@UpdaterProxy@@U?$less@I@std@@V?$allocator@U?$pair@$$CBIW4UpdateStatus@UpdaterProxy@@@std@@@4@$0A@@std@@@std@@@2@V?$_Tree_const_iterator@V?$_Tree_val@V?$_Tmap_traits@IW4UpdateStatus@UpdaterProxy@@U?$less@I@std@@V?$allocator@U?$pair@$$CBIW4UpdateStatus@UpdaterProxy@@@std@@@4@$0A@@std@@@std@@@2@0@Z 1000963d f i WebCommonLib:PluginManager.obj
 0001:0000868c       ?_Destroy@?$vector@UUpdateInfo@PluginManager@@V?$allocator@UUpdateInfo@PluginManager@@@std@@@std@@IAEXPAUUpdateInfo@PluginManager@@0@Z 1000968c f i WebCommonLib:PluginManager.obj
 0001:000086bf       ?_Reserve@?$vector@UUpdateInfo@PluginManager@@V?$allocator@UUpdateInfo@PluginManager@@@std@@@std@@IAEXI@Z 100096bf f i WebCommonLib:PluginManager.obj
 0001:00008716       ?_Lrotate@?$_Tree@V?$_Tmap_traits@IW4UpdateStatus@UpdaterProxy@@U?$less@I@std@@V?$allocator@U?$pair@$$CBIW4UpdateStatus@UpdaterProxy@@@std@@@4@$0A@@std@@@std@@IAEXPAU_Node@?$_Tree_nod@V?$_Tmap_traits@IW4UpdateStatus@UpdaterProxy@@U?$less@I@std@@V?$allocator@U?$pair@$$CBIW4UpdateStatus@UpdaterProxy@@@std@@@4@$0A@@std@@@2@@Z 10009716 f i WebCommonLib:PluginManager.obj
 0001:00008716       ?_Lrotate@?$_Tree@V?$_Tmap_traits@KPAVTimer@?A0xa59a0aab@@U?$less@K@std@@V?$allocator@U?$pair@$$CBKPAVTimer@?A0xa59a0aab@@@std@@@4@$0A@@std@@@std@@IAEXPAU_Node@?$_Tree_nod@V?$_Tmap_traits@KPAVTimer@?A0xa59a0aab@@U?$less@K@std@@V?$allocator@U?$pair@$$CBKPAVTimer@?A0xa59a0aab@@@std@@@4@$0A@@std@@@2@@Z 10009716 f i WebCommonLib:PluginManager.obj
 0001:00008759       ?_Rrotate@?$_Tree@V?$_Tmap_traits@KPAVTimer@?A0xa59a0aab@@U?$less@K@std@@V?$allocator@U?$pair@$$CBKPAVTimer@?A0xa59a0aab@@@std@@@4@$0A@@std@@@std@@IAEXPAU_Node@?$_Tree_nod@V?$_Tmap_traits@KPAVTimer@?A0xa59a0aab@@U?$less@K@std@@V?$allocator@U?$pair@$$CBKPAVTimer@?A0xa59a0aab@@@std@@@4@$0A@@std@@@2@@Z 10009759 f i WebCommonLib:PluginManager.obj
 0001:00008759       ?_Rrotate@?$_Tree@V?$_Tmap_traits@IW4UpdateStatus@UpdaterProxy@@U?$less@I@std@@V?$allocator@U?$pair@$$CBIW4UpdateStatus@UpdaterProxy@@@std@@@4@$0A@@std@@@std@@IAEXPAU_Node@?$_Tree_nod@V?$_Tmap_traits@IW4UpdateStatus@UpdaterProxy@@U?$less@I@std@@V?$allocator@U?$pair@$$CBIW4UpdateStatus@UpdaterProxy@@@std@@@4@$0A@@std@@@2@@Z 10009759 f i WebCommonLib:PluginManager.obj
 0001:0000879e       ?reserve@?$vector@UUpdateInfo@PluginManager@@V?$allocator@UUpdateInfo@PluginManager@@@std@@@std@@QAEXI@Z 1000979e f i WebCommonLib:PluginManager.obj
 0001:00008858       ??E?$_Tree_const_iterator@V?$_Tree_val@V?$_Tmap_traits@IW4UpdateStatus@UpdaterProxy@@U?$less@I@std@@V?$allocator@U?$pair@$$CBIW4UpdateStatus@UpdaterProxy@@@std@@@4@$0A@@std@@@std@@@std@@QAEAAV01@XZ 10009858 f i WebCommonLib:PluginManager.obj
 0001:00008858       ??E?$_Tree_const_iterator@V?$_Tree_val@V?$_Tmap_traits@PAVDownload@@PAU_NPStream@@U?$less@PAVDownload@@@std@@V?$allocator@U?$pair@QAVDownload@@PAU_NPStream@@@std@@@4@$0A@@std@@@std@@@std@@QAEAAV01@XZ 10009858 f i DownloadNetscape.obj
 0001:00008858       ??E?$_Tree_unchecked_const_iterator@V?$_Tree_val@V?$_Tmap_traits@KPAVTimer@?A0xa59a0aab@@U?$less@K@std@@V?$allocator@U?$pair@$$CBKPAVTimer@?A0xa59a0aab@@@std@@@4@$0A@@std@@@std@@U_Iterator_base0@2@@std@@QAEAAV01@XZ 10009858 f i WebCommonLib:PluginManager.obj
 0001:00008858       ??E?$_Tree_const_iterator@V?$_Tree_val@V?$_Tmap_traits@IPAVDownloaderNetscape@@U?$less@I@std@@V?$allocator@U?$pair@$$CBIPAVDownloaderNetscape@@@std@@@3@$0A@@std@@@std@@@std@@QAEAAV01@XZ 10009858 f i DownloadNetscape.obj
 0001:0000888e       ?_Chassign@?$basic_string@DU?$char_traits@D@std@@V?$allocator@D@2@@std@@QAEXIID@Z 1000988e f i WebCommonLib:PluginManager.obj
 0001:000088ca       ?allocate@?$allocator@UUpdateInfo@PluginManager@@@std@@QAEPAUUpdateInfo@PluginManager@@I@Z 100098ca f i WebCommonLib:PluginManager.obj
 0001:00008913       ??$ChangeStringFormat@PB_WV?$basic_string@DU?$char_traits@D@std@@V?$allocator@D@2@@std@@Uwide_to_multi_byte@detail@@@detail@@YAXABQB_WIAAV?$basic_string@DU?$char_traits@D@std@@V?$allocator@D@2@@std@@Uwide_to_multi_byte@0@@Z 10009913 f i WebCommonLib:PluginManager.obj
 0001:0000897c       ??$ConvertUnityPathNameImpl@V?$basic_string@DU?$char_traits@D@std@@V?$allocator@D@2@@std@@@detail@@YAXABV?$basic_string@DU?$char_traits@D@std@@V?$allocator@D@2@@std@@AAV?$basic_string@_WU?$char_traits@_W@std@@V?$allocator@_W@2@@2@@Z 1000997c f i WebCommonLib:PluginManager.obj
 0001:000089cd       ??$?HDU?$char_traits@D@std@@V?$allocator@D@1@@std@@YA?AV?$basic_string@DU?$char_traits@D@std@@V?$allocator@D@2@@0@PBD$$QAV10@@Z 100099cd f i WebCommonLib:PluginManager.obj
 0001:000089f3       ??$?HDU?$char_traits@D@std@@V?$allocator@D@1@@std@@YA?AV?$basic_string@DU?$char_traits@D@std@@V?$allocator@D@2@@0@$$QAV10@PBD@Z 100099f3 f i WebCommonLib:PluginManager.obj
 0001:00008a19       ??$?HDU?$char_traits@D@std@@V?$allocator@D@1@@std@@YA?AV?$basic_string@DU?$char_traits@D@std@@V?$allocator@D@2@@0@$$QAV10@ABV10@@Z 10009a19 f i WebCommonLib:PluginManager.obj
 0001:00008a39       ??$?HDU?$char_traits@D@std@@V?$allocator@D@1@@std@@YA?AV?$basic_string@DU?$char_traits@D@std@@V?$allocator@D@2@@0@ABV10@0@Z 10009a39 f i WebCommonLib:PluginManager.obj
 0001:00008a70       ?insert@?$basic_string@DU?$char_traits@D@std@@V?$allocator@D@2@@std@@QAEAAV12@IABV12@II@Z 10009a70 f i WebCommonLib:PluginManager.obj
 0001:00008b8c       ?insert@?$basic_string@DU?$char_traits@D@std@@V?$allocator@D@2@@std@@QAEAAV12@IPBDI@Z 10009b8c f i WebCommonLib:PluginManager.obj
 0001:00008c44       ?resize@?$basic_string@DU?$char_traits@D@std@@V?$allocator@D@2@@std@@QAEXID@Z 10009c44 f i WebCommonLib:PluginManager.obj
 0001:00008c6a       ?append@?$basic_string@DU?$char_traits@D@std@@V?$allocator@D@2@@std@@QAEAAV12@ID@Z 10009c6a f i WebCommonLib:PluginManager.obj
 0001:00008cca       ??$_Sort@PAPAVUnityWebPlayerPluginInstance@@HP6A_NPAV1@0@Z@std@@YAXPAPAVUnityWebPlayerPluginInstance@@0HP6A_NPAV1@1@Z@Z 10009cca f i WebCommonLib:PluginManager.obj
 0001:00008df2       ??$_Buynode@U?$pair@KPAVTimer@?A0xa59a0aab@@@std@@@?$_Tree_val@V?$_Tmap_traits@KPAVTimer@?A0xa59a0aab@@U?$less@K@std@@V?$allocator@U?$pair@$$CBKPAVTimer@?A0xa59a0aab@@@std@@@4@$0A@@std@@@std@@QAEPAU_Node@?$_Tree_nod@V?$_Tmap_traits@KPAVTimer@?A0xa59a0aab@@U?$less@K@std@@V?$allocator@U?$pair@$$CBKPAVTimer@?A0xa59a0aab@@@std@@@4@$0A@@std@@@1@$$QAU?$pair@KPAVTimer@?A0xa59a0aab@@@1@@Z 10009df2 f i WebCommonLib:PluginManager.obj
 0001:00008df2       ??$_Buynode@U?$pair@$$CBIW4UpdateStatus@UpdaterProxy@@@std@@@?$_Tree_val@V?$_Tmap_traits@IW4UpdateStatus@UpdaterProxy@@U?$less@I@std@@V?$allocator@U?$pair@$$CBIW4UpdateStatus@UpdaterProxy@@@std@@@4@$0A@@std@@@std@@QAEPAU_Node@?$_Tree_nod@V?$_Tmap_traits@IW4UpdateStatus@UpdaterProxy@@U?$less@I@std@@V?$allocator@U?$pair@$$CBIW4UpdateStatus@UpdaterProxy@@@std@@@4@$0A@@std@@@1@$$QAU?$pair@$$CBIW4UpdateStatus@UpdaterProxy@@@1@@Z 10009df2 f i WebCommonLib:UpdaterProxy.obj
 0001:00008e61       ??0UpdateInfo@PluginManager@@QAE@ABU01@@Z 10009e61 f i WebCommonLib:PluginManager.obj
 0001:00008e92       ??$_Replace@PA_W_W@std@@YAXPA_W0AB_W1@Z 10009e92 f i WebCommonLib:PluginManager.obj
 0001:00008eb8       ??$_Unguarded_partition@PAPAVUnityWebPlayerPluginInstance@@P6A_NPAV1@0@Z@std@@YA?AU?$pair@PAPAVUnityWebPlayerPluginInstance@@PAPAV1@@0@PAPAVUnityWebPlayerPluginInstance@@0P6A_NPAV2@1@Z@Z 10009eb8 f i WebCommonLib:PluginManager.obj
 0001:00009030       ??$_Insertion_sort@PAPAVUnityWebPlayerPluginInstance@@P6A_NPAV1@0@Z@std@@YAXPAPAVUnityWebPlayerPluginInstance@@0P6A_NPAV1@1@Z@Z 1000a030 f i WebCommonLib:PluginManager.obj
 0001:000090a8       ??$_Uninit_move@PAUUpdateInfo@PluginManager@@PAU12@V?$allocator@UUpdateInfo@PluginManager@@@std@@U12@@std@@YAPAUUpdateInfo@PluginManager@@PAU12@00AAV?$allocator@UUpdateInfo@PluginManager@@@0@0U_Nonscalar_ptr_iterator_tag@0@@Z 1000a0a8 f i WebCommonLib:PluginManager.obj
 0001:0000912f       ??$_Median@PAPAVUnityWebPlayerPluginInstance@@P6A_NPAV1@0@Z@std@@YAXPAPAVUnityWebPlayerPluginInstance@@00P6A_NPAV1@1@Z@Z 1000a12f f i WebCommonLib:PluginManager.obj
 0001:000091bf       ??$_Med3@PAPAVUnityWebPlayerPluginInstance@@P6A_NPAV1@0@Z@std@@YAXPAPAVUnityWebPlayerPluginInstance@@00P6A_NPAV1@1@Z@Z 1000a1bf f i WebCommonLib:PluginManager.obj
 0001:00009203       ??$_Adjust_heap@PAPAVUnityWebPlayerPluginInstance@@HPAV1@P6A_NPAV1@0@Z@std@@YAXPAPAVUnityWebPlayerPluginInstance@@HH$$QAPAV1@P6A_NPAV1@2@Z@Z 1000a203 f i WebCommonLib:PluginManager.obj
 0001:0000928c       ?GenerateGuidString@@YA?AV?$basic_string@DU?$char_traits@D@std@@V?$allocator@D@2@@std@@XZ 1000a28c f   WebCommonLib:WebPluginUtility.obj
 0001:000092fd       ?GetForceDevelopmentPlugin@@YA_NXZ 1000a2fd f   WebCommonLib:WebPluginUtility.obj
 0001:0000934b       ?GetDisableAutoUpdates@@YA_NXZ 1000a34b f   WebCommonLib:WebPluginUtility.obj
 0001:00009383       ?WebDebugLog@@YAXAAVLogger@@PBDZZ 1000a383 f   WebCommonLib:WebPluginUtility.obj
 0001:0000939d       ?GetKeepLogFiles@@YA_NXZ   1000a39d f   WebCommonLib:WebPluginUtility.obj
 0001:000093b7       ?GetNumericVersion@@YAHABV?$basic_string@DU?$char_traits@D@std@@V?$allocator@D@2@@std@@@Z 1000a3b7 f   WebCommonLib:WebPluginUtility.obj
 0001:00009519       ?VFormat@@YA?AV?$basic_string@DU?$char_traits@D@std@@V?$allocator@D@2@@std@@PBDPAD@Z 1000a519 f   WebCommonLib:WebPluginUtility.obj
 0001:00009554       ?Format@@YA?AV?$basic_string@DU?$char_traits@D@std@@V?$allocator@D@2@@std@@PBDZZ 1000a554 f   WebCommonLib:WebPluginUtility.obj
 0001:00009854       ?CreateDIBSectionFromBGRA@?A0x09aeca17@@YAPAUHBITMAP__@@PAUHDC__@@PBXHH@Z 1000a854 f   WebCommonLib:ProgressDisplayWin.obj
 0001:000098d2       ??0ProgressImage@@QAE@PAUHDC__@@I@Z 1000a8d2 f   WebCommonLib:ProgressDisplayWin.obj
 0001:00009971       ?Initialize@progress@@YAXAAVMutex@@PAUHINSTANCE__@@@Z 1000a971 f   WebCommonLib:ProgressDisplayWin.obj
 0001:00009af0       ?ShowProgress@progress@@YAXAAVSetup@1@PAUHDC__@@ABUtagRECT@@MABV?$basic_string@DU?$char_traits@D@std@@V?$allocator@D@2@@std@@AAH_N@Z 1000aaf0 f   WebCommonLib:ProgressDisplayWin.obj
 0001:00009ec2       ?LinkSubclassProc@ProgressLink@@CGJPAUHWND__@@IIJ@Z 1000aec2 f   WebCommonLib:ProgressDisplayWin.obj
 0001:00009f13       ?Draw@ProgressLink@@QAEXAAUtagDRAWITEMSTRUCT@@@Z 1000af13 f   WebCommonLib:ProgressDisplayWin.obj
 0001:0000a000       ?Create@ProgressLink@@QAEXPAUHINSTANCE__@@PAUHWND__@@HHW4Alignment@1@IABV?$basic_string@_WU?$char_traits@_W@std@@V?$allocator@_W@2@@std@@ABUColor@progress@@4@Z 1000b000 f   WebCommonLib:ProgressDisplayWin.obj
 0001:0000a125       ??0PluginError@@QAE@ABV?$basic_string@DU?$char_traits@D@std@@V?$allocator@D@2@@std@@0_N@Z 1000b125 f i WebCommonLib:PluginInstance.obj
 0001:0000a169       ?AddWwwDownload@PluginInstance@@QAEXPAVDownload@@@Z 1000b169 f i WebCommonLib:PluginInstance.obj
 0001:0000a1ea       ??0PluginInstance@@QAE@PAX0P6AX0@Z@Z 1000b1ea f   WebCommonLib:PluginInstance.obj
 0001:0000a59c       ??1PluginError@@QAE@XZ     1000b59c f i WebCommonLib:PluginInstance.obj
 0001:0000a5b4       ??1PluginInstance@@QAE@XZ  1000b5b4 f   WebCommonLib:PluginInstance.obj
 0001:0000a6f5       ?Validate@PluginInstance@@QAE?AW4PlayerHashValidationResult@@XZ 1000b6f5 f   WebCommonLib:PluginInstance.obj
 0001:0000a75d       ?DeleteTempFiles@PluginInstance@@QAEX_N@Z 1000b75d f   WebCommonLib:PluginInstance.obj
 0001:0000a7d2       ?SetError@PluginInstance@@QAEXABVPluginError@@@Z 1000b7d2 f   WebCommonLib:PluginInstance.obj
 0001:0000a825       ??4PluginError@@QAEAAV0@ABV0@@Z 1000b825 f i WebCommonLib:PluginInstance.obj
 0001:0000a84a       ?SetError@PluginInstance@@QAEXABV?$basic_string@DU?$char_traits@D@std@@V?$allocator@D@2@@std@@0_N@Z 1000b84a f   WebCommonLib:PluginInstance.obj
 0001:0000a873       ??Rcancelled_downloads@detail@@QBE_NPAVDownload@@@Z 1000b873 f i WebCommonLib:PluginInstance.obj
 0001:0000a89a       ?Tick@PluginInstance@@QAEXXZ 1000b89a f   WebCommonLib:PluginInstance.obj
 0001:0000a8f1       ?ParseDataHeader@PluginInstance@@AAEXXZ 1000b8f1 f   WebCommonLib:PluginInstance.obj
 0001:0000aa9d       ?UpdateDownloadDataFile@PluginInstance@@AAEXXZ 1000ba9d f   WebCommonLib:PluginInstance.obj
 0001:0000ab66       ?UpdateProgress@?A0x10dfc39b@@YAXIIAAI00@Z 1000bb66 f   WebCommonLib:PluginInstance.obj
 0001:0000ab91       ?UpdateProgress@PluginInstance@@AAEXXZ 1000bb91 f   WebCommonLib:PluginInstance.obj
 0001:0000ad02       ?IsReadyToLoad@PluginInstance@@QAE_NXZ 1000bd02 f   WebCommonLib:PluginInstance.obj
 0001:0000ad7d       ?Log@PluginInstance@@QAAXPBDZZ 1000bd7d f   WebCommonLib:PluginInstance.obj
 0001:0000ad99       ?AddSendMessage@PluginInstance@@QAEXPBD0ABUVariantValue@@@Z 1000bd99 f   WebCommonLib:PluginInstance.obj
 0001:0000ae70       ?StartDownloadBinding@@YAPAVDownload@@PBDPAX1P6AHPAV1@@Z@Z 1000be70 f   WebCommonLib:PluginInstance.obj
 0001:0000aee2       ?StartDownloadBinding2@@YAPAVDownload@@PBDPAX1P6AHPAV1@@ZPBXI4I@Z 1000bee2 f   WebCommonLib:PluginInstance.obj
 0001:0000af5a       ??1?$vector@UWebMessage@@V?$allocator@UWebMessage@@@std@@@std@@QAE@XZ 1000bf5a f i WebCommonLib:PluginInstance.obj
 0001:0000af8a       ?_Reserve@?$vector@UWebMessage@@V?$allocator@UWebMessage@@@std@@@std@@IAEXI@Z 1000bf8a f i WebCommonLib:PluginInstance.obj
 0001:0000afe1       ?_Reserve@?$vector@PAVUnityWebPlayerPluginInstance@@V?$allocator@PAVUnityWebPlayerPluginInstance@@@std@@@std@@IAEXI@Z 1000bfe1 f i WebCommonLib:PluginManager.obj
 0001:0000afe1       ?_Reserve@?$vector@PAVDownload@@V?$allocator@PAVDownload@@@std@@@std@@IAEXI@Z 1000bfe1 f i WebCommonLib:PluginInstance.obj
 0001:0000afe1       ?_Reserve@?$vector@PAVPluginInstance@@V?$allocator@PAVPluginInstance@@@std@@@std@@IAEXI@Z 1000bfe1 f i WebCommonLib:PluginManager.obj
 0001:0000b030       ?reserve@?$vector@UWebMessage@@V?$allocator@UWebMessage@@@std@@@std@@QAEXI@Z 1000c030 f i WebCommonLib:PluginInstance.obj
 0001:0000b10a       ?reserve@?$vector@PAVUnityWebPlayerPluginInstance@@V?$allocator@PAVUnityWebPlayerPluginInstance@@@std@@@std@@QAEXI@Z 1000c10a f i WebCommonLib:PluginManager.obj
 0001:0000b10a       ?reserve@?$vector@PAVPluginInstance@@V?$allocator@PAVPluginInstance@@@std@@@std@@QAEXI@Z 1000c10a f i WebCommonLib:PluginManager.obj
 0001:0000b10a       ?reserve@?$vector@PAVDownload@@V?$allocator@PAVDownload@@@std@@@std@@QAEXI@Z 1000c10a f i WebCommonLib:PluginInstance.obj
 0001:0000b1b0       ?allocate@?$allocator@UWebMessage@@@std@@QAEPAUWebMessage@@I@Z 1000c1b0 f i WebCommonLib:PluginInstance.obj
 0001:0000b1f9       ?allocate@?$allocator@PAVUnityWebPlayerPluginInstance@@@std@@QAEPAPAVUnityWebPlayerPluginInstance@@I@Z 1000c1f9 f i WebCommonLib:PluginManager.obj
 0001:0000b1f9       ?allocate@?$allocator@PAVPluginInstance@@@std@@QAEPAPAVPluginInstance@@I@Z 1000c1f9 f i WebCommonLib:PluginManager.obj
 0001:0000b1f9       ?allocate@?$allocator@PAVDownload@@@std@@QAEPAPAVDownload@@I@Z 1000c1f9 f i WebCommonLib:PluginInstance.obj
 0001:0000b244       ??$tick_downloads@V?$vector@PAVDownload@@V?$allocator@PAVDownload@@@std@@@std@@@@YAXAAV?$vector@PAVDownload@@V?$allocator@PAVDownload@@@std@@@std@@@Z 1000c244 f i WebCommonLib:PluginInstance.obj
 0001:0000b2ba       ??$_Cons_val@V?$allocator@UWebMessage@@@std@@UWebMessage@@U3@@std@@YAXAAV?$allocator@UWebMessage@@@0@PAUWebMessage@@$$QAU2@@Z 1000c2ba f i WebCommonLib:PluginInstance.obj
 0001:0000b2ef       ??$_Uninit_move@PAUWebMessage@@PAU1@V?$allocator@UWebMessage@@@std@@U1@@std@@YAPAUWebMessage@@PAU1@00AAV?$allocator@UWebMessage@@@0@0U_Nonscalar_ptr_iterator_tag@0@@Z 1000c2ef f i WebCommonLib:PluginInstance.obj
 0001:0000b359       ??$_Dest_val@V?$allocator@UWebMessage@@@std@@UWebMessage@@@std@@YAXAAV?$allocator@UWebMessage@@@0@PAUWebMessage@@@Z 1000c359 f i WebCommonLib:PluginInstance.obj
 0001:0000b37c       ?NotifyDWWM@BogusVistaDWWMNotifier@@QAEXPAUHWND__@@@Z 1000c37c f   WebCommonLib:WinWebUtils.obj
 0001:0000b3e0       ?GetTimeUSImpl@?A0x7b9a98a1@@YA_KXZ 1000c3e0 f   WebCommonLib:WinWebUtils.obj
 0001:0000b416       ?GetTimeUSImplWin7@?A0x7b9a98a1@@YA_KXZ 1000c416 f   WebCommonLib:WinWebUtils.obj
 0001:0000b436       ?InitializeGetTimeUS@?A0x7b9a98a1@@YAP6A_KXZXZ 1000c436 f   WebCommonLib:WinWebUtils.obj
 0001:0000b4a8       ?Start@UnityInstanceThread@@QAEXPAUHINSTANCE__@@AAVPluginInstance@@PAUHWND__@@HH@Z 1000c4a8 f   WebCommonLib:UnityInstanceThread.obj
 0001:0000b50a       ?Stop@UnityInstanceThread@@QAEXXZ 1000c50a f   WebCommonLib:UnityInstanceThread.obj
 0001:0000b549       ?Update@UnityInstanceThread@@QAEXPAUHWND__@@HH@Z 1000c549 f   WebCommonLib:UnityInstanceThread.obj
 0001:0000b5f5       ?SetParentInfo@UnityInstanceThread@@QAEXPAUHWND__@@HH_N@Z 1000c5f5 f   WebCommonLib:UnityInstanceThread.obj
 0001:0000b646       ?HandleForeground@UnityInstanceThread@@QAE_NXZ 1000c646 f   WebCommonLib:UnityInstanceThread.obj
 0001:0000b6a1       ?FetchExternalCalls@UnityInstanceThread@@QAE?AV?$basic_string@DU?$char_traits@D@std@@V?$allocator@D@2@@std@@XZ 1000c6a1 f   WebCommonLib:UnityInstanceThread.obj
 0001:0000b81b       ?LoadAndInitialize@UnityInstanceThread@@AAEXXZ 1000c81b f   WebCommonLib:UnityInstanceThread.obj
 0001:0000b8a7       ??$_Move@PAUWebMessage@@PAU1@@std@@YAPAUWebMessage@@PAU1@00@Z 1000c8a7 f i WebCommonLib:UnityInstanceThread.obj
 0001:0000b905       ??4VariantValue@@QAEAAU0@ABU0@@Z 1000c905 f i WebCommonLib:UnityInstanceThread.obj
 0001:0000b93f       ??_EDownload@@UAEPAXI@Z    1000c93f f i  CIL library: CIL module
 0001:0000b93f       ??_GDownload@@UAEPAXI@Z    1000c93f f i WebCommonLib:Download.obj
 0001:0000b93f       ??_GDownloaderNetscape@@UAEPAXI@Z 1000c93f f i DownloadNetscape.obj
 0001:0000b93f       ??_EDownloaderNetscape@@UAEPAXI@Z 1000c93f f i  CIL library: CIL module
 0001:0000b95e       ??1Download@@UAE@XZ        1000c95e f   WebCommonLib:Download.obj
 0001:0000b993       ?Append@Download@@QAEXPBXI@Z 1000c993 f   WebCommonLib:Download.obj
 0001:0000ba1f       ?HandleExternalDownloadComplete@Download@@QAEXXZ 1000ca1f f   WebCommonLib:Download.obj
 0001:0000ba3f       ?Parse@Color@progress@@QAE_NPBD@Z 1000ca3f f   WebCommonLib:ProgressDisplay.obj
 0001:0000bae4       ??1Setup@progress@@QAE@XZ  1000cae4 f   WebCommonLib:ProgressDisplay.obj
 0001:0000bb1b       ??0RequiredBundleRevision@@QAE@W4BundleID@@@Z 1000cb1b f i WebCommonLib:RevisionsQuery.obj
 0001:0000bb83       ??1RequiredBundleRevision@@QAE@XZ 1000cb83 f i WebCommonLib:RevisionsQuery.obj
 0001:0000bbc1       ?GetTime@@YA_KXZ           1000cbc1 f   WebCommonLib:RevisionsQuery.obj
 0001:0000bbcf       ?GetRevisionsRequestTimeout@?A0xf6e77619@@YAHXZ 1000cbcf f   WebCommonLib:RevisionsQuery.obj
 0001:0000bbed       ?DefaultAutoUpdateURL@@YA?AV?$basic_string@DU?$char_traits@D@std@@V?$allocator@D@2@@std@@W4AutoUpdateURL@@@Z 1000cbed f   WebCommonLib:RevisionsQuery.obj
 0001:0000bca7       ??0RevisionsQuery@@QAE@XZ  1000cca7 f   WebCommonLib:RevisionsQuery.obj
 0001:0000bdd1       ??1RevisionsQuery@@QAE@XZ  1000cdd1 f   WebCommonLib:RevisionsQuery.obj
 0001:0000be54       ?Tick@RevisionsQuery@@QAEXAAUUnityWebStreamHeader@@@Z 1000ce54 f   WebCommonLib:RevisionsQuery.obj
 0001:0000c282       ?URLEscape@@YA?AV?$basic_string@DU?$char_traits@D@std@@V?$allocator@D@2@@std@@ABV12@@Z 1000d282 f   WebCommonLib:RevisionsQuery.obj
 0001:0000c376       ?PluginStartDownloadingData@RevisionsQuery@@QAEXABV?$basic_string@DU?$char_traits@D@std@@V?$allocator@D@2@@std@@00@Z 1000d376 f   WebCommonLib:RevisionsQuery.obj
 0001:0000c71c       ?ValidatePlayerHash@RevisionsQuery@@QAE?AW4PlayerHashValidationResult@@ABV?$basic_string@DU?$char_traits@D@std@@V?$allocator@D@2@@std@@PBEI@Z 1000d71c f   WebCommonLib:RevisionsQuery.obj
 0001:0000cb66       ?UpdateRequiredPlayerVersion@RevisionsQuery@@AAEXAAURequiredBundleRevision@@ABUUnityWebStreamHeader@@@Z 1000db66 f   WebCommonLib:RevisionsQuery.obj
 0001:0000cc99       ?UpdateDownloadBundleRevisionIfNeeded@RequiredBundleRevision@@QAEXAAVRevisionsQuery@@@Z 1000dc99 f   WebCommonLib:RevisionsQuery.obj
 0001:0000d14f       ?IsReadyToLoad@RequiredBundleRevision@@QBE_NAAVRevisionsQuery@@@Z 1000e14f f   WebCommonLib:RevisionsQuery.obj
 0001:0000d216       ?UpdateRequiredMonoVersion@RevisionsQuery@@AAEXAAURequiredBundleRevision@@0@Z 1000e216 f   WebCommonLib:RevisionsQuery.obj
 0001:0000d67d       ?GetMinMaxRequiredRevision@RevisionsQuery@@QAE_NW4BundleID@@ABV?$basic_string@DU?$char_traits@D@std@@V?$allocator@D@2@@std@@PAV34@2PAH3@Z 1000e67d f   WebCommonLib:RevisionsQuery.obj
 0001:0000d730       ?GetMinMaxRequiredRevisionInternal@RevisionsQuery@@AAEXW4BundleID@@ABV?$basic_string@DU?$char_traits@D@std@@V?$allocator@D@2@@std@@AAVMiniXMLFile@@PAV34@3PAH4@Z 1000e730 f   WebCommonLib:RevisionsQuery.obj
 0001:0000da72       ?GetAutoUpdateURL@RevisionsQuery@@QAE?BV?$basic_string@DU?$char_traits@D@std@@V?$allocator@D@2@@std@@W4AutoUpdateURL@@_N@Z 1000ea72 f   WebCommonLib:RevisionsQuery.obj
 0001:0000db43       ?SetAutoUpdateURL@RevisionsQuery@@QAEXABV?$basic_string@DU?$char_traits@D@std@@V?$allocator@D@2@@std@@@Z 1000eb43 f   WebCommonLib:RevisionsQuery.obj
 0001:0000dc64       ?VerifyAutoUpdateURL@RevisionsQuery@@QAEXXZ 1000ec64 f   WebCommonLib:RevisionsQuery.obj
 0001:0000de23       ?replace@?$basic_string@DU?$char_traits@D@std@@V?$allocator@D@2@@std@@QAEAAV12@IIPBDI@Z 1000ee23 f i WebCommonLib:RevisionsQuery.obj
 0001:0000df58       ?insert@?$basic_string@DU?$char_traits@D@std@@V?$allocator@D@2@@std@@QAEAAV12@IID@Z 1000ef58 f i WebCommonLib:RevisionsQuery.obj
 0001:0000dfe8       ??$_Buynode@V?$basic_string@DU?$char_traits@D@std@@V?$allocator@D@2@@std@@@?$_Tree_val@V?$_Tset_traits@V?$basic_string@DU?$char_traits@D@std@@V?$allocator@D@2@@std@@U?$less@V?$basic_string@DU?$char_traits@D@std@@V?$allocator@D@2@@std@@@2@V?$allocator@V?$basic_string@DU?$char_traits@D@std@@V?$allocator@D@2@@std@@@2@$0A@@std@@@std@@QAEPAU_Node@?$_Tree_nod@V?$_Tset_traits@V?$basic_string@DU?$char_traits@D@std@@V?$allocator@D@2@@std@@U?$less@V?$basic_string@DU?$char_traits@D@std@@V?$allocator@D@2@@std@@@2@V?$allocator@V?$basic_string@DU?$char_traits@D@std@@V?$allocator@D@2@@std@@@2@$0A@@std@@@1@$$QAV?$basic_string@DU?$char_traits@D@std@@V?$allocator@D@2@@1@@Z 1000efe8 f i WebCommonLib:RevisionsQuery.obj
 0001:0000e059       ?GetCustomLogLocation@@YAPBDPBD@Z 1000f059 f   WebCommonLib:Logger.obj
 0001:0000e06e       ??0Logger@@QAE@ABV?$basic_string@DU?$char_traits@D@std@@V?$allocator@D@2@@std@@@Z 1000f06e f   WebCommonLib:Logger.obj
 0001:0000e10e       ?Close@Logger@@QAEXXZ      1000f10e f   WebCommonLib:Logger.obj
 0001:0000e121       ?Log@Logger@@QAAXPBDZZ     1000f121 f   WebCommonLib:Logger.obj
 0001:0000e132       ?VLog@Logger@@QAEXPBDPAD@Z 1000f132 f   WebCommonLib:Logger.obj
 0001:0000e1c9       ??0SimpleString@@QAE@PBDK@Z 1000f1c9 f   WebCommonLib:WebScripting.obj
 0001:0000e20e       ??0SimpleString@@QAE@ABU0@@Z 1000f20e f   WebCommonLib:WebScripting.obj
 0001:0000e23a       ??4SimpleString@@QAEXABU0@@Z 1000f23a f   WebCommonLib:WebScripting.obj
 0001:0000e275       ??1SimpleString@@QAE@XZ    1000f275 f   WebCommonLib:WebScripting.obj
 0001:0000e284       ??0VariantArray@VariantValue@@QAE@HPBU1@@Z 1000f284 f   WebCommonLib:WebScripting.obj
 0001:0000e301       ??_EVariantValue@@QAEPAXI@Z 1000f301 f i WebCommonLib:WebScripting.obj
 0001:0000e337       ??0VariantArray@VariantValue@@QAE@ABU01@@Z 1000f337 f   WebCommonLib:WebScripting.obj
 0001:0000e3d3       ??4VariantArray@VariantValue@@QAEXABU01@@Z 1000f3d3 f   WebCommonLib:WebScripting.obj
 0001:0000e486       ??1VariantArray@VariantValue@@QAE@XZ 1000f486 f   WebCommonLib:WebScripting.obj
 0001:0000e493       ??1MiniXMLFile@@QAE@XZ     1000f493 f   WebCommonLib:MiniXmlFile.obj
 0001:0000e4b3       ?Parse@MiniXMLFile@@QAE_NPBDI@Z 1000f4b3 f   WebCommonLib:MiniXmlFile.obj
 0001:0000e521       ?Parse@MiniXMLFile@@QAE_NABV?$basic_string@DU?$char_traits@D@std@@V?$allocator@D@2@@std@@@Z 1000f521 f   WebCommonLib:MiniXmlFile.obj
 0001:0000e627       ?GetStringValue@MiniXMLFile@@QAE?AV?$basic_string@DU?$char_traits@D@std@@V?$allocator@D@2@@std@@ABV23@PBX@Z 1000f627 f   WebCommonLib:MiniXmlFile.obj
 0001:0000e6b1       ?GetArrayCount@MiniXMLFile@@QAEHABV?$basic_string@DU?$char_traits@D@std@@V?$allocator@D@2@@std@@PBX@Z 1000f6b1 f   WebCommonLib:MiniXmlFile.obj
 0001:0000e724       ?GetArrayElementDict@MiniXMLFile@@QAEPBXABV?$basic_string@DU?$char_traits@D@std@@V?$allocator@D@2@@std@@HPBX@Z 1000f724 f   WebCommonLib:MiniXmlFile.obj
 0001:0000e79c       ?GetArrayElementString@MiniXMLFile@@QAE?AV?$basic_string@DU?$char_traits@D@std@@V?$allocator@D@2@@std@@ABV23@HPBX@Z 1000f79c f   WebCommonLib:MiniXmlFile.obj
 0001:0000e84b       ?Completed@UpdateOperation@UpdaterProxy@@SA_NABV?$ResourcePtr@VUpdateOperation@UpdaterProxy@@@@@Z 1000f84b f i WebCommonLib:UpdaterProxy.obj
 0001:0000e866       ??1UpdaterProxy@@QAE@XZ    1000f866 f i WebCommonLib:UpdaterProxy.obj
 0001:0000e922       ?Open@ServerPipe@UpdaterProxy@@QAE_NPB_WKKK@Z 1000f922 f   WebCommonLib:UpdaterProxy.obj
 0001:0000e976       ?Open@UpdateOperation@UpdaterProxy@@QAE_NABV?$Handle@PAXVFileHandleRoot@@$0PPPPPPPP@@@@Z 1000f976 f   WebCommonLib:UpdaterProxy.obj
 0001:0000e9e3       ?Close@UpdateOperation@UpdaterProxy@@QAEXXZ 1000f9e3 f   WebCommonLib:UpdaterProxy.obj
 0001:0000e9f6       ?BeginUpdate@UpdaterProxy@@QAEIPB_W_N00PAUHWND__@@1@Z 1000f9f6 f   WebCommonLib:UpdaterProxy.obj
 0001:0000edd9       ?UpdaterThread@?A0xf40a2a01@@YGKPAX@Z 1000fdd9 f   WebCommonLib:UpdaterProxy.obj
 0001:0000eeb3       ?LaunchUpdater@UpdaterProxy@@AAE_NPAUHWND__@@_N@Z 1000feb3 f   WebCommonLib:UpdaterProxy.obj
 0001:0000f1bd       ?GetUpdateStatus@UpdaterProxy@@QAE?AW4UpdateStatus@1@I@Z 100101bd f   WebCommonLib:UpdaterProxy.obj
 0001:0000f1f1       ?UpdateOperations@UpdaterProxy@@AAEXXZ 100101f1 f   WebCommonLib:UpdaterProxy.obj
 0001:0000f35e       ?Hold@?$ResourceRoot@VUpdaterProxy@@VIResource@@@@UAEXXZ 1001035e f i WebCommonLib:UpdaterProxy.obj
 0001:0000f35e       ?Hold@?$ResourceRoot@VUpdateMessage@Updater@@VIResource@@@@UAEXXZ 1001035e f i WebCommonLib:Updater.obj
 0001:0000f35e       ?Hold@?$ResourceRoot@VClientPipe@@VIResource@@@@UAEXXZ 1001035e f i WebCommonLib:Updater.obj
 0001:0000f35e       ?Hold@?$ResourceRoot@VUpdateOperation@UpdaterProxy@@VIResource@@@@UAEXXZ 1001035e f i WebCommonLib:UpdaterProxy.obj
 0001:0000f35e       ?Hold@?$ResourceRoot@VServerPipe@UpdaterProxy@@VIResource@@@@UAEXXZ 1001035e f i WebCommonLib:UpdaterProxy.obj
 0001:0000f362       ?Release@?$ResourceRoot@VUpdaterProxy@@VIResource@@@@UAEXXZ 10010362 f i WebCommonLib:UpdaterProxy.obj
 0001:0000f378       ?Release@?$ResourceRoot@VServerPipe@UpdaterProxy@@VIResource@@@@UAEXXZ 10010378 f i WebCommonLib:UpdaterProxy.obj
 0001:0000f378       ?Release@?$ResourceRoot@VClientPipe@@VIResource@@@@UAEXXZ 10010378 f i WebCommonLib:Updater.obj
 0001:0000f39c       ?Release@?$ResourceRoot@VUpdateOperation@UpdaterProxy@@VIResource@@@@UAEXXZ 1001039c f i WebCommonLib:UpdaterProxy.obj
 0001:0000f3b8       ?clear@?$list@V?$ResourcePtr@VUpdateOperation@UpdaterProxy@@@@V?$allocator@V?$ResourcePtr@VUpdateOperation@UpdaterProxy@@@@@std@@@std@@QAEXXZ 100103b8 f i WebCommonLib:UpdaterProxy.obj
 0001:0000f3ef       ?_Buynode@?$_List_val@V?$ResourcePtr@VUpdateOperation@UpdaterProxy@@@@V?$allocator@V?$ResourcePtr@VUpdateOperation@UpdaterProxy@@@@@std@@@std@@QAEPAU_Node@?$_List_nod@V?$ResourcePtr@VUpdateOperation@UpdaterProxy@@@@V?$allocator@V?$ResourcePtr@VUpdateOperation@UpdaterProxy@@@@@std@@@2@PAU342@0ABV?$ResourcePtr@VUpdateOperation@UpdaterProxy@@@@@Z 100103ef f i WebCommonLib:UpdaterProxy.obj
 0001:0000f45a       ?allocate@?$allocator@U_Node@?$_List_nod@V?$ResourcePtr@VUpdateOperation@UpdaterProxy@@@@V?$allocator@V?$ResourcePtr@VUpdateOperation@UpdaterProxy@@@@@std@@@std@@@std@@QAEPAU_Node@?$_List_nod@V?$ResourcePtr@VUpdateOperation@UpdaterProxy@@@@V?$allocator@V?$ResourcePtr@VUpdateOperation@UpdaterProxy@@@@@std@@@2@I@Z 1001045a f i WebCommonLib:UpdaterProxy.obj
 0001:0000f492       ?allocate@?$allocator@U_Node@?$_Tree_nod@V?$_Tmap_traits@IW4UpdateStatus@UpdaterProxy@@U?$less@I@std@@V?$allocator@U?$pair@$$CBIW4UpdateStatus@UpdaterProxy@@@std@@@4@$0A@@std@@@std@@@std@@QAEPAU_Node@?$_Tree_nod@V?$_Tmap_traits@IW4UpdateStatus@UpdaterProxy@@U?$less@I@std@@V?$allocator@U?$pair@$$CBIW4UpdateStatus@UpdaterProxy@@@std@@@4@$0A@@std@@@2@I@Z 10010492 f i WebCommonLib:UpdaterProxy.obj
 0001:0000f492       ?allocate@?$allocator@U_Node@?$_Tree_nod@V?$_Tmap_traits@KPAVTimer@?A0xa59a0aab@@U?$less@K@std@@V?$allocator@U?$pair@$$CBKPAVTimer@?A0xa59a0aab@@@std@@@4@$0A@@std@@@std@@@std@@QAEPAU_Node@?$_Tree_nod@V?$_Tmap_traits@KPAVTimer@?A0xa59a0aab@@U?$less@K@std@@V?$allocator@U?$pair@$$CBKPAVTimer@?A0xa59a0aab@@@std@@@4@$0A@@std@@@2@I@Z 10010492 f i WebCommonLib:PluginManager.obj
 0001:0000f492       ?allocate@?$allocator@U_Node@?$_Tree_nod@V?$_Tmap_traits@IPAVDownloaderNetscape@@U?$less@I@std@@V?$allocator@U?$pair@$$CBIPAVDownloaderNetscape@@@std@@@3@$0A@@std@@@std@@@std@@QAEPAU_Node@?$_Tree_nod@V?$_Tmap_traits@IPAVDownloaderNetscape@@U?$less@I@std@@V?$allocator@U?$pair@$$CBIPAVDownloaderNetscape@@@std@@@3@$0A@@std@@@2@I@Z 10010492 f i DownloadNetscape.obj
 0001:0000f492       ?allocate@?$allocator@U_Node@?$_Tree_nod@V?$_Tmap_traits@PAVDownload@@PAU_NPStream@@U?$less@PAVDownload@@@std@@V?$allocator@U?$pair@QAVDownload@@PAU_NPStream@@@std@@@4@$0A@@std@@@std@@@std@@QAEPAU_Node@?$_Tree_nod@V?$_Tmap_traits@PAVDownload@@PAU_NPStream@@U?$less@PAVDownload@@@std@@V?$allocator@U?$pair@QAVDownload@@PAU_NPStream@@@std@@@4@$0A@@std@@@2@I@Z 10010492 f i DownloadNetscape.obj
 0001:0000f4ca       ?Write@?$PipeRoot@VServerPipe@UpdaterProxy@@@@QAE?AW4Result@1@PBXKK@Z 100104ca f i WebCommonLib:UpdaterProxy.obj
 0001:0000f578       ?_Linsert@?$_Tree@V?$_Tmap_traits@IW4UpdateStatus@UpdaterProxy@@U?$less@I@std@@V?$allocator@U?$pair@$$CBIW4UpdateStatus@UpdaterProxy@@@std@@@4@$0A@@std@@@std@@QAE?AU?$pair@V?$_Tree_iterator@V?$_Tree_val@V?$_Tmap_traits@IW4UpdateStatus@UpdaterProxy@@U?$less@I@std@@V?$allocator@U?$pair@$$CBIW4UpdateStatus@UpdaterProxy@@@std@@@4@$0A@@std@@@std@@@std@@_N@2@PAU_Node@?$_Tree_nod@V?$_Tmap_traits@IW4UpdateStatus@UpdaterProxy@@U?$less@I@std@@V?$allocator@U?$pair@$$CBIW4UpdateStatus@UpdaterProxy@@@std@@@4@$0A@@std@@@2@_N@Z 10010578 f i WebCommonLib:UpdaterProxy.obj
 0001:0000f578       ?_Linsert@?$_Tree@V?$_Tmap_traits@KPAVTimer@?A0xa59a0aab@@U?$less@K@std@@V?$allocator@U?$pair@$$CBKPAVTimer@?A0xa59a0aab@@@std@@@4@$0A@@std@@@std@@QAE?AU?$pair@V?$_Tree_iterator@V?$_Tree_val@V?$_Tmap_traits@KPAVTimer@?A0xa59a0aab@@U?$less@K@std@@V?$allocator@U?$pair@$$CBKPAVTimer@?A0xa59a0aab@@@std@@@4@$0A@@std@@@std@@@std@@_N@2@PAU_Node@?$_Tree_nod@V?$_Tmap_traits@KPAVTimer@?A0xa59a0aab@@U?$less@K@std@@V?$allocator@U?$pair@$$CBKPAVTimer@?A0xa59a0aab@@@std@@@4@$0A@@std@@@2@_N@Z 10010578 f i WebCommonLib:PluginManager.obj
 0001:0000f63e       ?_Insert@?$_Tree@V?$_Tmap_traits@IW4UpdateStatus@UpdaterProxy@@U?$less@I@std@@V?$allocator@U?$pair@$$CBIW4UpdateStatus@UpdaterProxy@@@std@@@4@$0A@@std@@@std@@IAE?AV?$_Tree_iterator@V?$_Tree_val@V?$_Tmap_traits@IW4UpdateStatus@UpdaterProxy@@U?$less@I@std@@V?$allocator@U?$pair@$$CBIW4UpdateStatus@UpdaterProxy@@@std@@@4@$0A@@std@@@std@@@2@_NPAU_Node@?$_Tree_nod@V?$_Tmap_traits@IW4UpdateStatus@UpdaterProxy@@U?$less@I@std@@V?$allocator@U?$pair@$$CBIW4UpdateStatus@UpdaterProxy@@@std@@@4@$0A@@std@@@2@1@Z 1001063e f i WebCommonLib:UpdaterProxy.obj
 0001:0000f63e       ?_Insert@?$_Tree@V?$_Tmap_traits@KPAVTimer@?A0xa59a0aab@@U?$less@K@std@@V?$allocator@U?$pair@$$CBKPAVTimer@?A0xa59a0aab@@@std@@@4@$0A@@std@@@std@@IAE?AV?$_Tree_iterator@V?$_Tree_val@V?$_Tmap_traits@KPAVTimer@?A0xa59a0aab@@U?$less@K@std@@V?$allocator@U?$pair@$$CBKPAVTimer@?A0xa59a0aab@@@std@@@4@$0A@@std@@@std@@@2@_NPAU_Node@?$_Tree_nod@V?$_Tmap_traits@KPAVTimer@?A0xa59a0aab@@U?$less@K@std@@V?$allocator@U?$pair@$$CBKPAVTimer@?A0xa59a0aab@@@std@@@4@$0A@@std@@@2@1@Z 1001063e f i WebCommonLib:PluginManager.obj
 0001:0000f757       ??0UnityLoader@@QAE@AAVPluginInstance@@@Z 10010757 f   WebCommonLib:UnityLoader.obj
 0001:0000f883       ?Load@UnityLoader@@QAE_NPAUHINSTANCE__@@AAV?$basic_string@DU?$char_traits@D@std@@V?$allocator@D@2@@std@@@Z 10010883 f   WebCommonLib:UnityLoader.obj
 0001:0000fa73       ?CopyToTempPath@UnityLoader@@AAE_NAAV?$basic_string@DU?$char_traits@D@std@@V?$allocator@D@2@@std@@@Z 10010a73 f   WebCommonLib:UnityLoader.obj
 0001:0000fd27       ?LoadUnityDLL@UnityLoader@@AAE_NAAV?$basic_string@DU?$char_traits@D@std@@V?$allocator@D@2@@std@@@Z 10010d27 f   WebCommonLib:UnityLoader.obj
 0001:0000ff31       ??1UnityLoader@@QAE@XZ     10010f31 f   WebCommonLib:UnityLoader.obj
 0001:0001000a       ?GetHomePath@@YA?AV?$basic_string@DU?$char_traits@D@std@@V?$allocator@D@2@@std@@PAUHKEY__@@@Z 1001100a f   WebCommonLib:Pluginfor360Browser.obj
 0001:00010083       ?UseGreenVersionfor360Browser@@YA_NXZ 10011083 f   WebCommonLib:Pluginfor360Browser.obj
 0001:00010129       ?ConvertUnityPathName@@YAXPBDPA_WH@Z 10011129 f   WebCommonLib:PathUnicodeConversion.obj
 0001:0001015c       ?GetGlobalPreference@@YA?AV?$basic_string@DU?$char_traits@D@std@@V?$allocator@D@2@@std@@PBD@Z 1001115c f   WebCommonLib:GlobalPreferences.obj
 0001:000101df       ?SetGlobalPreference@@YAXPBDV?$basic_string@DU?$char_traits@D@std@@V?$allocator@D@2@@std@@@Z 100111df f   WebCommonLib:GlobalPreferences.obj
 0001:00010298       ?fopen_inmem_func@@YAPAXPAXPBDH@Z 10011298 f   WebCommonLib:Decompressor.obj
 0001:000102a4       ?fread_inmem_func@@YAKPAX00K@Z 100112a4 f   WebCommonLib:Decompressor.obj
 0001:000102de       ?ftell_inmem_func@@YAJPAX0@Z 100112de f   WebCommonLib:Decompressor.obj
 0001:000102e9       ?fseek_inmem_func@@YAJPAX0KH@Z 100112e9 f   WebCommonLib:Decompressor.obj
 0001:0001033d       ?fclose_inmem_func@@YAHPAX0@Z 1001133d f   WebCommonLib:Decompressor.obj
 0001:0001034b       ?ferror_inmem_func@@YAHPAX0@Z 1001134b f   WebCommonLib:Decompressor.obj
 0001:0001034b       ?fwrite_inmem_func@@YAKPAX0PBXK@Z 1001134b f   WebCommonLib:Decompressor.obj
 0001:0001034b       __matherr                  1001134b f   LIBCMT:_matherr_.obj
 0001:0001053d       ?Decompress@decomp@@YA_NPBXIABV?$basic_string@DU?$char_traits@D@std@@V?$allocator@D@2@@std@@@Z 1001153d f   WebCommonLib:Decompressor.obj
 0001:00010618       ?CreateFolderWide@fileutils@@YA_NABV?$basic_string@_WU?$char_traits@_W@std@@V?$allocator@_W@2@@std@@@Z 10011618 f   WebCommonLib:WebFileUtilities.obj
 0001:00010693       ?CreateFolder@fileutils@@YA_NABV?$basic_string@DU?$char_traits@D@std@@V?$allocator@D@2@@std@@@Z 10011693 f   WebCommonLib:WebFileUtilities.obj
 0001:000106ec       ?CreateFolderRecursive@fileutils@@YA_NABV?$basic_string@DU?$char_traits@D@std@@V?$allocator@D@2@@std@@@Z 100116ec f   WebCommonLib:WebFileUtilities.obj
 0001:000107b4       ?GetBaseTempFolder@fileutils@@YA?AV?$basic_string@DU?$char_traits@D@std@@V?$allocator@D@2@@std@@XZ 100117b4 f   WebCommonLib:WebFileUtilities.obj
 0001:00010830       ?RemoveFolderRecursiveWide@fileutils@@YA_NABV?$basic_string@_WU?$char_traits@_W@std@@V?$allocator@_W@2@@std@@@Z 10011830 f   WebCommonLib:WebFileUtilities.obj
 0001:00010a3f       ?RemoveFolderRecursive@fileutils@@YA_NABV?$basic_string@DU?$char_traits@D@std@@V?$allocator@D@2@@std@@_N@Z 10011a3f f   WebCommonLib:WebFileUtilities.obj
 0001:00010a9a       ?find@?$basic_string@_WU?$char_traits@_W@std@@V?$allocator@_W@2@@std@@QBEIPB_WII@Z 10011a9a f i WebCommonLib:WebFileUtilities.obj
 0001:00010b46       ??$?H_WU?$char_traits@_W@std@@V?$allocator@_W@1@@std@@YA?AV?$basic_string@_WU?$char_traits@_W@std@@V?$allocator@_W@2@@0@ABV10@_W@Z 10011b46 f i WebCommonLib:WebFileUtilities.obj
 0001:00010b8b       ??$?H_WU?$char_traits@_W@std@@V?$allocator@_W@1@@std@@YA?AV?$basic_string@_WU?$char_traits@_W@std@@V?$allocator@_W@2@@0@ABV10@PB_W@Z 10011b8b f i WebCommonLib:WebFileUtilities.obj
 0001:00010be4       ?reserve@?$basic_string@_WU?$char_traits@_W@std@@V?$allocator@_W@2@@std@@QAEXI@Z 10011be4 f i WebCommonLib:WebFileUtilities.obj
 0001:00010c1d       ?append@?$basic_string@_WU?$char_traits@_W@std@@V?$allocator@_W@2@@std@@QAEAAV12@ABV12@II@Z 10011c1d f i WebCommonLib:WebFileUtilities.obj
 0001:00010cc0       ?append@?$basic_string@_WU?$char_traits@_W@std@@V?$allocator@_W@2@@std@@QAEAAV12@PB_WI@Z 10011cc0 f i WebCommonLib:WebFileUtilities.obj
 0001:00010d61       ?UTF8ToWide@@YAXPBDPA_WH@Z 10011d61 f   WebCommonLib:WinUnicode.obj
 0001:00010e6a       ?AppendPathName@@YA?AV?$basic_string@DU?$char_traits@D@std@@V?$allocator@D@2@@std@@ABV12@0@Z 10011e6a f   WebCommonLib:PathNameUtility.obj
 0001:00010e82       ?append@?$basic_string@DU?$char_traits@D@std@@V?$allocator@D@2@@std@@QAEAAV12@V?$_String_const_iterator@DU?$char_traits@D@std@@V?$allocator@D@2@@2@0@Z 10011e82 f i WebCommonLib:PathNameUtility.obj
 0001:00010f6d       ??$_Assign@PBE@?$basic_string@DU?$char_traits@D@std@@V?$allocator@D@2@@std@@QAEAAV01@PBE0Uinput_iterator_tag@1@@Z 10011f6d f i WebCommonLib:UnityWebStreamHeader.obj
 0001:00010ff4       ??$_Construct@PBE@?$basic_string@DU?$char_traits@D@std@@V?$allocator@D@2@@std@@QAEXPBE0Uforward_iterator_tag@1@@Z 10011ff4 f i WebCommonLib:UnityWebStreamHeader.obj
 0001:0001105d       ?VerifySignature@@YA_NV?$basic_string@DU?$char_traits@D@std@@V?$allocator@D@2@@std@@0H@Z 1001205d f   WebCommonLib:Verification.obj
 0001:00011235       ?GenerateHash@@YA?AV?$basic_string@DU?$char_traits@D@std@@V?$allocator@D@2@@std@@PBEI@Z 10012235 f   WebCommonLib:Verification.obj
 0001:00011359       _ezxml_child               10012359 f   WebCommonLib:ezxml.obj
 0001:00011384       _ezxml_err                 10012384 f   WebCommonLib:ezxml.obj
 0001:000113d4       _ezxml_decode              100123d4 f   WebCommonLib:ezxml.obj
 0001:00011694       _ezxml_open_tag            10012694 f   WebCommonLib:ezxml.obj
 0001:000116c6       _ezxml_char_content        100126c6 f   WebCommonLib:ezxml.obj
 0001:00011788       _ezxml_close_tag           10012788 f   WebCommonLib:ezxml.obj
 0001:000117cd       _ezxml_ent_ok              100127cd f   WebCommonLib:ezxml.obj
 0001:00011861       _ezxml_proc_inst           10012861 f   WebCommonLib:ezxml.obj
 0001:00011a4e       _ezxml_internal_dtd        10012a4e f   WebCommonLib:ezxml.obj
 0001:00011f84       _ezxml_str2utf8            10012f84 f   WebCommonLib:ezxml.obj
 0001:0001213d       _ezxml_free_attr           1001313d f   WebCommonLib:ezxml.obj
 0001:000121a9       _ezxml_parse_str           100131a9 f   WebCommonLib:ezxml.obj
 0001:00012881       _ezxml_free                10013881 f   WebCommonLib:ezxml.obj
 0001:000129e9       _ezxml_add_child           100139e9 f   WebCommonLib:ezxml.obj
 0001:00012af5       ?Initialize@Updater@@QAE_NXZ 10013af5 f   WebCommonLib:Updater.obj
 0001:00012c97       ?Connect@Updater@@QAE_NPB_W@Z 10013c97 f   WebCommonLib:Updater.obj
 0001:00012db9       ?Run@Updater@@QAEHXZ       10013db9 f   WebCommonLib:Updater.obj
 0001:00012fac       ?MessageTrampoline@Updater@@CGKPAX@Z 10013fac f   WebCommonLib:Updater.obj
 0001:00012fd7       ?OnUpdateMessage@Updater@@AAEXABUUpdateMessageHeader@@ABV?$UpdateRequestBody@$00@@@Z 10013fd7 f   WebCommonLib:Updater.obj
 0001:00013096       ?PerformUpdate@Updater@@AAE_NIABV?$UpdateRequestBody@$00@@@Z 10014096 f   WebCommonLib:Updater.obj
 0001:00013274       ?GetFileTransactionSupport@Updater@@ABE_NPB_WPAX@Z 10014274 f   WebCommonLib:Updater.obj
 0001:000132b7       ?UpdateFile@Updater@@ABE_NIPB_W0W4Flags@UpdateItem@@PAX@Z 100142b7 f   WebCommonLib:Updater.obj
 0001:000134ad       ?UpdateSubfolder@Updater@@ABE_NIPB_W0W4Flags@UpdateItem@@PAX@Z 100144ad f   WebCommonLib:Updater.obj
 0001:00013670       ?CopyFileW@Updater@@ABE_NIPB_W0KPAX@Z 10014670 f   WebCommonLib:Updater.obj
 0001:000136aa       ?MoveFileW@Updater@@ABE_NIPB_W0KPAX@Z 100146aa f   WebCommonLib:Updater.obj
 0001:000136e1       ?CreateDirectoryW@Updater@@ABE_NIPB_W_NPAX@Z 100146e1 f   WebCommonLib:Updater.obj
 0001:00013800       ?DeleteDirectory@Updater@@ABE?AW4DeleteDirectoryResult@1@IPB_WPAX@Z 10014800 f   WebCommonLib:Updater.obj
 0001:00013a26       ?Release@?$ResourceRoot@VUpdateMessage@Updater@@VIResource@@@@UAEXXZ 10014a26 f i WebCommonLib:Updater.obj
 0001:00013a44       ?Read@?$PipeRoot@VClientPipe@@@@QAE?AW4Result@1@PAXKK@Z 10014a44 f i WebCommonLib:Updater.obj
 0001:00013af0       ?Write@?$PipeRoot@VClientPipe@@@@QAE?AW4Result@1@PBXKK@Z 10014af0 f i WebCommonLib:Updater.obj
 0001:00013b9b       ??0CPUInfo@@QAE@XZ         10014b9b f   WebCommonLib:CPUInfo.obj
 0001:00013c13       ?internalGetString@?A0xa57cb415@@YA_NPAUHKEY__@@ABV?$basic_string@DU?$char_traits@D@std@@V?$allocator@D@2@@std@@1AAV34@@Z 10014c13 f   WebCommonLib:Registry.obj
 0001:00013d32       ?getString@registry@@YA?AV?$basic_string@DU?$char_traits@D@std@@V?$allocator@D@2@@std@@ABV23@00@Z 10014d32 f   WebCommonLib:Registry.obj
 0001:00013dc5       ?Open@ClientPipe@@QAE_NPB_WK_NK@Z 10014dc5 f   WebCommonLib:ClientPipe.obj
 0001:00013e4a       ??1out_of_range@std@@UAE@XZ 10014e4a f i libcpmt:xthrow.obj
 0001:00013e4a       ??1length_error@std@@UAE@XZ 10014e4a f i libcpmt:xthrow.obj
 0001:00013e4f       ??0logic_error@std@@QAE@ABV01@@Z 10014e4f f i libcpmt:xthrow.obj
 0001:00013e6c       ?_Xlength_error@std@@YAXPBD@Z 10014e6c f   libcpmt:xthrow.obj
 0001:00013e9c       ??0length_error@std@@QAE@ABV01@@Z 10014e9c f i libcpmt:xthrow.obj
 0001:00013eb9       ?_Xout_of_range@std@@YAXPBD@Z 10014eb9 f   libcpmt:xthrow.obj
 0001:00013ee9       ??0out_of_range@std@@QAE@ABV01@@Z 10014ee9 f i libcpmt:xthrow.obj
 0001:00013f06       ??_Glogic_error@std@@UAEPAXI@Z 10014f06 f i libcpmt:xthrow.obj
 0001:00013f06       ??_Glength_error@std@@UAEPAXI@Z 10014f06 f i libcpmt:xthrow.obj
 0001:00013f06       ??_Elength_error@std@@UAEPAXI@Z 10014f06 f i libcpmt:xthrow.obj
 0001:00013f06       ??_Gout_of_range@std@@UAEPAXI@Z 10014f06 f i libcpmt:xthrow.obj
 0001:00013f06       ??_Elogic_error@std@@UAEPAXI@Z 10014f06 f i libcpmt:xthrow.obj
 0001:00013f06       ??_Eout_of_range@std@@UAEPAXI@Z 10014f06 f i libcpmt:xthrow.obj
 0001:00013f27       ??_U@YAPAXI@Z              10014f27 f   libcpmt:newaop.obj
 0001:00013f32       ??2@YAPAXI@Z               10014f32 f   LIBCMT:new.obj
 0001:00013fb2       ??3@YAXPAX@Z               10014fb2 f   LIBCMT:delete.obj
 0001:00014073       ___onexitinit              10015073 f   LIBCMT:onexit.obj
 0001:000140a4       __onexit                   100150a4 f   LIBCMT:onexit.obj
 0001:000140e0       _atexit                    100150e0 f   LIBCMT:onexit.obj
 0001:000140f7       ??0exception@std@@QAE@ABQBDH@Z 100150f7 f   LIBCMT:stdexcpt.obj
 0001:00014114       ?what@exception@std@@UBEPBDXZ 10015114 f   LIBCMT:stdexcpt.obj
 0001:00014121       ?_Copy_str@exception@std@@AAEXPBD@Z 10015121 f   LIBCMT:stdexcpt.obj
 0001:00014161       ?_Tidy@exception@std@@AAEXXZ 10015161 f   LIBCMT:stdexcpt.obj
 0001:0001417f       ??0exception@std@@QAE@ABQBD@Z 1001517f f   LIBCMT:stdexcpt.obj
 0001:000141a6       ??4exception@std@@QAEAAV01@ABV01@@Z 100151a6 f   LIBCMT:stdexcpt.obj
 0001:000141db       ??1exception@std@@UAE@XZ   100151db f   LIBCMT:stdexcpt.obj
 0001:000141e6       ??_Eexception@std@@UAEPAXI@Z 100151e6 f i LIBCMT:stdexcpt.obj
 0001:000141e6       ??_Gexception@std@@UAEPAXI@Z 100151e6 f i LIBCMT:stdexcpt.obj
 0001:0001420d       ??0exception@std@@QAE@ABV01@@Z 1001520d f   LIBCMT:stdexcpt.obj
 0001:00014232       ??1type_info@@UAE@XZ       10015232 f   LIBCMT:typinfo.obj
 0001:00014242       ??_Gtype_info@@UAEPAXI@Z   10015242 f i LIBCMT:typinfo.obj
 0001:00014242       ??_Etype_info@@UAEPAXI@Z   10015242 f i LIBCMT:typinfo.obj
 0001:00014263       ??8type_info@@QBE_NABV0@@Z 10015263 f   LIBCMT:typinfo.obj
 0001:00014290       _memcpy                    10015290 f   LIBCMT:memcpy.obj
 0001:00014600       _memmove                   10015600 f   LIBCMT:memmove.obj
 0001:00014961       _wcslen                    10015961 f   LIBCMT:wcslen.obj
 0001:00014980       _strlen                    10015980 f   LIBCMT:strlen.obj
 0001:00014a10       _strstr                    10015a10 f   LIBCMT:strstr.obj
 0001:00014a96       _memcmp                    10015a96 f   LIBCMT:memcmp.obj
 0001:00015ff0       _memset                    10016ff0 f   LIBCMT:memset.obj
 0001:0001606a       ??0_LocaleUpdate@@QAE@PAUlocaleinfo_struct@@@Z 1001706a f i LIBCMT:stricmp.obj
 0001:000160f1       ___ascii_stricmp           100170f1 f   LIBCMT:stricmp.obj
 0001:0001612a       __stricmp_l                1001712a f   LIBCMT:stricmp.obj
 0001:000161ea       __stricmp                  100171ea f   LIBCMT:stricmp.obj
 0001:00016231       ??_V@YAXPAX@Z              10017231 f   LIBCMT:delete2.obj
 0001:00016240       _memchr                    10017240 f   LIBCMT:memchr.obj
 0001:000162ed       _printf                    100172ed f   LIBCMT:printf.obj
 0001:00016394       __get_printf_count_output  10017394 f   LIBCMT:printf.obj
 0001:000163aa       __CRT_INIT@12              100173aa f   LIBCMT:dllcrt0.obj
 0001:00016604       __DllMainCRTStartup@12     10017604 f   LIBCMT:dllcrt0.obj
 0001:00016627       __wcsnicmp_l               10017627 f   LIBCMT:wcsnicmp.obj
 0001:0001670c       __wcsnicmp                 1001770c f   LIBCMT:wcsnicmp.obj
 0001:000167aa       __snprintf                 100177aa f   LIBCMT:snprintf.obj
 0001:00016856       __vsnprintf_l              10017856 f   LIBCMT:vsnprint.obj
 0001:00016902       __vsnprintf                10017902 f   LIBCMT:vsnprint.obj
 0001:0001691f       __getenv_helper_nolock     1001791f f   LIBCMT:getenv.obj
 0001:000169a6       _getenv                    100179a6 f   LIBCMT:getenv.obj
 0001:00016a20       ??_U@YAPAXIABUnothrow_t@std@@@Z 10017a20 f   LIBCMT:newaopnt.obj
 0001:00016a2b       _free                      10017a2b f   LIBCMT:free.obj
 0001:00016a65       _calloc                    10017a65 f   LIBCMT:calloc.obj
 0001:00016ab0       _strcpy                    10017ab0 f   LIBCMT:strcat.obj
 0001:00016ac0       _strcat                    10017ac0 f   LIBCMT:strcat.obj
 0001:00016ba8       __tolower_l                10017ba8 f   LIBCMT:tolower.obj
 0001:00016cbd       _tolower                   10017cbd f   LIBCMT:tolower.obj
 0001:00016ce9       _atol                      10017ce9 f   LIBCMT:atox.obj
 0001:00016cff       _atoi                      10017cff f   LIBCMT:atox.obj
 0001:00016d0a       __flush                    10017d0a f   LIBCMT:fflush.obj
 0001:00016d72       __fflush_nolock            10017d72 f   LIBCMT:fflush.obj
 0001:00016e94       _fflush                    10017e94 f   LIBCMT:fflush.obj
 0001:00016ee7       __flushall                 10017ee7 f   LIBCMT:fflush.obj
 0001:00016ef0       __wfsopen                  10017ef0 f   LIBCMT:wfopen.obj
 0001:00016fae       __wfopen                   10017fae f   LIBCMT:wfopen.obj
 0001:00016fc5       _fprintf                   10017fc5 f   LIBCMT:fprintf.obj
 0001:000170d1       __localtime64_s            100180d1 f   LIBCMT:loctim64.obj
 0001:00017359       __localtime64              10018359 f   LIBCMT:loctim64.obj
 0001:00017380       __fclose_nolock            10018380 f   LIBCMT:fclose.obj
 0001:000173ed       _fclose                    100183ed f   LIBCMT:fclose.obj
 0001:00017461       __time64                   10018461 f   LIBCMT:time64.obj
 0001:000174b2       __fread_nolock_s           100184b2 f   LIBCMT:fread.obj
 0001:0001766e       _fread_s                   1001866e f   LIBCMT:fread.obj
 0001:000176fc       _fread                     100186fc f   LIBCMT:fread.obj
 0001:00017720       _strcmp                    10018720 f   LIBCMT:strcmp.obj
 0001:000177a8       __ftell_nolock             100187a8 f   LIBCMT:ftell.obj
 0001:0001793c       _ftell                     1001893c f   LIBCMT:ftell.obj
 0001:000179a1       __fseek_nolock             100189a1 f   LIBCMT:fseek.obj
 0001:00017a2b       _fseek                     10018a2b f   LIBCMT:fseek.obj
 0001:00017aa7       _wcscpy_s                  10018aa7 f   LIBCMT:wcscpy_s.obj
 0001:00017b0a       _wcsstr                    10018b0a f   LIBCMT:wcsstr.obj
 0001:00017b6a       __fwrite_nolock            10018b6a f   LIBCMT:fwrite.obj
 0001:00017cc1       _fwrite                    10018cc1 f   LIBCMT:fwrite.obj
 0001:00017d3b       _wcscmp                    10018d3b f   LIBCMT:wcscmp.obj
 0001:00017d79       _sprintf                   10018d79 f   LIBCMT:sprintf.obj
 0001:00017dfd       _malloc                    10018dfd f   LIBCMT:malloc.obj
 0001:00017e91       _strncmp                   10018e91 f   LIBCMT:strncmp.obj
 0001:00017f51       __isalpha_l                10018f51 f i LIBCMT:_ctype.obj
 0001:00017fa7       _isalpha                   10018fa7 f i LIBCMT:_ctype.obj
 0001:00017fd7       __isdigit_l                10018fd7 f i LIBCMT:_ctype.obj
 0001:00018028       _isdigit                   10019028 f i LIBCMT:_ctype.obj
 0001:00018056       __isspace_l                10019056 f i LIBCMT:_ctype.obj
 0001:000180a7       _isspace                   100190a7 f i LIBCMT:_ctype.obj
 0001:000180f0       _strchr                    100190f0 f   LIBCMT:strchr.obj
 0001:000180f6       ___from_strstr_to_strchr   100190f6     LIBCMT:strchr.obj
 0001:000183d9       _strtol                    100193d9 f   LIBCMT:strtol.obj
 0001:00018410       _strncpy                   10019410 f   LIBCMT:strncpy.obj
 0001:00018534       __strdup                   10019534 f   LIBCMT:strdup.obj
 0001:00018590       _strspn                    10019590 f   LIBCMT:strspn.obj
 0001:000185e0       _strcspn                   100195e0 f   LIBCMT:strcspn.obj
 0001:00018626       _realloc                   10019626 f   LIBCMT:realloc.obj
 0001:000186d3       __CxxThrowException@8      100196d3 f   LIBCMT:throw.obj
 0001:0001871f       __initp_heap_handler       1001971f f   LIBCMT:handler.obj
 0001:0001872e       __callnewh                 1001972e f   LIBCMT:handler.obj
 0001:00018756       __malloc_crt               10019756 f   LIBCMT:crtheap.obj
 0001:0001879b       __calloc_crt               1001979b f   LIBCMT:crtheap.obj
 0001:000187e7       __realloc_crt              100197e7 f   LIBCMT:crtheap.obj
 0001:00018835       __recalloc_crt             10019835 f   LIBCMT:crtheap.obj
 0001:00018887       __msize                    10019887 f   LIBCMT:msize.obj
 0001:000188ba       ___crtCorExitProcess       100198ba f   LIBCMT:crt0dat.obj
 0001:000188e5       ___crtExitProcess          100198e5 f   LIBCMT:crt0dat.obj
 0001:000188fd       __lockexit                 100198fd f   LIBCMT:crt0dat.obj
 0001:00018906       __unlockexit               10019906 f   LIBCMT:crt0dat.obj
 0001:0001890f       __init_pointers            1001990f f   LIBCMT:crt0dat.obj
 0001:00018942       __initterm_e               10019942 f   LIBCMT:crt0dat.obj
 0001:00018966       __cinit                    10019966 f   LIBCMT:crt0dat.obj
 0001:00018b3d       __exit                     10019b3d f   LIBCMT:crt0dat.obj
 0001:00018b53       __cexit                    10019b53 f   LIBCMT:crt0dat.obj
 0001:00018b62       __amsg_exit                10019b62 f   LIBCMT:crt0dat.obj
 0001:00018b80       __SEH_prolog4              10019b80 f   LIBCMT:sehprolg4.obj
 0001:00018bc5       __SEH_epilog4              10019bc5 f   LIBCMT:sehprolg4.obj
 0001:00018be0       __except_handler4          10019be0 f   LIBCMT:chandler4.obj
 0001:00018d6f       _strcpy_s                  10019d6f f   LIBCMT:strcpy_s.obj
 0001:00018dce       ?_Type_info_dtor@type_info@@CAXPAV1@@Z 10019dce f   LIBCMT:typname.obj
 0001:00018e3e       __VEC_memcpy               10019e3e f   LIBCMT:p4_memcpy.obj
 0001:00018f41       ___sse2_available_init     10019f41 f   LIBCMT:cpu_disp.obj
 0001:00018f51       __initp_misc_invarg        10019f51 f   LIBCMT:invarg.obj
 0001:00018f60       __call_reportfault         10019f60 f   LIBCMT:invarg.obj
 0001:00019089       __invoke_watson            1001a089 f   LIBCMT:invarg.obj
 0001:000190ae       __invalid_parameter        1001a0ae f   LIBCMT:invarg.obj
 0001:000190db       __invalid_parameter_noinfo 1001a0db f   LIBCMT:invarg.obj
 0001:000190eb       __get_errno_from_oserr     1001a0eb f   LIBCMT:dosmap.obj
 0001:0001912d       __errno                    1001a12d f   LIBCMT:dosmap.obj
 0001:00019140       ___doserrno                1001a140 f   LIBCMT:dosmap.obj
 0001:00019153       __dosmaperr                1001a153 f   LIBCMT:dosmap.obj
 0001:00019176       _abort                     1001a176 f   LIBCMT:abort.obj
 0001:000191a9       __GET_RTERRMSG             1001a1a9 f   LIBCMT:crt0msg.obj
 0001:000191cf       __NMSG_WRITE               1001a1cf f   LIBCMT:crt0msg.obj
 0001:0001937e       __FF_MSGBANNER             1001a37e f   LIBCMT:crt0msg.obj
 0001:000193b7       __initp_misc_purevirt      1001a3b7 f   LIBCMT:inithelp.obj
 0001:000193c6       __VEC_memzero              1001a3c6 f   LIBCMT:p4_memset.obj
 0001:000196a3       ___updatetmbcinfo          1001a6a3 f   LIBCMT:mbctype.obj
 0001:000197c3       __setmbcp_nolock           1001a7c3 f   LIBCMT:mbctype.obj
 0001:000199ac       __setmbcp                  1001a9ac f   LIBCMT:mbctype.obj
 0001:00019b46       ___initmbctable            1001ab46 f   LIBCMT:mbctype.obj
 0001:00019b64       ___addlocaleref            1001ab64 f   LIBCMT:localref.obj
 0001:00019bf3       ___removelocaleref         1001abf3 f   LIBCMT:localref.obj
 0001:00019c8c       ___freetlocinfo            1001ac8c f   LIBCMT:localref.obj
 0001:00019dd7       __updatetlocinfoEx_nolock  1001add7 f   LIBCMT:localref.obj
 0001:00019e24       ___updatetlocinfo          1001ae24 f   LIBCMT:localref.obj
 0001:00019e9d       __encoded_null             1001ae9d f   LIBCMT:tidtable.obj
 0001:00019ea6       ___crtTlsAlloc@4           1001aea6 f   LIBCMT:tidtable.obj
 0001:00019eaf       ___set_flsgetvalue         1001aeaf f   LIBCMT:tidtable.obj
 0001:00019ee3       __mtterm                   1001aee3 f   LIBCMT:tidtable.obj
 0001:00019f20       __initptd                  1001af20 f   LIBCMT:tidtable.obj
 0001:00019fd4       __getptd_noexit            1001afd4 f   LIBCMT:tidtable.obj
 0001:0001a04d       __getptd                   1001b04d f   LIBCMT:tidtable.obj
 0001:0001a067       __freefls@4                1001b067 f   LIBCMT:tidtable.obj
 0001:0001a196       __freeptd                  1001b196 f   LIBCMT:tidtable.obj
 0001:0001a204       __mtinit                   1001b204 f   LIBCMT:tidtable.obj
 0001:0001a37f       ___iob_func                1001b37f f   LIBCMT:_file.obj
 0001:0001a385       ___initstdio               1001b385 f   LIBCMT:_file.obj
 0001:0001a436       ___endstdio                1001b436 f   LIBCMT:_file.obj
 0001:0001a456       __lock_file                1001b456 f   LIBCMT:_file.obj
 0001:0001a497       __lock_file2               1001b497 f   LIBCMT:_file.obj
 0001:0001a4c9       __unlock_file              1001b4c9 f   LIBCMT:_file.obj
 0001:0001a505       __unlock_file2             1001b505 f   LIBCMT:_file.obj
 0001:0001a534       __stbuf                    1001b534 f   LIBCMT:_sftbuf.obj
 0001:0001a5d0       __ftbuf                    1001b5d0 f   LIBCMT:_sftbuf.obj
 0001:0001a699       __output_l                 1001b699 f   LIBCMT:output.obj
 0001:0001b2a1       __ioinit                   1001c2a1 f   LIBCMT:ioinit.obj
 0001:0001b4e6       __ioterm                   1001c4e6 f   LIBCMT:ioinit.obj
 0001:0001b539       __setenvp                  1001c539 f   LIBCMT:stdenvp.obj
 0001:0001b7af       __setargv                  1001c7af f   LIBCMT:stdargv.obj
 0001:0001b86a       ___crtGetEnvironmentStringsA 1001c86a f   LIBCMT:a_env.obj
 0001:0001b901       __RTC_Initialize           1001c901 f   LIBCMT:_initsect_.obj
 0001:0001b927       __RTC_Terminate            1001c927 f   LIBCMT:_initsect_.obj
 0001:0001b94d       __heap_init                1001c94d f   LIBCMT:heapinit.obj
 0001:0001b96b       __heap_term                1001c96b f   LIBCMT:heapinit.obj
 0001:0001b97f       __XcptFilter               1001c97f f   LIBCMT:winxfltr.obj
 0001:0001bac9       ___CppXcptFilter           1001cac9 f   LIBCMT:winxfltr.obj
 0001:0001bae9       ___security_init_cookie    1001cae9 f   LIBCMT:gs_support.obj
 0001:0001bb84       __towlower_l               1001cb84 f   LIBCMT:towlower.obj
 0001:0001bc24       __flsbuf                   1001cc24 f   LIBCMT:_flsbuf.obj
 0001:0001bd88       __mbsnbicoll_l             1001cd88 f   LIBCMT:mbsnbico.obj
 0001:0001be66       __mbsnbicoll               1001ce66 f   LIBCMT:mbsnbico.obj
 0001:0001be80       ___wtomb_environ           1001ce80 f   LIBCMT:wtombenv.obj
 0001:0001bf17       __mtinitlocks              1001cf17 f   LIBCMT:mlock.obj
 0001:0001bf61       __mtdeletelocks            1001cf61 f   LIBCMT:mlock.obj
 0001:0001bfb8       __unlock                   1001cfb8 f   LIBCMT:mlock.obj
 0001:0001bfcf       __mtinitlocknum            1001cfcf f   LIBCMT:mlock.obj
 0001:0001c091       __lock                     1001d091 f   LIBCMT:mlock.obj
 0001:0001c0c4       _strnlen                   1001d0c4 f   LIBCMT:strlen_s.obj
 0001:0001c0e1       ??2@YAPAXIABUnothrow_t@std@@@Z 1001d0e1 f   LIBCMT:newopnt.obj
 0001:0001c110       __calloc_impl              1001d110 f   LIBCMT:calloc_impl.obj
 0001:0001c192       __freea                    1001d192 f i LIBCMT:a_map.obj
 0001:0001c399       ___crtLCMapStringA         1001d399 f   LIBCMT:a_map.obj
 0001:0001c3df       __isleadbyte_l             1001d3df f i LIBCMT:_wctype.obj
 0001:0001c417       _isleadbyte                1001d417 f i LIBCMT:_wctype.obj
 0001:0001c42a       __isctype_l                1001d42a f   LIBCMT:isctype.obj
 0001:0001c4e2       __write_nolock             1001d4e2 f   LIBCMT:write.obj
 0001:0001cbdf       __write                    1001dbdf f   LIBCMT:write.obj
 0001:0001ccb3       __fileno                   1001dcb3 f   LIBCMT:fileno.obj
 0001:0001ccd9       __commit                   1001dcd9 f   LIBCMT:commit.obj
 0001:0001cdb2       __wopenfile                1001ddb2 f   LIBCMT:_wopen.obj
 0001:0001d06b       __getstream                1001e06b f   LIBCMT:stream.obj
 0001:0001d1a0       __local_unwind4            1001e1a0 f   LIBCMT:exsup4.obj
 0001:0001d276       __seh_longjmp_unwind4@4    1001e276 f   LIBCMT:exsup4.obj
 0001:0001d292       @_EH4_CallFilterFunc@8     1001e292 f   LIBCMT:exsup4.obj
 0001:0001d2a9       @_EH4_TransferToHandler@8  1001e2a9 f   LIBCMT:exsup4.obj
 0001:0001d2c2       @_EH4_GlobalUnwind2@8      1001e2c2 f   LIBCMT:exsup4.obj
 0001:0001d2db       @_EH4_LocalUnwind@16       1001e2db f   LIBCMT:exsup4.obj
 0001:0001d9d3       ___tzset                   1001e9d3 f   LIBCMT:tzset.obj
 0001:0001da22       __isindst                  1001ea22 f   LIBCMT:tzset.obj
 0001:0001da63       __gmtime64_s               1001ea63 f   LIBCMT:gmtime64.obj
 0001:0001dc9c       __get_daylight             1001ec9c f   LIBCMT:timeset.obj
 0001:0001dcc9       __get_dstbias              1001ecc9 f   LIBCMT:timeset.obj
 0001:0001dcf6       __get_timezone             1001ecf6 f   LIBCMT:timeset.obj
 0001:0001dd23       ___daylight                1001ed23 f   LIBCMT:timeset.obj
 0001:0001dd29       ___dstbias                 1001ed29 f   LIBCMT:timeset.obj
 0001:0001dd2f       ___timezone                1001ed2f f   LIBCMT:timeset.obj
 0001:0001dd35       ___tzname                  1001ed35 f   LIBCMT:timeset.obj
 0001:0001dd40       __alldiv                   1001ed40 f   LIBCMT:lldiv.obj
 0001:0001ddf0       __allrem                   1001edf0 f   LIBCMT:llrem.obj
 0001:0001dea2       ___getgmtimebuf            1001eea2 f   LIBCMT:gmtime.obj
 0001:0001ded9       __close_nolock             1001eed9 f   LIBCMT:close.obj
 0001:0001df75       __close                    1001ef75 f   LIBCMT:close.obj
 0001:0001e039       __freebuf                  1001f039 f   LIBCMT:_freebuf.obj
 0001:0001e070       __aulldiv                  1001f070 f   LIBCMT:ulldiv.obj
 0001:0001e0d8       __filbuf                   1001f0d8 f   LIBCMT:_filbuf.obj
 0001:0001e1fa       __read_nolock              1001f1fa f   LIBCMT:read.obj
 0001:0001e7b1       __read                     1001f7b1 f   LIBCMT:read.obj
 0001:0001e8a7       _memcpy_s                  1001f8a7 f   LIBCMT:memcpy_s.obj
 0001:0001e91c       __lseek_nolock             1001f91c f   LIBCMT:lseek.obj
 0001:0001e991       __lseek                    1001f991 f   LIBCMT:lseek.obj
 0001:0001ea65       __recalloc                 1001fa65 f   LIBCMT:recalloc.obj
 0001:0001ead3       ?terminate@@YAXXZ          1001fad3 f   LIBCMT:hooks.obj
 0001:0001eb0c       ?unexpected@@YAXXZ         1001fb0c f   LIBCMT:hooks.obj
 0001:0001eb1f       ?_inconsistency@@YAXXZ     1001fb1f f   LIBCMT:hooks.obj
 0001:0001eb57       __initp_eh_hooks           1001fb57 f   LIBCMT:hooks.obj
 0001:0001eb68       __initp_misc_winsig        1001fb68 f   LIBCMT:winsig.obj
 0001:0001ebbd       ___get_sigabrt             1001fbbd f   LIBCMT:winsig.obj
 0001:0001ebca       _raise                     1001fbca f   LIBCMT:winsig.obj
 0001:0001ed6d       __initp_misc_rand_s        1001fd6d f   LIBCMT:rand_s.obj
 0001:0001ed7c       __initp_misc_cfltcvt_tab   1001fd7c f   LIBCMT:cmiscdat.obj
 0001:0001eda0       __ValidateImageBase        1001fda0 f   LIBCMT:pesect.obj
 0001:0001ede0       __FindPESection            1001fde0 f   LIBCMT:pesect.obj
 0001:0001ee30       __IsNonwritableInCurrentImage 1001fe30 f   LIBCMT:pesect.obj
 0001:0001eeec       @__security_check_cookie@4 1001feec f   LIBCMT:secchk.obj
 0001:0001eefb       __crt_debugger_hook        1001fefb f   LIBCMT:dbghook.obj
 0001:0001ef03       __mbtowc_l                 1001ff03 f   LIBCMT:mbtowc.obj
 0001:0001f019       _mbtowc                    10020019 f   LIBCMT:mbtowc.obj
 0001:0001f040       __allmul                   10020040 f   LIBCMT:llmul.obj
 0001:0001f074       ___crtMessageBoxW          10020074 f   LIBCMT:crtmboxw.obj
 0001:0001f1e0       _wcscat_s                  100201e0 f   LIBCMT:wcscat_s.obj
 0001:0001f255       _wcsncpy_s                 10020255 f   LIBCMT:wcsncpy_s.obj
 0001:0001f322       __set_error_mode           10020322 f   LIBCMT:errmode.obj
 0001:0001f361       _strncpy_s                 10020361 f   LIBCMT:strncpy_s.obj
 0001:0001f4fd       ___crtGetStringTypeA       100204fd f   LIBCMT:a_str.obj
 0001:0001f53d       ___free_lc_time            1002053d f   LIBCMT:inittime.obj
 0001:0001f8b4       ___free_lconv_num          100208b4 f   LIBCMT:initnum.obj
 0001:0001f91d       ___free_lconv_mon          1002091d f   LIBCMT:initmon.obj
 0001:0001fa1b       ____lc_codepage_func       10020a1b f   LIBCMT:initctyp.obj
 0001:0001fa50       _strpbrk                   10020a50 f   LIBCMT:strpbrk.obj
 0001:0001fa90       __fcloseall                10020a90 f   LIBCMT:closeall.obj
 0001:0001fb2c       __isatty                   10020b2c f   LIBCMT:isatty.obj
 0001:0001fb82       __wctomb_s_l               10020b82 f   LIBCMT:wctomb.obj
 0001:0001fcd7       _wctomb_s                  10020cd7 f   LIBCMT:wctomb.obj
 0001:0001fd00       __aulldvrm                 10020d00 f   LIBCMT:ulldvrm.obj
 0001:0001fde8       __ismbblead                10020de8 f   LIBCMT:ismbbyte.obj
 0001:0001fe00       ___crtLCMapStringW         10020e00 f   LIBCMT:w_map.obj
 0001:0001fe2f       _iswctype                  10020e2f f   LIBCMT:iswctype.obj
 0001:0001fe84       __lseeki64_nolock          10020e84 f   LIBCMT:lseeki64.obj
 0001:0001ff09       __lseeki64                 10020f09 f   LIBCMT:lseeki64.obj
 0001:0001fff3       __getbuf                   10020ff3 f   LIBCMT:_getbuf.obj
 0001:000202aa       ___crtCompareStringA       100212aa f   LIBCMT:a_cmp.obj
 0001:000202ec       __strnicoll_l              100212ec f   LIBCMT:strnicol.obj
 0001:00020488       ___crtsetenv               10021488 f   LIBCMT:setenv.obj
 0001:000206ca       ?_JumpToContinuation@@YGXPAXPAUEHRegistrationNode@@@Z 100216ca f   LIBCMT:_trnsctrl_.obj
 0001:000206fc       ?_CallMemberFunction1@@YGXPAX00@Z 100216fc f   LIBCMT:_trnsctrl_.obj
 0001:000206fc       ?_CallMemberFunction0@@YGXPAX0@Z 100216fc f   LIBCMT:_trnsctrl_.obj
 0001:000206fc       ?_CallMemberFunction2@@YGXPAX00H@Z 100216fc f   LIBCMT:_trnsctrl_.obj
 0001:00020703       ?_UnwindNestedFrames@@YGXPAUEHRegistrationNode@@PAUEHExceptionRecord@@@Z 10021703 f   LIBCMT:_trnsctrl_.obj
 0001:00020757       ___CxxFrameHandler3        10021757 f   LIBCMT:_trnsctrl_.obj
 0001:000207c0       ?_CallSETranslator@@YAHPAUEHExceptionRecord@@PAUEHRegistrationNode@@PAX2PBU_s_FuncInfo@@H1@Z 100217c0 f   LIBCMT:_trnsctrl_.obj
 0001:00020936       ?_GetRangeOfTrysToCheck@@YAPBU_s_TryBlockMapEntry@@PBU_s_FuncInfo@@HHPAI1@Z 10021936 f   LIBCMT:_trnsctrl_.obj
 0001:000209a9       __CreateFrameInfo          100219a9 f   LIBCMT:_trnsctrl_.obj
 0001:000209d5       __IsExceptionObjectToBeDestroyed 100219d5 f   LIBCMT:_trnsctrl_.obj
 0001:000209fc       __FindAndUnlinkFrame       100219fc f   LIBCMT:_trnsctrl_.obj
 0001:00020a4e       ?_CallCatchBlock2@@YAPAXPAUEHRegistrationNode@@PBU_s_FuncInfo@@PAXHK@Z 10021a4e f   LIBCMT:_trnsctrl_.obj
 0001:00020aae       __EH_prolog3_catch         10021aae f   LIBCMT:ehprolg3.obj
 0001:00020ae4       __EH_epilog3               10021ae4 f   LIBCMT:ehprolg3.obj
 0001:00020b00       __alloca_probe_16          10021b00 f   LIBCMT:alloca16.obj
 0001:00020b16       __alloca_probe_8           10021b16     LIBCMT:alloca16.obj
 0001:00020b2c       __putwch_nolock            10021b2c f   LIBCMT:putwch.obj
 0001:00020b70       __chkstk                   10021b70 f   LIBCMT:chkstk.obj
 0001:00020b70       __alloca_probe             10021b70     LIBCMT:chkstk.obj
 0001:00020b9b       __set_osfhnd               10021b9b f   LIBCMT:osfinfo.obj
 0001:00020c1c       __free_osfhnd              10021c1c f   LIBCMT:osfinfo.obj
 0001:00020ca2       __get_osfhandle            10021ca2 f   LIBCMT:osfinfo.obj
 0001:00020d0b       ___lock_fhandle            10021d0b f   LIBCMT:osfinfo.obj
 0001:00020daa       __unlock_fhandle           10021daa f   LIBCMT:osfinfo.obj
 0001:00020dd1       __alloc_osfhnd             10021dd1 f   LIBCMT:osfinfo.obj
 0001:0002169f       __wsopen_helper            1002269f f   LIBCMT:wopen.obj
 0001:00021763       __wsopen_s                 10022763 f   LIBCMT:wopen.obj
 0001:00021783       _wcsncmp                   10022783 f   LIBCMT:wcsncmp.obj
 0001:000217c0       __global_unwind2           100227c0 f   LIBCMT:exsup.obj
 0001:00021825       __local_unwind2            10022825 f   LIBCMT:exsup.obj
 0001:000218a9       __abnormal_termination     100228a9 f   LIBCMT:exsup.obj
 0001:000218cc       __NLG_Notify1              100228cc f   LIBCMT:exsup.obj
 0001:000218d5       __NLG_Notify               100228d5 f   LIBCMT:exsup.obj
 0001:000218ec       __NLG_Dispatch2            100228ec     LIBCMT:exsup.obj
 0001:000218ec       __NLG_Dispatch             100228ec     LIBCMT:exsup.obj
 0001:000218f4       __NLG_Call                 100228f4 f   LIBCMT:exsup.obj
 0001:000218f6       __NLG_Return2              100228f6     LIBCMT:exsup.obj
 0001:000218f7       __fptrap                   100228f7 f   LIBCMT:crt0fp.obj
 0001:00021900       ___report_gsfailure        10022900 f   LIBCMT:gs_report.obj
 0001:00021a06       __strnicmp_l               10022a06 f   LIBCMT:strnicmp.obj
 0001:00021ae8       __strnicmp                 10022ae8 f   LIBCMT:strnicmp.obj
 0001:00021b3b       _wcsnlen                   10022b3b f   LIBCMT:wcslen_s.obj
 0001:00021b5b       __mbschr_l                 10022b5b f   LIBCMT:mbschr.obj
 0001:00021c0b       __mbschr                   10022c0b f   LIBCMT:mbschr.obj
 0001:00021c22       ??1bad_exception@std@@UAE@XZ 10022c22 f i LIBCMT:frame.obj
 0001:00021c2d       ??_Ebad_exception@std@@UAEPAXI@Z 10022c2d f i LIBCMT:frame.obj
 0001:00021c2d       ??_Gbad_exception@std@@UAEPAXI@Z 10022c2d f i LIBCMT:frame.obj
 0001:00021c54       ___TypeMatch               10022c54 f   LIBCMT:frame.obj
 0001:00021cb3       ___FrameUnwindFilter       10022cb3 f   LIBCMT:frame.obj
 0001:00021d02       ___FrameUnwindToState      10022d02 f   LIBCMT:frame.obj
 0001:00021e23       ___DestructExceptionObject 10022e23 f   LIBCMT:frame.obj
 0001:00021e78       ___AdjustPointer           10022e78 f   LIBCMT:frame.obj
 0001:000220fc       ___BuildCatchObjectHelper  100230fc f   LIBCMT:frame.obj
 0001:0002227b       ___BuildCatchObject        1002327b f   LIBCMT:frame.obj
 0001:000227f7       ??0bad_exception@std@@QAE@ABV01@@Z 100237f7 f i LIBCMT:frame.obj
 0001:00022814       ___InternalCxxFrameHandler 10023814 f   LIBCMT:frame.obj
 0001:00022900       __CallSettingFrame@12      10023900 f   LIBCMT:lowhelpr.obj
 0001:00022927       __NLG_Return               10023927     LIBCMT:lowhelpr.obj
 0001:0002294c       ___initconout              1002394c f   LIBCMT:initcon.obj
 0001:0002296b       ___termconout              1002396b f   LIBCMT:initcon.obj
 0001:00022982       __chsize_nolock            10023982 f   LIBCMT:chsize.obj
 0001:00022b38       __setmode_nolock           10023b38 f   LIBCMT:setmode.obj
 0001:00022bf3       __get_fmode                10023bf3 f   LIBCMT:setmode.obj
 0001:00022c20       ___ascii_strnicmp          10023c20 f   LIBCMT:_strnicm.obj
 0001:00022c81       ?_ValidateExecute@@YAHP6GHXZ@Z 10023c81 f   LIBCMT:validate.obj
 0001:00022c81       ?_ValidateWrite@@YAHPAXI@Z 10023c81 f   LIBCMT:validate.obj
 0001:00022c81       ?_ValidateRead@@YAHPBXI@Z  10023c81 f   LIBCMT:validate.obj
 0001:00022c94       _RtlUnwind@16              10023c94 f   kernel32:KERNEL32.dll
 0001:00022c9a       _png_get_valid             10023c9a f   pnglib:pngget.obj
 0001:00022cb6       _png_get_gAMA              10023cb6 f   pnglib:pngget.obj
 0001:00022ce1       _png_get_IHDR              10023ce1 f   pnglib:pngget.obj
 0001:00022df1       _png_set_strip_16          10023df1 f   pnglib:pngrtran.obj
 0001:00022e04       _png_set_gamma             10023e04 f   pnglib:pngrtran.obj
 0001:00022e5e       _png_set_expand            10023e5e f   pnglib:pngrtran.obj
 0001:00022e71       _png_set_gray_to_rgb       10023e71 f   pnglib:pngrtran.obj
 0001:00022e80       _png_read_transform_info   10023e80 f   pnglib:pngrtran.obj
 0001:00022fa7       _png_do_chop               10023fa7 f   pnglib:pngrtran.obj
 0001:00022fee       _png_do_read_swap_alpha    10023fee f   pnglib:pngrtran.obj
 0001:000230f0       _png_do_read_invert_alpha  100240f0 f   pnglib:pngrtran.obj
 0001:0002319e       _png_do_read_filler        1002419e f   pnglib:pngrtran.obj
 0001:000233dd       _png_do_gray_to_rgb        100243dd f   pnglib:pngrtran.obj
 0001:0002352a       _png_do_background         1002452a f   pnglib:pngrtran.obj
 0001:000243e1       _png_do_gamma              100253e1 f   pnglib:pngrtran.obj
 0001:00024763       _png_do_expand_palette     10025763 f   pnglib:pngrtran.obj
 0001:0002495f       _png_do_expand             1002595f f   pnglib:pngrtran.obj
 0001:00024ce3       _png_build_gamma_table     10025ce3 f   pnglib:pngrtran.obj
 0001:000252d7       _png_init_read_transformations 100262d7 f   pnglib:pngrtran.obj
 0001:00025d6d       _png_do_read_transformations 10026d6d f   pnglib:pngrtran.obj
 0001:00025fd2       _png_create_read_struct_2  10026fd2 f   pnglib:pngread.obj
 0001:000261b0       _png_read_info             100271b0 f   pnglib:pngread.obj
 0001:00026679       _png_read_update_info      10027679 f   pnglib:pngread.obj
 0001:000266ad       _png_read_row              100276ad f   pnglib:pngread.obj
 0001:00026b22       _png_read_rows             10027b22 f   pnglib:pngread.obj
 0001:00026ba2       _png_read_end              10027ba2 f   pnglib:pngread.obj
 0001:00026f87       _png_read_destroy          10027f87 f   pnglib:pngread.obj
 0001:00027197       _png_create_read_struct    10028197 f   pnglib:pngread.obj
 0001:000271b5       _png_destroy_read_struct   100281b5 f   pnglib:pngread.obj
 0001:00027270       _png_set_bgr               10028270 f   pnglib:pngtrans.obj
 0001:00027280       _png_set_packing           10028280 f   pnglib:pngtrans.obj
 0001:000272a0       _png_set_interlace_handling 100282a0 f   pnglib:pngtrans.obj
 0001:000272c1       _png_set_filler            100282c1 f   pnglib:pngtrans.obj
 0001:0002731b       _png_do_bgr                1002831b f   pnglib:pngtrans.obj
 0001:000273da       _png_sig_cmp               100283da f   pnglib:png.obj
 0001:0002742e       _png_check_sig             1002842e f   pnglib:png.obj
 0001:00027448       _png_zalloc                10028448 f   pnglib:png.obj
 0001:0002748f       _png_zfree                 1002848f f   pnglib:png.obj
 0001:00027498       _png_reset_crc             10028498 f   pnglib:png.obj
 0001:000274b3       _png_calculate_crc         100284b3 f   pnglib:png.obj
 0001:000274f7       _png_info_init_3           100284f7 f   pnglib:png.obj
 0001:00027530       _png_free_data             10028530 f   pnglib:png.obj
 0001:000278d3       _png_info_destroy          100288d3 f   pnglib:png.obj
 0001:00027929       _png_handle_as_unknown     10028929 f   pnglib:png.obj
 0001:00027986       _png_create_info_struct    10028986 f   pnglib:png.obj
 0001:000279c4       _png_read_data             100289c4 f   pnglib:pngrio.obj
 0001:000279ee       _png_default_read_data     100289ee f   pnglib:pngrio.obj
 0001:00027a21       _png_set_read_fn           10028a21 f   pnglib:pngrio.obj
 0001:00027bf1       _png_set_error_fn          10028bf1 f   pnglib:pngerror.obj
 0001:00027c0f       _png_error                 10028c0f f   pnglib:pngerror.obj
 0001:00027c9c       _png_warning               10028c9c f   pnglib:pngerror.obj
 0001:00027ce5       _png_chunk_error           10028ce5 f   pnglib:pngerror.obj
 0001:00027d1b       _png_chunk_warning         10028d1b f   pnglib:pngerror.obj
 0001:00027d51       _png_create_struct_2       10028d51 f   pnglib:pngmem.obj
 0001:00027db0       _png_destroy_struct_2      10028db0 f   pnglib:pngmem.obj
 0001:00027de3       _png_malloc_default        10028de3 f   pnglib:pngmem.obj
 0001:00027e01       _png_free_default          10028e01 f   pnglib:pngmem.obj
 0001:00027e1b       _png_memcpy_check          10028e1b f   pnglib:pngmem.obj
 0001:00027e31       _png_memset_check          10028e31 f   pnglib:pngmem.obj
 0001:00027e47       _png_set_mem_fn            10028e47 f   pnglib:pngmem.obj
 0001:00027e6e       _png_create_struct         10028e6e f   pnglib:pngmem.obj
 0001:00027e82       _png_destroy_struct        10028e82 f   pnglib:pngmem.obj
 0001:00027e93       _png_malloc                10028e93 f   pnglib:pngmem.obj
 0001:00027ee4       _png_free                  10028ee4 f   pnglib:pngmem.obj
 0001:00027f0f       _png_malloc_warn           10028f0f f   pnglib:pngmem.obj
 0001:00027f3e       _png_get_uint_32           10028f3e f   pnglib:pngrutil.obj
 0001:00027f3e       _png_get_int_32            10028f3e f   pnglib:pngrutil.obj
 0001:00027f64       _png_get_uint_16           10028f64 f   pnglib:pngrutil.obj
 0001:00027f7f       _png_crc_read              10028f7f f   pnglib:pngrutil.obj
 0001:00027fa1       _png_crc_error             10028fa1 f   pnglib:pngrutil.obj
 0001:00028002       _png_decompress_chunk      10029002 f   pnglib:pngrutil.obj
 0001:00028315       _png_check_chunk_name      10029315 f   pnglib:pngrutil.obj
 0001:00028379       _png_combine_row           10029379 f   pnglib:pngrutil.obj
 0001:0002856a       _png_do_read_interlace     1002956a f   pnglib:pngrutil.obj
 0001:0002883a       _png_read_filter_row       1002983a f   pnglib:pngrutil.obj
 0001:000289cf       _png_read_start_row        100299cf f   pnglib:pngrutil.obj
 0001:00028c13       _png_get_uint_31           10029c13 f   pnglib:pngrutil.obj
 0001:00028c3e       _png_crc_finish            10029c3e f   pnglib:pngrutil.obj
 0001:00028cd2       _png_handle_IHDR           10029cd2 f   pnglib:pngrutil.obj
 0001:00028dfc       _png_handle_PLTE           10029dfc f   pnglib:pngrutil.obj
 0001:00028f46       _png_handle_IEND           10029f46 f   pnglib:pngrutil.obj
 0001:00028f8a       _png_handle_gAMA           10029f8a f   pnglib:pngrutil.obj
 0001:000290cf       _png_handle_sBIT           1002a0cf f   pnglib:pngrutil.obj
 0001:000291df       _png_handle_cHRM           1002a1df f   pnglib:pngrutil.obj
 0001:00029577       _png_handle_sRGB           1002a577 f   pnglib:pngrutil.obj
 0001:00029756       _png_handle_iCCP           1002a756 f   pnglib:pngrutil.obj
 0001:000298c9       _png_handle_sPLT           1002a8c9 f   pnglib:pngrutil.obj
 0001:00029a9b       _png_handle_tRNS           1002aa9b f   pnglib:pngrutil.obj
 0001:00029c65       _png_handle_bKGD           1002ac65 f   pnglib:pngrutil.obj
 0001:00029de8       _png_handle_hIST           1002ade8 f   pnglib:pngrutil.obj
 0001:00029ee8       _png_handle_pHYs           1002aee8 f   pnglib:pngrutil.obj
 0001:00029f89       _png_handle_oFFs           1002af89 f   pnglib:pngrutil.obj
 0001:0002a02d       _png_handle_pCAL           1002b02d f   pnglib:pngrutil.obj
 0001:0002a21c       _png_handle_sCAL           1002b21c f   pnglib:pngrutil.obj
 0001:0002a36c       _png_handle_tIME           1002b36c f   pnglib:pngrutil.obj
 0001:0002a430       _png_handle_tEXt           1002b430 f   pnglib:pngrutil.obj
 0001:0002a530       _png_handle_zTXt           1002b530 f   pnglib:pngrutil.obj
 0001:0002a67a       _png_handle_unknown        1002b67a f   pnglib:pngrutil.obj
 0001:0002a7b0       _png_read_finish_row       1002b7b0 f   pnglib:pngrutil.obj
 0001:0002aa05       _png_set_bKGD              1002ba05 f   pnglib:pngset.obj
 0001:0002aa2e       _png_set_cHRM              1002ba2e f   pnglib:pngset.obj
 0001:0002ac51       _png_set_cHRM_fixed        1002bc51 f   pnglib:pngset.obj
 0001:0002ae05       _png_set_gAMA              1002be05 f   pnglib:pngset.obj
 0001:0002ae7d       _png_set_gAMA_fixed        1002be7d f   pnglib:pngset.obj
 0001:0002aef3       _png_set_hIST              1002bef3 f   pnglib:pngset.obj
 0001:0002af96       _png_set_IHDR              1002bf96 f   pnglib:pngset.obj
 0001:0002b14b       _png_set_oFFs              1002c14b f   pnglib:pngset.obj
 0001:0002b176       _png_set_pCAL              1002c176 f   pnglib:pngset.obj
 0001:0002b2d4       _png_set_sCAL              1002c2d4 f   pnglib:pngset.obj
 0001:0002b308       _png_set_pHYs              1002c308 f   pnglib:pngset.obj
 0001:0002b333       _png_set_PLTE              1002c333 f   pnglib:pngset.obj
 0001:0002b3e4       _png_set_sBIT              1002c3e4 f   pnglib:pngset.obj
 0001:0002b40d       _png_set_sRGB              1002c40d f   pnglib:pngset.obj
 0001:0002b42c       _png_set_sRGB_gAMA_and_cHRM 1002c42c f   pnglib:pngset.obj
 0001:0002b4fd       _png_set_iCCP              1002c4fd f   pnglib:pngset.obj
 0001:0002b5d8       _png_set_text_2            1002c5d8 f   pnglib:pngset.obj
 0001:0002b77e       _png_set_tIME              1002c77e f   pnglib:pngset.obj
 0001:0002b7b3       _png_set_tRNS              1002c7b3 f   pnglib:pngset.obj
 0001:0002b852       _png_set_sPLT              1002c852 f   pnglib:pngset.obj
 0001:0002b966       _png_set_unknown_chunks    1002c966 f   pnglib:pngset.obj
 0001:0002bcc4       _unzGetGlobalInfo          1002ccc4 f   zlib:unzip.obj
 0001:0002c01b       _unzGetCurrentFileInfo     1002d01b f   zlib:unzip.obj
 0001:0002c042       _unzGoToFirstFile          1002d042 f   zlib:unzip.obj
 0001:0002c087       _unzGoToNextFile           1002d087 f   zlib:unzip.obj
 0001:0002c2d8       _unzReadCurrentFile        1002d2d8 f   zlib:unzip.obj
 0001:0002c505       _unzCloseCurrentFile       1002d505 f   zlib:unzip.obj
 0001:0002c57e       _unzOpen2                  1002d57e f   zlib:unzip.obj
 0001:0002c797       _unzClose                  1002d797 f   zlib:unzip.obj
 0001:0002c7ce       _unzOpenCurrentFile3       1002d7ce f   zlib:unzip.obj
 0001:0002ca57       _unzOpenCurrentFile        1002da57 f   zlib:unzip.obj
 0001:0002ca6d       _inflateReset              1002da6d f   zlib:inflate.obj
 0001:0002cacc       _inflateInit2_             1002dacc f   zlib:inflate.obj
 0001:0002cb86       _inflateInit_              1002db86 f   zlib:inflate.obj
 0001:0002cc74       _inflate                   1002dc74 f   zlib:inflate.obj
 0001:0002deb0       _inflateEnd                1002eeb0 f   zlib:inflate.obj
 0001:0002def1       _get_crc_table             1002eef1 f   zlib:crc32.obj
 0001:0002e165       _crc32                     1002f165 f   zlib:crc32.obj
 0001:0002e181       _fopen_file_func           1002f181 f   zlib:ioapi.obj
 0001:0002e1c8       _fread_file_func           1002f1c8 f   zlib:ioapi.obj
 0001:0002e1e0       _fwrite_file_func          1002f1e0 f   zlib:ioapi.obj
 0001:0002e1f8       _ftell_file_func           1002f1f8 f   zlib:ioapi.obj
 0001:0002e206       _fseek_file_func           1002f206 f   zlib:ioapi.obj
 0001:0002e23b       _fclose_file_func          1002f23b f   zlib:ioapi.obj
 0001:0002e249       _ferror_file_func          1002f249 f   zlib:ioapi.obj
 0001:0002e257       _fill_fopen_filefunc       1002f257 f   zlib:ioapi.obj
 0001:0002e293       _zcalloc                   1002f293 f   zlib:zutil.obj
 0001:0002e2a6       _zcfree                    1002f2a6 f   zlib:zutil.obj
 0001:0002e2b4       _inflate_fast              1002f2b4 f   zlib:inffast.obj
 0001:0002e6a6       _inflate_table             1002f6a6 f   zlib:inftrees.obj
 0001:0002ea54       _adler32                   1002fa54 f   zlib:adler32.obj
 0001:0002ec75       ?RemoveFromList@ListElement@@QAE_NXZ 1002fc75 f i CrashHandlerLib:CrashHandler.obj
 0001:0002ec95       ?InsertInList@ListElement@@QAEXPAV1@@Z 1002fc95 f i CrashHandlerLib:CrashHandler.obj
 0001:0002f668       ?clear@?$List@VStringNode@@@@QAEXXZ 10030668 f i CrashHandlerLib:CrashHandler.obj
 0001:0002f668       ?clear@?$List@VSFileDetail@@@@QAEXXZ 10030668 f i CrashHandlerLib:CrashHandler.obj
 0001:0002f685       ?Uninstall@CrashHandlerImpl@@QAEXXZ 10030685 f   CrashHandlerLib:CrashHandler.obj
 0001:0002f69e       ?Uninstall@CrashHandler@@QAEXXZ 1003069e f   CrashHandlerLib:CrashHandler.obj
 0001:0002f6a5       ?IsInstalled@CrashHandler@@QBE_NXZ 100306a5 f   CrashHandlerLib:CrashHandler.obj
 0001:0002f6b3       ?SetCrashCallback@CrashHandler@@QAEXP6AXPBD@Z_N@Z 100306b3 f   CrashHandlerLib:CrashHandler.obj
 0001:0002fdbe       ?Install@CrashHandlerImpl@@QAE_NXZ 10030dbe f   CrashHandlerLib:CrashHandler.obj
 0001:0002fdf3       ?Install@CrashHandler@@QAE_NXZ 10030df3 f   CrashHandlerLib:CrashHandler.obj
 0001:0002fdfa       ??1StringNode@@QAE@XZ      10030dfa f i CrashHandlerLib:CrashHandler.obj
 0001:0002fe11       ??1SFileDetail@@QAE@XZ     10030e11 f i CrashHandlerLib:CrashHandler.obj
 0001:0002fe40       ??$delete_elements@V?$ListIterator@VStringNode@@@@@@YAXV?$ListIterator@VStringNode@@@@0@Z 10030e40 f i CrashHandlerLib:CrashHandler.obj
 0001:0002fe6d       ??$delete_elements@V?$ListIterator@VSFileDetail@@@@@@YAXV?$ListIterator@VSFileDetail@@@@0@Z 10030e6d f i CrashHandlerLib:CrashHandler.obj
 0001:0002fe9a       ??$_Find_if@V?$ListIterator@VSFileDetail@@@@Uelement_name@@@std@@YA?AV?$ListIterator@VSFileDetail@@@@V1@0Uelement_name@@@Z 10030e9a f i CrashHandlerLib:CrashHandler.obj
 0001:0002fe9a       ??$_Find_if@V?$ListIterator@VStringNode@@@@Uelement_name@@@std@@YA?AV?$ListIterator@VStringNode@@@@V1@0Uelement_name@@@Z 10030e9a f i CrashHandlerLib:CrashHandler.obj
 0001:0002fecb       ??1CrashHandlerImpl@@QAE@XZ 10030ecb f   CrashHandlerLib:CrashHandler.obj
 0001:0002ffa3       ??$find_if@V?$ListIterator@VStringNode@@@@Uelement_name@@@std@@YA?AV?$ListIterator@VStringNode@@@@V1@0Uelement_name@@@Z 10030fa3 f i CrashHandlerLib:CrashHandler.obj
 0001:0002ffa3       ??$find_if@V?$ListIterator@VSFileDetail@@@@Uelement_name@@@std@@YA?AV?$ListIterator@VSFileDetail@@@@V1@0Uelement_name@@@Z 10030fa3 f i CrashHandlerLib:CrashHandler.obj
 0001:0002ffc5       ??1?$auto_ptr@VCrashHandlerImpl@@@std@@QAE@XZ 10030fc5 f i CrashHandlerLib:CrashHandler.obj
 0001:0002ffdc       ??$remove_from_intrusive_list@V?$List@VSFileDetail@@@@Uelement_name@@@@YAXAAV?$List@VSFileDetail@@@@Uelement_name@@@Z 10030fdc f i CrashHandlerLib:CrashHandler.obj
 0001:0003001c       ??$remove_from_intrusive_list@V?$List@VStringNode@@@@Uelement_name@@@@YAXAAV?$List@VStringNode@@@@Uelement_name@@@Z 1003101c f i CrashHandlerLib:CrashHandler.obj
 0001:0003005c       ?AddFolderToDelete@CrashHandlerImpl@@QAEXPBD@Z 1003105c f   CrashHandlerLib:CrashHandler.obj
 0001:00030094       ?RemoveFile@CrashHandlerImpl@@QAEXPBD@Z 10031094 f   CrashHandlerLib:CrashHandler.obj
 0001:000300a9       ?RemoveFolderToDelete@CrashHandlerImpl@@QAEXPBD@Z 100310a9 f   CrashHandlerLib:CrashHandler.obj
 0001:000300be       ??1CrashHandler@@QAE@XZ    100310be f   CrashHandlerLib:CrashHandler.obj
 0001:000300d0       ?RemoveFile@CrashHandler@@QAEXPBD@Z 100310d0 f   CrashHandlerLib:CrashHandler.obj
 0001:000300db       ?AddFolderToDelete@CrashHandler@@QAEXPBD@Z 100310db f   CrashHandlerLib:CrashHandler.obj
 0001:000300e6       ?RemoveFolderToDelete@CrashHandler@@QAEXPBD@Z 100310e6 f   CrashHandlerLib:CrashHandler.obj
 0001:000300f1       ??$?HDU?$char_traits@D@std@@V?$allocator@D@1@@std@@YA?AV?$basic_string@DU?$char_traits@D@std@@V?$allocator@D@2@@0@ABV10@D@Z 100310f1 f i CrashHandlerLib:CrashHandler.obj
 0001:00030134       ??$?HDU?$char_traits@D@std@@V?$allocator@D@1@@std@@YA?AV?$basic_string@DU?$char_traits@D@std@@V?$allocator@D@2@@0@$$QAV10@0@Z 10031134 f i CrashHandlerLib:CrashHandler.obj
 0001:00030181       ??$?HDU?$char_traits@D@std@@V?$allocator@D@1@@std@@YA?AV?$basic_string@DU?$char_traits@D@std@@V?$allocator@D@2@@0@ABV10@PBD@Z 10031181 f i CrashHandlerLib:CrashHandler.obj
 0001:000301d8       ??0SFileDetail@@QAE@PBD0@Z 100311d8 f i CrashHandlerLib:CrashHandler.obj
 0001:00030279       ??0CrashHandlerImpl@@QAE@PBD000@Z 10031279 f   CrashHandlerLib:CrashHandler.obj
 0001:000306d0       ?AddFile@CrashHandlerImpl@@QAEXPBD0@Z 100316d0 f   CrashHandlerLib:CrashHandler.obj
 0001:00030703       ??0CrashHandler@@QAE@PBD000@Z 10031703 f   CrashHandlerLib:CrashHandler.obj
 0001:00030738       ?AddFile@CrashHandler@@QAEXPBD0@Z 10031738 f   CrashHandlerLib:CrashHandler.obj
 0001:00030743       ?Release@CMiniVersion@@QAEXXZ 10031743 f   CrashHandlerLib:MiniVersion.obj
 0001:00030758       ?GetFileVersion@CMiniVersion@@QAEXPAG@Z 10031758 f   CrashHandlerLib:MiniVersion.obj
 0001:00030779       ?GetProductVersion@CMiniVersion@@QAEXPAG@Z 10031779 f   CrashHandlerLib:MiniVersion.obj
 0001:0003079a       ?GetCompanyName@CMiniVersion@@QAEHPADH@Z 1003179a f   CrashHandlerLib:MiniVersion.obj
 0001:000307dd       ?GetFileDescription@CMiniVersion@@QAEHPADH@Z 100317dd f   CrashHandlerLib:MiniVersion.obj
 0001:00030820       ?GetProductName@CMiniVersion@@QAEHPADH@Z 10031820 f   CrashHandlerLib:MiniVersion.obj
 0001:00030863       ?GetFixedInfo@CMiniVersion@@IAEHAAUtagVS_FIXEDFILEINFO@@@Z 10031863 f   CrashHandlerLib:MiniVersion.obj
 0001:000308a3       ?GetStringInfo@CMiniVersion@@IAEHPBDPAD@Z 100318a3 f   CrashHandlerLib:MiniVersion.obj
 0001:00030931       ?Init@CMiniVersion@@QAE_NXZ 10031931 f   CrashHandlerLib:MiniVersion.obj
 0001:00030a30       ??0CMiniVersion@@QAE@PB_W@Z 10031a30 f   CrashHandlerLib:MiniVersion.obj
 0001:00030acf       ?GetFilePart@crhfileutils@@YAPBDPBD@Z 10031acf f   CrashHandlerLib:FileUtilities.obj
 0001:00030aea       ?GetTempDirectoryWide@crhfileutils@@YA?AV?$basic_string@_WU?$char_traits@_W@std@@V?$allocator@_W@2@@std@@XZ 10031aea f   CrashHandlerLib:FileUtilities.obj
 0001:00030b28       ?ConvertWideToUTF8String@@YAXABV?$basic_string@_WU?$char_traits@_W@std@@V?$allocator@_W@2@@std@@AAV?$basic_string@DU?$char_traits@D@std@@V?$allocator@D@2@@2@@Z 10031b28 f i CrashHandlerLib:FileUtilities.obj
 0001:00030b58       ??$ConvertWindowsPathNameImpl@V?$basic_string@_WU?$char_traits@_W@std@@V?$allocator@_W@2@@std@@@detail@@YAXABV?$basic_string@_WU?$char_traits@_W@std@@V?$allocator@_W@2@@std@@AAV?$basic_string@DU?$char_traits@D@std@@V?$allocator@D@2@@2@@Z 10031b58 f i CrashHandlerLib:FileUtilities.obj
 0001:00030b9a       ?GetTempDirectory@crhfileutils@@YA?AV?$basic_string@DU?$char_traits@D@std@@V?$allocator@D@2@@std@@XZ 10031b9a f   CrashHandlerLib:FileUtilities.obj
 0001:00030bd9       ?GenerateGuidString@crhfileutils@@YA?AV?$basic_string@DU?$char_traits@D@std@@V?$allocator@D@2@@std@@XZ 10031bd9 f   CrashHandlerLib:FileUtilities.obj
 0001:00030c4f       ?RemoveDirectoryRecursiveWide@crhfileutils@@YA_NABV?$basic_string@_WU?$char_traits@_W@std@@V?$allocator@_W@2@@std@@@Z 10031c4f f   CrashHandlerLib:FileUtilities.obj
 0001:00030e34       ?RemoveDirectoryRecursive@crhfileutils@@YA_NABV?$basic_string@DU?$char_traits@D@std@@V?$allocator@D@2@@std@@@Z 10031e34 f   CrashHandlerLib:FileUtilities.obj
 0001:00030e77       ?flush@IniFile@@QAEXXZ     10031e77 f   CrashHandlerLib:IniFile.obj
 0001:00030e91       ??0IniFile@@QAE@XZ         10031e91 f   CrashHandlerLib:IniFile.obj
 0001:00030ea4       ??1IniFile@@QAE@XZ         10031ea4 f   CrashHandlerLib:IniFile.obj
 0001:00030eb9       ?ConvertUTF8ToWideString@@YAXPBDAAV?$basic_string@_WU?$char_traits@_W@std@@V?$allocator@_W@2@@std@@@Z 10031eb9 f i CrashHandlerLib:IniFile.obj
 0001:00030ee3       ??$ConvertUnityPathNameImpl@PBD@detail@@YAXABQBDAAV?$basic_string@_WU?$char_traits@_W@std@@V?$allocator@_W@2@@std@@@Z 10031ee3 f i CrashHandlerLib:IniFile.obj
 0001:00030f36       ??$Utf8ToWideImpl@PBD@detail@@YA?AV?$basic_string@_WU?$char_traits@_W@std@@V?$allocator@_W@2@@std@@ABQBD@Z 10031f36 f i CrashHandlerLib:IniFile.obj
 0001:00030f5f       ?setFileName@IniFile@@QAEXPBD_N@Z 10031f5f f   CrashHandlerLib:IniFile.obj
 0001:00030fcf       ?writeString@IniFile@@QBE_NPB_W0PBD@Z 10031fcf f   CrashHandlerLib:IniFile.obj
 0001:0003103f       __cfltcvt_init             1003203f f   LIBCMT:_fpinit_.obj
 0001:0003109f       __fpmath                   1003209f f   LIBCMT:_fpinit_.obj
 0001:000310b8       _fabs                      100320b8 f   LIBCMT:_fabs_.obj
 0001:00031180       _pow                       10032180 f   LIBCMT:_pow_.obj
 0001:000311c0       __CIpow                    100321c0 f   LIBCMT:_pow_.obj
 0001:000311fb       __CIpow_default            100321fb f   LIBCMT:_pow_.obj
 0001:00031214       __pow_default              10032214     LIBCMT:_pow_.obj
 0001:00031410       __ftol2_sse                10032410 f   LIBCMT:ftol2.obj
 0001:00031419       __ftol2_pentium4           10032419 f   LIBCMT:ftol2.obj
 0001:0003142c       __ftol2_sse_excpt          1003242c f   LIBCMT:ftol2.obj
 0001:00031446       __ftol2                    10032446 f   LIBCMT:ftol2.obj
 0001:000314c0       __setjmp3                  100324c0 f   LIBCMT:setjmp3.obj
 0001:00031540       _longjmp                   10032540 f   LIBCMT:longjmp.obj
 0001:000315f1       __strtod_l                 100325f1 f   LIBCMT:strtod.obj
 0001:00031714       _strtod                    10032714 f   LIBCMT:strtod.obj
 0001:0003172b       __fsopen                   1003272b f   LIBCMT:fopen.obj
 0001:000317e7       _fopen                     100327e7 f   LIBCMT:fopen.obj
 0001:000317fe       _ferror                    100327fe f   LIBCMT:feoferr.obj
 0001:00031826       __vswprintf_helper         10032826 f   LIBCMT:vswprnc.obj
 0001:0003191c       __vswprintf_c_l            1003291c f   LIBCMT:vswprnc.obj
 0001:00031950       __SEH_prolog               10032950 f   LIBCMT:sehprolg.obj
 0001:0003198b       __SEH_epilog               1003298b f   LIBCMT:sehprolg.obj
 0001:000319a8       __except_handler3          100329a8 f   LIBCMT:exsup3.obj
 0001:00031aa6       __seh_longjmp_unwind@4     10032aa6 f   LIBCMT:exsup3.obj
 0001:00031ac4       __EH_prolog                10032ac4 f   LIBCMT:ehprolog.obj
 0001:00031af0       _strrchr                   10032af0 f   LIBCMT:strrchr.obj
 0001:00031b1d       __forcdecpt_l              10032b1d f   LIBCMT:cvt.obj
 0001:00031b91       __cropzeros_l              10032b91 f   LIBCMT:cvt.obj
 0001:00031c13       __positive                 10032c13 f   LIBCMT:cvt.obj
 0001:00031c2f       __fassign_l                10032c2f f   LIBCMT:cvt.obj
 0001:00031c71       __fassign                  10032c71 f   LIBCMT:cvt.obj
 0001:00031caa       __forcdecpt                10032caa f   LIBCMT:cvt.obj
 0001:00031cbd       __cropzeros                10032cbd f   LIBCMT:cvt.obj
 0001:00031e31       __cftoe_l                  10032e31 f   LIBCMT:cvt.obj
 0001:00031ef8       __cftoe                    10032ef8 f   LIBCMT:cvt.obj
 0001:00031f18       __cftoa_l                  10032f18 f   LIBCMT:cvt.obj
 0001:00032391       __cftof_l                  10033391 f   LIBCMT:cvt.obj
 0001:00032452       __cftog_l                  10033452 f   LIBCMT:cvt.obj
 0001:0003253f       __cfltcvt_l                1003353f f   LIBCMT:cvt.obj
 0001:000325c7       __cfltcvt                  100335c7 f   LIBCMT:cvt.obj
 0001:000325ea       __setdefaultprecision      100335ea f   LIBCMT:fp8.obj
 0001:00032612       __raise_exc_ex             10033612 f   LIBCMT:_fpexcept_.obj
 0001:000328ee       __raise_exc                100338ee f   LIBCMT:_fpexcept_.obj
 0001:00032911       __handle_exc               10033911 f   LIBCMT:_fpexcept_.obj
 0001:00032af5       __set_errno_from_matherr   10033af5 f   LIBCMT:_fpexcept_.obj
 0001:00032b22       __errcode                  10033b22 f   LIBCMT:_fpexcept_.obj
 0001:00032b56       __umatherr                 10033b56 f   LIBCMT:_fpexcept_.obj
 0001:00032bf6       __handle_qnan1             10033bf6 f   LIBCMT:_fpexcept_.obj
 0001:00032c4b       __except1                  10033c4b f   LIBCMT:_fpexcept_.obj
 0001:00032d15       __set_exp                  10033d15 f   LIBCMT:_util_.obj
 0001:00032d42       __sptype                   10033d42 f   LIBCMT:_util_.obj
 0001:00032da8       __decomp                   10033da8 f   LIBCMT:_util_.obj
 0001:00032e6b       __statfp                   10033e6b f   LIBCMT:_fpctrl_.obj
 0001:00032e7b       __clrfp                    10033e7b f   LIBCMT:_fpctrl_.obj
 0001:00032e8c       __ctrlfp                   10033e8c f   LIBCMT:_fpctrl_.obj
 0001:00032eb7       __set_statfp               10033eb7 f   LIBCMT:_fpctrl_.obj
 0001:00032f0f       ___set_fpsr_sse2           10033f0f f   LIBCMT:_fpctrl_.obj
 0001:00032f81       __sse2_mathfcns_init       10033f81 f   LIBCMT:_mathfcns_.obj
 0001:00032fa0       __CIpow_pentium4           10033fa0 f   LIBCMT:_pow_pentium4_.obj
 0001:00032fb9       __pow_pentium4             10033fb9     LIBCMT:_pow_pentium4_.obj
 0001:00033b11       __fFEXP                    10034b11     LIBCMT:_87tran_.obj
 0001:00033b68       __rtinfpopse               10034b68     LIBCMT:_87tran_.obj
 0001:00033b6a       __rtinfnpopse              10034b6a     LIBCMT:_87tran_.obj
 0001:00033b7a       __fFLN                     10034b7a     LIBCMT:_87tran_.obj
 0001:00033c2f       __rtinfpop                 10034c2f     LIBCMT:_87tran_.obj
 0001:00033c31       __rtinfnpop                10034c31     LIBCMT:_87tran_.obj
 0001:00033c4e       __ffexpm1                  10034c4e     LIBCMT:_87tran_.obj
 0001:00033d00       __trandisp1                10034d00 f   LIBCMT:_87disp_.obj
 0001:00033d67       __trandisp2                10034d67 f   LIBCMT:_87disp_.obj
 0001:00033df3       __rttospopde               10034df3     LIBCMT:_87disp_.obj
 0001:00033df8       __rttospop                 10034df8     LIBCMT:_87disp_.obj
 0001:00033dfa       __rtnospop                 10034dfa     LIBCMT:_87disp_.obj
 0001:00033dfc       __rttosnpop                10034dfc     LIBCMT:_87disp_.obj
 0001:00033dfd       __rtnospopde               10034dfd     LIBCMT:_87disp_.obj
 0001:00033e04       __rtzeropop                10034e04     LIBCMT:_87disp_.obj
 0001:00033e06       __rtzeronpop               10034e06     LIBCMT:_87disp_.obj
 0001:00033e0b       __rtonepop                 10034e0b     LIBCMT:_87disp_.obj
 0001:00033e0d       __rtonenpop                10034e0d     LIBCMT:_87disp_.obj
 0001:00033e12       __tosnan1                  10034e12     LIBCMT:_87disp_.obj
 0001:00033e3d       __nosnan2                  10034e3d     LIBCMT:_87disp_.obj
 0001:00033e3f       __tosnan2                  10034e3f     LIBCMT:_87disp_.obj
 0001:00033e67       __nan2                     10034e67     LIBCMT:_87disp_.obj
 0001:00033ea6       __rtindfpop                10034ea6     LIBCMT:_87disp_.obj
 0001:00033ea8       __rtindfnpop               10034ea8     LIBCMT:_87disp_.obj
 0001:00033eb9       __rttosnpopde              10034eb9     LIBCMT:_87disp_.obj
 0001:00033ec3       __rtchsifneg               10034ec3     LIBCMT:_87disp_.obj
 0001:00033ed0       __startTwoArgErrorHandling 10034ed0 f   LIBCMT:_genexcep_.obj
 0001:00033ee7       __startOneArgErrorHandling 10034ee7 f   LIBCMT:_genexcep_.obj
 0001:00033f30       __twoToTOS                 10034f30 f   LIBCMT:_common_.obj
 0001:00033f45       __load_CW                  10034f45 f   LIBCMT:_common_.obj
 0001:00033f5c       __convertTOStoQNaN         10034f5c f   LIBCMT:_common_.obj
 0001:00033f75       __fload_withFB             10034f75 f   LIBCMT:_common_.obj
 0001:00033fb8       __checkTOS_withFB          10034fb8 f   LIBCMT:_common_.obj
 0001:00033fce       __fast_exit                10034fce f   LIBCMT:_common_.obj
 0001:00033fdb       __math_exit                10034fdb f   LIBCMT:_common_.obj
 0001:00034005       __check_overflow_exit      10035005 f   LIBCMT:_common_.obj
 0001:00034019       __check_range_exit         10035019 f   LIBCMT:_common_.obj
 0001:000340bc       __d_inttype                100350bc f   LIBCMT:_powhlp_.obj
 0001:00034126       __powhlp                   10035126 f   LIBCMT:_powhlp_.obj
 0001:00034251       __rt_probe_read4@4         10035251 f   LIBCMT:sehsupp.obj
 0001:000342a0       __fltin2                   100352a0 f   LIBCMT:_cfin_.obj
 0001:00034347       __openfile                 10035347 f   LIBCMT:_open.obj
 0001:00034674       __woutput_l                10035674 f   LIBCMT:woutput.obj
 0001:0003523c       _CallDestructExceptionObject 1003623c f   LIBCMT:calldtor.obj
 0001:00035340       __ValidateEH3RN            10036340 f   LIBCMT:eh3valid.obj
 0001:00035686       __atodbl_l                 10036686 f   LIBCMT:atodbl.obj
 0001:0003572e       __atoflt_l                 1003672e f   LIBCMT:atodbl.obj
 0001:000357d6       __fptostr                  100367d6 f   LIBCMT:_fptostr.obj
 0001:00035889       ___dtold                   10036889 f   LIBCMT:_cfout_.obj
 0001:0003593c       __fltout2                  1003693c f   LIBCMT:_cfout_.obj
 0001:000359d0       __alldvrm                  100369d0 f   LIBCMT:lldvrm.obj
 0001:00035ab0       __aullshr                  10036ab0 f   LIBCMT:ullshr.obj
 0001:00035acf       __controlfp_s              10036acf f   LIBCMT:_contrlfp_.obj
 0001:00035b2e       ___libm_error_support      10036b2e f   LIBCMT:_libm_error_.obj
 0001:00035dfa       __87except                 10036dfa f   LIBCMT:_87except_.obj
 0001:00035f39       __frnd                     10036f39 f   LIBCMT:_frnd_.obj
 0001:00035f4d       __fpclass                  10036f4d f   LIBCMT:_ieeemisc_.obj
 0001:00035fea       __ld12tod                  10036fea f   LIBCMT:_intrncvt_.obj
 0001:0003653b       __ld12tof                  1003753b f   LIBCMT:_intrncvt_.obj
 0001:00036a8c       ___strgtold12_l            10037a8c f   LIBCMT:_strgtold_.obj
 0001:0003789c       __sopen_helper             1003889c f   LIBCMT:open.obj
 0001:00037960       __sopen_s                  10038960 f   LIBCMT:open.obj
 0001:00037980       __mbsnbicmp_l              10038980 f   LIBCMT:mbsnbicm.obj
 0001:00037b84       __mbsnbicmp                10038b84 f   LIBCMT:mbsnbicm.obj
 0001:00037b9e       __mbsnbcmp_l               10038b9e f   LIBCMT:mbsnbcmp.obj
 0001:00037cea       __mbsnbcmp                 10038cea f   LIBCMT:mbsnbcmp.obj
 0001:00037d04       __fputwc_nolock            10038d04 f   LIBCMT:fputwc.obj
 0001:00037e8b       _$I10_OUTPUT               10038e8b f   LIBCMT:_x10fout_.obj
 0001:000388b1       __control87                100398b1 f i LIBCMT:_ieee87_.obj
 0001:00038bc3       ___mtold12                 10039bc3 f   LIBCMT:_mantold_.obj
 0001:00038da7       __flswbuf                  10039da7 f   LIBCMT:_flswbuf.obj
 0001:00038f1c       _VerQueryValueA@16         10039f1c f   version:VERSION.dll
 0001:00038f22       _GetFileVersionInfoW@16    10039f22 f   version:VERSION.dll
 0001:00038f28       _GetFileVersionInfoSizeW@8 10039f28 f   version:VERSION.dll
 0002:00000000       __imp__GetUserNameA@8      1003b000     advapi32:ADVAPI32.dll
 0002:00000004       __imp__OpenProcessToken@12 1003b004     advapi32:ADVAPI32.dll
 0002:00000008       __imp__OpenThreadToken@16  1003b008     advapi32:ADVAPI32.dll
 0002:0000000c       __imp__GetTokenInformation@20 1003b00c     advapi32:ADVAPI32.dll
 0002:00000010       __imp__RegQueryValueExW@24 1003b010     advapi32:ADVAPI32.dll
 0002:00000014       __imp__RegOpenKeyW@12      1003b014     advapi32:ADVAPI32.dll
 0002:00000018       __imp__AllocateAndInitializeSid@44 1003b018     advapi32:ADVAPI32.dll
 0002:0000001c       __imp__FreeSid@4           1003b01c     advapi32:ADVAPI32.dll
 0002:00000020       __imp__CheckTokenMembership@12 1003b020     advapi32:ADVAPI32.dll
 0002:00000024       __imp__RegCloseKey@4       1003b024     advapi32:ADVAPI32.dll
 0002:00000028       __imp__CryptGetHashParam@20 1003b028     advapi32:ADVAPI32.dll
 0002:0000002c       __imp__CryptAcquireContextW@20 1003b02c     advapi32:ADVAPI32.dll
 0002:00000030       __imp__CryptVerifySignatureW@24 1003b030     advapi32:ADVAPI32.dll
 0002:00000034       __imp__CryptReleaseContext@8 1003b034     advapi32:ADVAPI32.dll
 0002:00000038       __imp__CryptImportKey@24   1003b038     advapi32:ADVAPI32.dll
 0002:0000003c       __imp__CryptCreateHash@20  1003b03c     advapi32:ADVAPI32.dll
 0002:00000040       __imp__CryptDestroyKey@4   1003b040     advapi32:ADVAPI32.dll
 0002:00000044       __imp__CryptDestroyHash@4  1003b044     advapi32:ADVAPI32.dll
 0002:00000048       __imp__CryptHashData@16    1003b048     advapi32:ADVAPI32.dll
 0002:0000004c       __imp__RegSetValueExA@24   1003b04c     advapi32:ADVAPI32.dll
 0002:00000050       __imp__RegOpenKeyExA@20    1003b050     advapi32:ADVAPI32.dll
 0002:00000054       __imp__RegCreateKeyA@12    1003b054     advapi32:ADVAPI32.dll
 0002:00000058       __imp__RegQueryValueExA@24 1003b058     advapi32:ADVAPI32.dll
 0002:0000005c       \177ADVAPI32_NULL_THUNK_DATA 1003b05c     advapi32:ADVAPI32.dll
 0002:00000060       __imp__CreateFontW@56      1003b060     gdi32:GDI32.dll
 0002:00000064       __imp__CreateSolidBrush@4  1003b064     gdi32:GDI32.dll
 0002:00000068       __imp__CreateCompatibleBitmap@12 1003b068     gdi32:GDI32.dll
 0002:0000006c       __imp__DeleteDC@4          1003b06c     gdi32:GDI32.dll
 0002:00000070       __imp__BitBlt@36           1003b070     gdi32:GDI32.dll
 0002:00000074       __imp__Polygon@12          1003b074     gdi32:GDI32.dll
 0002:00000078       __imp__Polyline@12         1003b078     gdi32:GDI32.dll
 0002:0000007c       __imp__CreatePen@12        1003b07c     gdi32:GDI32.dll
 0002:00000080       __imp__CreateCompatibleDC@4 1003b080     gdi32:GDI32.dll
 0002:00000084       __imp__SetTextColor@8      1003b084     gdi32:GDI32.dll
 0002:00000088       __imp__SetBkMode@8         1003b088     gdi32:GDI32.dll
 0002:0000008c       __imp__GetObjectW@12       1003b08c     gdi32:GDI32.dll
 0002:00000090       __imp__GetTextExtentPoint32W@16 1003b090     gdi32:GDI32.dll
 0002:00000094       __imp__GetTextMetricsW@8   1003b094     gdi32:GDI32.dll
 0002:00000098       __imp__SelectObject@8      1003b098     gdi32:GDI32.dll
 0002:0000009c       __imp__DeleteObject@4      1003b09c     gdi32:GDI32.dll
 0002:000000a0       __imp__CreateFontIndirectW@4 1003b0a0     gdi32:GDI32.dll
 0002:000000a4       __imp__Rectangle@20        1003b0a4     gdi32:GDI32.dll
 0002:000000a8       __imp__CreateDIBSection@24 1003b0a8     gdi32:GDI32.dll
 0002:000000ac       __imp__GetCurrentObject@8  1003b0ac     gdi32:GDI32.dll
 0002:000000b0       \177GDI32_NULL_THUNK_DATA  1003b0b0     gdi32:GDI32.dll
 0002:000000b4       __imp__DisableThreadLibraryCalls@4 1003b0b4     kernel32:KERNEL32.dll
 0002:000000b8       __imp__GetTickCount@0      1003b0b8     kernel32:KERNEL32.dll
 0002:000000bc       __imp__GetProcessHeap@0    1003b0bc     kernel32:KERNEL32.dll
 0002:000000c0       __imp__SetEndOfFile@4      1003b0c0     kernel32:KERNEL32.dll
 0002:000000c4       __imp__SetStdHandle@8      1003b0c4     kernel32:KERNEL32.dll
 0002:000000c8       __imp__WriteConsoleW@20    1003b0c8     kernel32:KERNEL32.dll
 0002:000000cc       __imp__CreateFileA@28      1003b0cc     kernel32:KERNEL32.dll
 0002:000000d0       __imp__WritePrivateProfileStringW@16 1003b0d0     kernel32:KERNEL32.dll
 0002:000000d4       __imp__lstrcpynW@12        1003b0d4     kernel32:KERNEL32.dll
 0002:000000d8       __imp__lstrcpynA@12        1003b0d8     kernel32:KERNEL32.dll
 0002:000000dc       __imp__SetErrorMode@4      1003b0dc     kernel32:KERNEL32.dll
 0002:000000e0       __imp__CreateProcessW@40   1003b0e0     kernel32:KERNEL32.dll
 0002:000000e4       __imp__lstrcpyA@8          1003b0e4     kernel32:KERNEL32.dll
 0002:000000e8       __imp__GlobalMemoryStatus@4 1003b0e8     kernel32:KERNEL32.dll
 0002:000000ec       __imp__GetSystemInfo@4     1003b0ec     kernel32:KERNEL32.dll
 0002:000000f0       __imp__VirtualQuery@12     1003b0f0     kernel32:KERNEL32.dll
 0002:000000f4       __imp__GetFileSize@8       1003b0f4     kernel32:KERNEL32.dll
 0002:000000f8       __imp__GetFileTime@16      1003b0f8     kernel32:KERNEL32.dll
 0002:000000fc       __imp__lstrlenA@4          1003b0fc     kernel32:KERNEL32.dll
 0002:00000100       __imp__FileTimeToLocalFileTime@8 1003b100     kernel32:KERNEL32.dll
 0002:00000104       __imp__FileTimeToDosDateTime@12 1003b104     kernel32:KERNEL32.dll
 0002:00000108       __imp__SetEnvironmentVariableA@8 1003b108     kernel32:KERNEL32.dll
 0002:0000010c       __imp__CompareStringW@24   1003b10c     kernel32:KERNEL32.dll
 0002:00000110       __imp__WaitForSingleObjectEx@12 1003b110     kernel32:KERNEL32.dll
 0002:00000114       __imp__InitializeCriticalSection@4 1003b114     kernel32:KERNEL32.dll
 0002:00000118       __imp__LeaveCriticalSection@4 1003b118     kernel32:KERNEL32.dll
 0002:0000011c       __imp__EnterCriticalSection@4 1003b11c     kernel32:KERNEL32.dll
 0002:00000120       __imp__CreateMutexA@12     1003b120     kernel32:KERNEL32.dll
 0002:00000124       __imp__DeleteCriticalSection@4 1003b124     kernel32:KERNEL32.dll
 0002:00000128       __imp__ReleaseMutex@4      1003b128     kernel32:KERNEL32.dll
 0002:0000012c       __imp__CloseHandle@4       1003b12c     kernel32:KERNEL32.dll
 0002:00000130       __imp__CreateTimerQueue@0  1003b130     kernel32:KERNEL32.dll
 0002:00000134       __imp__DeleteTimerQueueEx@8 1003b134     kernel32:KERNEL32.dll
 0002:00000138       __imp__FreeLibrary@4       1003b138     kernel32:KERNEL32.dll
 0002:0000013c       __imp__GetCurrentProcess@0 1003b13c     kernel32:KERNEL32.dll
 0002:00000140       __imp__GetCurrentThread@0  1003b140     kernel32:KERNEL32.dll
 0002:00000144       __imp__WideCharToMultiByte@32 1003b144     kernel32:KERNEL32.dll
 0002:00000148       __imp__LoadLibraryW@4      1003b148     kernel32:KERNEL32.dll
 0002:0000014c       __imp__GetModuleFileNameW@12 1003b14c     kernel32:KERNEL32.dll
 0002:00000150       __imp__GetProcAddress@8    1003b150     kernel32:KERNEL32.dll
 0002:00000154       __imp__CreateTimerQueueTimer@28 1003b154     kernel32:KERNEL32.dll
 0002:00000158       __imp__SetCurrentDirectoryW@4 1003b158     kernel32:KERNEL32.dll
 0002:0000015c       __imp__GetCurrentThreadId@0 1003b15c     kernel32:KERNEL32.dll
 0002:00000160       __imp__GetVersion@0        1003b160     kernel32:KERNEL32.dll
 0002:00000164       __imp__DeleteFileW@4       1003b164     kernel32:KERNEL32.dll
 0002:00000168       __imp__FindResourceW@12    1003b168     kernel32:KERNEL32.dll
 0002:0000016c       __imp__LoadResource@8      1003b16c     kernel32:KERNEL32.dll
 0002:00000170       __imp__SizeofResource@8    1003b170     kernel32:KERNEL32.dll
 0002:00000174       __imp__LockResource@4      1003b174     kernel32:KERNEL32.dll
 0002:00000178       __imp__QueryPerformanceCounter@4 1003b178     kernel32:KERNEL32.dll
 0002:0000017c       __imp__GetVersionExW@4     1003b17c     kernel32:KERNEL32.dll
 0002:00000180       __imp__QueryPerformanceFrequency@4 1003b180     kernel32:KERNEL32.dll
 0002:00000184       __imp__WaitForSingleObject@8 1003b184     kernel32:KERNEL32.dll
 0002:00000188       __imp__ConnectNamedPipe@8  1003b188     kernel32:KERNEL32.dll
 0002:0000018c       __imp__CreateNamedPipeW@32 1003b18c     kernel32:KERNEL32.dll
 0002:00000190       __imp__WriteFile@20        1003b190     kernel32:KERNEL32.dll
 0002:00000194       __imp__ReadFile@20         1003b194     kernel32:KERNEL32.dll
 0002:00000198       __imp__GetOverlappedResult@16 1003b198     kernel32:KERNEL32.dll
 0002:0000019c       __imp__GetLastError@0      1003b19c     kernel32:KERNEL32.dll
 0002:000001a0       __imp__CreateEventW@16     1003b1a0     kernel32:KERNEL32.dll
 0002:000001a4       __imp__CreateThread@24     1003b1a4     kernel32:KERNEL32.dll
 0002:000001a8       __imp__CopyFileW@12        1003b1a8     kernel32:KERNEL32.dll
 0002:000001ac       __imp__FindFirstFileW@8    1003b1ac     kernel32:KERNEL32.dll
 0002:000001b0       __imp__MoveFileExW@12      1003b1b0     kernel32:KERNEL32.dll
 0002:000001b4       __imp__CreateDirectoryW@8  1003b1b4     kernel32:KERNEL32.dll
 0002:000001b8       __imp__CreateFileW@28      1003b1b8     kernel32:KERNEL32.dll
 0002:000001bc       __imp__GetTempPathW@8      1003b1bc     kernel32:KERNEL32.dll
 0002:000001c0       __imp__FindClose@4         1003b1c0     kernel32:KERNEL32.dll
 0002:000001c4       __imp__RemoveDirectoryW@4  1003b1c4     kernel32:KERNEL32.dll
 0002:000001c8       __imp__FindNextFileW@8     1003b1c8     kernel32:KERNEL32.dll
 0002:000001cc       __imp__SetFileAttributesW@8 1003b1cc     kernel32:KERNEL32.dll
 0002:000001d0       __imp__GetFullPathNameW@16 1003b1d0     kernel32:KERNEL32.dll
 0002:000001d4       __imp__CreateMutexW@12     1003b1d4     kernel32:KERNEL32.dll
 0002:000001d8       __imp__CopyFileExW@24      1003b1d8     kernel32:KERNEL32.dll
 0002:000001dc       __imp__FindFirstFileExW@24 1003b1dc     kernel32:KERNEL32.dll
 0002:000001e0       __imp__TerminateThread@8   1003b1e0     kernel32:KERNEL32.dll
 0002:000001e4       __imp__lstrlenW@4          1003b1e4     kernel32:KERNEL32.dll
 0002:000001e8       __imp__OpenMutexW@12       1003b1e8     kernel32:KERNEL32.dll
 0002:000001ec       __imp__WaitForMultipleObjects@16 1003b1ec     kernel32:KERNEL32.dll
 0002:000001f0       __imp__lstrcmpiW@8         1003b1f0     kernel32:KERNEL32.dll
 0002:000001f4       __imp__lstrcpyW@8          1003b1f4     kernel32:KERNEL32.dll
 0002:000001f8       __imp__GetVolumeInformationW@32 1003b1f8     kernel32:KERNEL32.dll
 0002:000001fc       __imp__ExpandEnvironmentStringsA@12 1003b1fc     kernel32:KERNEL32.dll
 0002:00000200       __imp__SetNamedPipeHandleState@16 1003b200     kernel32:KERNEL32.dll
 0002:00000204       __imp__EncodePointer@4     1003b204     kernel32:KERNEL32.dll
 0002:00000208       __imp__DecodePointer@4     1003b208     kernel32:KERNEL32.dll
 0002:0000020c       __imp__GetCommandLineA@0   1003b20c     kernel32:KERNEL32.dll
 0002:00000210       __imp__HeapFree@12         1003b210     kernel32:KERNEL32.dll
 0002:00000214       __imp__GetSystemTimeAsFileTime@4 1003b214     kernel32:KERNEL32.dll
 0002:00000218       __imp__HeapAlloc@12        1003b218     kernel32:KERNEL32.dll
 0002:0000021c       __imp__HeapReAlloc@16      1003b21c     kernel32:KERNEL32.dll
 0002:00000220       __imp__RaiseException@16   1003b220     kernel32:KERNEL32.dll
 0002:00000224       __imp__Sleep@4             1003b224     kernel32:KERNEL32.dll
 0002:00000228       __imp__HeapSize@12         1003b228     kernel32:KERNEL32.dll
 0002:0000022c       __imp__GetModuleHandleW@4  1003b22c     kernel32:KERNEL32.dll
 0002:00000230       __imp__ExitProcess@4       1003b230     kernel32:KERNEL32.dll
 0002:00000234       __imp__IsProcessorFeaturePresent@4 1003b234     kernel32:KERNEL32.dll
 0002:00000238       __imp__UnhandledExceptionFilter@4 1003b238     kernel32:KERNEL32.dll
 0002:0000023c       __imp__SetUnhandledExceptionFilter@4 1003b23c     kernel32:KERNEL32.dll
 0002:00000240       __imp__IsDebuggerPresent@0 1003b240     kernel32:KERNEL32.dll
 0002:00000244       __imp__TerminateProcess@8  1003b244     kernel32:KERNEL32.dll
 0002:00000248       __imp__GetStdHandle@4      1003b248     kernel32:KERNEL32.dll
 0002:0000024c       __imp__GetCPInfo@8         1003b24c     kernel32:KERNEL32.dll
 0002:00000250       __imp__InterlockedIncrement@4 1003b250     kernel32:KERNEL32.dll
 0002:00000254       __imp__InterlockedDecrement@4 1003b254     kernel32:KERNEL32.dll
 0002:00000258       __imp__GetACP@0            1003b258     kernel32:KERNEL32.dll
 0002:0000025c       __imp__GetOEMCP@0          1003b25c     kernel32:KERNEL32.dll
 0002:00000260       __imp__IsValidCodePage@4   1003b260     kernel32:KERNEL32.dll
 0002:00000264       __imp__TlsAlloc@0          1003b264     kernel32:KERNEL32.dll
 0002:00000268       __imp__TlsGetValue@4       1003b268     kernel32:KERNEL32.dll
 0002:0000026c       __imp__TlsSetValue@8       1003b26c     kernel32:KERNEL32.dll
 0002:00000270       __imp__TlsFree@4           1003b270     kernel32:KERNEL32.dll
 0002:00000274       __imp__SetLastError@4      1003b274     kernel32:KERNEL32.dll
 0002:00000278       __imp__SetHandleCount@4    1003b278     kernel32:KERNEL32.dll
 0002:0000027c       __imp__InitializeCriticalSectionAndSpinCount@8 1003b27c     kernel32:KERNEL32.dll
 0002:00000280       __imp__GetFileType@4       1003b280     kernel32:KERNEL32.dll
 0002:00000284       __imp__GetStartupInfoW@4   1003b284     kernel32:KERNEL32.dll
 0002:00000288       __imp__GetModuleFileNameA@12 1003b288     kernel32:KERNEL32.dll
 0002:0000028c       __imp__FreeEnvironmentStringsW@4 1003b28c     kernel32:KERNEL32.dll
 0002:00000290       __imp__GetEnvironmentStringsW@0 1003b290     kernel32:KERNEL32.dll
 0002:00000294       __imp__HeapCreate@12       1003b294     kernel32:KERNEL32.dll
 0002:00000298       __imp__HeapDestroy@4       1003b298     kernel32:KERNEL32.dll
 0002:0000029c       __imp__GetCurrentProcessId@0 1003b29c     kernel32:KERNEL32.dll
 0002:000002a0       __imp__LCMapStringW@24     1003b2a0     kernel32:KERNEL32.dll
 0002:000002a4       __imp__GetConsoleCP@0      1003b2a4     kernel32:KERNEL32.dll
 0002:000002a8       __imp__GetConsoleMode@8    1003b2a8     kernel32:KERNEL32.dll
 0002:000002ac       __imp__FlushFileBuffers@4  1003b2ac     kernel32:KERNEL32.dll
 0002:000002b0       __imp__RtlUnwind@16        1003b2b0     kernel32:KERNEL32.dll
 0002:000002b4       __imp__GetTimeZoneInformation@4 1003b2b4     kernel32:KERNEL32.dll
 0002:000002b8       __imp__SetFilePointer@16   1003b2b8     kernel32:KERNEL32.dll
 0002:000002bc       __imp__GetStringTypeW@16   1003b2bc     kernel32:KERNEL32.dll
 0002:000002c0       __imp__MultiByteToWideChar@24 1003b2c0     kernel32:KERNEL32.dll
 0002:000002c4       \177KERNEL32_NULL_THUNK_DATA 1003b2c4     kernel32:KERNEL32.dll
 0002:000002c8       __imp__AlphaBlend@44       1003b2c8     MSImg32:MSIMG32.dll
 0002:000002cc       \177MSIMG32_NULL_THUNK_DATA 1003b2cc     MSImg32:MSIMG32.dll
 0002:000002d0       __imp__ShellExecuteExW@4   1003b2d0     shell32:SHELL32.dll
 0002:000002d4       __imp__SHGetFolderPathW@20 1003b2d4     shell32:SHELL32.dll
 0002:000002d8       \177SHELL32_NULL_THUNK_DATA 1003b2d8     shell32:SHELL32.dll
 0002:000002dc       __imp__PathSkipRootW@4     1003b2dc     WebCommonLib:SHLWAPI.dll
 0002:000002e0       __imp__PathRemoveFileSpecW@4 1003b2e0     WebCommonLib:SHLWAPI.dll
 0002:000002e4       __imp__PathCombineW@12     1003b2e4     WebCommonLib:SHLWAPI.dll
 0002:000002e8       __imp__PathAppendW@8       1003b2e8     WebCommonLib:SHLWAPI.dll
 0002:000002ec       __imp__PathStripToRootW@4  1003b2ec     WebCommonLib:SHLWAPI.dll
 0002:000002f0       \177SHLWAPI_NULL_THUNK_DATA 1003b2f0     WebCommonLib:SHLWAPI.dll
 0002:000002f4       __imp__CallWindowProcW@20  1003b2f4     user32:USER32.dll
 0002:000002f8       __imp__GetSystemMetrics@4  1003b2f8     user32:USER32.dll
 0002:000002fc       __imp__GetWindowTextW@12   1003b2fc     user32:USER32.dll
 0002:00000300       __imp__LoadCursorW@8       1003b300     user32:USER32.dll
 0002:00000304       __imp__SetCursor@4         1003b304     user32:USER32.dll
 0002:00000308       __imp__GetForegroundWindow@0 1003b308     user32:USER32.dll
 0002:0000030c       __imp__GetParent@4         1003b30c     user32:USER32.dll
 0002:00000310       __imp__MessageBoxW@16      1003b310     user32:USER32.dll
 0002:00000314       __imp__wsprintfW           1003b314     user32:USER32.dll
 0002:00000318       __imp__CreatePopupMenu@0   1003b318     user32:USER32.dll
 0002:0000031c       __imp__GetSubMenu@8        1003b31c     user32:USER32.dll
 0002:00000320       __imp__EnableMenuItem@12   1003b320     user32:USER32.dll
 0002:00000324       __imp__LoadMenuW@8         1003b324     user32:USER32.dll
 0002:00000328       __imp__GetWindowRect@8     1003b328     user32:USER32.dll
 0002:0000032c       __imp__MessageBoxA@16      1003b32c     user32:USER32.dll
 0002:00000330       __imp__GetClientRect@8     1003b330     user32:USER32.dll
 0002:00000334       __imp__DrawTextW@20        1003b334     user32:USER32.dll
 0002:00000338       __imp__InflateRect@12      1003b338     user32:USER32.dll
 0002:0000033c       __imp__GetSysColorBrush@4  1003b33c     user32:USER32.dll
 0002:00000340       __imp__FillRect@12         1003b340     user32:USER32.dll
 0002:00000344       __imp__GetSysColor@4       1003b344     user32:USER32.dll
 0002:00000348       __imp__InvalidateRect@12   1003b348     user32:USER32.dll
 0002:0000034c       __imp__PtInRect@12         1003b34c     user32:USER32.dll
 0002:00000350       __imp__AdjustWindowRectEx@16 1003b350     user32:USER32.dll
 0002:00000354       __imp__CopyRect@8          1003b354     user32:USER32.dll
 0002:00000358       __imp__ReleaseDC@8         1003b358     user32:USER32.dll
 0002:0000035c       __imp__SetRect@20          1003b35c     user32:USER32.dll
 0002:00000360       __imp__GetDC@4             1003b360     user32:USER32.dll
 0002:00000364       __imp__IsRectEmpty@4       1003b364     user32:USER32.dll
 0002:00000368       __imp__GetMenuItemCount@4  1003b368     user32:USER32.dll
 0002:0000036c       __imp__EndPaint@8          1003b36c     user32:USER32.dll
 0002:00000370       __imp__BeginPaint@8        1003b370     user32:USER32.dll
 0002:00000374       __imp__ShowWindow@8        1003b374     user32:USER32.dll
 0002:00000378       __imp__SetWindowPos@28     1003b378     user32:USER32.dll
 0002:0000037c       __imp__DestroyWindow@4     1003b37c     user32:USER32.dll
 0002:00000380       __imp__CreateWindowExW@48  1003b380     user32:USER32.dll
 0002:00000384       __imp__wvsprintfA@12       1003b384     user32:USER32.dll
 0002:00000388       __imp__wsprintfA           1003b388     user32:USER32.dll
 0002:0000038c       __imp__PostMessageW@16     1003b38c     user32:USER32.dll
 0002:00000390       __imp__IsWindow@4          1003b390     user32:USER32.dll
 0002:00000394       __imp__AppendMenuW@16      1003b394     user32:USER32.dll
 0002:00000398       __imp__RemoveMenu@12       1003b398     user32:USER32.dll
 0002:0000039c       __imp__LoadBitmapW@8       1003b39c     user32:USER32.dll
 0002:000003a0       __imp__SystemParametersInfoW@16 1003b3a0     user32:USER32.dll
 0002:000003a4       __imp__GetWindowLongW@8    1003b3a4     user32:USER32.dll
 0002:000003a8       __imp__SetWindowLongW@12   1003b3a8     user32:USER32.dll
 0002:000003ac       __imp__DestroyMenu@4       1003b3ac     user32:USER32.dll
 0002:000003b0       __imp__GetClassLongW@8     1003b3b0     user32:USER32.dll
 0002:000003b4       __imp__GetAncestor@8       1003b3b4     user32:USER32.dll
 0002:000003b8       __imp__ClientToScreen@8    1003b3b8     user32:USER32.dll
 0002:000003bc       __imp__WindowFromPoint@8   1003b3bc     user32:USER32.dll
 0002:000003c0       __imp__UnregisterClassW@8  1003b3c0     user32:USER32.dll
 0002:000003c4       __imp__RegisterClassExW@4  1003b3c4     user32:USER32.dll
 0002:000003c8       __imp__LoadImageW@24       1003b3c8     user32:USER32.dll
 0002:000003cc       __imp__DefWindowProcW@16   1003b3cc     user32:USER32.dll
 0002:000003d0       __imp__SendMessageW@16     1003b3d0     user32:USER32.dll
 0002:000003d4       __imp__SetCapture@4        1003b3d4     user32:USER32.dll
 0002:000003d8       __imp__SendInput@12        1003b3d8     user32:USER32.dll
 0002:000003dc       __imp__ReleaseCapture@0    1003b3dc     user32:USER32.dll
 0002:000003e0       __imp__GetMenuItemInfoW@16 1003b3e0     user32:USER32.dll
 0002:000003e4       \177USER32_NULL_THUNK_DATA 1003b3e4     user32:USER32.dll
 0002:000003e8       __imp__GetFileVersionInfoSizeW@8 1003b3e8     version:VERSION.dll
 0002:000003ec       __imp__GetFileVersionInfoW@16 1003b3ec     version:VERSION.dll
 0002:000003f0       __imp__VerQueryValueA@16   1003b3f0     version:VERSION.dll
 0002:000003f4       \177VERSION_NULL_THUNK_DATA 1003b3f4     version:VERSION.dll
 0002:000003f8       __imp__timeGetTime@0       1003b3f8     winmm:WINMM.dll
 0002:000003fc       \177WINMM_NULL_THUNK_DATA  1003b3fc     winmm:WINMM.dll
 0002:00000400       __imp__CoTaskMemFree@4     1003b400     ole32:ole32.dll
 0002:00000404       __imp__CoCreateGuid@4      1003b404     ole32:ole32.dll
 0002:00000408       __imp__StringFromGUID2@12  1003b408     ole32:ole32.dll
 0002:0000040c       \177ole32_NULL_THUNK_DATA  1003b40c     ole32:ole32.dll
 0002:00000410       ___xc_a                    1003b410     LIBCMT:crt0init.obj
 0002:0000043c       ___xc_z                    1003b43c     LIBCMT:crt0init.obj
 0002:00000440       ___xi_a                    1003b440     LIBCMT:crt0init.obj
 0002:00000458       ___xi_z                    1003b458     LIBCMT:crt0init.obj
 0002:0000045c       ___xp_a                    1003b45c     LIBCMT:crt0init.obj
 0002:00000468       ___xp_z                    1003b468     LIBCMT:crt0init.obj
 0002:0000046c       ___xt_a                    1003b46c     LIBCMT:crt0init.obj
 0002:00000470       ___xt_z                    1003b470     LIBCMT:crt0init.obj
 0002:000004a0       ??_7logic_error@std@@6B@   1003b4a0     libcpmt:xthrow.obj
 0002:000004ac       ??_7length_error@std@@6B@  1003b4ac     libcpmt:xthrow.obj
 0002:000004b8       ??_7out_of_range@std@@6B@  1003b4b8     libcpmt:xthrow.obj
 0002:000004c4       ??_7bad_alloc@std@@6B@     1003b4c4     LIBCMT:new.obj
 0002:000004cc       ??_C@_0P@GHFPNOJB@bad?5allocation?$AA@ 1003b4cc     LIBCMT:new.obj
 0002:000004e0       ??_7exception@std@@6B@     1003b4e0     LIBCMT:stdexcpt.obj
 0002:000004e8       ??_C@_0BC@EOODALEL@Unknown?5exception?$AA@ 1003b4e8     LIBCMT:stdexcpt.obj
 0002:00000500       ??_7type_info@@6B@         1003b500     LIBCMT:typinfo.obj
 0002:00000504       __pDefaultRawDllMain       1003b504     LIBCMT:dllcrt0.obj
 0002:00000504       __pRawDllMain              1003b504     LIBCMT:dllcrt0.obj
 0002:00000528       ??_C@_0P@MIGLKIOC@CorExitProcess?$AA@ 1003b528     LIBCMT:crt0dat.obj
 0002:00000538       ??_C@_1BI@BGOHAHKC@?$AAm?$AAs?$AAc?$AAo?$AAr?$AAe?$AAe?$AA?4?$AAd?$AAl?$AAl?$AA?$AA@ 1003b538     LIBCMT:crt0dat.obj
 0002:00000550       ??_C@_1BO@BKOMIGKJ@?$AAr?$AAu?$AAn?$AAt?$AAi?$AAm?$AAe?$AA?5?$AAe?$AAr?$AAr?$AAo?$AAr?$AA?5?$AA?$AA@ 1003b550     LIBCMT:crt0msg.obj
 0002:00000570       ??_C@_15JNBOKNOG@?$AA?$AN?$AA?6?$AA?$AA@ 1003b570     LIBCMT:crt0msg.obj
 0002:00000578       ??_C@_1BM@JBBEPPHI@?$AAT?$AAL?$AAO?$AAS?$AAS?$AA?5?$AAe?$AAr?$AAr?$AAo?$AAr?$AA?$AN?$AA?6?$AA?$AA@ 1003b578     LIBCMT:crt0msg.obj
 0002:00000594       ??_C@_1BK@KMOMNAAI@?$AAS?$AAI?$AAN?$AAG?$AA?5?$AAe?$AAr?$AAr?$AAo?$AAr?$AA?$AN?$AA?6?$AA?$AA@ 1003b594     LIBCMT:crt0msg.obj
 0002:000005b0       ??_C@_1BO@BFCDCGC@?$AAD?$AAO?$AAM?$AAA?$AAI?$AAN?$AA?5?$AAe?$AAr?$AAr?$AAo?$AAr?$AA?$AN?$AA?6?$AA?$AA@ 1003b5b0     LIBCMT:crt0msg.obj
 0002:000005d0       ??_C@_1BOO@KGEDBGAJ@?$AAR?$AA6?$AA0?$AA3?$AA3?$AA?$AN?$AA?6?$AA?9?$AA?5?$AAA?$AAt?$AAt?$AAe?$AAm?$AAp?$AAt?$AA?5?$AAt?$AAo?$AA?5?$AAu?$AAs?$AAe?$AA?5?$AAM?$AAS?$AAI?$AAL?$AA?5?$AAc?$AAo?$AAd@ 1003b5d0     LIBCMT:crt0msg.obj
 0002:000007c0       ??_C@_1GG@GOPILAJP@?$AAR?$AA6?$AA0?$AA3?$AA2?$AA?$AN?$AA?6?$AA?9?$AA?5?$AAn?$AAo?$AAt?$AA?5?$AAe?$AAn?$AAo?$AAu?$AAg?$AAh?$AA?5?$AAs?$AAp?$AAa?$AAc?$AAe?$AA?5?$AAf?$AAo?$AAr?$AA?5?$AAl?$AAo@ 1003b7c0     LIBCMT:crt0msg.obj
 0002:00000828       ??_C@_1MG@ENCOOIDF@?$AAR?$AA6?$AA0?$AA3?$AA1?$AA?$AN?$AA?6?$AA?9?$AA?5?$AAA?$AAt?$AAt?$AAe?$AAm?$AAp?$AAt?$AA?5?$AAt?$AAo?$AA?5?$AAi?$AAn?$AAi?$AAt?$AAi?$AAa?$AAl?$AAi?$AAz?$AAe?$AA?5?$AAt@ 1003b828     LIBCMT:crt0msg.obj
 0002:000008f0       ??_C@_1DO@BMFCDCD@?$AAR?$AA6?$AA0?$AA3?$AA0?$AA?$AN?$AA?6?$AA?9?$AA?5?$AAC?$AAR?$AAT?$AA?5?$AAn?$AAo?$AAt?$AA?5?$AAi?$AAn?$AAi?$AAt?$AAi?$AAa?$AAl?$AAi?$AAz?$AAe?$AAd?$AA?$AN?$AA?6?$AA?$AA@ 1003b8f0     LIBCMT:crt0msg.obj
 0002:00000930       ??_C@_1EK@HHFLMAOL@?$AAR?$AA6?$AA0?$AA2?$AA8?$AA?$AN?$AA?6?$AA?9?$AA?5?$AAu?$AAn?$AAa?$AAb?$AAl?$AAe?$AA?5?$AAt?$AAo?$AA?5?$AAi?$AAn?$AAi?$AAt?$AAi?$AAa?$AAl?$AAi?$AAz?$AAe?$AA?5?$AAh?$AAe@ 1003b930     LIBCMT:crt0msg.obj
 0002:00000980       ??_C@_1GK@MFGOKLAG@?$AAR?$AA6?$AA0?$AA2?$AA7?$AA?$AN?$AA?6?$AA?9?$AA?5?$AAn?$AAo?$AAt?$AA?5?$AAe?$AAn?$AAo?$AAu?$AAg?$AAh?$AA?5?$AAs?$AAp?$AAa?$AAc?$AAe?$AA?5?$AAf?$AAo?$AAr?$AA?5?$AAl?$AAo@ 1003b980     LIBCMT:crt0msg.obj
 0002:000009f0       ??_C@_1GK@MCAAGJMO@?$AAR?$AA6?$AA0?$AA2?$AA6?$AA?$AN?$AA?6?$AA?9?$AA?5?$AAn?$AAo?$AAt?$AA?5?$AAe?$AAn?$AAo?$AAu?$AAg?$AAh?$AA?5?$AAs?$AAp?$AAa?$AAc?$AAe?$AA?5?$AAf?$AAo?$AAr?$AA?5?$AAs?$AAt@ 1003b9f0     LIBCMT:crt0msg.obj
 0002:00000a60       ??_C@_1EM@MAADIHMB@?$AAR?$AA6?$AA0?$AA2?$AA5?$AA?$AN?$AA?6?$AA?9?$AA?5?$AAp?$AAu?$AAr?$AAe?$AA?5?$AAv?$AAi?$AAr?$AAt?$AAu?$AAa?$AAl?$AA?5?$AAf?$AAu?$AAn?$AAc?$AAt?$AAi?$AAo?$AAn?$AA?5?$AAc@ 1003ba60     LIBCMT:crt0msg.obj
 0002:00000ab0       ??_C@_1GK@FHCKBEFA@?$AAR?$AA6?$AA0?$AA2?$AA4?$AA?$AN?$AA?6?$AA?9?$AA?5?$AAn?$AAo?$AAt?$AA?5?$AAe?$AAn?$AAo?$AAu?$AAg?$AAh?$AA?5?$AAs?$AAp?$AAa?$AAc?$AAe?$AA?5?$AAf?$AAo?$AAr?$AA?5?$AA_?$AAo@ 1003bab0     LIBCMT:crt0msg.obj
 0002:00000b20       ??_C@_1FC@ECHBIFBC@?$AAR?$AA6?$AA0?$AA1?$AA9?$AA?$AN?$AA?6?$AA?9?$AA?5?$AAu?$AAn?$AAa?$AAb?$AAl?$AAe?$AA?5?$AAt?$AAo?$AA?5?$AAo?$AAp?$AAe?$AAn?$AA?5?$AAc?$AAo?$AAn?$AAs?$AAo?$AAl?$AAe?$AA?5@ 1003bb20     LIBCMT:crt0msg.obj
 0002:00000b78       ??_C@_1EC@JIBHAOPH@?$AAR?$AA6?$AA0?$AA1?$AA8?$AA?$AN?$AA?6?$AA?9?$AA?5?$AAu?$AAn?$AAe?$AAx?$AAp?$AAe?$AAc?$AAt?$AAe?$AAd?$AA?5?$AAh?$AAe?$AAa?$AAp?$AA?5?$AAe?$AAr?$AAr?$AAo?$AAr?$AA?$AN?$AA?6@ 1003bb78     LIBCMT:crt0msg.obj
 0002:00000bc0       ??_C@_1FK@BEOGODMC@?$AAR?$AA6?$AA0?$AA1?$AA7?$AA?$AN?$AA?6?$AA?9?$AA?5?$AAu?$AAn?$AAe?$AAx?$AAp?$AAe?$AAc?$AAt?$AAe?$AAd?$AA?5?$AAm?$AAu?$AAl?$AAt?$AAi?$AAt?$AAh?$AAr?$AAe?$AAa?$AAd?$AA?5@ 1003bbc0     LIBCMT:crt0msg.obj
 0002:00000c20       ??_C@_1FI@LOGNIKDM@?$AAR?$AA6?$AA0?$AA1?$AA6?$AA?$AN?$AA?6?$AA?9?$AA?5?$AAn?$AAo?$AAt?$AA?5?$AAe?$AAn?$AAo?$AAu?$AAg?$AAh?$AA?5?$AAs?$AAp?$AAa?$AAc?$AAe?$AA?5?$AAf?$AAo?$AAr?$AA?5?$AAt?$AAh@ 1003bc20     LIBCMT:crt0msg.obj
 0002:00000c78       ??_C@_1EG@BEHAGFJD@?$AAR?$AA6?$AA0?$AA1?$AA0?$AA?$AN?$AA?6?$AA?9?$AA?5?$AAa?$AAb?$AAo?$AAr?$AAt?$AA?$CI?$AA?$CJ?$AA?5?$AAh?$AAa?$AAs?$AA?5?$AAb?$AAe?$AAe?$AAn?$AA?5?$AAc?$AAa?$AAl?$AAl?$AAe?$AAd@ 1003bc78     LIBCMT:crt0msg.obj
 0002:00000cc0       ??_C@_1FI@HONFMGBI@?$AAR?$AA6?$AA0?$AA0?$AA9?$AA?$AN?$AA?6?$AA?9?$AA?5?$AAn?$AAo?$AAt?$AA?5?$AAe?$AAn?$AAo?$AAu?$AAg?$AAh?$AA?5?$AAs?$AAp?$AAa?$AAc?$AAe?$AA?5?$AAf?$AAo?$AAr?$AA?5?$AAe?$AAn@ 1003bcc0     LIBCMT:crt0msg.obj
 0002:00000d18       ??_C@_1FE@LLNEDJMD@?$AAR?$AA6?$AA0?$AA0?$AA8?$AA?$AN?$AA?6?$AA?9?$AA?5?$AAn?$AAo?$AAt?$AA?5?$AAe?$AAn?$AAo?$AAu?$AAg?$AAh?$AA?5?$AAs?$AAp?$AAa?$AAc?$AAe?$AA?5?$AAf?$AAo?$AAr?$AA?5?$AAa?$AAr@ 1003bd18     LIBCMT:crt0msg.obj
 0002:00000d70       ??_C@_1FK@PGACCAFB@?$AAR?$AA6?$AA0?$AA0?$AA2?$AA?$AN?$AA?6?$AA?9?$AA?5?$AAf?$AAl?$AAo?$AAa?$AAt?$AAi?$AAn?$AAg?$AA?5?$AAp?$AAo?$AAi?$AAn?$AAt?$AA?5?$AAs?$AAu?$AAp?$AAp?$AAo?$AAr?$AAt?$AA?5@ 1003bd70     LIBCMT:crt0msg.obj
 0002:00000e80       ??_C@_1EK@MBDPDCGA@?$AAM?$AAi?$AAc?$AAr?$AAo?$AAs?$AAo?$AAf?$AAt?$AA?5?$AAV?$AAi?$AAs?$AAu?$AAa?$AAl?$AA?5?$AAC?$AA?$CL?$AA?$CL?$AA?5?$AAR?$AAu?$AAn?$AAt?$AAi?$AAm?$AAe?$AA?5?$AAL?$AAi?$AAb@ 1003be80     LIBCMT:crt0msg.obj
 0002:00000ecc       ??_C@_15IABLJNFO@?$AA?6?$AA?6?$AA?$AA@ 1003becc     LIBCMT:crt0msg.obj
 0002:00000ed4       ??_C@_17LGKOMLJ@?$AA?4?$AA?4?$AA?4?$AA?$AA@ 1003bed4     LIBCMT:crt0msg.obj
 0002:00000edc       ??_C@_1CO@EAEJAADC@?$AA?$DM?$AAp?$AAr?$AAo?$AAg?$AAr?$AAa?$AAm?$AA?5?$AAn?$AAa?$AAm?$AAe?$AA?5?$AAu?$AAn?$AAk?$AAn?$AAo?$AAw?$AAn?$AA?$DO?$AA?$AA@ 1003bedc     LIBCMT:crt0msg.obj
 0002:00000f0c       ??_C@_1DE@JNGNBFGO@?$AAR?$AAu?$AAn?$AAt?$AAi?$AAm?$AAe?$AA?5?$AAE?$AAr?$AAr?$AAo?$AAr?$AA?$CB?$AA?6?$AA?6?$AAP?$AAr?$AAo?$AAg?$AAr?$AAa?$AAm?$AA?3?$AA?5?$AA?$AA@ 1003bf0c     LIBCMT:crt0msg.obj
 0002:00000f40       ??_C@_1BC@GDGBMEMK@?$AAH?$AAH?$AA?3?$AAm?$AAm?$AA?3?$AAs?$AAs?$AA?$AA@ 1003bf40     LIBCMT:nlsdata2.obj
 0002:00000f54       ??_C@_1CI@KNAKOEBC@?$AAd?$AAd?$AAd?$AAd?$AA?0?$AA?5?$AAM?$AAM?$AAM?$AAM?$AA?5?$AAd?$AAd?$AA?0?$AA?5?$AAy?$AAy?$AAy?$AAy?$AA?$AA@ 1003bf54     LIBCMT:nlsdata2.obj
 0002:00000f7c       ??_C@_1BC@IEBCMHCM@?$AAM?$AAM?$AA?1?$AAd?$AAd?$AA?1?$AAy?$AAy?$AA?$AA@ 1003bf7c     LIBCMT:nlsdata2.obj
 0002:00000f90       ??_C@_15CLMNNGEL@?$AAP?$AAM?$AA?$AA@ 1003bf90     LIBCMT:nlsdata2.obj
 0002:00000f98       ??_C@_15ODEHAHHF@?$AAA?$AAM?$AA?$AA@ 1003bf98     LIBCMT:nlsdata2.obj
 0002:00000fa0       ??_C@_1BC@FEMKIFH@?$AAD?$AAe?$AAc?$AAe?$AAm?$AAb?$AAe?$AAr?$AA?$AA@ 1003bfa0     LIBCMT:nlsdata2.obj
 0002:00000fb4       ??_C@_1BC@BGLIFPF@?$AAN?$AAo?$AAv?$AAe?$AAm?$AAb?$AAe?$AAr?$AA?$AA@ 1003bfb4     LIBCMT:nlsdata2.obj
 0002:00000fc8       ??_C@_1BA@EPANDLNG@?$AAO?$AAc?$AAt?$AAo?$AAb?$AAe?$AAr?$AA?$AA@ 1003bfc8     LIBCMT:nlsdata2.obj
 0002:00000fd8       ??_C@_1BE@DKAAMBJL@?$AAS?$AAe?$AAp?$AAt?$AAe?$AAm?$AAb?$AAe?$AAr?$AA?$AA@ 1003bfd8     LIBCMT:nlsdata2.obj
 0002:00000fec       ??_C@_1O@PAHLKOAC@?$AAA?$AAu?$AAg?$AAu?$AAs?$AAt?$AA?$AA@ 1003bfec     LIBCMT:nlsdata2.obj
 0002:00000ffc       ??_C@_19BIFMLPCD@?$AAJ?$AAu?$AAl?$AAy?$AA?$AA@ 1003bffc     LIBCMT:nlsdata2.obj
 0002:00001008       ??_C@_19EPFLPGAP@?$AAJ?$AAu?$AAn?$AAe?$AA?$AA@ 1003c008     LIBCMT:nlsdata2.obj
 0002:00001014       ??_C@_1M@GJNLMHFD@?$AAA?$AAp?$AAr?$AAi?$AAl?$AA?$AA@ 1003c014     LIBCMT:nlsdata2.obj
 0002:00001020       ??_C@_1M@IKEENEDF@?$AAM?$AAa?$AAr?$AAc?$AAh?$AA?$AA@ 1003c020     LIBCMT:nlsdata2.obj
 0002:0000102c       ??_C@_1BC@JGDDFFAM@?$AAF?$AAe?$AAb?$AAr?$AAu?$AAa?$AAr?$AAy?$AA?$AA@ 1003c02c     LIBCMT:nlsdata2.obj
 0002:00001040       ??_C@_1BA@EFMEIEBA@?$AAJ?$AAa?$AAn?$AAu?$AAa?$AAr?$AAy?$AA?$AA@ 1003c040     LIBCMT:nlsdata2.obj
 0002:00001050       ??_C@_17EGKACKIF@?$AAD?$AAe?$AAc?$AA?$AA@ 1003c050     LIBCMT:nlsdata2.obj
 0002:00001058       ??_C@_17BBDMLCIG@?$AAN?$AAo?$AAv?$AA?$AA@ 1003c058     LIBCMT:nlsdata2.obj
 0002:00001060       ??_C@_17FNLKOI@?$AAO?$AAc?$AAt?$AA?$AA@ 1003c060     LIBCMT:nlsdata2.obj
 0002:00001068       ??_C@_17HCHCOKMG@?$AAS?$AAe?$AAp?$AA?$AA@ 1003c068     LIBCMT:nlsdata2.obj
 0002:00001070       ??_C@_17ICPELBCN@?$AAA?$AAu?$AAg?$AA?$AA@ 1003c070     LIBCMT:nlsdata2.obj
 0002:00001078       ??_C@_17IJPCKHK@?$AAJ?$AAu?$AAl?$AA?$AA@ 1003c078     LIBCMT:nlsdata2.obj
 0002:00001080       ??_C@_17KCJGOCPB@?$AAJ?$AAu?$AAn?$AA?$AA@ 1003c080     LIBCMT:nlsdata2.obj
 0002:00001088       ??_C@_17PNNKMEED@?$AAM?$AAa?$AAy?$AA?$AA@ 1003c088     LIBCMT:nlsdata2.obj
 0002:00001090       ??_C@_17LFPOIHDD@?$AAA?$AAp?$AAr?$AA?$AA@ 1003c090     LIBCMT:nlsdata2.obj
 0002:00001098       ??_C@_17CKNLEDEC@?$AAM?$AAa?$AAr?$AA?$AA@ 1003c098     LIBCMT:nlsdata2.obj
 0002:000010a0       ??_C@_17LMDJEKJN@?$AAF?$AAe?$AAb?$AA?$AA@ 1003c0a0     LIBCMT:nlsdata2.obj
 0002:000010a8       ??_C@_17DKNBKCHM@?$AAJ?$AAa?$AAn?$AA?$AA@ 1003c0a8     LIBCMT:nlsdata2.obj
 0002:000010b0       ??_C@_1BC@ENMNNPAJ@?$AAS?$AAa?$AAt?$AAu?$AAr?$AAd?$AAa?$AAy?$AA?$AA@ 1003c0b0     LIBCMT:nlsdata2.obj
 0002:000010c4       ??_C@_1O@PDICJHAG@?$AAF?$AAr?$AAi?$AAd?$AAa?$AAy?$AA?$AA@ 1003c0c4     LIBCMT:nlsdata2.obj
 0002:000010d4       ??_C@_1BC@HHMNLIHE@?$AAT?$AAh?$AAu?$AAr?$AAs?$AAd?$AAa?$AAy?$AA?$AA@ 1003c0d4     LIBCMT:nlsdata2.obj
 0002:000010e8       ??_C@_1BE@EBOGMDOH@?$AAW?$AAe?$AAd?$AAn?$AAe?$AAs?$AAd?$AAa?$AAy?$AA?$AA@ 1003c0e8     LIBCMT:nlsdata2.obj
 0002:000010fc       ??_C@_1BA@ENFBFFEK@?$AAT?$AAu?$AAe?$AAs?$AAd?$AAa?$AAy?$AA?$AA@ 1003c0fc     LIBCMT:nlsdata2.obj
 0002:0000110c       ??_C@_1O@MMNBFLIA@?$AAM?$AAo?$AAn?$AAd?$AAa?$AAy?$AA?$AA@ 1003c10c     LIBCMT:nlsdata2.obj
 0002:0000111c       ??_C@_1O@IHNHDHPB@?$AAS?$AAu?$AAn?$AAd?$AAa?$AAy?$AA?$AA@ 1003c11c     LIBCMT:nlsdata2.obj
 0002:0000112c       ??_C@_17GGIBDPIH@?$AAS?$AAa?$AAt?$AA?$AA@ 1003c12c     LIBCMT:nlsdata2.obj
 0002:00001134       ??_C@_17HFOLPPLP@?$AAF?$AAr?$AAi?$AA?$AA@ 1003c134     LIBCMT:nlsdata2.obj
 0002:0000113c       ??_C@_17PDPHAADD@?$AAT?$AAh?$AAu?$AA?$AA@ 1003c13c     LIBCMT:nlsdata2.obj
 0002:00001144       ??_C@_17CJEDCEPE@?$AAW?$AAe?$AAd?$AA?$AA@ 1003c144     LIBCMT:nlsdata2.obj
 0002:0000114c       ??_C@_17BMKGEGOJ@?$AAT?$AAu?$AAe?$AA?$AA@ 1003c14c     LIBCMT:nlsdata2.obj
 0002:00001154       ??_C@_17KBOMKBF@?$AAM?$AAo?$AAn?$AA?$AA@ 1003c154     LIBCMT:nlsdata2.obj
 0002:0000115c       ??_C@_17MBGCMIPB@?$AAS?$AAu?$AAn?$AA?$AA@ 1003c15c     LIBCMT:nlsdata2.obj
 0002:00001164       ??_C@_08JCCMCCIL@HH?3mm?3ss?$AA@ 1003c164     LIBCMT:nlsdata2.obj
 0002:00001170       ??_C@_0BE@CKGJFCPC@dddd?0?5MMMM?5dd?0?5yyyy?$AA@ 1003c170     LIBCMT:nlsdata2.obj
 0002:00001184       ??_C@_08BPBNCDIB@MM?1dd?1yy?$AA@ 1003c184     LIBCMT:nlsdata2.obj
 0002:00001190       ??_C@_02CJNFDJBF@PM?$AA@   1003c190     LIBCMT:nlsdata2.obj
 0002:00001194       ??_C@_02DEDBPAFC@AM?$AA@   1003c194     LIBCMT:nlsdata2.obj
 0002:00001198       ??_C@_08EDHMEBNP@December?$AA@ 1003c198     LIBCMT:nlsdata2.obj
 0002:000011a4       ??_C@_08HCHEGEOA@November?$AA@ 1003c1a4     LIBCMT:nlsdata2.obj
 0002:000011b0       ??_C@_07JJNFCEND@October?$AA@ 1003c1b0     LIBCMT:nlsdata2.obj
 0002:000011b8       ??_C@_09BHHEALKD@September?$AA@ 1003c1b8     LIBCMT:nlsdata2.obj
 0002:000011c4       ??_C@_06LBBHFDDG@August?$AA@ 1003c1c4     LIBCMT:nlsdata2.obj
 0002:000011cc       ??_C@_04MIEPOIFP@July?$AA@ 1003c1cc     LIBCMT:nlsdata2.obj
 0002:000011d4       ??_C@_04CNLMGBGM@June?$AA@ 1003c1d4     LIBCMT:nlsdata2.obj
 0002:000011dc       ??_C@_05DMJDNLEJ@April?$AA@ 1003c1dc     LIBCMT:nlsdata2.obj
 0002:000011e4       ??_C@_05HPCKOFNC@March?$AA@ 1003c1e4     LIBCMT:nlsdata2.obj
 0002:000011ec       ??_C@_08GNJGEPFN@February?$AA@ 1003c1ec     LIBCMT:nlsdata2.obj
 0002:000011f8       ??_C@_07CGJPFGJA@January?$AA@ 1003c1f8     LIBCMT:nlsdata2.obj
 0002:00001200       ??_C@_03MKABNOCG@Dec?$AA@  1003c200     LIBCMT:nlsdata2.obj
 0002:00001204       ??_C@_03JPJOFNIA@Nov?$AA@  1003c204     LIBCMT:nlsdata2.obj
 0002:00001208       ??_C@_03BMAOKBAD@Oct?$AA@  1003c208     LIBCMT:nlsdata2.obj
 0002:0000120c       ??_C@_03GGCAPAJC@Sep?$AA@  1003c20c     LIBCMT:nlsdata2.obj
 0002:00001210       ??_C@_03IFJFEIGA@Aug?$AA@  1003c210     LIBCMT:nlsdata2.obj
 0002:00001214       ??_C@_03LBGABGKK@Jul?$AA@  1003c214     LIBCMT:nlsdata2.obj
 0002:00001218       ??_C@_03IDFGHECI@Jun?$AA@  1003c218     LIBCMT:nlsdata2.obj
 0002:0000121c       ??_C@_03CNMDKL@May?$AA@    1003c21c     LIBCMT:nlsdata2.obj
 0002:00001220       ??_C@_03LEOLGMJP@Apr?$AA@  1003c220     LIBCMT:nlsdata2.obj
 0002:00001224       ??_C@_03ODNJBKGA@Mar?$AA@  1003c224     LIBCMT:nlsdata2.obj
 0002:00001228       ??_C@_03HJBDCHOM@Feb?$AA@  1003c228     LIBCMT:nlsdata2.obj
 0002:0000122c       ??_C@_03JIHJHPIE@Jan?$AA@  1003c22c     LIBCMT:nlsdata2.obj
 0002:00001230       ??_C@_08INBOOONO@Saturday?$AA@ 1003c230     LIBCMT:nlsdata2.obj
 0002:0000123c       ??_C@_06JECMNKMI@Friday?$AA@ 1003c23c     LIBCMT:nlsdata2.obj
 0002:00001244       ??_C@_08HACCIKIA@Thursday?$AA@ 1003c244     LIBCMT:nlsdata2.obj
 0002:00001250       ??_C@_09DLIGFAKA@Wednesday?$AA@ 1003c250     LIBCMT:nlsdata2.obj
 0002:0000125c       ??_C@_07BAAGCFCM@Tuesday?$AA@ 1003c25c     LIBCMT:nlsdata2.obj
 0002:00001264       ??_C@_06JLEDEDGH@Monday?$AA@ 1003c264     LIBCMT:nlsdata2.obj
 0002:0000126c       ??_C@_06OOPIFAJ@Sunday?$AA@ 1003c26c     LIBCMT:nlsdata2.obj
 0002:00001274       ??_C@_03FEFJNEK@Sat?$AA@   1003c274     LIBCMT:nlsdata2.obj
 0002:00001278       ??_C@_03IDIOELNC@Fri?$AA@  1003c278     LIBCMT:nlsdata2.obj
 0002:0000127c       ??_C@_03IOFIKPDN@Thu?$AA@  1003c27c     LIBCMT:nlsdata2.obj
 0002:00001280       ??_C@_03MHOMLAJA@Wed?$AA@  1003c280     LIBCMT:nlsdata2.obj
 0002:00001284       ??_C@_03NAGEINEP@Tue?$AA@  1003c284     LIBCMT:nlsdata2.obj
 0002:00001288       ??_C@_03PDAGKDH@Mon?$AA@   1003c288     LIBCMT:nlsdata2.obj
 0002:0000128c       ??_C@_03KOEHGMDN@Sun?$AA@  1003c28c     LIBCMT:nlsdata2.obj
 0002:00001290       ??_C@_1BK@DBDEIDLH@?$AAK?$AAE?$AAR?$AAN?$AAE?$AAL?$AA3?$AA2?$AA?4?$AAD?$AAL?$AAL?$AA?$AA@ 1003c290     LIBCMT:tidtable.obj
 0002:000012ac       ??_C@_07PEJMOBNF@FlsFree?$AA@ 1003c2ac     LIBCMT:tidtable.obj
 0002:000012b4       ??_C@_0M@JCPCPOEF@FlsSetValue?$AA@ 1003c2b4     LIBCMT:tidtable.obj
 0002:000012c0       ??_C@_0M@GDNOONDI@FlsGetValue?$AA@ 1003c2c0     LIBCMT:tidtable.obj
 0002:000012cc       ??_C@_08KNHFBNJ@FlsAlloc?$AA@ 1003c2cc     LIBCMT:tidtable.obj
 0002:00001358       ??_C@_01NEMOKFLO@?$DN?$AA@ 1003c358     LIBCMT:setlocal.obj
 0002:0000135c       ??_C@_1O@CEDCILHN@?$AA?$CI?$AAn?$AAu?$AAl?$AAl?$AA?$CJ?$AA?$AA@ 1003c35c     LIBCMT:output.obj
 0002:0000136c       ??_C@_06OJHGLDPL@?$CInull?$CJ?$AA@ 1003c36c     LIBCMT:output.obj
 0002:00001378       ___lookuptable             1003c378     LIBCMT:output.obj
 0002:000013d8       __XcptActTab               1003c3d8     LIBCMT:winxfltr.obj
 0002:00001468       __First_FPE_Indx           1003c468     LIBCMT:winxfltr.obj
 0002:0000146c       __Num_FPE                  1003c46c     LIBCMT:winxfltr.obj
 0002:00001470       __XcptActTabSize           1003c470     LIBCMT:winxfltr.obj
 0002:00001474       __XcptActTabCount          1003c474     LIBCMT:winxfltr.obj
 0002:000014b0       ??_C@_02CLFPBFFP@TZ?$AA@   1003c4b0     LIBCMT:tzset.obj
 0002:000014b4       ___dnames                  1003c4b4     LIBCMT:timeset.obj
 0002:000014cc       ___mnames                  1003c4cc     LIBCMT:timeset.obj
 0002:000014f4       ??_C@_0BK@CFCOFLF@?5Complete?5Object?5Locator?8?$AA@ 1003c4f4     LIBCMT:undname.obj
 0002:00001510       ??_C@_0BN@MECKDCOJ@?5Class?5Hierarchy?5Descriptor?8?$AA@ 1003c510     LIBCMT:undname.obj
 0002:00001530       ??_C@_0BD@LGICGFMM@?5Base?5Class?5Array?8?$AA@ 1003c530     LIBCMT:undname.obj
 0002:00001544       ??_C@_0BM@LDKODKLH@?5Base?5Class?5Descriptor?5at?5?$CI?$AA@ 1003c544     LIBCMT:undname.obj
 0002:00001560       ??_C@_0BC@DAFEJGAK@?5Type?5Descriptor?8?$AA@ 1003c560     LIBCMT:undname.obj
 0002:00001574       ??_C@_0BM@PMGGMLDN@?$GAlocal?5static?5thread?5guard?8?$AA@ 1003c574     LIBCMT:undname.obj
 0002:00001590       ??_C@_0CL@FGIJHLCE@?$GAmanaged?5vector?5copy?5constructor@ 1003c590     LIBCMT:undname.obj
 0002:000015bc       ??_C@_0CJ@GJELGAMM@?$GAvector?5vbase?5copy?5constructor?5i@ 1003c5bc     LIBCMT:undname.obj
 0002:000015e8       ??_C@_0CD@CGAJBKEJ@?$GAvector?5copy?5constructor?5iterato@ 1003c5e8     LIBCMT:undname.obj
 0002:0000160c       ??_C@_0CB@PDBIFEP@?$GAdynamic?5atexit?5destructor?5for?5?8@ 1003c60c     LIBCMT:undname.obj
 0002:00001630       ??_C@_0BL@CLIPGLGB@?$GAdynamic?5initializer?5for?5?8?$AA@ 1003c630     LIBCMT:undname.obj
 0002:0000164c       ??_C@_0CM@FCBBDIGB@?$GAeh?5vector?5vbase?5copy?5constructo@ 1003c64c     LIBCMT:undname.obj
 0002:00001678       ??_C@_0CG@HLDDJMAG@?$GAeh?5vector?5copy?5constructor?5iter@ 1003c678     LIBCMT:undname.obj
 0002:000016a0       ??_C@_0CF@IMGKMJNO@?$GAmanaged?5vector?5destructor?5itera@ 1003c6a0     LIBCMT:undname.obj
 0002:000016c8       ??_C@_0CG@CFDHKGGD@?$GAmanaged?5vector?5constructor?5iter@ 1003c6c8     LIBCMT:undname.obj
 0002:000016f0       ??_C@_0BN@CKNJLHMB@?$GAplacement?5delete?$FL?$FN?5closure?8?$AA@ 1003c6f0     LIBCMT:undname.obj
 0002:00001710       ??_C@_0BL@CNOONJFP@?$GAplacement?5delete?5closure?8?$AA@ 1003c710     LIBCMT:undname.obj
 0002:0000172c       ??_C@_0P@HJKNJFNN@?$GAomni?5callsig?8?$AA@ 1003c72c     LIBCMT:undname.obj
 0002:0000173c       ??_C@_09LBNFPBCA@?5delete?$FL?$FN?$AA@ 1003c73c     LIBCMT:undname.obj
 0002:00001748       ??_C@_06FHBGPFGH@?5new?$FL?$FN?$AA@ 1003c748     LIBCMT:undname.obj
 0002:00001750       ??_C@_0CE@IIHCMGGL@?$GAlocal?5vftable?5constructor?5closu@ 1003c750     LIBCMT:undname.obj
 0002:00001774       ??_C@_0BA@KKLDJDLB@?$GAlocal?5vftable?8?$AA@ 1003c774     LIBCMT:undname.obj
 0002:00001784       ??_C@_05KHLCHHI@?$GARTTI?$AA@ 1003c784     LIBCMT:undname.obj
 0002:0000178c       ??_C@_03KLGMFNMG@?$GAEH?$AA@ 1003c78c     LIBCMT:undname.obj
 0002:00001790       ??_C@_0BA@KBCDOMBN@?$GAudt?5returning?8?$AA@ 1003c790     LIBCMT:undname.obj
 0002:000017a0       ??_C@_0BL@LLKPOHJI@?$GAcopy?5constructor?5closure?8?$AA@ 1003c7a0     LIBCMT:undname.obj
 0002:000017bc       ??_C@_0CH@OOJPLCPH@?$GAeh?5vector?5vbase?5constructor?5ite@ 1003c7bc     LIBCMT:undname.obj
 0002:000017e4       ??_C@_0CA@GCEOPDGL@?$GAeh?5vector?5destructor?5iterator?8?$AA@ 1003c7e4     LIBCMT:undname.obj
 0002:00001804       ??_C@_0CB@JONCMFFK@?$GAeh?5vector?5constructor?5iterator?8@ 1003c804     LIBCMT:undname.obj
 0002:00001828       ??_C@_0BL@NILFHHPC@?$GAvirtual?5displacement?5map?8?$AA@ 1003c828     LIBCMT:undname.obj
 0002:00001844       ??_C@_0CE@IKBNEHA@?$GAvector?5vbase?5constructor?5iterat@ 1003c844     LIBCMT:undname.obj
 0002:00001868       ??_C@_0BN@LFPFMEDL@?$GAvector?5destructor?5iterator?8?$AA@ 1003c868     LIBCMT:undname.obj
 0002:00001888       ??_C@_0BO@PFGOCPJJ@?$GAvector?5constructor?5iterator?8?$AA@ 1003c888     LIBCMT:undname.obj
 0002:000018a8       ??_C@_0BN@IMDCHIKM@?$GAscalar?5deleting?5destructor?8?$AA@ 1003c8a8     LIBCMT:undname.obj
 0002:000018c8       ??_C@_0BO@OBMKPJIG@?$GAdefault?5constructor?5closure?8?$AA@ 1003c8c8     LIBCMT:undname.obj
 0002:000018e8       ??_C@_0BN@DEGPLNFK@?$GAvector?5deleting?5destructor?8?$AA@ 1003c8e8     LIBCMT:undname.obj
 0002:00001908       ??_C@_0BD@JDLKDPAB@?$GAvbase?5destructor?8?$AA@ 1003c908     LIBCMT:undname.obj
 0002:0000191c       ??_C@_08OBABFOLI@?$GAstring?8?$AA@ 1003c91c     LIBCMT:undname.obj
 0002:00001928       ??_C@_0BF@KDPPACIK@?$GAlocal?5static?5guard?8?$AA@ 1003c928     LIBCMT:undname.obj
 0002:00001940       ??_C@_08LLFFHHDJ@?$GAtypeof?8?$AA@ 1003c940     LIBCMT:undname.obj
 0002:0000194c       ??_C@_07FEEIOKP@?$GAvcall?8?$AA@ 1003c94c     LIBCMT:undname.obj
 0002:00001954       ??_C@_09BLBHBJP@?$GAvbtable?8?$AA@ 1003c954     LIBCMT:undname.obj
 0002:00001960       ??_C@_09IFPLHPGF@?$GAvftable?8?$AA@ 1003c960     LIBCMT:undname.obj
 0002:0000196c       ??_C@_02MHEGNOJ@?$FO?$DN?$AA@ 1003c96c     LIBCMT:undname.obj
 0002:00001970       ??_C@_02DHLNPPGH@?$HM?$DN?$AA@ 1003c970     LIBCMT:undname.obj
 0002:00001974       ??_C@_02FGJGFEAB@?$CG?$DN?$AA@ 1003c974     LIBCMT:undname.obj
 0002:00001978       ??_C@_03CDNPDDLA@?$DM?$DM?$DN?$AA@ 1003c978     LIBCMT:undname.obj
 0002:0000197c       ??_C@_03IKFCCPFF@?$DO?$DO?$DN?$AA@ 1003c97c     LIBCMT:undname.obj
 0002:00001980       ??_C@_02FENAOKFI@?$CF?$DN?$AA@ 1003c980     LIBCMT:undname.obj
 0002:00001984       ??_C@_02FJEHGPIO@?1?$DN?$AA@ 1003c984     LIBCMT:undname.obj
 0002:00001988       ??_C@_02FKMDLLOA@?9?$DN?$AA@ 1003c988     LIBCMT:undname.obj
 0002:0000198c       ??_C@_02FOEOMHFC@?$CL?$DN?$AA@ 1003c98c     LIBCMT:undname.obj
 0002:00001990       ??_C@_02FPIMKNGF@?$CK?$DN?$AA@ 1003c990     LIBCMT:undname.obj
 0002:00001994       ??_C@_02NONPIBCD@?$HM?$HM?$AA@ 1003c994     LIBCMT:undname.obj
 0002:00001998       ??_C@_02PPKAJPJL@?$CG?$CG?$AA@ 1003c998     LIBCMT:undname.obj
 0002:0000199c       ??_C@_01DNKMNLPK@?$HM?$AA@ 1003c99c     LIBCMT:undname.obj
 0002:000019a0       ??_C@_01JKBOJNNK@?$FO?$AA@ 1003c9a0     LIBCMT:undname.obj
 0002:000019a4       ??_C@_01PJKLJHI@?$HO?$AA@  1003c9a4     LIBCMT:undname.obj
 0002:000019a8       ??_C@_02HCKGKOFO@?$CI?$CJ?$AA@ 1003c9a8     LIBCMT:undname.obj
 0002:000019ac       ??_C@_01IHBHIGKO@?0?$AA@   1003c9ac     LIBCMT:undname.obj
 0002:000019b0       ??_C@_02EEKDKGMJ@?$DO?$DN?$AA@ 1003c9b0     LIBCMT:undname.obj
 0002:000019b4       ??_C@_02EHCHHCKH@?$DM?$DN?$AA@ 1003c9b4     LIBCMT:undname.obj
 0002:000019b8       ??_C@_01FGNFDNOH@?$CF?$AA@ 1003c9b8     LIBCMT:undname.obj
 0002:000019bc       ??_C@_03MNHNFDLC@?9?$DO?$CK?$AA@ 1003c9bc     LIBCMT:undname.obj
 0002:000019c0       ??_C@_01MIFGBAGJ@?$CL?$AA@ 1003c9c0     LIBCMT:undname.obj
 0002:000019c4       ??_C@_02ECNGHCIF@?$CL?$CL?$AA@ 1003c9c4     LIBCMT:undname.obj
 0002:000019c8       ??_C@_02HBOOOICD@?9?$DO?$AA@ 1003c9c8     LIBCMT:undname.obj
 0002:000019cc       ??_C@_08LHJFAFGD@operator?$AA@ 1003c9cc     LIBCMT:undname.obj
 0002:000019d8       ??_C@_02GPECMEKF@?$FL?$FN?$AA@ 1003c9d8     LIBCMT:undname.obj
 0002:000019dc       ??_C@_02FDNJECIE@?$CB?$DN?$AA@ 1003c9dc     LIBCMT:undname.obj
 0002:000019e0       ??_C@_02EGOFBIJA@?$DN?$DN?$AA@ 1003c9e0     LIBCMT:undname.obj
 0002:000019e4       ??_C@_01DCLJPIOD@?$CB?$AA@ 1003c9e4     LIBCMT:undname.obj
 0002:000019e8       ??_C@_02FODMEDOG@?$DM?$DM?$AA@ 1003c9e8     LIBCMT:undname.obj
 0002:000019ec       ??_C@_02GPIOPFAK@?$DO?$DO?$AA@ 1003c9ec     LIBCMT:undname.obj
 0002:000019f0       ??_C@_07FPCDHGMM@?5delete?$AA@ 1003c9f0     LIBCMT:undname.obj
 0002:000019f8       ??_C@_04NIHEBCM@?5new?$AA@ 1003c9f8     LIBCMT:undname.obj
 0002:00001a00       ??_C@_0M@GFIIJFMG@__unaligned?$AA@ 1003ca00     LIBCMT:undname.obj
 0002:00001a0c       ??_C@_0L@PILCLIHE@__restrict?$AA@ 1003ca0c     LIBCMT:undname.obj
 0002:00001a18       ??_C@_07JOMMBBKO@__ptr64?$AA@ 1003ca18     LIBCMT:undname.obj
 0002:00001a20       ??_C@_06GHPCKEAG@__eabi?$AA@ 1003ca20     LIBCMT:undname.obj
 0002:00001a28       ??_C@_09HIJEGCPM@__clrcall?$AA@ 1003ca28     LIBCMT:undname.obj
 0002:00001a34       ??_C@_0L@JMKHOMEK@__fastcall?$AA@ 1003ca34     LIBCMT:undname.obj
 0002:00001a40       ??_C@_0L@NPHFGOKO@__thiscall?$AA@ 1003ca40     LIBCMT:undname.obj
 0002:00001a4c       ??_C@_09IFJBGAPI@__stdcall?$AA@ 1003ca4c     LIBCMT:undname.obj
 0002:00001a58       ??_C@_08GHMPAG@__pascal?$AA@ 1003ca58     LIBCMT:undname.obj
 0002:00001a64       ??_C@_07KOLFKCDI@__cdecl?$AA@ 1003ca64     LIBCMT:undname.obj
 0002:00001a6c       ??_C@_08EHJDFFNH@__based?$CI?$AA@ 1003ca6c     LIBCMT:undname.obj
 0002:00001bfc       ??_C@_0BI@DFKBFLJE@GetProcessWindowStation?$AA@ 1003cbfc     LIBCMT:crtmboxw.obj
 0002:00001c14       ??_C@_0BK@DEKFELLI@GetUserObjectInformationW?$AA@ 1003cc14     LIBCMT:crtmboxw.obj
 0002:00001c30       ??_C@_0BD@HHGDFDBJ@GetLastActivePopup?$AA@ 1003cc30     LIBCMT:crtmboxw.obj
 0002:00001c44       ??_C@_0BA@HNOPNCHB@GetActiveWindow?$AA@ 1003cc44     LIBCMT:crtmboxw.obj
 0002:00001c54       ??_C@_0M@DLDCCGNP@MessageBoxW?$AA@ 1003cc54     LIBCMT:crtmboxw.obj
 0002:00001c60       ??_C@_1BG@GOEBHBDC@?$AAU?$AAS?$AAE?$AAR?$AA3?$AA2?$AA?4?$AAD?$AAL?$AAL?$AA?$AA@ 1003cc60     LIBCMT:crtmboxw.obj
 0002:00001c78       ___newctype                1003cc78     LIBCMT:ctype.obj
 0002:00001f78       __wctype                   1003cf78     LIBCMT:ctype.obj
 0002:00002180       ___newclmap                1003d180     LIBCMT:ctype.obj
 0002:00002300       ___newcumap                1003d300     LIBCMT:ctype.obj
 0002:00002480       ___lookuptable_s           1003d480     LIBCMT:outputs.obj
 0002:000024e4       __pDestructExceptionObject 1003d4e4     LIBCMT:frame.obj
 0002:000024ec       ??_7bad_exception@std@@6B@ 1003d4ec     LIBCMT:frame.obj
 0002:000024f4       ??_C@_0O@DPKOEFFH@bad?5exception?$AA@ 1003d4f4     LIBCMT:frame.obj
 0002:00002504       ??_C@_1BA@BALFACEM@?$AAC?$AAO?$AAN?$AAO?$AAU?$AAT?$AA$?$AA?$AA@ 1003d504     LIBCMT:initcon.obj
 0002:00002514       _FOLDERID_LocalAppDataLow  1003d514     uuid:shguids.obj
 0002:00002524       ??_C@_0DC@MHGEAIEM@Width?5too?5large?5for?5libpng?5to?5pr@ 1003d524     pnglib:pngget.obj
 0002:00002558       ??_C@_0BF@IBPIFLEG@Invalid?5image?5height?$AA@ 1003d558     pnglib:pngget.obj
 0002:00002570       ??_C@_0BE@MKFPKGEK@Invalid?5image?5width?$AA@ 1003d570     pnglib:pngget.obj
 0002:00002584       ??_C@_0BD@JPMLPKHD@Invalid?5color?5type?$AA@ 1003d584     pnglib:pngget.obj
 0002:00002598       ??_C@_0BC@IIDONEMJ@Invalid?5bit?5depth?$AA@ 1003d598     pnglib:pngget.obj
 0002:000025d0       __real@3fa999999999999a    1003d5d0     pnglib:pngrtran.obj
 0002:000025d8       __real@40efffe000000000    1003d5d8     pnglib:pngrtran.obj
 0002:000025e0       __real@3f70000000000000    1003d5e0     pnglib:pngrtran.obj
 0002:000025e8       __real@41f0000000000000    1003d5e8     pnglib:pngrtran.obj
 0002:000025f0       __real@406fe00000000000    1003d5f0     pnglib:pngrtran.obj
 0002:000025f8       __real@3eb0c6f7a0b5ed8d    1003d5f8     pnglib:pngrtran.obj
 0002:00002600       ??_C@_0CF@HEFPFJHN@NULL?5row?5buffer?5for?5row?5?$CFld?0?5pas@ 1003d600     pnglib:pngrtran.obj
 0002:00002628       ??_C@_0BD@LBMCPKOE@zlib?5version?5error?$AA@ 1003d628     pnglib:pngread.obj
 0002:0000263c       ??_C@_0BC@MCPIPOGP@zlib?5memory?5error?$AA@ 1003d63c     pnglib:pngread.obj
 0002:00002650       ??_C@_0BD@CPDHIJBA@Unknown?5zlib?5error?$AA@ 1003d650     pnglib:pngread.obj
 0002:00002664       ??_C@_05GDHACFMB@1?42?43?$AA@ 1003d664     pnglib:pngread.obj
 0002:0000266c       ??_C@_0DH@LDFDLODO@Incompatible?5libpng?5version?5in?5a@ 1003d66c     pnglib:pngread.obj
 0002:000026a4       ??_C@_0DG@CCNLMKFB@Application?5?5is?5?5running?5with?5pn@ 1003d6a4     pnglib:pngread.obj
 0002:000026dc       ??_C@_0DG@OGOEMJOC@Application?5was?5compiled?5with?5pn@ 1003d6dc     pnglib:pngread.obj
 0002:00002714       ??_C@_0BJ@LAKDHAPN@Missing?5PLTE?5before?5IDAT?$AA@ 1003d714     pnglib:pngread.obj
 0002:00002730       ??_C@_0BJ@FFGICIDJ@Missing?5IHDR?5before?5IDAT?$AA@ 1003d730     pnglib:pngread.obj
 0002:0000274c       ??_C@_0CH@NMANOLCN@PNG?5file?5corrupted?5by?5ASCII?5conv@ 1003d74c     pnglib:pngread.obj
 0002:00002774       ??_C@_0P@KIMIGLKH@Not?5a?5PNG?5file?$AA@ 1003d774     pnglib:pngread.obj
 0002:00002788       ??_C@_0EH@CHENFKEM@Ignoring?5extra?5png_read_update_i@ 1003d788     pnglib:pngread.obj
 0002:000027d0       ??_C@_0BG@OKGHHCLP@Extra?5compressed?5data?$AA@ 1003d7d0     pnglib:pngread.obj
 0002:000027e8       ??_C@_0BE@JMOGBNJB@Decompression?5error?$AA@ 1003d7e8     pnglib:pngread.obj
 0002:000027fc       ??_C@_0BG@EIEOOJHA@Not?5enough?5image?5data?$AA@ 1003d7fc     pnglib:pngread.obj
 0002:00002814       ??_C@_0CB@KCPNIGFM@Invalid?5attempt?5to?5read?5row?5data@ 1003d814     pnglib:pngread.obj
 0002:00002838       ??_C@_0CI@BENEDNPA@PNG_READ_SWAP_SUPPORTED?5is?5not?5d@ 1003d838     pnglib:pngread.obj
 0002:00002860       ??_C@_0CJ@IFNPHJKM@PNG_READ_SHIFT_SUPPORTED?5is?5not?5@ 1003d860     pnglib:pngread.obj
 0002:0000288c       ??_C@_0CI@CMHDPOOG@PNG_READ_PACK_SUPPORTED?5is?5not?5d@ 1003d88c     pnglib:pngread.obj
 0002:000028b4       ??_C@_0CM@EEPCCKAP@PNG_READ_PACKSWAP_SUPPORTED?5is?5n@ 1003d8b4     pnglib:pngread.obj
 0002:000028e0       ??_C@_0CK@IMAIGNJJ@PNG_READ_INVERT_SUPPORTED?5is?5not@ 1003d8e0     pnglib:pngread.obj
 0002:0000290c       ??_C@_0BG@JAHFDNP@Too?5many?5IDAT?8s?5found?$AA@ 1003d90c     pnglib:pngread.obj
 0002:00002c28       _png_libpng_ver            1003dc28     pnglib:png.obj
 0002:00002c3c       _png_sig                   1003dc3c     pnglib:png.obj
 0002:00002c44       _png_IHDR                  1003dc44     pnglib:png.obj
 0002:00002c4c       _png_IDAT                  1003dc4c     pnglib:png.obj
 0002:00002c54       _png_IEND                  1003dc54     pnglib:png.obj
 0002:00002c5c       _png_PLTE                  1003dc5c     pnglib:png.obj
 0002:00002c64       _png_bKGD                  1003dc64     pnglib:png.obj
 0002:00002c6c       _png_cHRM                  1003dc6c     pnglib:png.obj
 0002:00002c74       _png_gAMA                  1003dc74     pnglib:png.obj
 0002:00002c7c       _png_hIST                  1003dc7c     pnglib:png.obj
 0002:00002c84       _png_iCCP                  1003dc84     pnglib:png.obj
 0002:00002c8c       _png_iTXt                  1003dc8c     pnglib:png.obj
 0002:00002c94       _png_oFFs                  1003dc94     pnglib:png.obj
 0002:00002c9c       _png_pCAL                  1003dc9c     pnglib:png.obj
 0002:00002ca4       _png_sCAL                  1003dca4     pnglib:png.obj
 0002:00002cac       _png_pHYs                  1003dcac     pnglib:png.obj
 0002:00002cb4       _png_sBIT                  1003dcb4     pnglib:png.obj
 0002:00002cbc       _png_sPLT                  1003dcbc     pnglib:png.obj
 0002:00002cc4       _png_sRGB                  1003dcc4     pnglib:png.obj
 0002:00002ccc       _png_tEXt                  1003dccc     pnglib:png.obj
 0002:00002cd4       _png_tIME                  1003dcd4     pnglib:png.obj
 0002:00002cdc       _png_tRNS                  1003dcdc     pnglib:png.obj
 0002:00002ce4       _png_zTXt                  1003dce4     pnglib:png.obj
 0002:00002cec       _png_pass_start            1003dcec     pnglib:png.obj
 0002:00002d08       _png_pass_inc              1003dd08     pnglib:png.obj
 0002:00002d24       _png_pass_ystart           1003dd24     pnglib:png.obj
 0002:00002d40       _png_pass_yinc             1003dd40     pnglib:png.obj
 0002:00002d5c       _png_pass_mask             1003dd5c     pnglib:png.obj
 0002:00002d78       _png_pass_dsp_mask         1003dd78     pnglib:png.obj
 0002:00002dc4       ??_C@_0CD@PGGPKBFM@Potential?5overflow?5in?5png_zalloc@ 1003ddc4     pnglib:png.obj
 0002:00002de8       ??_C@_0BL@GPADEDKN@Call?5to?5NULL?5read?5function?$AA@ 1003dde8     pnglib:pngrio.obj
 0002:00002e04       ??_C@_0L@BAFDDAPG@Read?5Error?$AA@ 1003de04     pnglib:pngrio.obj
 0002:00002e10       ??_C@_0DC@EOBOCMJO@same?5structure?4?5?5Resetting?5write@ 1003de10     pnglib:pngrio.obj
 0002:00002e48       ??_C@_0EB@NJKELLKM@It?8s?5an?5error?5to?5set?5both?5read_d@ 1003de48     pnglib:pngrio.obj
 0002:00002e9c       ??_C@_0BC@MFANGAPN@libpng?5error?3?5?$CFs?6?$AA@ 1003de9c     pnglib:pngerror.obj
 0002:00002eb0       ??_C@_0BN@HLDBDDID@libpng?5error?3?5?$CFs?0?5offset?$DN?$CFd?6?$AA@ 1003deb0     pnglib:pngerror.obj
 0002:00002ed0       ??_C@_0BJ@LPAEKCLO@libpng?5error?5no?4?5?$CFs?3?5?$CFs?6?$AA@ 1003ded0     pnglib:pngerror.obj
 0002:00002eec       ??_C@_0BE@LNAJCNP@libpng?5warning?3?5?$CFs?6?$AA@ 1003deec     pnglib:pngerror.obj
 0002:00002f00       ??_C@_0BL@FIILBAME@libpng?5warning?5no?4?5?$CFs?3?5?$CFs?6?$AA@ 1003df00     pnglib:pngerror.obj
 0002:00002f1c       ??_C@_0P@PFFMKGBN@Out?5of?5Memory?$CB?$AA@ 1003df1c     pnglib:pngmem.obj
 0002:00002f4c       ??_C@_0CB@MCDBJLEK@Unknown?5zTXt?5compression?5type?5?$CFd@ 1003df4c     pnglib:pngrutil.obj
 0002:00002f70       ??_C@_0BM@JFPBMAIB@Not?5enough?5memory?5for?5text?4?$AA@ 1003df70     pnglib:pngrutil.obj
 0002:00002f8c       ??_C@_0CN@DJANJIKN@Incomplete?5compressed?5datastream@ 1003df8c     pnglib:pngrutil.obj
 0002:00002fbc       ??_C@_0DA@FNMACPCD@Data?5error?5in?5compressed?5datastr@ 1003dfbc     pnglib:pngrutil.obj
 0002:00002fec       ??_C@_0DC@PEAPBHCI@Buffer?5error?5in?5compressed?5datas@ 1003dfec     pnglib:pngrutil.obj
 0002:00003020       ??_C@_0CG@CPNAANEJ@Not?5enough?5memory?5to?5decompress?5@ 1003e020     pnglib:pngrutil.obj
 0002:00003048       ??_C@_0CI@GGNOMFOH@Not?5enough?5memory?5to?5decompress?5@ 1003e048     pnglib:pngrutil.obj
 0002:00003070       ??_C@_0CH@ECICABF@Not?5enough?5memory?5to?5decompress?5@ 1003e070     pnglib:pngrutil.obj
 0002:00003098       ??_C@_0BD@GFBMLKLH@invalid?5chunk?5type?$AA@ 1003e098     pnglib:pngrutil.obj
 0002:000030ac       ??_C@_0CC@FECADCN@Ignoring?5bad?5adaptive?5filter?5typ@ 1003e0ac     pnglib:pngrutil.obj
 0002:000030d0       ??_C@_0CO@BIJGDGNC@Row?5has?5too?5many?5bytes?5to?5alloca@ 1003e0d0     pnglib:pngrutil.obj
 0002:00003100       ??_C@_0CD@EOPDCPFH@PNG?5unsigned?5integer?5out?5of?5rang@ 1003e100     pnglib:pngrutil.obj
 0002:00003124       ??_C@_09BJGMGMHA@CRC?5error?$AA@ 1003e124     pnglib:pngrutil.obj
 0002:00003130       ??_C@_0BD@CLODLFAN@Invalid?5IHDR?5chunk?$AA@ 1003e130     pnglib:pngrutil.obj
 0002:00003144       ??_C@_0BC@KBAKFAAH@Out?5of?5place?5IHDR?$AA@ 1003e144     pnglib:pngrutil.obj
 0002:00003158       ??_C@_0CM@LODLIOMP@Truncating?5incorrect?5info?5tRNS?5c@ 1003e158     pnglib:pngrutil.obj
 0002:00003184       ??_C@_0CH@GNNEJFAH@Truncating?5incorrect?5tRNS?5chunk?5@ 1003e184     pnglib:pngrutil.obj
 0002:000031ac       ??_C@_0BG@HHEHMEJK@Invalid?5palette?5chunk?$AA@ 1003e1ac     pnglib:pngrutil.obj
 0002:000031c4       ??_C@_0CF@FFJHLJE@Ignoring?5PLTE?5chunk?5in?5grayscale@ 1003e1c4     pnglib:pngrutil.obj
 0002:000031ec       ??_C@_0BF@PMKDIIMG@Duplicate?5PLTE?5chunk?$AA@ 1003e1ec     pnglib:pngrutil.obj
 0002:00003204       ??_C@_0BI@GEKPHPN@Invalid?5PLTE?5after?5IDAT?$AA@ 1003e204     pnglib:pngrutil.obj
 0002:0000321c       ??_C@_0BJ@LEBILHKO@Missing?5IHDR?5before?5PLTE?$AA@ 1003e21c     pnglib:pngrutil.obj
 0002:00003238       ??_C@_0BM@PFCLLCBO@Incorrect?5IEND?5chunk?5length?$AA@ 1003e238     pnglib:pngrutil.obj
 0002:00003254       ??_C@_0BB@BLPFHNNN@No?5image?5in?5file?$AA@ 1003e254     pnglib:pngrutil.obj
 0002:00003268       __real@40f86a0000000000    1003e268     pnglib:pngrutil.obj
 0002:00003270       ??_C@_0BF@BDHDCHJF@gamma?5?$DN?5?$CI?$CFd?1100000?$CJ?6?$AA@ 1003e270     pnglib:pngrutil.obj
 0002:00003288       ??_C@_0DI@KINMKNNO@Ignoring?5incorrect?5gAMA?5value?5wh@ 1003e288     pnglib:pngrutil.obj
 0002:000032c0       ??_C@_0CB@NAEALNDI@Ignoring?5gAMA?5chunk?5with?5gamma?$DN0@ 1003e2c0     pnglib:pngrutil.obj
 0002:000032e4       ??_C@_0BM@NIAHDFBB@Incorrect?5gAMA?5chunk?5length?$AA@ 1003e2e4     pnglib:pngrutil.obj
 0002:00003300       ??_C@_0BF@IMCFKHDJ@Duplicate?5gAMA?5chunk?$AA@ 1003e300     pnglib:pngrutil.obj
 0002:00003318       ??_C@_0BI@JEEHFLME@Out?5of?5place?5gAMA?5chunk?$AA@ 1003e318     pnglib:pngrutil.obj
 0002:00003330       ??_C@_0BI@POPIJBNN@Invalid?5gAMA?5after?5IDAT?$AA@ 1003e330     pnglib:pngrutil.obj
 0002:00003348       ??_C@_0BJ@CCOIFGBO@Missing?5IHDR?5before?5gAMA?$AA@ 1003e348     pnglib:pngrutil.obj
 0002:00003364       ??_C@_0BM@NECIIMI@Incorrect?5sBIT?5chunk?5length?$AA@ 1003e364     pnglib:pngrutil.obj
 0002:00003380       ??_C@_0BF@BAIKMFDA@Duplicate?5sBIT?5chunk?$AA@ 1003e380     pnglib:pngrutil.obj
 0002:00003398       ??_C@_0BI@IOIDJMN@Out?5of?5place?5sBIT?5chunk?$AA@ 1003e398     pnglib:pngrutil.obj
 0002:000033b0       ??_C@_0BI@GNBHBDGP@Invalid?5sBIT?5after?5IDAT?$AA@ 1003e3b0     pnglib:pngrutil.obj
 0002:000033c8       ??_C@_0BJ@JFIBIGHK@Missing?5IHDR?5before?5sBIT?$AA@ 1003e3c8     pnglib:pngrutil.obj
 0002:000033e4       ??_C@_0BJ@FAHLKGEB@Invalid?5cHRM?5white?5point?$AA@ 1003e3e4     pnglib:pngrutil.obj
 0002:00003400       ??_C@_0BM@IACKJHOF@gx?$DN?$CFf?0?5gy?$DN?$CFf?0?5bx?$DN?$CFf?0?5by?$DN?$CFf?6?$AA@ 1003e400     pnglib:pngrutil.obj
 0002:0000341c       ??_C@_0BM@NBPNPEHL@wx?$DN?$CFf?0?5wy?$DN?$CFf?0?5rx?$DN?$CFf?0?5ry?$DN?$CFf?6?$AA@ 1003e41c     pnglib:pngrutil.obj
 0002:00003438       ??_C@_0DI@MIMDNNAG@Ignoring?5incorrect?5cHRM?5value?5wh@ 1003e438     pnglib:pngrutil.obj
 0002:00003470       ??_C@_0BI@GNBEGBIO@Invalid?5cHRM?5blue?5point?$AA@ 1003e470     pnglib:pngrutil.obj
 0002:00003488       ??_C@_0BJ@OMNHHNBI@Invalid?5cHRM?5green?5point?$AA@ 1003e488     pnglib:pngrutil.obj
 0002:000034a4       ??_C@_0BH@MNPFDHMO@Invalid?5cHRM?5red?5point?$AA@ 1003e4a4     pnglib:pngrutil.obj
 0002:000034bc       ??_C@_0BM@JPCBJGIK@Incorrect?5cHRM?5chunk?5length?$AA@ 1003e4bc     pnglib:pngrutil.obj
 0002:000034d8       ??_C@_0BF@OEDPGHJO@Duplicate?5cHRM?5chunk?$AA@ 1003e4d8     pnglib:pngrutil.obj
 0002:000034f0       ??_C@_0BJ@PEGEEMNB@Missing?5PLTE?5before?5cHRM?$AA@ 1003e4f0     pnglib:pngrutil.obj
 0002:0000350c       ??_C@_0BI@PGCHPLFE@Invalid?5cHRM?5after?5IDAT?$AA@ 1003e50c     pnglib:pngrutil.obj
 0002:00003524       ??_C@_0BJ@BBKPBEBF@Missing?5IHDR?5before?5cHRM?$AA@ 1003e524     pnglib:pngrutil.obj
 0002:00003540       ??_C@_0BN@PPEBNPGC@incorrect?5gamma?$DN?$CI?$CFd?1100000?$CJ?6?$AA@ 1003e540     pnglib:pngrutil.obj
 0002:00003560       ??_C@_0BE@CEGOJHBA@Unknown?5sRGB?5intent?$AA@ 1003e560     pnglib:pngrutil.obj
 0002:00003574       ??_C@_0BM@FMAJKMKD@Incorrect?5sRGB?5chunk?5length?$AA@ 1003e574     pnglib:pngrutil.obj
 0002:00003590       ??_C@_0BF@EFDCKHOG@Duplicate?5sRGB?5chunk?$AA@ 1003e590     pnglib:pngrutil.obj
 0002:000035a8       ??_C@_0BI@FNFAFLBL@Out?5of?5place?5sRGB?5chunk?$AA@ 1003e5a8     pnglib:pngrutil.obj
 0002:000035c0       ??_C@_0BI@PGAMKAKH@Invalid?5sRGB?5after?5IDAT?$AA@ 1003e5c0     pnglib:pngrutil.obj
 0002:000035d8       ??_C@_0BJ@NDJOEJDI@Missing?5IHDR?5before?5sRGB?$AA@ 1003e5d8     pnglib:pngrutil.obj
 0002:000035f4       ??_C@_0CL@DPOBKPIG@Profile?5size?5field?5missing?5from?5@ 1003e5f4     pnglib:pngrutil.obj
 0002:00003620       ??_C@_0CB@EGBHHAKA@Ignoring?5truncated?5iCCP?5profile?4@ 1003e620     pnglib:pngrutil.obj
 0002:00003644       ??_C@_0DA@PBEFIAOD@Ignoring?5nonzero?5compression?5typ@ 1003e644     pnglib:pngrutil.obj
 0002:00003674       ??_C@_0BF@NLNNCHCP@Malformed?5iCCP?5chunk?$AA@ 1003e674     pnglib:pngrutil.obj
 0002:0000368c       ??_C@_0BF@KCHFLGCF@Duplicate?5iCCP?5chunk?$AA@ 1003e68c     pnglib:pngrutil.obj
 0002:000036a4       ??_C@_0BI@LKBHEKNI@Out?5of?5place?5iCCP?5chunk?$AA@ 1003e6a4     pnglib:pngrutil.obj
 0002:000036bc       ??_C@_0BI@NEPGPMDI@Invalid?5iCCP?5after?5IDAT?$AA@ 1003e6bc     pnglib:pngrutil.obj
 0002:000036d4       ??_C@_0BJ@GOJGCOOO@Missing?5IHDR?5before?5iCCP?$AA@ 1003e6d4     pnglib:pngrutil.obj
 0002:000036f0       ??_C@_0CE@MCMAFPMA@sPLT?5chunk?5requires?5too?5much?5mem@ 1003e6f0     pnglib:pngrutil.obj
 0002:00003714       ??_C@_0BE@HJCMKPPM@sPLT?5chunk?5too?5long?$AA@ 1003e714     pnglib:pngrutil.obj
 0002:00003728       ??_C@_0BK@FFJLCLGE@sPLT?5chunk?5has?5bad?5length?$AA@ 1003e728     pnglib:pngrutil.obj
 0002:00003744       ??_C@_0BF@JHCGGFHI@malformed?5sPLT?5chunk?$AA@ 1003e744     pnglib:pngrutil.obj
 0002:0000375c       ??_C@_0BI@FFAFDNM@Invalid?5sPLT?5after?5IDAT?$AA@ 1003e75c     pnglib:pngrutil.obj
 0002:00003774       ??_C@_0BJ@GJFKNLIF@Missing?5IHDR?5before?5sPLT?$AA@ 1003e774     pnglib:pngrutil.obj
 0002:00003790       ??_C@_0CK@JMGMOHJA@tRNS?5chunk?5not?5allowed?5with?5alph@ 1003e790     pnglib:pngrutil.obj
 0002:000037bc       ??_C@_0BH@JJNMONHM@Zero?5length?5tRNS?5chunk?$AA@ 1003e7bc     pnglib:pngrutil.obj
 0002:000037d4       ??_C@_0BJ@NIHNNFHD@Missing?5PLTE?5before?5tRNS?$AA@ 1003e7d4     pnglib:pngrutil.obj
 0002:000037f0       ??_C@_0BF@HALLDFIL@Duplicate?5tRNS?5chunk?$AA@ 1003e7f0     pnglib:pngrutil.obj
 0002:00003808       ??_C@_0BI@MMDCNIMN@Invalid?5tRNS?5after?5IDAT?$AA@ 1003e808     pnglib:pngrutil.obj
 0002:00003820       ??_C@_0BM@JNMFOMLO@Incorrect?5tRNS?5chunk?5length?$AA@ 1003e820     pnglib:pngrutil.obj
 0002:0000383c       ??_C@_0BJ@DNLGINLH@Missing?5IHDR?5before?5tRNS?$AA@ 1003e83c     pnglib:pngrutil.obj
 0002:00003858       ??_C@_0CB@NACPDIGJ@Incorrect?5bKGD?5chunk?5index?5value@ 1003e858     pnglib:pngrutil.obj
 0002:0000387c       ??_C@_0BM@MJOFIPAI@Incorrect?5bKGD?5chunk?5length?$AA@ 1003e87c     pnglib:pngrutil.obj
 0002:00003898       ??_C@_0BF@DHJOBPEI@Duplicate?5bKGD?5chunk?$AA@ 1003e898     pnglib:pngrutil.obj
 0002:000038b0       ??_C@_0BJ@BAJOBAFN@Missing?5PLTE?5before?5bKGD?$AA@ 1003e8b0     pnglib:pngrutil.obj
 0002:000038cc       ??_C@_0BI@CMLGFIFF@Invalid?5bKGD?5after?5IDAT?$AA@ 1003e8cc     pnglib:pngrutil.obj
 0002:000038e4       ??_C@_0BJ@PFFFEIJJ@Missing?5IHDR?5before?5bKGD?$AA@ 1003e8e4     pnglib:pngrutil.obj
 0002:00003900       ??_C@_0BM@HJCIDHBG@Incorrect?5hIST?5chunk?5length?$AA@ 1003e900     pnglib:pngrutil.obj
 0002:0000391c       ??_C@_0BF@FMFDLFKH@Duplicate?5hIST?5chunk?$AA@ 1003e91c     pnglib:pngrutil.obj
 0002:00003934       ??_C@_0BJ@KBMKNJIK@Missing?5PLTE?5before?5hIST?$AA@ 1003e934     pnglib:pngrutil.obj
 0002:00003950       ??_C@_0BI@LLJKEGEF@Invalid?5hIST?5after?5IDAT?$AA@ 1003e950     pnglib:pngrutil.obj
 0002:00003968       ??_C@_0BJ@EEABIBEO@Missing?5IHDR?5before?5hIST?$AA@ 1003e968     pnglib:pngrutil.obj
 0002:00003984       ??_C@_0BF@MBDJBKMG@Duplicate?5pHYs?5chunk?$AA@ 1003e984     pnglib:pngrutil.obj
 0002:0000399c       ??_C@_0BI@ILGPKLEK@Invalid?5pHYs?5after?5IDAT?$AA@ 1003e99c     pnglib:pngrutil.obj
 0002:000039b4       ??_C@_0BM@CAALIFOJ@Incorrect?5pHYs?5chunk?5length?$AA@ 1003e9b4     pnglib:pngrutil.obj
 0002:000039d0       ??_C@_0BJ@HLHPANNL@Missing?5IHDR?5before?5pHYs?$AA@ 1003e9d0     pnglib:pngrutil.obj
 0002:000039ec       ??_C@_0BF@JBIHJHNI@Duplicate?5oFFs?5chunk?$AA@ 1003e9ec     pnglib:pngrutil.obj
 0002:00003a04       ??_C@_0BI@DOPHGCAB@Invalid?5oFFs?5after?5IDAT?$AA@ 1003ea04     pnglib:pngrutil.obj
 0002:00003a1c       ??_C@_0BM@NBDONMKL@Incorrect?5oFFs?5chunk?5length?$AA@ 1003ea1c     pnglib:pngrutil.obj
 0002:00003a38       ??_C@_0BJ@GOGKJOPG@Missing?5IHDR?5before?5oFFs?$AA@ 1003ea38     pnglib:pngrutil.obj
 0002:00003a54       ??_C@_0BL@ELFLIGPP@No?5memory?5for?5pCAL?5params?4?$AA@ 1003ea54     pnglib:pngrutil.obj
 0002:00003a70       ??_C@_0CK@GBCGFDCK@Unrecognized?5equation?5type?5for?5p@ 1003ea70     pnglib:pngrutil.obj
 0002:00003a9c       ??_C@_0CK@ONFOCIAG@Invalid?5pCAL?5parameters?5for?5equa@ 1003ea9c     pnglib:pngrutil.obj
 0002:00003ac8       ??_C@_0BC@KNEPBMNA@Invalid?5pCAL?5data?$AA@ 1003eac8     pnglib:pngrutil.obj
 0002:00003adc       ??_C@_0BF@HCCMEAIJ@Duplicate?5pCAL?5chunk?$AA@ 1003eadc     pnglib:pngrutil.obj
 0002:00003af4       ??_C@_0BI@CAHJBHPE@Invalid?5pCAL?5after?5IDAT?$AA@ 1003eaf4     pnglib:pngrutil.obj
 0002:00003b0c       ??_C@_0BM@BADKGCIJ@No?5memory?5for?5pCAL?5purpose?4?$AA@ 1003eb0c     pnglib:pngrutil.obj
 0002:00003b28       ??_C@_0BJ@OGJFFCCO@Missing?5IHDR?5before?5pCAL?$AA@ 1003eb28     pnglib:pngrutil.obj
 0002:00003b44       ??_C@_0BC@EGHIKHND@Invalid?5sCAL?5data?$AA@ 1003eb44     pnglib:pngrutil.obj
 0002:00003b58       ??_C@_0CG@ILPCKGAK@malformed?5height?5string?5in?5sCAL?5@ 1003eb58     pnglib:pngrutil.obj
 0002:00003b80       ??_C@_0CF@LLNCAD@malformed?5width?5string?5in?5sCAL?5c@ 1003eb80     pnglib:pngrutil.obj
 0002:00003ba8       ??_C@_0BF@OLMOCGII@Duplicate?5sCAL?5chunk?$AA@ 1003eba8     pnglib:pngrutil.obj
 0002:00003bc0       ??_C@_0BI@JLBKDAG@Invalid?5sCAL?5after?5IDAT?$AA@ 1003ebc0     pnglib:pngrutil.obj
 0002:00003bd8       ??_C@_0CK@IHKBDLGD@Out?5of?5memory?5while?5processing?5s@ 1003ebd8     pnglib:pngrutil.obj
 0002:00003c04       ??_C@_0BJ@KBDFCIPO@Missing?5IHDR?5before?5sCAL?$AA@ 1003ec04     pnglib:pngrutil.obj
 0002:00003c20       ??_C@_0BF@CMKMELPN@Duplicate?5tIME?5chunk?$AA@ 1003ec20     pnglib:pngrutil.obj
 0002:00003c38       ??_C@_0BM@HAEOJOJG@Incorrect?5tIME?5chunk?5length?$AA@ 1003ec38     pnglib:pngrutil.obj
 0002:00003c54       ??_C@_0BI@DEMOLHAA@Out?5of?5place?5tIME?5chunk?$AA@ 1003ec54     pnglib:pngrutil.obj
 0002:00003c6c       ??_C@_0CL@OGIJCCIO@Insufficient?5memory?5to?5process?5t@ 1003ec6c     pnglib:pngrutil.obj
 0002:00003c98       ??_C@_0CJ@FOHJNEOL@Not?5enough?5memory?5to?5process?5tex@ 1003ec98     pnglib:pngrutil.obj
 0002:00003cc4       ??_C@_0CB@EKMLANHJ@No?5memory?5to?5process?5text?5chunk?4@ 1003ecc4     pnglib:pngrutil.obj
 0002:00003ce8       ??_C@_0BJ@DCBGIPDG@Missing?5IHDR?5before?5tEXt?$AA@ 1003ece8     pnglib:pngrutil.obj
 0002:00003d04       ??_C@_0CJ@KDPACLDH@Insufficient?5memory?5to?5store?5zTX@ 1003ed04     pnglib:pngrutil.obj
 0002:00003d30       ??_C@_0CJ@BBPBJAPJ@Not?5enough?5memory?5to?5process?5zTX@ 1003ed30     pnglib:pngrutil.obj
 0002:00003d5c       ??_C@_0CH@KHHIIBBM@Unknown?5compression?5type?5in?5zTXt@ 1003ed5c     pnglib:pngrutil.obj
 0002:00003d84       ??_C@_0BH@OKNNOGIJ@Zero?5length?5zTXt?5chunk?$AA@ 1003ed84     pnglib:pngrutil.obj
 0002:00003d9c       ??_C@_0CF@INOJJBEP@Out?5of?5memory?5processing?5zTXt?5ch@ 1003ed9c     pnglib:pngrutil.obj
 0002:00003dc4       ??_C@_0BJ@GFIDABKN@Missing?5IHDR?5before?5zTXt?$AA@ 1003edc4     pnglib:pngrutil.obj
 0002:00003de0       ??_C@_0BE@IFBNEDBM@error?5in?5user?5chunk?$AA@ 1003ede0     pnglib:pngrutil.obj
 0002:00003df4       ??_C@_0BH@OMJPKJPP@unknown?5critical?5chunk?$AA@ 1003edf4     pnglib:pngrutil.obj
 0002:00003e0c       ??_C@_0BH@KJLLHDND@Extra?5compression?5data?$AA@ 1003ee0c     pnglib:pngrutil.obj
 0002:00003e24       ??_C@_0BH@FADDMAED@Extra?5compressed?5data?4?$AA@ 1003ee24     pnglib:pngrutil.obj
 0002:00003e3c       ??_C@_0BE@JLEKBIKH@Decompression?5Error?$AA@ 1003ee3c     pnglib:pngrutil.obj
 0002:00003e50       ??_C@_0DE@IIKHIEFN@Ignoring?5attempt?5to?5set?5negative@ 1003ee50     pnglib:pngset.obj
 0002:00003e84       ??_C@_0DO@EEGLKLJK@Ignoring?5attempt?5to?5set?5chromati@ 1003ee84     pnglib:pngset.obj
 0002:00003ec8       __real@40d4f8b51eb851ec    1003eec8     pnglib:pngset.obj
 0002:00003ed0       __real@41dfffffffc00000    1003eed0     pnglib:pngset.obj
 0002:00003ed8       ??_C@_0BA@FODJPOMI@Setting?5gamma?$DN0?$AA@ 1003eed8     pnglib:pngset.obj
 0002:00003ee8       ??_C@_0BL@OOPLOBFJ@Limiting?5gamma?5to?521474?483?$AA@ 1003eee8     pnglib:pngset.obj
 0002:00003f04       ??_C@_0BP@BJIADBMD@Setting?5negative?5gamma?5to?5zero?$AA@ 1003ef04     pnglib:pngset.obj
 0002:00003f24       ??_C@_0CP@KJELKCMD@Invalid?5palette?5size?0?5hIST?5alloc@ 1003ef24     pnglib:pngset.obj
 0002:00003f54       ??_C@_0CJ@HIIPIHBM@Insufficient?5memory?5for?5hIST?5chu@ 1003ef54     pnglib:pngset.obj
 0002:00003f80       ??_C@_0BO@KOOEGEDO@Unknown?5filter?5method?5in?5IHDR?$AA@ 1003ef80     pnglib:pngset.obj
 0002:00003fa0       ??_C@_0CD@DDOOCEDP@Unknown?5compression?5method?5in?5IH@ 1003efa0     pnglib:pngset.obj
 0002:00003fc4       ??_C@_0CB@EMHJMLOA@Unknown?5interlace?5method?5in?5IHDR@ 1003efc4     pnglib:pngset.obj
 0002:00003fe8       ??_C@_0DB@FGMBGHOJ@Invalid?5color?5type?1bit?5depth?5com@ 1003efe8     pnglib:pngset.obj
 0002:0000401c       ??_C@_0BL@KPIFPGMP@Invalid?5color?5type?5in?5IHDR?$AA@ 1003f01c     pnglib:pngset.obj
 0002:00004038       ??_C@_0BK@OAKOLNFJ@Invalid?5bit?5depth?5in?5IHDR?$AA@ 1003f038     pnglib:pngset.obj
 0002:00004054       ??_C@_0DA@KJHOLOOI@Width?5is?5too?5large?5for?5libpng?5to@ 1003f054     pnglib:pngset.obj
 0002:00004084       ??_C@_0BL@PKEOJJBA@Invalid?5image?5size?5in?5IHDR?$AA@ 1003f084     pnglib:pngset.obj
 0002:000040a0       ??_C@_0CH@MBJMGPKM@image?5size?5exceeds?5user?5limits?5i@ 1003f0a0     pnglib:pngset.obj
 0002:000040c8       ??_C@_0CG@OEFPMCG@Image?5width?5or?5height?5is?5zero?5in@ 1003f0c8     pnglib:pngset.obj
 0002:000040f0       ??_C@_0CI@BJJAJFBL@Insufficient?5memory?5for?5pCAL?5par@ 1003f0f0     pnglib:pngset.obj
 0002:00004118       ??_C@_0CF@FNBJPHKN@Insufficient?5memory?5for?5pCAL?5par@ 1003f118     pnglib:pngset.obj
 0002:00004140       ??_C@_0CE@GHAOJDBK@Insufficient?5memory?5for?5pCAL?5uni@ 1003f140     pnglib:pngset.obj
 0002:00004164       ??_C@_0CG@JFEJBACA@Insufficient?5memory?5for?5pCAL?5pur@ 1003f164     pnglib:pngset.obj
 0002:0000418c       ??_C@_0BH@IKBNLCFC@Invalid?5palette?5length?$AA@ 1003f18c     pnglib:pngset.obj
 0002:000041a8       __real@3fd40346e0000000    1003f1a8     pnglib:pngset.obj
 0002:000041b0       __real@3fd50e5600000000    1003f1b0     pnglib:pngset.obj
 0002:000041b8       __real@3fe47ae140000000    1003f1b8     pnglib:pngset.obj
 0002:000041c0       __real@3fd51eb860000000    1003f1c0     pnglib:pngset.obj
 0002:000041c8       __real@3fd3333340000000    1003f1c8     pnglib:pngset.obj
 0002:000041d0       __real@3fe3333340000000    1003f1d0     pnglib:pngset.obj
 0002:000041d8       __real@3fc3333340000000    1003f1d8     pnglib:pngset.obj
 0002:000041e0       __real@3faeb851e0000000    1003f1e0     pnglib:pngset.obj
 0002:000041e8       __real@3fdd1758e0000000    1003f1e8     pnglib:pngset.obj
 0002:000041f0       ??_C@_0CN@LIEAHFGD@Insufficient?5memory?5to?5process?5i@ 1003f1f0     pnglib:pngset.obj
 0002:00004220       ??_C@_0CL@FFBJCBGI@Insufficient?5memory?5to?5process?5i@ 1003f220     pnglib:pngset.obj
 0002:0000424c       ??_C@_0BK@DENNMICD@iTXt?5chunk?5not?5supported?4?$AA@ 1003f24c     pnglib:pngset.obj
 0002:00004268       ??_C@_0BN@MLELJANO@No?5memory?5for?5sPLT?5palettes?4?$AA@ 1003f268     pnglib:pngset.obj
 0002:00004288       ??_C@_0CI@ICGKPKMD@Out?5of?5memory?5processing?5unknown@ 1003f288     pnglib:pngset.obj
 0002:000042b0       ??_C@_0CO@KHAGOEON@Out?5of?5memory?5while?5processing?5u@ 1003f2b0     pnglib:pngset.obj
 0002:000042e0       _unz_copyright             1003f2e0     zlib:unzip.obj
 0002:00004be0       ??_C@_0BH@FGKKJGOC@incorrect?5length?5check?$AA@ 1003fbe0     zlib:inflate.obj
 0002:00004bf8       ??_C@_0BF@MEIGEHBE@incorrect?5data?5check?$AA@ 1003fbf8     zlib:inflate.obj
 0002:00004c10       ??_C@_0BO@ECPMAOGG@invalid?5distance?5too?5far?5back?$AA@ 1003fc10     zlib:inflate.obj
 0002:00004c30       ??_C@_0BG@LBKINIKP@invalid?5distance?5code?$AA@ 1003fc30     zlib:inflate.obj
 0002:00004c48       ??_C@_0BM@FFFLPBBC@invalid?5literal?1length?5code?$AA@ 1003fc48     zlib:inflate.obj
 0002:00004c64       ??_C@_0BG@GMDFCBGP@invalid?5distances?5set?$AA@ 1003fc64     zlib:inflate.obj
 0002:00004c7c       ??_C@_0BM@IIMGAINC@invalid?5literal?1lengths?5set?$AA@ 1003fc7c     zlib:inflate.obj
 0002:00004c98       ??_C@_0BK@BMMPFBBH@invalid?5bit?5length?5repeat?$AA@ 1003fc98     zlib:inflate.obj
 0002:00004cb4       ??_C@_0BJ@HDEPPGOH@invalid?5code?5lengths?5set?$AA@ 1003fcb4     zlib:inflate.obj
 0002:00004cd0       ??_C@_0CE@GMIGFPBB@too?5many?5length?5or?5distance?5symb@ 1003fcd0     zlib:inflate.obj
 0002:00004cf4       ??_C@_0BN@LGAADGOK@invalid?5stored?5block?5lengths?$AA@ 1003fcf4     zlib:inflate.obj
 0002:00004d14       ??_C@_0BD@PJCBIDD@invalid?5block?5type?$AA@ 1003fd14     zlib:inflate.obj
 0002:00004d28       ??_C@_0BE@GONKLEPM@header?5crc?5mismatch?$AA@ 1003fd28     zlib:inflate.obj
 0002:00004d3c       ??_C@_0BJ@BLBBCOMO@unknown?5header?5flags?5set?$AA@ 1003fd3c     zlib:inflate.obj
 0002:00004d58       ??_C@_0BH@LIBMMIGA@incorrect?5header?5check?$AA@ 1003fd58     zlib:inflate.obj
 0002:00004d70       ??_C@_0BE@EMOGCLGO@invalid?5window?5size?$AA@ 1003fd70     zlib:inflate.obj
 0002:00004d84       ??_C@_0BL@IHKGDAEE@unknown?5compression?5method?$AA@ 1003fd84     zlib:inflate.obj
 0002:00006da0       ??_C@_02GMLFBBN@wb?$AA@    10041da0     zlib:ioapi.obj
 0002:00006da4       ??_C@_03HMFOOINA@r?$CLb?$AA@ 10041da4     zlib:ioapi.obj
 0002:00006da8       ??_C@_02JDPG@rb?$AA@       10041da8     zlib:ioapi.obj
 0002:00006dac       ??_C@_0BF@CJFPCCEG@incompatible?5version?$AA@ 10041dac     zlib:zutil.obj
 0002:00006dc4       ??_C@_0N@DFPGLBGC@buffer?5error?$AA@ 10041dc4     zlib:zutil.obj
 0002:00006dd4       ??_C@_0BE@OGGJBMCE@insufficient?5memory?$AA@ 10041dd4     zlib:zutil.obj
 0002:00006de8       ??_C@_0L@HAHMBNLP@data?5error?$AA@ 10041de8     zlib:zutil.obj
 0002:00006df4       ??_C@_0N@MKKNPMJD@stream?5error?$AA@ 10041df4     zlib:zutil.obj
 0002:00006e04       ??_C@_0L@KIJFAKBJ@file?5error?$AA@ 10041e04     zlib:zutil.obj
 0002:00006e10       ??_C@_0L@FNAOCBOG@stream?5end?$AA@ 10041e10     zlib:zutil.obj
 0002:00006e1c       ??_C@_0BA@MOKMMFOD@need?5dictionary?$AA@ 10041e1c     zlib:zutil.obj
 0002:00006e2c       _z_errmsg                  10041e2c     zlib:zutil.obj
 0002:00006e58       _inflate_copyright         10041e58     zlib:inftrees.obj
 0002:00006f88       ??_C@_0M@GNHGCLPL@Flash9g?4ocx?$AA@ 10041f88     CrashHandlerLib:CrashHandler.obj
 0002:00006f94       ??_C@_0M@KGCKPIFO@Flash9f?4ocx?$AA@ 10041f94     CrashHandlerLib:CrashHandler.obj
 0002:00006fa0       ??_C@_0M@CALOIKPA@Flash9e?4ocx?$AA@ 10041fa0     CrashHandlerLib:CrashHandler.obj
 0002:00006fac       ??_C@_0M@OLOCFJFF@Flash9d?4ocx?$AA@ 10041fac     CrashHandlerLib:CrashHandler.obj
 0002:00006fb8       ??_C@_0M@PGOHGJON@Flash9c?4ocx?$AA@ 10041fb8     CrashHandlerLib:CrashHandler.obj
 0002:00006fc4       ??_C@_0M@DNLLLKEI@Flash9b?4ocx?$AA@ 10041fc4     CrashHandlerLib:CrashHandler.obj
 0002:00006fd0       ??_C@_0BH@FJLNIMJF@Shockwave?53d?5Asset?4x32?$AA@ 10041fd0     CrashHandlerLib:CrashHandler.obj
 0002:00006fe8       ??_C@_0BB@IKCEGOCJ@AcroIEHelper?4dll?$AA@ 10041fe8     CrashHandlerLib:CrashHandler.obj
 0002:00006ffc       ??_C@_0O@CLCBIAFH@WebHelper?4dll?$AA@ 10041ffc     CrashHandlerLib:CrashHandler.obj
 0002:0000700c       ??_C@_0N@IAEGOPOO@Download?4dll?$AA@ 1004200c     CrashHandlerLib:CrashHandler.obj
 0002:0000701c       ??_C@_09IMMMOKKM@ole32?4dll?$AA@ 1004201c     CrashHandlerLib:CrashHandler.obj
 0002:00007028       ??_C@_0M@BLDKPNFN@mswsock?4dll?$AA@ 10042028     CrashHandlerLib:CrashHandler.obj
 0002:00007034       ??_C@_0L@BKDAKGAC@dirapi?4dll?$AA@ 10042034     CrashHandlerLib:CrashHandler.obj
 0002:00007040       ??_C@_0M@PONHDOCA@ieframe?4dll?$AA@ 10042040     CrashHandlerLib:CrashHandler.obj
 0002:0000704c       ??_C@_0L@KIABCLL@mshtml?4dll?$AA@ 1004204c     CrashHandlerLib:CrashHandler.obj
 0002:00007058       ??_C@_0L@PHODAIAG@RPCRT4?4dll?$AA@ 10042058     CrashHandlerLib:CrashHandler.obj
 0002:00007064       ??_C@_0N@BIPHMCIB@wmnetmgr?4dll?$AA@ 10042064     CrashHandlerLib:CrashHandler.obj
 0002:00007074       ??_C@_0BC@DIMOMKIE@QuickTimeH264?4qtx?$AA@ 10042074     CrashHandlerLib:CrashHandler.obj
 0002:00007088       ??_C@_0N@IIMHDAPA@Explorer?4EXE?$AA@ 10042088     CrashHandlerLib:CrashHandler.obj
 0002:00007098       ??_C@_09FLKFJBLM@ntdll?4dll?$AA@ 10042098     CrashHandlerLib:CrashHandler.obj
 0002:000070a4       ??_C@_0L@CDHGNOIF@Flash9?4ocx?$AA@ 100420a4     CrashHandlerLib:CrashHandler.obj
 0002:000070b0       ??_C@_0M@DAPOODEJ@firefox?4exe?$AA@ 100420b0     CrashHandlerLib:CrashHandler.obj
 0002:000070bc       ??_C@_0N@NLIHOLOP@iexplore?4exe?$AA@ 100420bc     CrashHandlerLib:CrashHandler.obj
 0002:000070cc       ??_C@_0BK@LFBKEMAM@?$CFd?9?$CF02d?9?$CF02d_?$CF02d?$CF02d?$CF02d?$AA@ 100420cc     CrashHandlerLib:CrashHandler.obj
 0002:000070e8       ??_C@_0BC@MNIKNFKD@MiniDumpWriteDump?$AA@ 100420e8     CrashHandlerLib:CrashHandler.obj
 0002:000070fc       ??_C@_1BI@NIJBKGEB@?$AAD?$AAB?$AAG?$AAH?$AAE?$AAL?$AAP?$AA?4?$AAD?$AAL?$AAL?$AA?$AA@ 100420fc     CrashHandlerLib:CrashHandler.obj
 0002:00007114       ??_C@_02PCIJFNDE@?$AN?6?$AA@ 10042114     CrashHandlerLib:CrashHandler.obj
 0002:00007118       ??_C@_0BN@MIOLEDFL@?5?5?5ProdVer?3?5?5?5?5?$CFd?4?$CFd?4?$CFd?4?$CFd?$AN?6?$AA@ 10042118     CrashHandlerLib:CrashHandler.obj
 0002:00007138       ??_C@_0BN@NPPLIEOE@?5?5?5FileVer?3?5?5?5?5?$CFd?4?$CFd?4?$CFd?4?$CFd?$AN?6?$AA@ 10042138     CrashHandlerLib:CrashHandler.obj
 0002:00007158       ??_C@_0BE@BINIANHA@?5?5?5FileDesc?3?5?5?5?$CFs?$AN?6?$AA@ 10042158     CrashHandlerLib:CrashHandler.obj
 0002:0000716c       ??_C@_0BE@PIDFFMIN@?5?5?5Product?3?5?5?5?5?$CFs?$AN?6?$AA@ 1004216c     CrashHandlerLib:CrashHandler.obj
 0002:00007180       ??_C@_0BE@KFIOGAPA@?5?5?5Company?3?5?5?5?5?$CFs?$AN?6?$AA@ 10042180     CrashHandlerLib:CrashHandler.obj
 0002:00007194       ??_C@_0L@GDBIPFOJ@Version?3?$AN?6?$AA@ 10042194     CrashHandlerLib:CrashHandler.obj
 0002:000071a0       ??_C@_0CE@LFDKMBCN@File?5Size?3?5?5?$CF?910d?5?5File?5Time?3?5?5?$CF@ 100421a0     CrashHandlerLib:CrashHandler.obj
 0002:000071c4       ??_C@_0CJ@KDNBAJGK@Image?5Base?3?50x?$CF08x?5?5Image?5Size?3?5@ 100421c4     CrashHandlerLib:CrashHandler.obj
 0002:000071f0       ??_C@_04LLEBNMDN@?$CFs?$AN?6?$AA@ 100421f0     CrashHandlerLib:CrashHandler.obj
 0002:000071f8       ??_C@_0M@JNMGKHJJ@Module?5?$CFd?$AN?6?$AA@ 100421f8     CrashHandlerLib:CrashHandler.obj
 0002:00007204       ??_C@_0CJ@EHIHMCME@?$CFd?5MB?5user?5address?5space?5?$FL?$CFd?5MB?5@ 10042204     CrashHandlerLib:CrashHandler.obj
 0002:00007230       ??_C@_0CC@DEEBIKPO@?$CFd?5MB?5paging?5file?5?$FL?$CFd?5MB?5free?$FN?4?$AN@ 10042230     CrashHandlerLib:CrashHandler.obj
 0002:00007254       ??_C@_0CG@CEBKILLG@?$CFd?5MB?5physical?5memory?5?$FL?$CFd?5MB?5fre@ 10042254     CrashHandlerLib:CrashHandler.obj
 0002:0000727c       ??_C@_0BG@KCAIBNBE@?$CFd?$CF?$CF?5memory?5in?5use?4?$AN?6?$AA@ 1004227c     CrashHandlerLib:CrashHandler.obj
 0002:00007294       ??_C@_0BB@GEKHAOPD@?$CFs?0?5run?5by?5?$CFs?4?$AN?6?$AA@ 10042294     CrashHandlerLib:CrashHandler.obj
 0002:000072a8       ??_C@_07NBCGADJA@Unknown?$AA@ 100422a8     CrashHandlerLib:CrashHandler.obj
 0002:000072b0       ??_C@_0BI@JNCPBKJH@Error?5occurred?5at?5?$CFs?4?$AN?6?$AA@ 100422b0     CrashHandlerLib:CrashHandler.obj
 0002:000072c8       ??_C@_0BK@KPJFIGIL@an?5Unknown?5exception?5type?$AA@ 100422c8     CrashHandlerLib:CrashHandler.obj
 0002:000072e4       ??_C@_0BK@HOJFPEEB@a?5Microsoft?5C?$CL?$CL?5Exception?$AA@ 100422e4     CrashHandlerLib:CrashHandler.obj
 0002:00007300       ??_C@_0BM@LDHCKNKI@a?5DLL?5Initialization?5Failed?$AA@ 10042300     CrashHandlerLib:CrashHandler.obj
 0002:0000731c       ??_C@_0BB@LJENMGNL@a?5Stack?5Overflow?$AA@ 1004231c     CrashHandlerLib:CrashHandler.obj
 0002:00007330       ??_C@_0BJ@HMGNLHOK@a?5Privileged?5Instruction?$AA@ 10042330     CrashHandlerLib:CrashHandler.obj
 0002:0000734c       ??_C@_0BE@CDPGECPC@an?5Integer?5Overflow?$AA@ 1004234c     CrashHandlerLib:CrashHandler.obj
 0002:00007360       ??_C@_0BK@FNOEEFCK@an?5Integer?5Divide?5by?5Zero?$AA@ 10042360     CrashHandlerLib:CrashHandler.obj
 0002:0000737c       ??_C@_0BC@CICINNDB@a?5Float?5Underflow?$AA@ 1004237c     CrashHandlerLib:CrashHandler.obj
 0002:00007390       ??_C@_0BE@DOBFFDCD@a?5Float?5Stack?5Check?$AA@ 10042390     CrashHandlerLib:CrashHandler.obj
 0002:000073a4       ??_C@_0BB@LAJAGHGH@a?5Float?5Overflow?$AA@ 100423a4     CrashHandlerLib:CrashHandler.obj
 0002:000073b8       ??_C@_0BK@NACDCIPD@a?5Float?5Invalid?5Operation?$AA@ 100423b8     CrashHandlerLib:CrashHandler.obj
 0002:000073d4       ??_C@_0BH@HGODNPMP@a?5Float?5Inexact?5Result?$AA@ 100423d4     CrashHandlerLib:CrashHandler.obj
 0002:000073ec       ??_C@_0BH@PIHGMMNI@a?5Float?5Divide?5by?5Zero?$AA@ 100423ec     CrashHandlerLib:CrashHandler.obj
 0002:00007404       ??_C@_0BJ@LCJBHHL@a?5Float?5Denormal?5Operand?$AA@ 10042404     CrashHandlerLib:CrashHandler.obj
 0002:00007420       ??_C@_0BI@DFIFOIBG@a?5Array?5Bounds?5Exceeded?$AA@ 10042420     CrashHandlerLib:CrashHandler.obj
 0002:00007438       ??_C@_0BH@HOHCDFKK@an?5Invalid?5Disposition?$AA@ 10042438     CrashHandlerLib:CrashHandler.obj
 0002:00007450       ??_C@_0BL@DFCKDLHL@a?5Noncontinuable?5Exception?$AA@ 10042450     CrashHandlerLib:CrashHandler.obj
 0002:0000746c       ??_C@_0BH@CMGOADMI@an?5Illegal?5Instruction?$AA@ 1004246c     CrashHandlerLib:CrashHandler.obj
 0002:00007484       ??_C@_0M@JNBECNGI@a?5No?5Memory?$AA@ 10042484     CrashHandlerLib:CrashHandler.obj
 0002:00007490       ??_C@_0BB@DKICMMFA@an?5In?5Page?5Error?$AA@ 10042490     CrashHandlerLib:CrashHandler.obj
 0002:000074a4       ??_C@_0BE@GLOKLDAN@an?5Access?5Violation?$AA@ 100424a4     CrashHandlerLib:CrashHandler.obj
 0002:000074b8       ??_C@_0N@JLDHOHAI@a?5Breakpoint?$AA@ 100424b8     CrashHandlerLib:CrashHandler.obj
 0002:000074c8       ??_C@_0BI@IPDDFHBH@a?5Datatype?5Misalignment?$AA@ 100424c8     CrashHandlerLib:CrashHandler.obj
 0002:000074e0       ??_C@_0BA@MNEFCPPO@a?5Control?9Break?$AA@ 100424e0     CrashHandlerLib:CrashHandler.obj
 0002:000074f0       ??_C@_0M@FNOJOPNP@a?5Control?9C?$AA@ 100424f0     CrashHandlerLib:CrashHandler.obj
 0002:000074fc       ??_C@_0CL@OMKINDCC@Exception?5encountered?5during?5sta@ 100424fc     CrashHandlerLib:CrashHandler.obj
 0002:00007528       ??_C@_02HAOIJKIC@?$CFc?$AA@ 10042528     CrashHandlerLib:CrashHandler.obj
 0002:0000752c       ??_C@_09CMIEKKHO@?5?5?5?5?5?5?5?5?5?$AA@ 1004252c     CrashHandlerLib:CrashHandler.obj
 0002:00007538       ??_C@_08FCCPIPOA@0x?$CF08x?3?5?$AA@ 10042538     CrashHandlerLib:CrashHandler.obj
 0002:00007544       ??_C@_05ECIELPFL@?$CF08x?5?$AA@ 10042544     CrashHandlerLib:CrashHandler.obj
 0002:0000754c       ??_C@_0N@MCABBBJA@?$AN?6?$AN?6Stack?3?$AN?6?$AA@ 1004254c     CrashHandlerLib:CrashHandler.obj
 0002:0000755c       ??_C@_0CN@DPHIKGID@EFlags?3?50x?$CF08x?5?5ESP?3?50x?$CF08x?5?5Seg@ 1004255c     CrashHandlerLib:CrashHandler.obj
 0002:0000758c       ??_C@_0CN@FNEAJLBC@EIP?3?5?5?5?50x?$CF08x?5?5EBP?3?50x?$CF08x?5?5Seg@ 1004258c     CrashHandlerLib:CrashHandler.obj
 0002:000075bc       ??_C@_0CN@HMCEKAPI@EBX?3?5?5?5?50x?$CF08x?5?5ECX?3?50x?$CF08x?5?5EDX@ 100425bc     CrashHandlerLib:CrashHandler.obj
 0002:000075ec       ??_C@_0CN@HFPOGCDG@EDI?3?5?5?5?50x?$CF08x?5?5ESI?3?50x?$CF08x?5?5EAX@ 100425ec     CrashHandlerLib:CrashHandler.obj
 0002:0000761c       ??_C@_0L@BIIJGCKB@Context?3?$AN?6?$AA@ 1004261c     CrashHandlerLib:CrashHandler.obj
 0002:00007628       ??_C@_1M@NPFJGIEI@?$AAO?$AAo?$AAp?$AAs?$AA?$CB?$AA?$AA@ 10042628     CrashHandlerLib:CrashHandler.obj
 0002:00007638       ??_C@_0IP@KBGJLEGI@The?5game?5crashed?4?6The?5crash?5repo@ 10042638     CrashHandlerLib:CrashHandler.obj
 0002:000076c8       ??_C@_1BG@OPOAEFEM@?$AAD?$AAe?$AAl?$AAe?$AAt?$AAe?$AA?$CF?$AA0?$AA2?$AAd?$AA?$AA@ 100426c8     CrashHandlerLib:CrashHandler.obj
 0002:000076e0       ??_C@_0BG@OJAHPGIL@?$AN?6?$DN?$DN?5?$FLend?5of?5?$CFs?$FN?5?$DN?$DN?$AN?6?$AA@ 100426e0     CrashHandlerLib:CrashHandler.obj
 0002:000076f8       ??_C@_09EGLJBNGG@error?4log?$AA@ 100426f8     CrashHandlerLib:CrashHandler.obj
 0002:00007704       ??_C@_03MMEAEOBL@?$DP?$DP?5?$AA@ 10042704     CrashHandlerLib:CrashHandler.obj
 0002:00007708       ??_C@_05CNDJFPDP@?$CF02x?5?$AA@ 10042708     CrashHandlerLib:CrashHandler.obj
 0002:00007710       ??_C@_0BF@PEDFBGMK@?$AN?6Bytes?5at?5CS?3EIP?3?$AN?6?$AA@ 10042710     CrashHandlerLib:CrashHandler.obj
 0002:00007728       ??_C@_02DKCKIIND@?$CFs?$AA@ 10042728     CrashHandlerLib:CrashHandler.obj
 0002:0000772c       ??_C@_0CP@PADPOHII@?$CFs?5location?5?$CF08x?5caused?5an?5acces@ 1004272c     CrashHandlerLib:CrashHandler.obj
 0002:0000775c       ??_C@_08CPFAPHAF@Write?5to?$AA@ 1004275c     CrashHandlerLib:CrashHandler.obj
 0002:00007768       ??_C@_09JHOILLPP@Read?5from?$AA@ 10042768     CrashHandlerLib:CrashHandler.obj
 0002:00007774       ??_C@_19NLLMBBJO@?$AAT?$AAi?$AAm?$AAe?$AA?$AA@ 10042774     CrashHandlerLib:CrashHandler.obj
 0002:00007780       ??_C@_0DI@HKPLNEGL@?$CFs?5caused?5?$CFs?5?$CI0x?$CF08x?$CJ?$AN?6?5?5in?5modu@ 10042780     CrashHandlerLib:CrashHandler.obj
 0002:000077b8       ??_C@_0BF@KGHEJPDC@?$CFs?5?$FLversion?3?5?$CFs?$FN?$AN?6?$AN?6?$AA@ 100427b8     CrashHandlerLib:CrashHandler.obj
 0002:000077d0       ??_C@_1BC@PLJCHAJ@?$AAF?$AAi?$AAl?$AAe?$AA?$CF?$AA0?$AA2?$AAd?$AA?$AA@ 100427d0     CrashHandlerLib:CrashHandler.obj
 0002:000077e4       ??_C@_1BE@FAIENDFF@?$AAF?$AAi?$AAl?$AAe?$AAs?$AAP?$AAa?$AAt?$AAh?$AA?$AA@ 100427e4     CrashHandlerLib:CrashHandler.obj
 0002:000077f8       ??_C@_19GFDACHI@?$AAI?$AAn?$AAf?$AAo?$AA?$AA@ 100427f8     CrashHandlerLib:CrashHandler.obj
 0002:00007804       ??_C@_1CE@LMLLJEJL@?$AAU?$AAn?$AAi?$AAt?$AAy?$AAC?$AAr?$AAa?$AAs?$AAh?$AAH?$AAa?$AAn?$AAd?$AAl?$AAe?$AAr?$AA?$AA@ 10042804     CrashHandlerLib:CrashHandler.obj
 0002:00007828       ??_C@_1BA@HJNHGNPD@?$AAA?$AAp?$AAp?$AAN?$AAa?$AAm?$AAe?$AA?$AA@ 10042828     CrashHandlerLib:CrashHandler.obj
 0002:00007838       ??_C@_02JPEBCGCN@?5?$CC?$AA@ 10042838     CrashHandlerLib:CrashHandler.obj
 0002:0000783c       ??_C@_0L@DFHNJDMN@Error?5dump?$AA@ 1004283c     CrashHandlerLib:CrashHandler.obj
 0002:00007848       ??_C@_09LGNEKANH@Error?5log?$AA@ 10042848     CrashHandlerLib:CrashHandler.obj
 0002:00007854       ??_C@_09HIBDPELJ@crash?4dmp?$AA@ 10042854     CrashHandlerLib:CrashHandler.obj
 0002:00007860       ??_C@_0L@NJHNIKCK@report?4ini?$AA@ 10042860     CrashHandlerLib:CrashHandler.obj
 0002:0000786c       ??_C@_06DIBIFALP@crash_?$AA@ 1004286c     CrashHandlerLib:CrashHandler.obj
 0002:00007874       ??_C@_06PHKFGJCD@Crash_?$AA@ 10042874     CrashHandlerLib:CrashHandler.obj
 0002:0000787c       ??_C@_01KICIPPFI@?2?$AA@   1004287c     CrashHandlerLib:MiniVersion.obj
 0002:00007880       ??_C@_0BM@CEKPECKE@?2StringFileInfo?2?$CF04x?$CF04x?2?$CFs?$AA@ 10042880     CrashHandlerLib:MiniVersion.obj
 0002:0000789c       ??_C@_0BJ@KPNNKBCP@?2VarFileInfo?2Translation?$AA@ 1004289c     CrashHandlerLib:MiniVersion.obj
 0002:000078b8       ??_C@_0M@MNPNDAHP@ProductName?$AA@ 100428b8     CrashHandlerLib:MiniVersion.obj
 0002:000078c4       ??_C@_0BA@IMJFJNNG@FileDescription?$AA@ 100428c4     CrashHandlerLib:MiniVersion.obj
 0002:000078d4       ??_C@_0M@DHIAIDA@CompanyName?$AA@ 100428d4     CrashHandlerLib:MiniVersion.obj
 0002:000078f0       __FPinit                   100428f0     LIBCMT:_fpinit_.obj
 0002:000078f4       ??_C@_05KLBDPFGC@e?$CL000?$AA@ 100428f4     LIBCMT:cvt.obj
 0002:000078fc       ??_C@_0L@KDOEJCKC@_nextafter?$AA@ 100428fc     LIBCMT:_fpexcept_.obj
 0002:00007908       ??_C@_05JGDBENOH@_logb?$AA@ 10042908     LIBCMT:_fpexcept_.obj
 0002:00007910       ??_C@_03ONILCKOB@_yn?$AA@  10042910     LIBCMT:_fpexcept_.obj
 0002:00007914       ??_C@_03NAKIGLHK@_y1?$AA@  10042914     LIBCMT:_fpexcept_.obj
 0002:00007918       ??_C@_03MJLDFKDL@_y0?$AA@  10042918     LIBCMT:_fpexcept_.obj
 0002:0000791c       ??_C@_05GKKHEGJL@frexp?$AA@ 1004291c     LIBCMT:_fpexcept_.obj
 0002:00007924       ??_C@_04KEPJIHGP@fmod?$AA@ 10042924     LIBCMT:_fpexcept_.obj
 0002:0000792c       ??_C@_06MEIMCGCF@_hypot?$AA@ 1004292c     LIBCMT:_fpexcept_.obj
 0002:00007934       ??_C@_05KBKMEMPO@_cabs?$AA@ 10042934     LIBCMT:_fpexcept_.obj
 0002:0000793c       ??_C@_05CEJMAHNP@ldexp?$AA@ 1004293c     LIBCMT:_fpexcept_.obj
 0002:00007944       ??_C@_04EHEDPDJG@modf?$AA@ 10042944     LIBCMT:_fpexcept_.obj
 0002:0000794c       ??_C@_04ODHECPBC@fabs?$AA@ 1004294c     LIBCMT:_fpexcept_.obj
 0002:00007954       ??_C@_05PBJFFIGL@floor?$AA@ 10042954     LIBCMT:_fpexcept_.obj
 0002:0000795c       ??_C@_04GFPJNGEK@ceil?$AA@ 1004295c     LIBCMT:_fpexcept_.obj
 0002:00007964       ??_C@_03IIINPABG@tan?$AA@  10042964     LIBCMT:_fpexcept_.obj
 0002:00007968       ??_C@_03LALBNOCG@cos?$AA@  10042968     LIBCMT:_fpexcept_.obj
 0002:0000796c       ??_C@_03BLEJJJBH@sin?$AA@  1004296c     LIBCMT:_fpexcept_.obj
 0002:00007970       ??_C@_04EIAKFFMI@sqrt?$AA@ 10042970     LIBCMT:_fpexcept_.obj
 0002:00007978       ??_C@_05KNGEOGJB@atan2?$AA@ 10042978     LIBCMT:_fpexcept_.obj
 0002:00007980       ??_C@_04MLLJIGOK@atan?$AA@ 10042980     LIBCMT:_fpexcept_.obj
 0002:00007988       ??_C@_04PDIFKINK@acos?$AA@ 10042988     LIBCMT:_fpexcept_.obj
 0002:00007990       ??_C@_04FIHNOPOL@asin?$AA@ 10042990     LIBCMT:_fpexcept_.obj
 0002:00007998       ??_C@_04FJHINJAO@tanh?$AA@ 10042998     LIBCMT:_fpexcept_.obj
 0002:000079a0       ??_C@_04HPJJNFIM@cosh?$AA@ 100429a0     LIBCMT:_fpexcept_.obj
 0002:000079a8       ??_C@_04COOMCNPB@sinh?$AA@ 100429a8     LIBCMT:_fpexcept_.obj
 0002:000079b0       ??_C@_05HGHHAHAP@log10?$AA@ 100429b0     LIBCMT:_fpexcept_.obj
 0002:000079b8       ??_C@_03JGHBODFD@pow?$AA@  100429b8     LIBCMT:_fpexcept_.obj
 0002:000079bc       ??_C@_03KHJOGHMM@exp?$AA@  100429bc     LIBCMT:_fpexcept_.obj
 0002:0000b300       __infinity                 10046300     LIBCMT:_87tran_.obj
 0002:0000b30a       __minfinity                1004630a     LIBCMT:_87tran_.obj
 0002:0000b314       __logemax                  10046314     LIBCMT:_87tran_.obj
 0002:0000b33a       __OP_EXPjmptab             1004633a     LIBCMT:_87tran_.obj
 0002:0000b360       __indefinite               10046360     LIBCMT:_87disp_.obj
 0002:0000b36a       __piby2                    1004636a     LIBCMT:_87disp_.obj
 0002:0000b398       __DEFAULT_CW_in_mem        10046398     LIBCMT:_common_.obj
 0002:0000b39a       __pi_by_2_to_61            1004639a     LIBCMT:_common_.obj
 0002:0000b460       ??_C@_05EOHGHCHD@exp10?$AA@ 10046460     LIBCMT:_libm_error_.obj
 0002:0000b468       ??_C@_06IMKFLFPG@1?$CDQNAN?$AA@ 10046468     LIBCMT:_x10fout_.obj
 0002:0000b470       ??_C@_05DNEBIAHO@1?$CDINF?$AA@ 10046470     LIBCMT:_x10fout_.obj
 0002:0000b478       ??_C@_05PHHOCPM@1?$CDIND?$AA@ 10046478     LIBCMT:_x10fout_.obj
 0002:0000b480       ??_C@_06PGGFOGJG@1?$CDSNAN?$AA@ 10046480     LIBCMT:_x10fout_.obj
 0002:0000b488       ??_C@_1CK@OEHDHPKK@?$AAU?$AAn?$AAi?$AAt?$AAy?$AA?4?$AAC?$AAo?$AAn?$AAt?$AAe?$AAx?$AAt?$AAS?$AAu?$AAb?$AAm?$AAe?$AAn?$AAu?$AA?$AA@ 10046488     ContextMenuWindowClass.obj
 0002:0000b4b4       ??_C@_0BD@OLBABOEK@vector?$DMT?$DO?5too?5long?$AA@ 100464b4     ContextSubmenu.obj
 0002:0000b4c8       ??_C@_0BI@CFPLBAOH@invalid?5string?5position?$AA@ 100464c8     ContextSubmenu.obj
 0002:0000b4e0       ??_C@_0BA@JFNIOLAK@string?5too?5long?$AA@ 100464e0     ContextSubmenu.obj
 0002:0000b4f0       ??_C@_00CNPNBAHC@?$AA@     100464f0     UnityWebPlayerPlugin.obj
 0002:0000b4f4       ??_C@_0M@BICCDHJH@AppleWebKit?$AA@ 100464f4     UnityWebPlayerPlugin.obj
 0002:0000b500       ??_C@_06MFKEHBAP@Safari?$AA@ 10046500     UnityWebPlayerPlugin.obj
 0002:0000b508       ??_C@_06ELAFFBDJ@Chrome?$AA@ 10046508     UnityWebPlayerPlugin.obj
 0002:0000b510       ??_C@_07MGBJGBAB@Firefox?$AA@ 10046510     UnityWebPlayerPlugin.obj
 0002:0000b518       ??_C@_1CE@HHEHNMBK@?$AAU?$AAn?$AAi?$AAt?$AAy?$AAI?$AAn?$AAt?$AAe?$AAr?$AAm?$AAe?$AAd?$AAi?$AAa?$AAt?$AAe?$AA?$AA@ 10046518     UnityWebPlayerPlugin.obj
 0002:0000b53c       ??_C@_1O@MOBNNEMB@?$AAB?$AAU?$AAT?$AAT?$AAO?$AAN?$AA?$AA@ 1004653c     UnityWebPlayerPlugin.obj
 0002:0000b54c       ??_C@_0BP@GHHJGHOC@document?4location?4reload?$CItrue?$CJ?$AA@ 1004654c     UnityWebPlayerPlugin.obj
 0002:0000b56c       ??_C@_0BG@FFDHPOJA@Closing?5plugin?5window?$AA@ 1004656c     UnityWebPlayerPlugin.obj
 0002:0000b584       ??_C@_0BN@GMFCBLJI@Error?5launching?5Unity?5Player?$AA@ 10046584     UnityWebPlayerPlugin.obj
 0002:0000b5a4       ??_C@_0P@GDACEMPM@Unknown?5error?4?$AA@ 100465a4     UnityWebPlayerPlugin.obj
 0002:0000b5b4       ??_C@_0BP@JBAAPNFM@Times?3?5download?5?$CF?41f?5load?5?$CF?41f?$AA@ 100465b4     UnityWebPlayerPlugin.obj
 0002:0000b5d4       ??_C@_1BM@GMKBAEMF@?$AAE?$AAr?$AAr?$AAo?$AAr?$AA?5?$AAd?$AAe?$AAt?$AAa?$AAi?$AAl?$AAs?$AA?$AA@ 100465d4     UnityWebPlayerPlugin.obj
 0002:0000b5f0       ??_C@_1CC@BKDLMOOJ@?$AAI?$AAn?$AAs?$AAt?$AAa?$AAl?$AAl?$AA?5?$AAM?$AAa?$AAn?$AAu?$AAa?$AAl?$AAl?$AAy?$AA?$AA@ 100465f0     UnityWebPlayerPlugin.obj
 0002:0000b614       ??_C@_1BI@FILNOEDB@?$AAD?$AAe?$AAv?$AAe?$AAl?$AAo?$AAp?$AAm?$AAe?$AAn?$AAt?$AA?$AA@ 10046614     UnityWebPlayerPlugin.obj
 0002:0000b62c       ??_C@_1CA@KODCIAHP@?$AAR?$AAe?$AAl?$AAe?$AAa?$AAs?$AAe?$AA?5?$AAC?$AAh?$AAa?$AAn?$AAn?$AAe?$AAl?$AA?$AA@ 1004662c     UnityWebPlayerPlugin.obj
 0002:0000b64c       ??_C@_0DC@DGACCBPE@http?3?1?1www?4unity3d?4com?1about?9uni@ 1004664c     UnityWebPlayerPlugin.obj
 0002:0000b680       ??_C@_1CK@DCMJIOOF@?$AAU?$AAn?$AAi?$AAt?$AAy?$AA?5?$AAP?$AAl?$AAa?$AAy?$AAe?$AAr?$AA?5?$AA4?$AA?4?$AA1?$AA?4?$AA2?$AAf?$AA1?$AA?$AA@ 10046680     UnityWebPlayerPlugin.obj
 0002:0000b6ac       ??_C@_0CH@ELMAAEIA@http?3?1?1webplayer?4unity3d?4com?1set@ 100466ac     UnityWebPlayerPlugin.obj
 0002:0000b6d4       ??_C@_04LHHJCNI@_top?$AA@  100466d4     UnityWebPlayerPlugin.obj
 0002:0000b6dc       ??_C@_0DC@MMAFCOPA@http?3?1?1www?4unity3d?4com?1unity?9web@ 100466dc     UnityWebPlayerPlugin.obj
 0002:0000b710       ??_C@_0BM@PAPJHAGI@invalid?5map?1set?$DMT?$DO?5iterator?$AA@ 10046710     UnityWebPlayerPlugin.obj
 0002:0000b72c       ??_C@_0BE@JONHPENG@map?1set?$DMT?$DO?5too?5long?$AA@ 1004672c     UnityWebPlayerPlugin.obj
 0002:0000b740       ??_7UnityWebPlayerPluginInstance@@6B@ 10046740     UnityWebPlayerPlugin.obj
 0002:0000b778       ??_C@_04LOAJBDKD@true?$AA@ 10046778     DownloadNetscape.obj
 0002:0000b780       ??_C@_03ICICOMAL@yes?$AA@  10046780     DownloadNetscape.obj
 0002:0000b784       ??_C@_01HIHLOKLC@1?$AA@    10046784     DownloadNetscape.obj
 0002:0000b788       ??_C@_03LOJEKLML@src?$AA@  10046788     DownloadNetscape.obj
 0002:0000b78c       ??_C@_0O@OLMICJDB@autoupdateURL?$AA@ 1004678c     DownloadNetscape.obj
 0002:0000b79c       ??_C@_0BH@CDKCOKGN@autoupdateURLSignature?$AA@ 1004679c     DownloadNetscape.obj
 0002:0000b7b4       ??_C@_0BE@OEKLEGFK@disableExternalCall?$AA@ 100467b4     DownloadNetscape.obj
 0002:0000b7c8       ??_C@_0BC@FIFCEAOE@disableFullscreen?$AA@ 100467c8     DownloadNetscape.obj
 0002:0000b7dc       ??_C@_0BA@DBLEKPBD@enableDebugging?$AA@ 100467dc     DownloadNetscape.obj
 0002:0000b7ec       ??_C@_0BD@MKIFFFNJ@disableContextMenu?$AA@ 100467ec     DownloadNetscape.obj
 0002:0000b800       ??_C@_0BD@BOENNFHP@firstFrameCallback?$AA@ 10046800     DownloadNetscape.obj
 0002:0000b814       ??_7Download@@6B@          10046814     WebCommonLib:Download.obj
 0002:0000b814       ??_7DownloaderNetscape@@6B@ 10046814     DownloadNetscape.obj
 0002:0000b820       ??_C@_0BA@FDMAGDNN@GetUnityVersion?$AA@ 10046820     NetscapeScriptablePlugin.obj
 0002:0000b830       ??_C@_0BB@HGPINCD@GetPluginVersion?$AA@ 10046830     NetscapeScriptablePlugin.obj
 0002:0000b844       ??_C@_0M@KOLHOMFC@SendMessage?$AA@ 10046844     NetscapeScriptablePlugin.obj
 0002:0000b850       ??_C@_0BK@NPGCJGFE@send?5to?5obj?5?$CFs?5method?5?$CFs?6?$AA@ 10046850     NetscapeScriptablePlugin.obj
 0002:0000b86c       ??_C@_0BP@MPGKJOHA@SendMessage?3?5Array?5is?5too?5deep?$AA@ 1004686c     NetscapeScriptablePlugin.obj
 0002:0000b88c       ??_C@_06IJDLPEM@length?$AA@ 1004688c     NetscapeScriptablePlugin.obj
 0002:0000b894       ??_C@_0CB@CDBINFIN@SendMessage?3?5Bad?5array?5size?5?$FL?$CFi?$FN@ 10046894     NetscapeScriptablePlugin.obj
 0002:0000b8b8       ??_C@_0CE@CAHBBMFM@SendMessage?3?5Object?5is?5not?5an?5ar@ 100468b8     NetscapeScriptablePlugin.obj
 0002:0000b8dc       ??_C@_0CJ@EJOGFANH@SendMessage?3?5Unsupported?5value?5t@ 100468dc     NetscapeScriptablePlugin.obj
 0002:0000b908       ??_C@_07GFCKPKLH@4?41?42f1?$AA@ 10046908     NetscapeScriptablePlugin.obj
 0002:0000b910       ??_C@_0BJ@LFKILBNM@Could?5not?5window?5object?4?$AA@ 10046910     NetscapeScriptablePlugin.obj
 0002:0000b92c       ??_C@_08CBBFJFMD@location?$AA@ 1004692c     NetscapeScriptablePlugin.obj
 0002:0000b938       ??_C@_04CMBCJJJD@href?$AA@ 10046938     NetscapeScriptablePlugin.obj
 0002:0000b940       ??_C@_0BM@CJHJDNMP@Could?5not?5get?5href?5property?$AA@ 10046940     NetscapeScriptablePlugin.obj
 0002:0000b95c       ??_C@_0CA@GHNAICC@Could?5not?5get?5location?5property?$AA@ 1004695c     NetscapeScriptablePlugin.obj
 0002:0000b97c       ??_C@_1CK@HMNJKCPC@?$AAU?$AAn?$AAi?$AAt?$AAy?$AA?2?$AAU?$AAn?$AAi?$AAt?$AAy?$AAW?$AAe?$AAb?$AAP?$AAl?$AAa?$AAy?$AAe?$AAr?$AA?$AA@ 1004697c     WebCommonLib:PluginManager.obj
 0002:0000b9a8       ??_C@_1CA@DPHJPKMD@?$AAU?$AAn?$AAi?$AAt?$AAy?$AA?2?$AAW?$AAe?$AAb?$AAP?$AAl?$AAa?$AAy?$AAe?$AAr?$AA?$AA@ 100469a8     WebCommonLib:PluginManager.obj
 0002:0000b9c8       ??_C@_0BK@KNADHGF@UnityWebPlayerUpdateMutex?$AA@ 100469c8     WebCommonLib:PluginManager.obj
 0002:0000b9e4       ??_C@_04FKNHOCAN@Mono?$AA@ 100469e4     WebCommonLib:PluginManager.obj
 0002:0000b9ec       ??_C@_0M@KMGBBLKI@UnityPlayer?$AA@ 100469ec     WebCommonLib:PluginManager.obj
 0002:0000b9f8       ??_C@_0M@GGKKKOHP@UnityPlugin?$AA@ 100469f8     WebCommonLib:PluginManager.obj
 0002:0000ba04       ??_C@_1CO@OIDNHGMC@?$AAU?$AAn?$AAi?$AAt?$AAy?$AA?4?$AAT?$AAi?$AAm?$AAe?$AAr?$AAW?$AAi?$AAn?$AAd?$AAo?$AAw?$AAC?$AAl?$AAa?$AAs?$AAs?$AA?$AA@ 10046a04     WebCommonLib:PluginManager.obj
 0002:0000ba34       ??_C@_0BN@HPKFFGJB@UnityWebPlayerReleaseChannel?$AA@ 10046a34     WebCommonLib:PluginManager.obj
 0002:0000ba54       ??_C@_06IMCHFAKP@Stable?$AA@ 10046a54     WebCommonLib:PluginManager.obj
 0002:0000ba5c       ??_C@_0BK@JHGENDFB@UnityWebPlayerDevelopment?$AA@ 10046a5c     WebCommonLib:PluginManager.obj
 0002:0000ba78       ??_C@_0N@GOEEHPBL@?9Development?$AA@ 10046a78     WebCommonLib:PluginManager.obj
 0002:0000ba88       ??_C@_06JECEJHIJ@loader?$AA@ 10046a88     WebCommonLib:PluginManager.obj
 0002:0000ba90       ??_C@_06BALNJMNP@player?$AA@ 10046a90     WebCommonLib:PluginManager.obj
 0002:0000ba98       ??_C@_04JLBGMNAJ@mono?$AA@ 10046a98     WebCommonLib:PluginManager.obj
 0002:0000baa0       ??_C@_03MGHMBJCF@log?$AA@  10046aa0     WebCommonLib:PluginManager.obj
 0002:0000baa4       ??_C@_0BC@DPLABALD@manager_debug?4txt?$AA@ 10046aa4     WebCommonLib:PluginManager.obj
 0002:0000bab8       ??_C@_04LCMACLFG@?4txt?$AA@ 10046ab8     WebCommonLib:PluginManager.obj
 0002:0000bac0       ??_C@_08PNAGJHAJ@manager_?$AA@ 10046ac0     WebCommonLib:PluginManager.obj
 0002:0000bacc       ??_C@_0BJ@IFIALDCJ@UNITY_WEBPLAYER_LOG_FILE?$AA@ 10046acc     WebCommonLib:PluginManager.obj
 0002:0000bae8       ??_C@_0BF@HJNHEAON@4?41?42f1_911c7369eeac?$AA@ 10046ae8     WebCommonLib:PluginManager.obj
 0002:0000bb00       ??_C@_0BN@LIIMKABC@Manager?5starting?0?5version?5?$CFs?$AA@ 10046b00     WebCommonLib:PluginManager.obj
 0002:0000bb20       ??_C@_0BF@ODJKNKKD@UnityBugReporter?4exe?$AA@ 10046b20     WebCommonLib:PluginManager.obj
 0002:0000bb38       ??_C@_0BL@KJKHBLOK@Unity?54?41?42f1_911c7369eeac?$AA@ 10046b38     WebCommonLib:PluginManager.obj
 0002:0000bb54       ??_C@_0BB@CDIOOPAI@Unity?5Web?5Player?$AA@ 10046b54     WebCommonLib:PluginManager.obj
 0002:0000bb68       ??_C@_0BB@IJAGOILP@Manager?5log?5file?$AA@ 10046b68     WebCommonLib:PluginManager.obj
 0002:0000bb7c       ??_C@_0N@LGMFGCMI@Log?5file?5?$CD?$CFi?$AA@ 10046b7c     WebCommonLib:PluginManager.obj
 0002:0000bb8c       ??_C@_01KMDKNFGN@?1?$AA@   10046b8c     WebCommonLib:PluginManager.obj
 0002:0000bb90       ??_C@_0BD@HAHLKBOP@Getting?5update?3?5?$CFs?$AA@ 10046b90     WebCommonLib:PluginManager.obj
 0002:0000bba4       ??_C@_02DJGKEECL@?4?4?$AA@ 10046ba4     WebCommonLib:PluginManager.obj
 0002:0000bba8       ??_C@_0L@MFNFJPGK@info?4plist?$AA@ 10046ba8     WebCommonLib:PluginManager.obj
 0002:0000bbb4       ??_C@_0BA@ELDKACDE@CFBundleVersion?$AA@ 10046bb4     WebCommonLib:PluginManager.obj
 0002:0000bbc4       ??_C@_0BA@PGBPBICB@ApplySelfUpdate?$AA@ 10046bc4     WebCommonLib:PluginManager.obj
 0002:0000bbd4       ??_C@_0BG@GINNJFIF@Unity?9WebPlugin?9Self?9?$AA@ 10046bd4     WebCommonLib:PluginManager.obj
 0002:0000bbec       ??_C@_0CF@PCNNNLPK@ApplySelfUpdate?5failed?5to?5decomp@ 10046bec     WebCommonLib:PluginManager.obj
 0002:0000bc14       ??_C@_0DE@FGMCEABG@ApplySelfUpdate?5failed?3?5update?5h@ 10046c14     WebCommonLib:PluginManager.obj
 0002:0000bc48       ??_C@_1BK@MBABLNAI@?$AAP?$AAl?$AAu?$AAg?$AAi?$AAn?$AAB?$AAu?$AAn?$AAd?$AAl?$AAe?$AA?$AA@ 10046c48     WebCommonLib:PluginManager.obj
 0002:0000bc64       ??_C@_0CI@FAEBKPCE@ApplyUpdate?3?5got?5unknown?5bundle?$DN@ 10046c64     WebCommonLib:PluginManager.obj
 0002:0000bc8c       ??_C@_0CC@EHDNDOCH@ApplyUpdate?3?5bundle?$DN?$CFi?5version?$DN?$CF@ 10046c8c     WebCommonLib:PluginManager.obj
 0002:0000bcb0       ??_C@_0BG@PILFFPEF@UnityWebPluginUpdate?9?$AA@ 10046cb0     WebCommonLib:PluginManager.obj
 0002:0000bcc8       ??_C@_0DI@LNOAKKEP@ApplyUpdate?5?$CIbundle?$DN?$CFi?5version?$DN?$CF@ 10046cc8     WebCommonLib:PluginManager.obj
 0002:0000bd00       ??_C@_0CB@GAMJOCB@Invalid?5auto?9update?5file?5format?4@ 10046d00     WebCommonLib:PluginManager.obj
 0002:0000bd24       ??_C@_0DP@FDNCFAOI@ApplyUpdate?5?$CIbundle?$DN?$CFi?5version?$DN?$CF@ 10046d24     WebCommonLib:PluginManager.obj
 0002:0000bd64       ??_C@_0DD@JKBPMOIH@Invalid?5auto?9update?5file?5?$CIno?5rev@ 10046d64     WebCommonLib:PluginManager.obj
 0002:0000bd98       ??_C@_0DM@DGDPIJJK@ApplyUpdate?5?$CIbundle?$DN?$CFi?5version?$DN?$CF@ 10046d98     WebCommonLib:PluginManager.obj
 0002:0000bdd4       ??_C@_0DE@KONPCKPF@Invalid?5auto?9update?5file?5?$CIrevisi@ 10046dd4     WebCommonLib:PluginManager.obj
 0002:0000be08       ??_C@_1BK@JAJFBAFH@?$AAP?$AAl?$AAa?$AAy?$AAe?$AAr?$AAB?$AAu?$AAn?$AAd?$AAl?$AAe?$AA?$AA@ 10046e08     WebCommonLib:PluginManager.obj
 0002:0000be24       ??_C@_1BG@IBPLJLGK@?$AAM?$AAo?$AAn?$AAo?$AAB?$AAu?$AAn?$AAd?$AAl?$AAe?$AA?$AA@ 10046e24     WebCommonLib:PluginManager.obj
 0002:0000be3c       ??_C@_1DC@MGMCFNCA@?$AAS?$AAO?$AAF?$AAT?$AAW?$AAA?$AAR?$AAE?$AA?2?$AAU?$AAn?$AAi?$AAt?$AAy?$AA?2?$AAW?$AAe?$AAb?$AAP?$AAl?$AAa?$AAy?$AAe?$AAr?$AA?$AA@ 10046e3c     WebCommonLib:PluginManager.obj
 0002:0000be70       ??_C@_1BE@DNDHOCGP@?$AAD?$AAi?$AAr?$AAe?$AAc?$AAt?$AAo?$AAr?$AAy?$AA?$AA@ 10046e70     WebCommonLib:PluginManager.obj
 0002:0000be84       ??_C@_1BI@BNFKGMFK@?$AAs?$AAh?$AAe?$AAl?$AAl?$AA3?$AA2?$AA?4?$AAd?$AAl?$AAl?$AA?$AA@ 10046e84     WebCommonLib:PluginManager.obj
 0002:0000be9c       ??_C@_0BF@OMOLCJCE@SHGetKnownFolderPath?$AA@ 10046e9c     WebCommonLib:PluginManager.obj
 0002:0000beb4       ??_C@_1DC@JDEHIBLG@?$AAU?$AAn?$AAi?$AAt?$AAy?$AAW?$AAe?$AAb?$AAP?$AAl?$AAa?$AAy?$AAe?$AAr?$AAU?$AAp?$AAd?$AAa?$AAt?$AAe?$AA?4?$AAe?$AAx?$AAe?$AA?$AA@ 10046eb4     WebCommonLib:PluginManager.obj
 0002:0000bee8       ??_C@_05MJJMKKFN@3?4x?4x?$AA@ 10046ee8     WebCommonLib:PluginManager.obj
 0002:0000bef0       ??_C@_0BN@HFHEPJHB@Failed?5to?5apply?5auto?9update?4?$AA@ 10046ef0     WebCommonLib:PluginManager.obj
 0002:0000bf10       ??_C@_0BC@KIADFMKJ@Update?5failed?3?5?$CFs?$AA@ 10046f10     WebCommonLib:PluginManager.obj
 0002:0000bf24       ??_C@_0L@DKDHNGPJ@?9win32?4zip?$AA@ 10046f24     WebCommonLib:PluginManager.obj
 0002:0000bf40       ??_C@_0BP@IBDLJFM@UNITY_FORCE_DEVELOPMENT_PLUGIN?$AA@ 10046f40     WebCommonLib:WebPluginUtility.obj
 0002:0000bf60       ??_C@_03IPHJCBHH@YES?$AA@  10046f60     WebCommonLib:WebPluginUtility.obj
 0002:0000bf64       ??_C@_0BN@BDCNAGEB@UNITY_DISABLE_PLUGIN_UPDATES?$AA@ 10046f64     WebCommonLib:WebPluginUtility.obj
 0002:0000bf84       ??_C@_02KAJCLHKP@no?$AA@   10046f84     WebCommonLib:WebPluginUtility.obj
 0002:0000bf88       ??_C@_0BO@LIBNJOEH@UNITY_FORCE_WEBPLAYER_VERSION?$AA@ 10046f88     WebCommonLib:WebPluginUtility.obj
 0002:0000bfa8       ??_C@_0BF@KOAHENNH@UNITY_KEEP_LOG_FILES?$AA@ 10046fa8     WebCommonLib:WebPluginUtility.obj
 0002:0000bfc0       ??_C@_06PIBLOKJG@1?42?418?$AA@ 10046fc0     WebCommonLib:ProgressDisplayWin.obj
 0002:0000bfc8       ??_C@_1O@LBFOCELB@?$AAB?$AAI?$AAN?$AAA?$AAR?$AAY?$AA?$AA@ 10046fc8     WebCommonLib:ProgressDisplayWin.obj
 0002:0000bfd8       ??_C@_1BA@DNKKBBGG@?$AAV?$AAe?$AAr?$AAd?$AAa?$AAn?$AAa?$AA?$AA@ 10046fd8     WebCommonLib:ProgressDisplayWin.obj
 0002:0000bfe8       ??_C@_04FGEHGIFJ@temp?$AA@ 10046fe8     WebCommonLib:PluginInstance.obj
 0002:0000bff0       ??_C@_0O@GKOJBPMP@log_debug?4txt?$AA@ 10046ff0     WebCommonLib:PluginInstance.obj
 0002:0000c000       ??_C@_04HGOBOJMF@log_?$AA@ 10047000     WebCommonLib:PluginInstance.obj
 0002:0000c008       ??_C@_0FO@PJADLOEP@Instance?5starting?0?5version?5?$CFs?0?5U@ 10047008     WebCommonLib:PluginInstance.obj
 0002:0000c068       ??_C@_0BK@EMKBLCLG@Instance?5?$CFs?5shutting?5down?$AA@ 10047068     WebCommonLib:PluginInstance.obj
 0002:0000c084       ??_C@_0M@COEHNKPE@Datafile?5?$CFs?$AA@ 10047084     WebCommonLib:PluginInstance.obj
 0002:0000c090       ??_C@_0DF@BKLMMMBO@Setting?5error?5display?3?5?8?$CFs?8?0?5det@ 10047090     WebCommonLib:PluginInstance.obj
 0002:0000c0c8       ??_C@_0DD@EECEFDD@Data?5file?5is?5corrupt?5?$CInot?5a?5Unit@ 100470c8     WebCommonLib:PluginInstance.obj
 0002:0000c0fc       ??_C@_0BC@IFGHNOGB@Invalid?5data?5file?$AA@ 100470fc     WebCommonLib:PluginInstance.obj
 0002:0000c110       ??_C@_0BO@HCOGIMBD@Download?5failed?0?5please?5retry?$AA@ 10047110     WebCommonLib:PluginInstance.obj
 0002:0000c130       ??_C@_0BN@FOIBJCAM@Failed?5to?5download?5data?5file?$AA@ 10047130     WebCommonLib:PluginInstance.obj
 0002:0000c150       ??_C@_0BI@DHBJAJGP@Unknown?5download?5status?$AA@ 10047150     WebCommonLib:PluginInstance.obj
 0002:0000c168       ??_C@_0P@DHEBFDOP@Internal?5error?$AA@ 10047168     WebCommonLib:PluginInstance.obj
 0002:0000c178       ??_C@_0CK@KENKOJJH@SendMessage?3?5no?5object?5or?5functi@ 10047178     WebCommonLib:PluginInstance.obj
 0002:0000c1a4       ??_C@_1BC@GDMECMAK@?$AAk?$AAe?$AAr?$AAn?$AAe?$AAl?$AA3?$AA2?$AA?$AA@ 100471a4     WebCommonLib:WinWebUtils.obj
 0002:0000c1b8       ??_C@_0BL@OLEDJOGO@QueryUnbiasedInterruptTime?$AA@ 100471b8     WebCommonLib:WinWebUtils.obj
 0002:0000c1d4       ??_C@_0M@CJNAABJD@bordercolor?$AA@ 100471d4     WebCommonLib:ProgressDisplay.obj
 0002:0000c1e0       ??_C@_09CIMBEKCH@textcolor?$AA@ 100471e0     WebCommonLib:ProgressDisplay.obj
 0002:0000c1ec       ??_C@_0BA@CPFCGCFN@backgroundcolor?$AA@ 100471ec     WebCommonLib:ProgressDisplay.obj
 0002:0000c1fc       ??_C@_0BA@NPDBPKI@backgroundimage?$AA@ 100471fc     WebCommonLib:ProgressDisplay.obj
 0002:0000c20c       ??_C@_09GLHFJHOD@logoimage?$AA@ 1004720c     WebCommonLib:ProgressDisplay.obj
 0002:0000c218       ??_C@_0BD@BJGAMFCN@progressframeimage?$AA@ 10047218     WebCommonLib:ProgressDisplay.obj
 0002:0000c22c       ??_C@_0BB@GINBNKCI@progressbarimage?$AA@ 1004722c     WebCommonLib:ProgressDisplay.obj
 0002:0000c240       ??_C@_0BA@NMIHJOMC@revisions?4plist?$AA@ 10047240     WebCommonLib:RevisionsQuery.obj
 0002:0000c250       ??_C@_0CA@PKLBIJDO@UNITY_REVISIONS_REQUEST_TIMEOUT?$AA@ 10047250     WebCommonLib:RevisionsQuery.obj
 0002:0000c270       ??_C@_0BO@HHGNNPHA@http?3?1?1webplayer?4unity3d?4com?1?$AA@ 10047270     WebCommonLib:RevisionsQuery.obj
 0002:0000c290       ??_C@_0CH@FIMIHNAK@http?3?1?1autoupdate?9revision?4unity@ 10047290     WebCommonLib:RevisionsQuery.obj
 0002:0000c2b8       ??_C@_0CC@LNCCEEBP@http?3?1?1wp?9360?4unity3d?4com?1unity3@ 100472b8     WebCommonLib:RevisionsQuery.obj
 0002:0000c2dc       ??_C@_0BP@DGOBBOLP@UNITY_REDIRECT_DOWNLOAD_FOLDER?$AA@ 100472dc     WebCommonLib:RevisionsQuery.obj
 0002:0000c2fc       ??_C@_0CA@HFPCIPFM@UNITY_REDIRECT_REVISIONS_FOLDER?$AA@ 100472fc     WebCommonLib:RevisionsQuery.obj
 0002:0000c31c       ??_C@_0BM@MAKDHPEO@autodownload_webplugin?93?4x?1?$AA@ 1004731c     WebCommonLib:RevisionsQuery.obj
 0002:0000c338       ??_C@_0CF@OMJMJMID@Global?5revisions?5download?5failed@ 10047338     WebCommonLib:RevisionsQuery.obj
 0002:0000c360       ??_C@_0FI@HHFPKAIA@Requesting?5plugin?5update?4?5Requir@ 10047360     WebCommonLib:RevisionsQuery.obj
 0002:0000c3b8       ??_C@_0CF@LDGGDADO@Failed?5to?5parse?5global?5revisions@ 100473b8     WebCommonLib:RevisionsQuery.obj
 0002:0000c3e0       ??_C@_0BC@LGPIDHBK@?5?$EA?$CG?$DL?3?$DM?$DO?$DN?$DP?$CC?8?1?2?$CB?$CD?$CF?$CL?$AA@ 100473e0     WebCommonLib:RevisionsQuery.obj
 0002:0000c3f4       ??_C@_05EHJIPHKB@?$CF?$CF?$CF2x?$AA@ 100473f4     WebCommonLib:RevisionsQuery.obj
 0002:0000c3fc       ??_C@_0O@JOAPDPIB@Referer?3?5?$CFs?$AN?6?$AA@ 100473fc     WebCommonLib:RevisionsQuery.obj
 0002:0000c40c       ??_C@_01HNPIGOCE@?$CG?$AA@ 1004740c     WebCommonLib:RevisionsQuery.obj
 0002:0000c410       ??_C@_08INNCGMHH@content?$DN?$AA@ 10047410     WebCommonLib:RevisionsQuery.obj
 0002:0000c41c       ??_C@_05GDEIIDKP@page?$DN?$AA@ 1004741c     WebCommonLib:RevisionsQuery.obj
 0002:0000c424       ??_C@_06FKKAOKII@secid?$DN?$AA@ 10047424     WebCommonLib:RevisionsQuery.obj
 0002:0000c42c       ??_C@_04GFJLOHHD@?$CF?43f?$AA@ 1004742c     WebCommonLib:RevisionsQuery.obj
 0002:0000c434       ??_C@_0P@NIODGODB@lastQueryTime?$DN?$AA@ 10047434     WebCommonLib:RevisionsQuery.obj
 0002:0000c444       ??_C@_08BBLDJMAO@runtime?$DN?$AA@ 10047444     WebCommonLib:RevisionsQuery.obj
 0002:0000c450       ??_C@_06FOAKIDDH@https?3?$AA@ 10047450     WebCommonLib:RevisionsQuery.obj
 0002:0000c458       ??_C@_01OGPIMHDM@?$DP?$AA@ 10047458     WebCommonLib:RevisionsQuery.obj
 0002:0000c45c       ??_C@_07BGIEAJGJ@unsecid?$AA@ 1004745c     WebCommonLib:RevisionsQuery.obj
 0002:0000c464       ??_C@_01JOAMLHOP@?9?$AA@   10047464     WebCommonLib:RevisionsQuery.obj
 0002:0000c468       ??_C@_0BP@DJADOAJD@Player?5hash?5?$CFs?5is?5blacklisted?6?$AA@ 10047468     WebCommonLib:RevisionsQuery.obj
 0002:0000c488       ??_C@_05PNFNNPOP@secid?$AA@ 10047488     WebCommonLib:RevisionsQuery.obj
 0002:0000c490       ??_C@_0BK@KIOKMILI@Player?5hash?5?$CFs?5not?5known?6?$AA@ 10047490     WebCommonLib:RevisionsQuery.obj
 0002:0000c4ac       ??_C@_0CA@DBIFNPPH@Player?5hash?5?$CFs?5not?5whitelisted?6?$AA@ 100474ac     WebCommonLib:RevisionsQuery.obj
 0002:0000c4d0       ??_C@_0IF@MJHJDOBI@Can?8t?5load?5web?5player?5because?5it@ 100474d0     WebCommonLib:RevisionsQuery.obj
 0002:0000c558       ??_C@_0CF@MGBJCOC@Can?8t?5load?4?5Built?5with?5beta?5rele@ 10047558     WebCommonLib:RevisionsQuery.obj
 0002:0000c580       ??_C@_0HA@ILEEAHN@A?5newer?5version?5of?5Unity?5Web?5Pla@ 10047580     WebCommonLib:RevisionsQuery.obj
 0002:0000c5f0       ??_C@_0CC@PAAOMCCF@Failed?5to?5update?5Unity?5Web?5Playe@ 100475f0     WebCommonLib:RevisionsQuery.obj
 0002:0000c614       ??_C@_0BL@GBHABEEF@?6Please?5install?5manually?4?6?$AA@ 10047614     WebCommonLib:RevisionsQuery.obj
 0002:0000c630       ??_C@_0EO@LLGLLLGC@A?5newer?5version?5of?5Unity?5Web?5Pla@ 10047630     WebCommonLib:RevisionsQuery.obj
 0002:0000c680       ??_C@_0HK@MMHHMMNH@A?5newer?5version?5of?5Unity?5Web?5Pla@ 10047680     WebCommonLib:RevisionsQuery.obj
 0002:0000c700       ??_C@_0FF@NCGMFGFL@A?5newer?5version?5of?5Unity?5Web?5Pla@ 10047700     WebCommonLib:RevisionsQuery.obj
 0002:0000c758       ??_C@_0GA@HFIKEGB@Requesting?5bundle?5?$CFd?5?$CI?$CFs?$CJ?5update@ 10047758     WebCommonLib:RevisionsQuery.obj
 0002:0000c7b8       ??_C@_0HF@OFPOGCGI@Unity?5Web?5Player?5update?5finished@ 100477b8     WebCommonLib:RevisionsQuery.obj
 0002:0000c830       ??_C@_0BM@FLNDFOHO@Failed?5to?5parse?5version?3?5?$CFs?$AA@ 10047830     WebCommonLib:RevisionsQuery.obj
 0002:0000c850       ??_C@_0FG@LHGJBAHM@Some?5files?5are?5missing?5or?5corrup@ 10047850     WebCommonLib:RevisionsQuery.obj
 0002:0000c8a8       ??_C@_0CM@LDJOMPHD@Unity?5Web?5Player?5is?5not?5installe@ 100478a8     WebCommonLib:RevisionsQuery.obj
 0002:0000c8d4       ??_C@_0M@PBILJBFF@monoVersion?$AA@ 100478d4     WebCommonLib:RevisionsQuery.obj
 0002:0000c8e0       ??_C@_0BE@OOGBEEJL@monoMinimumRevision?$AA@ 100478e0     WebCommonLib:RevisionsQuery.obj
 0002:0000c8f4       ??_C@_0DN@JAFFBJDE@Required?5mono?5revision?5is?50?5?$CIver@ 100478f4     WebCommonLib:RevisionsQuery.obj
 0002:0000c934       ??_C@_08PAMBCCJ@channels?$AA@ 10047934     WebCommonLib:RevisionsQuery.obj
 0002:0000c940       ??_C@_07CPCPJPKL@version?$AA@ 10047940     WebCommonLib:RevisionsQuery.obj
 0002:0000c948       ??_C@_0M@MEHAGKFI@channelName?$AA@ 10047948     WebCommonLib:RevisionsQuery.obj
 0002:0000c954       ??_C@_04IBOFHAPJ@hide?$AA@ 10047954     WebCommonLib:RevisionsQuery.obj
 0002:0000c95c       ??_C@_0P@EIKOPGFE@latestRevision?$AA@ 1004795c     WebCommonLib:RevisionsQuery.obj
 0002:0000c96c       ??_C@_0BA@OAPHKLHO@minimumRevision?$AA@ 1004796c     WebCommonLib:RevisionsQuery.obj
 0002:0000c97c       ??_C@_0BA@FLBBEFO@updateFilesPath?$AA@ 1004797c     WebCommonLib:RevisionsQuery.obj
 0002:0000c98c       ??_C@_0CB@NEDKDKML@Timed?5out?5on?5global?5version?5info@ 1004798c     WebCommonLib:RevisionsQuery.obj
 0002:0000c9b0       ??_C@_0N@IPLGBNNJ@https?3?1?1ssl?9?$AA@ 100479b0     WebCommonLib:RevisionsQuery.obj
 0002:0000c9c0       ??_C@_03GACAABJG@?3?1?1?$AA@ 100479c0     WebCommonLib:RevisionsQuery.obj
 0002:0000c9c4       ??_C@_07FGAOOBMN@http?3?1?1?$AA@ 100479c4     WebCommonLib:RevisionsQuery.obj
 0002:0000c9cc       ??_C@_0CD@BDPMEBHI@Verification?5of?5update?5URL?5faile@ 100479cc     WebCommonLib:RevisionsQuery.obj
 0002:0000c9f0       ??_C@_15GJMILFGI@?$AAa?$AAt?$AA?$AA@ 100479f0     WebCommonLib:Logger.obj
 0002:0000c9f8       ??_C@_0DN@GJNGJFP@?9?9?9?9?9?9?9?9?9?9?9?9?9?9?9?9?9?9?9?9?9?9?9?9?9?9?9?9?9?9?9?9@ 100479f8     WebCommonLib:Logger.obj
 0002:0000ca38       ??_C@_0CA@FLJOKIJ@?$CF02i?$CF02i?$CF02i?5?$CF02i?3?$CF02i?3?$CF02i?5?$CFs?6?$AA@ 10047a38     WebCommonLib:Logger.obj
 0002:0000ca58       ??_C@_04BCIDKIGN@dict?$AA@ 10047a58     WebCommonLib:MiniXmlFile.obj
 0002:0000ca60       ??_C@_15JJPIMNBO@?$AAr?$AAb?$AA?$AA@ 10047a60     WebCommonLib:MiniXmlFile.obj
 0002:0000ca68       ??_C@_03ICHNJLJF@key?$AA@  10047a68     WebCommonLib:MiniXmlFile.obj
 0002:0000ca6c       ??_C@_06ICGJLFIM@string?$AA@ 10047a6c     WebCommonLib:MiniXmlFile.obj
 0002:0000ca74       ??_C@_05HIFJDKLD@array?$AA@ 10047a74     WebCommonLib:MiniXmlFile.obj
 0002:0000ca7c       ??_C@_1BM@LBJAMDKE@?$AAU?$AAn?$AAi?$AAn?$AAs?$AAt?$AAa?$AAl?$AAl?$AA?4?$AAe?$AAx?$AAe?$AA?$AA@ 10047a7c     WebCommonLib:UpdaterProxy.obj
 0002:0000ca98       ??_C@_1CK@BFGAMPFN@?$AAU?$AAn?$AAi?$AAt?$AAy?$AAB?$AAu?$AAg?$AAR?$AAe?$AAp?$AAo?$AAr?$AAt?$AAe?$AAr?$AA?4?$AAe?$AAx?$AAe?$AA?$AA@ 10047a98     WebCommonLib:UpdaterProxy.obj
 0002:0000cac4       ??_C@_1BG@JMKNCDKP@?$AAi?$AAn?$AAf?$AAo?$AA?4?$AAp?$AAl?$AAi?$AAs?$AAt?$AA?$AA@ 10047ac4     WebCommonLib:UpdaterProxy.obj
 0002:0000cadc       ??_C@_1CK@NCFLLGJH@?$AAU?$AAn?$AAi?$AAt?$AAy?$AAW?$AAe?$AAb?$AAP?$AAl?$AAu?$AAg?$AAi?$AAn?$AAA?$AAX?$AA?4?$AAo?$AAc?$AAx?$AA?$AA@ 10047adc     WebCommonLib:UpdaterProxy.obj
 0002:0000cb08       ??_C@_1O@CBCBFMLE@?$AAl?$AAo?$AAa?$AAd?$AAe?$AAr?$AA?$AA@ 10047b08     WebCommonLib:UpdaterProxy.obj
 0002:0000cb18       ??_C@_1CA@JGJHDGMC@?$AAn?$AAp?$AAU?$AAn?$AAi?$AAt?$AAy?$AA3?$AAD?$AA3?$AA2?$AA?4?$AAd?$AAl?$AAl?$AA?$AA@ 10047b18     WebCommonLib:UpdaterProxy.obj
 0002:0000cb38       ??_C@_0DD@BIOBGEOC@Failed?5to?5create?5update?4?5Failed?5@ 10047b38     WebCommonLib:UpdaterProxy.obj
 0002:0000cb6c       ??_C@_0CJ@LOPGJMBA@Failed?5to?5create?5update?4?5Pipe?5is@ 10047b6c     WebCommonLib:UpdaterProxy.obj
 0002:0000cb98       ??_C@_0DM@EMLCFPKN@Failed?5to?5create?5update?4?5Failed?5@ 10047b98     WebCommonLib:UpdaterProxy.obj
 0002:0000cc04       ??_C@_0DH@PCGLNNFL@Failed?5to?5create?5update?4?5Failed?5@ 10047c04     WebCommonLib:UpdaterProxy.obj
 0002:0000cc3c       ??_C@_0DI@GCCNECDH@Failed?5to?5create?5update?4?5Failed?5@ 10047c3c     WebCommonLib:UpdaterProxy.obj
 0002:0000cc74       ??_C@_0DG@DFPGGFLG@Failed?5to?5create?5update?4?5Failed?5@ 10047c74     WebCommonLib:UpdaterProxy.obj
 0002:0000ccac       ??_C@_0CC@GKAFOGEI@Failed?5to?5accept?5update?5response@ 10047cac     WebCommonLib:UpdaterProxy.obj
 0002:0000cd14       ??_C@_0DG@LGACJHHO@Failed?5to?5launch?5updater?4?5Failed@ 10047d14     WebCommonLib:UpdaterProxy.obj
 0002:0000cd4c       ??_C@_0CP@MICENAMK@Failed?5to?5launch?5updater?4?5Failed@ 10047d4c     WebCommonLib:UpdaterProxy.obj
 0002:0000cd7c       ??_C@_19BDAJEHDN@?$AAo?$AAp?$AAe?$AAn?$AA?$AA@ 10047d7c     WebCommonLib:UpdaterProxy.obj
 0002:0000cd88       ??_C@_0CD@HEBOMJCL@Failed?5to?5launch?5external?5update@ 10047d88     WebCommonLib:UpdaterProxy.obj
 0002:0000cdac       ??_C@_0CD@NIICJOFE@Failed?5to?5launch?5internal?5update@ 10047dac     WebCommonLib:UpdaterProxy.obj
 0002:0000cdd0       ??_C@_0BJ@NKDJFPPG@Updater?5did?5not?5connect?4?$AA@ 10047dd0     WebCommonLib:UpdaterProxy.obj
 0002:0000cdec       ??_C@_0CC@EAEPNBDL@Updater?5did?5not?5accept?5handshake@ 10047dec     WebCommonLib:UpdaterProxy.obj
 0002:0000ce10       ??_C@_0CI@HLLNFCOL@Updater?5did?5not?5respond?5with?5han@ 10047e10     WebCommonLib:UpdaterProxy.obj
 0002:0000ce38       ??_C@_0CE@KEMKOFOB@Invalid?5updater?5handshake?5respon@ 10047e38     WebCommonLib:UpdaterProxy.obj
 0002:0000ce5c       ??_C@_0BB@MOGOBHAF@list?$DMT?$DO?5too?5long?$AA@ 10047e5c     WebCommonLib:UpdaterProxy.obj
 0002:0000ce70       ??_7UpdaterProxy@@6B@      10047e70     WebCommonLib:UpdaterProxy.obj
 0002:0000ce78       ??_7UpdateOperation@UpdaterProxy@@6B@ 10047e78     WebCommonLib:UpdaterProxy.obj
 0002:0000ce80       ??_C@_0DB@FBNNHDJM@This?5machine?5does?5not?5support?5SS@ 10047e80     WebCommonLib:UnityLoader.obj
 0002:0000ceb4       ??_C@_02MFDMBIJM@ok?$AA@   10047eb4     WebCommonLib:UnityLoader.obj
 0002:0000ceb8       ??_C@_06OHCJKBJM@FAILED?$AA@ 10047eb8     WebCommonLib:UnityLoader.obj
 0002:0000cec0       ??_C@_0BB@ELCMOPBJ@loader?3?5start?5?$CFs?$AA@ 10047ec0     WebCommonLib:UnityLoader.obj
 0002:0000ced4       ??_C@_0BP@CANPMPBP@Failed?5to?5start?5Unity?5Player?4?6?$AA@ 10047ed4     WebCommonLib:UnityLoader.obj
 0002:0000cef4       ??_C@_0N@CMIJEDLE@wrap_oal?4dll?$AA@ 10047ef4     WebCommonLib:UnityLoader.obj
 0002:0000cf04       ??_C@_0BC@PFFLDINN@webplayer_win?4dll?$AA@ 10047f04     WebCommonLib:UnityLoader.obj
 0002:0000cf18       ??_C@_0BL@BNOMLOGP@Failed?5to?5copy?5Unity?5dll?4?6?$AA@ 10047f18     WebCommonLib:UnityLoader.obj
 0002:0000cf34       ??_C@_0BM@DGPLHPLG@Failed?5to?5copy?5OpenAL?5dll?4?6?$AA@ 10047f34     WebCommonLib:UnityLoader.obj
 0002:0000cf50       ??_C@_0CJ@IGGKBPOL@loader?3?5FAILED?5to?5copy?5player?5te@ 10047f50     WebCommonLib:UnityLoader.obj
 0002:0000cf7c       ??_C@_0O@JMNNPPIE@mono?91?9vc?4dll?$AA@ 10047f7c     WebCommonLib:UnityLoader.obj
 0002:0000cf8c       ??_C@_0BK@JFDOPLNN@Failed?5to?5copy?5Mono?5dll?4?6?$AA@ 10047f8c     WebCommonLib:UnityLoader.obj
 0002:0000cfa8       ??_C@_0CH@CIMGECCG@loader?3?5FAILED?5to?5copy?5mono?5temp@ 10047fa8     WebCommonLib:UnityLoader.obj
 0002:0000cfd0       ??_C@_0CA@HJKHEOFG@loader?3?5unity?5dll?5not?5found?3?5?$CFs?$AA@ 10047fd0     WebCommonLib:UnityLoader.obj
 0002:0000cff0       ??_C@_0BL@PHLPIFCK@Failed?5to?5load?5Unity?5dll?4?6?$AA@ 10047ff0     WebCommonLib:UnityLoader.obj
 0002:0000d00c       ??_C@_0BF@ELKIJPCM@UnityWinWebStartData?$AA@ 1004800c     WebCommonLib:UnityLoader.obj
 0002:0000d024       ??_C@_0BJ@BANHEFED@UnityWinWebSetParentInfo?$AA@ 10048024     WebCommonLib:UnityLoader.obj
 0002:0000d040       ??_C@_0BM@IGHMBOFJ@UnityWinWebToggleFullscreen?$AA@ 10048040     WebCommonLib:UnityLoader.obj
 0002:0000d05c       ??_C@_0BI@OFPLCJFB@UnityWinWebIsFullscreen?$AA@ 1004805c     WebCommonLib:UnityLoader.obj
 0002:0000d074       ??_C@_0BB@KNLHMBLE@UnityWinWebClose?$AA@ 10048074     WebCommonLib:UnityLoader.obj
 0002:0000d088       ??_C@_0BI@GJABDPMF@UnityWinWebFinalCleanup?$AA@ 10048088     WebCommonLib:UnityLoader.obj
 0002:0000d0a0       ??_C@_0BE@PFIBMPDC@UnityWinWebSetPause?$AA@ 100480a0     WebCommonLib:UnityLoader.obj
 0002:0000d0b4       ??_C@_0BE@PCFJFBPD@UnityWinWebSetFocus?$AA@ 100480b4     WebCommonLib:UnityLoader.obj
 0002:0000d0c8       ??_C@_0BA@FGFJAMEB@UnityWinWebLoop?$AA@ 100480c8     WebCommonLib:UnityLoader.obj
 0002:0000d0d8       ??_C@_0BK@OCHBDOFG@UnityGetDisableFullscreen?$AA@ 100480d8     WebCommonLib:UnityLoader.obj
 0002:0000d0f4       ??_C@_0BF@MCDHKKPD@UnitySendWebMessages?$AA@ 100480f4     WebCommonLib:UnityLoader.obj
 0002:0000d10c       ??_C@_0BJ@NAEOKBPF@UnityExternalCallsLength?$AA@ 1004810c     WebCommonLib:UnityLoader.obj
 0002:0000d128       ??_C@_0BI@LDLIAKNK@UnityFetchExternalCalls?$AA@ 10048128     WebCommonLib:UnityLoader.obj
 0002:0000d140       ??_C@_0BL@OIPDKBAD@UnityShouldShowContextMenu?$AA@ 10048140     WebCommonLib:UnityLoader.obj
 0002:0000d15c       ??_C@_0BK@MJHFKCBF@UnityProgressDataDownload?$AA@ 1004815c     WebCommonLib:UnityLoader.obj
 0002:0000d178       ??_C@_0BD@JHGPBAOD@UnityIsReadyToPlay?$AA@ 10048178     WebCommonLib:UnityLoader.obj
 0002:0000d18c       ??_C@_0O@PBEJMPLL@UnityGetError?$AA@ 1004818c     WebCommonLib:UnityLoader.obj
 0002:0000d19c       ??_C@_0BI@EMJOBHMM@UnityGetPlayerTargetFPS?$AA@ 1004819c     WebCommonLib:UnityLoader.obj
 0002:0000d1b4       ??_C@_0BD@NGNLJPKE@UnitySetParentInfo?$AA@ 100481b4     WebCommonLib:UnityLoader.obj
 0002:0000d1c8       ??_C@_0BG@IFAGFBPB@loader?3?5final?5cleanup?$AA@ 100481c8     WebCommonLib:UnityLoader.obj
 0002:0000d1e0       ??_C@_0BJ@CFLMAIAB@loader?3?5unload?5unity?5dll?$AA@ 100481e0     WebCommonLib:UnityLoader.obj
 0002:0000d1fc       ??_C@_1BE@CNNBFHHP@?$AA3?$AA6?$AA0?$AAs?$AAe?$AA?4?$AAe?$AAx?$AAe?$AA?$AA@ 100481fc     WebCommonLib:Pluginfor360Browser.obj
 0002:0000d210       ??_C@_0BJ@JBDKPHIM@Software?2Unity?2WebPlayer?$AA@ 10048210     WebCommonLib:GlobalPreferences.obj
 0002:0000d22c       ??_C@_15MJDFFMKN@?$AAw?$AAb?$AA?$AA@ 1004822c     WebCommonLib:Decompressor.obj
 0002:0000d234       ??_C@_01NBENCBCI@?$CK?$AA@ 10048234     WebCommonLib:WebFileUtilities.obj
 0002:0000d238       ??_C@_0P@JLFAABJN@UnityWebPlayer?$AA@ 10048238     WebCommonLib:WebFileUtilities.obj
 0002:0000d248       ??_C@_13JOFGPIOO@?$AA?4?$AA?$AA@ 10048248     WebCommonLib:WebFileUtilities.obj
 0002:0000d24c       ??_C@_15DDHGOCBH@?$AA?4?$AA?4?$AA?$AA@ 1004824c     WebCommonLib:WebFileUtilities.obj
 0002:0000d254       ??_C@_08NBAAKOEL@UnityWeb?$AA@ 10048254     WebCommonLib:UnityWebStreamHeader.obj
 0002:0000d38c       ??_C@_0CK@BHABGMFL@Verify?3?5failed?5to?5acquire?5contex@ 1004838c     WebCommonLib:Verification.obj
 0002:0000d3b8       ??_C@_0CE@ENIIMKEC@Verify?3?5failed?5to?5import?5public?5@ 100483b8     WebCommonLib:Verification.obj
 0002:0000d3dc       ??_C@_0BO@JOMKDGLN@Verify?3?5failed?5to?5create?5hash?$AA@ 100483dc     WebCommonLib:Verification.obj
 0002:0000d3fc       ??_C@_0BM@GFHCJDCH@Verify?3?5failed?5to?5hash?5data?$AA@ 100483fc     WebCommonLib:Verification.obj
 0002:0000d418       ??_C@_0DA@NNMFAGAK@GenerateHash?3?5failed?5to?5acquire?5@ 10048418     WebCommonLib:Verification.obj
 0002:0000d448       ??_C@_0CO@OCMOPENC@GenerateHash?3?5failed?5to?5create?5h@ 10048448     WebCommonLib:Verification.obj
 0002:0000d478       ??_C@_0CK@LOGAKBCB@GenerateHash?3?5failed?5to?5hash?5dat@ 10048478     WebCommonLib:Verification.obj
 0002:0000d4a4       ??_C@_0CP@IOPFFNJK@GenerateHash?3?5failed?5to?5get?5hash@ 100484a4     WebCommonLib:Verification.obj
 0002:0000d4d4       ??_C@_04NOJCDH@?$CF02x?$AA@ 100484d4     WebCommonLib:Verification.obj
 0002:0000d4dc       ??_C@_05ONPNOBPM@?$CG?$CD38?$DL?$AA@ 100484dc     WebCommonLib:ezxml.obj
 0002:0000d4e4       ??_C@_04DMIAPOKJ@amp?$DL?$AA@ 100484e4     WebCommonLib:ezxml.obj
 0002:0000d4ec       ??_C@_05OMDPILML@?$CG?$CD39?$DL?$AA@ 100484ec     WebCommonLib:ezxml.obj
 0002:0000d4f4       ??_C@_05HNAHLMAI@apos?$DL?$AA@ 100484f4     WebCommonLib:ezxml.obj
 0002:0000d4fc       ??_C@_05OEOHBIJI@?$CG?$CD34?$DL?$AA@ 100484fc     WebCommonLib:ezxml.obj
 0002:0000d504       ??_C@_05LDHOCHGG@quot?$DL?$AA@ 10048504     WebCommonLib:ezxml.obj
 0002:0000d50c       ??_C@_05NHLEJEBI@?$CG?$CD62?$DL?$AA@ 1004850c     WebCommonLib:ezxml.obj
 0002:0000d514       ??_C@_03BHAAMAON@gt?$DL?$AA@ 10048514     WebCommonLib:ezxml.obj
 0002:0000d518       ??_C@_05NEDAEAHG@?$CG?$CD60?$DL?$AA@ 10048518     WebCommonLib:ezxml.obj
 0002:0000d520       ??_C@_03MAABEHOM@lt?$DL?$AA@ 10048520     WebCommonLib:ezxml.obj
 0002:0000d524       ??_C@_0BJ@OKJBEMCM@?$FLerror?5near?5line?5?$CFd?$FN?3?5?$CFs?$AA@ 10048524     WebCommonLib:ezxml.obj
 0002:0000d540       ??_C@_02ICNHGLNO@?$CG?$CD?$AA@ 10048540     WebCommonLib:ezxml.obj
 0002:0000d544       ??_C@_01CLKCMJKC@?5?$AA@   10048544     WebCommonLib:ezxml.obj
 0002:0000d548       ??_C@_0BN@EKAANKPM@unexpected?5closing?5tag?5?$DM?1?$CFs?$DO?$AA@ 10048548     WebCommonLib:ezxml.obj
 0002:0000d568       ??_C@_04FOLEBDDK@?7?$AN?6?5?$AA@ 10048568     WebCommonLib:ezxml.obj
 0002:0000d570       ??_C@_03PJHHNEEI@xml?$AA@  10048570     WebCommonLib:ezxml.obj
 0002:0000d574       ??_C@_0L@FLHGMILF@standalone?$AA@ 10048574     WebCommonLib:ezxml.obj
 0002:0000d580       ??_C@_07BMOOGACG@?7?$AN?6?5?$DN?8?$CC?$AA@ 10048580     WebCommonLib:ezxml.obj
 0002:0000d588       ??_C@_01PPODPGHN@?$DO?$AA@ 10048588     WebCommonLib:ezxml.obj
 0002:0000d58c       ??_C@_01MNNFJEPP@?$DM?$AA@ 1004858c     WebCommonLib:ezxml.obj
 0002:0000d590       ??_C@_08OMANJFFA@?$DM?$CBENTITY?$AA@ 10048590     WebCommonLib:ezxml.obj
 0002:0000d59c       ??_C@_05COKBLNEG@?7?$AN?6?5?$CF?$AA@ 1004859c     WebCommonLib:ezxml.obj
 0002:0000d5a4       ??_C@_0CA@HIBIOLGK@circular?5entity?5declaration?5?$CG?$CFs?$AA@ 100485a4     WebCommonLib:ezxml.obj
 0002:0000d5c4       ??_C@_09JFLAIMKP@?$DM?$CBATTLIST?$AA@ 100485c4     WebCommonLib:ezxml.obj
 0002:0000d5d0       ??_C@_0BD@JECACICL@unclosed?5?$DM?$CBATTLIST?$AA@ 100485d0     WebCommonLib:ezxml.obj
 0002:0000d5e4       ??_C@_05IHJHHGNM@?7?$AN?6?5?$DO?$AA@ 100485e4     WebCommonLib:ezxml.obj
 0002:0000d5ec       ??_C@_0BE@OPHFANMD@malformed?5?$DM?$CBATTLIST?$AA@ 100485ec     WebCommonLib:ezxml.obj
 0002:0000d600       ??_C@_05MLPNBPGH@CDATA?$AA@ 10048600     WebCommonLib:ezxml.obj
 0002:0000d608       ??_C@_08NCDGCBCC@NOTATION?$AA@ 10048608     WebCommonLib:ezxml.obj
 0002:0000d614       ??_C@_05ICBEPCEK@?7?$AN?6?5?$CJ?$AA@ 10048614     WebCommonLib:ezxml.obj
 0002:0000d61c       ??_C@_06PMNJDCKO@?$CDFIXED?$AA@ 1004861c     WebCommonLib:ezxml.obj
 0002:0000d624       ??_C@_04FFDNBKGC@?$DM?$CB?9?9?$AA@ 10048624     WebCommonLib:ezxml.obj
 0002:0000d62c       ??_C@_03PNLDJJMO@?9?9?$DO?$AA@ 1004862c     WebCommonLib:ezxml.obj
 0002:0000d630       ??_C@_02HFBBBACF@?$DM?$DP?$AA@ 10048630     WebCommonLib:ezxml.obj
 0002:0000d634       ??_C@_02GOEMJPDN@?$DP?$DO?$AA@ 10048634     WebCommonLib:ezxml.obj
 0002:0000d638       ??_C@_0BB@CIDLNPKI@root?5tag?5missing?$AA@ 10048638     WebCommonLib:ezxml.obj
 0002:0000d64c       ??_C@_0BP@EFHCLHOB@markup?5outside?5of?5root?5element?$AA@ 1004864c     WebCommonLib:ezxml.obj
 0002:0000d66c       ??_C@_06NDMDNLLD@?7?$AN?6?5?1?$DO?$AA@ 1004866c     WebCommonLib:ezxml.obj
 0002:0000d674       ??_C@_07PEIKGMMD@?7?$AN?6?5?$DN?1?$DO?$AA@ 10048674     WebCommonLib:ezxml.obj
 0002:0000d67c       ??_C@_05KMLKCFBP@?7?$AN?6?5?$DN?$AA@ 1004867c     WebCommonLib:ezxml.obj
 0002:0000d684       ??_C@_0L@BOJNAMOF@missing?5?$CFc?$AA@ 10048684     WebCommonLib:ezxml.obj
 0002:0000d690       ??_C@_09OBHDHGOK@missing?5?$DO?$AA@ 10048690     WebCommonLib:ezxml.obj
 0002:0000d69c       ??_C@_03NGIKGHOE@?$CB?9?9?$AA@ 1004869c     WebCommonLib:ezxml.obj
 0002:0000d6a0       ??_C@_02BAABKJLB@?9?9?$AA@ 100486a0     WebCommonLib:ezxml.obj
 0002:0000d6a4       ??_C@_0O@NEODEGIL@unclosed?5?$DM?$CB?9?9?$AA@ 100486a4     WebCommonLib:ezxml.obj
 0002:0000d6b4       ??_C@_08GMPBDPNL@?$CB?$FLCDATA?$FL?$AA@ 100486b4     WebCommonLib:ezxml.obj
 0002:0000d6c0       ??_C@_03MCHNFBAC@?$FN?$FN?$DO?$AA@ 100486c0     WebCommonLib:ezxml.obj
 0002:0000d6c4       ??_C@_0BD@BKCNIFDB@unclosed?5?$DM?$CB?$FLCDATA?$FL?$AA@ 100486c4     WebCommonLib:ezxml.obj
 0002:0000d6d8       ??_C@_08IAAAHACH@?$CBDOCTYPE?$AA@ 100486d8     WebCommonLib:ezxml.obj
 0002:0000d6e4       ??_C@_03OHBGAONO@?$FL?$FN?$DO?$AA@ 100486e4     WebCommonLib:ezxml.obj
 0002:0000d6e8       ??_C@_0BD@PGNMMKMN@unclosed?5?$DM?$CBDOCTYPE?$AA@ 100486e8     WebCommonLib:ezxml.obj
 0002:0000d6fc       ??_C@_0M@IPLLBBLK@unclosed?5?$DM?$DP?$AA@ 100486fc     WebCommonLib:ezxml.obj
 0002:0000d708       ??_C@_0N@LOEDOFDJ@unexpected?5?$DM?$AA@ 10048708     WebCommonLib:ezxml.obj
 0002:0000d718       ??_C@_0BC@EONPOLEO@unclosed?5tag?5?$DM?$CFs?$DO?$AA@ 10048718     WebCommonLib:ezxml.obj
 0002:0000d72c       ??_C@_01BJJEKLCA@?$CC?$AA@ 1004872c     WebCommonLib:ezxml.obj
 0002:0000d730       ??_C@_1BG@GLKFLKB@?$AAk?$AAt?$AAm?$AAw?$AA3?$AA2?$AA?4?$AAd?$AAl?$AAl?$AA?$AA@ 10048730     WebCommonLib:Updater.obj
 0002:0000d748       ??_C@_0BC@GAOFHPNA@CreateTransaction?$AA@ 10048748     WebCommonLib:Updater.obj
 0002:0000d75c       ??_C@_0BC@OLDFEAHM@CommitTransaction?$AA@ 1004875c     WebCommonLib:Updater.obj
 0002:0000d770       ??_C@_1BK@MGMFAEKH@?$AAk?$AAe?$AAr?$AAn?$AAe?$AAl?$AA3?$AA2?$AA?4?$AAd?$AAl?$AAl?$AA?$AA@ 10048770     WebCommonLib:Updater.obj
 0002:0000d78c       ??_C@_0BL@KILOLGEA@GetFullPathNameTransactedW?$AA@ 1004878c     WebCommonLib:Updater.obj
 0002:0000d7a8       ??_C@_0BN@KGIPEFFF@SetFileAttributesTransactedW?$AA@ 100487a8     WebCommonLib:Updater.obj
 0002:0000d7c8       ??_C@_0BJ@KAJEEPGD@FindFirstFileTransactedW?$AA@ 100487c8     WebCommonLib:Updater.obj
 0002:0000d7e4       ??_C@_0BG@DHJMHDAN@DeleteFileTransactedW?$AA@ 100487e4     WebCommonLib:Updater.obj
 0002:0000d7fc       ??_C@_0BL@DOLECCBH@CreateDirectoryTransactedW?$AA@ 100487fc     WebCommonLib:Updater.obj
 0002:0000d818       ??_C@_0BL@NPHAJMON@RemoveDirectoryTransactedW?$AA@ 10048818     WebCommonLib:Updater.obj
 0002:0000d834       ??_C@_0BE@HKBCBLNP@CopyFileTransactedW?$AA@ 10048834     WebCommonLib:Updater.obj
 0002:0000d848       ??_C@_0BE@OPNPBNBB@MoveFileTransactedW?$AA@ 10048848     WebCommonLib:Updater.obj
 0002:0000d85c       ??_C@_1DE@KJGGILOD@?$AAU?$AAn?$AAi?$AAt?$AAy?$AAW?$AAe?$AAb?$AAP?$AAl?$AAa?$AAy?$AAe?$AAr?$AAU?$AAp?$AAd?$AAa?$AAt?$AAe?$AAM?$AAu?$AAt?$AAe?$AAx?$AA?$AA@ 1004885c     WebCommonLib:Updater.obj
 0002:0000d890       ??_C@_1BA@GKAOCBBO@?$AA?$CF?$AAs?$AA?4?$AA?$CF?$AA?4?$AA3?$AAd?$AA?$AA@ 10048890     WebCommonLib:Updater.obj
 0002:0000d8a0       ??_C@_17LDPNGHAG@?$AAo?$AAc?$AAx?$AA?$AA@ 100488a0     WebCommonLib:Updater.obj
 0002:0000d8a8       ??_C@_1CA@HCBCOPKN@?$AAO?$AAC?$AAX?$AAU?$AAp?$AAd?$AAa?$AAt?$AAe?$AAF?$AAa?$AAi?$AAl?$AAe?$AAd?$AA?$AA@ 100488a8     WebCommonLib:Updater.obj
 0002:0000d8c8       ??_C@_13BBDEGPLJ@?$AA?$CK?$AA?$AA@ 100488c8     WebCommonLib:Updater.obj
 0002:0000d8cc       ??_7ClientPipe@@6B@        100488cc     WebCommonLib:Updater.obj
 0002:0000d8cc       ??_7ServerPipe@UpdaterProxy@@6B@ 100488cc     WebCommonLib:UpdaterProxy.obj
 0002:0000d8d4       ??_7UpdateMessage@Updater@@6B@ 100488d4     WebCommonLib:Updater.obj
 0002:0000d8e0       __real@408f400000000000    100488e0      CIL library: CIL module
 0002:0000d8e8       __real@4000000000000000    100488e8      CIL library: CIL module
 0002:0000d8f0       __real@0000000000000000    100488f0      CIL library: CIL module
 0002:0000d8f8       __real@3fdccccccccccccd    100488f8      CIL library: CIL module
 0002:0000d900       __real@3ff0000000000000    10048900      CIL library: CIL module
 0002:0000d908       __real@4f800000            10048908      CIL library: CIL module
 0002:0000d90c       __real@bf800000            1004890c      CIL library: CIL module
 0002:0000d910       __real@3fe0000000000000    10048910      CIL library: CIL module
 0002:0000d918       __real@3fdcccccc0000000    10048918      CIL library: CIL module
 0002:0000d920       __real@41cdcd6500000000    10048920      CIL library: CIL module
 0002:0000d928       __real@3f50624de0000000    10048928      CIL library: CIL module
 0002:0000d930       __load_config_used         10048930     LIBCMT:loadcfg.obj
 0002:0000d9e4       ??_R4logic_error@std@@6B@  100489e4     libcpmt:xthrow.obj
 0002:0000d9f8       ??_R3logic_error@std@@8    100489f8     libcpmt:xthrow.obj
 0002:0000da08       ??_R2logic_error@std@@8    10048a08     libcpmt:xthrow.obj
 0002:0000da14       ??_R1A@?0A@EA@logic_error@std@@8 10048a14     libcpmt:xthrow.obj
 0002:0000da30       ??_R1A@?0A@EA@exception@std@@8 10048a30     libcpmt:xthrow.obj
 0002:0000da4c       ??_R3exception@std@@8      10048a4c     libcpmt:xthrow.obj
 0002:0000da5c       ??_R2exception@std@@8      10048a5c     libcpmt:xthrow.obj
 0002:0000da64       ??_R4length_error@std@@6B@ 10048a64     libcpmt:xthrow.obj
 0002:0000da78       ??_R3length_error@std@@8   10048a78     libcpmt:xthrow.obj
 0002:0000da88       ??_R2length_error@std@@8   10048a88     libcpmt:xthrow.obj
 0002:0000da98       ??_R1A@?0A@EA@length_error@std@@8 10048a98     libcpmt:xthrow.obj
 0002:0000dab4       ??_R4out_of_range@std@@6B@ 10048ab4     libcpmt:xthrow.obj
 0002:0000dac8       ??_R3out_of_range@std@@8   10048ac8     libcpmt:xthrow.obj
 0002:0000dad8       ??_R2out_of_range@std@@8   10048ad8     libcpmt:xthrow.obj
 0002:0000dae8       ??_R1A@?0A@EA@out_of_range@std@@8 10048ae8     libcpmt:xthrow.obj
 0002:0000db04       ??_R4bad_alloc@std@@6B@    10048b04     LIBCMT:new.obj
 0002:0000db18       ??_R3bad_alloc@std@@8      10048b18     LIBCMT:new.obj
 0002:0000db28       ??_R2bad_alloc@std@@8      10048b28     LIBCMT:new.obj
 0002:0000db34       ??_R1A@?0A@EA@bad_alloc@std@@8 10048b34     LIBCMT:new.obj
 0002:0000db50       ??_R4exception@std@@6B@    10048b50     LIBCMT:stdexcpt.obj
 0002:0000db64       ??_R4type_info@@6B@        10048b64     LIBCMT:typinfo.obj
 0002:0000db78       ??_R3type_info@@8          10048b78     LIBCMT:typinfo.obj
 0002:0000db88       ??_R2type_info@@8          10048b88     LIBCMT:typinfo.obj
 0002:0000db90       ??_R1A@?0A@EA@type_info@@8 10048b90     LIBCMT:typinfo.obj
 0002:0000dbac       ??_R4bad_exception@std@@6B@ 10048bac     LIBCMT:frame.obj
 0002:0000dbc0       ??_R3bad_exception@std@@8  10048bc0     LIBCMT:frame.obj
 0002:0000dbd0       ??_R2bad_exception@std@@8  10048bd0     LIBCMT:frame.obj
 0002:0000dbdc       ??_R1A@?0A@EA@bad_exception@std@@8 10048bdc     LIBCMT:frame.obj
 0002:0000dc00       ___safe_se_handler_table   10048c00     <linker-defined>
 0002:0000dc70       ___rtc_iaa                 10048c70     LIBCMT:_initsect_.obj
 0002:0000dc74       ___rtc_izz                 10048c74     LIBCMT:_initsect_.obj
 0002:0000dc78       ___rtc_taa                 10048c78     LIBCMT:_initsect_.obj
 0002:0000dc7c       ___rtc_tzz                 10048c7c     LIBCMT:_initsect_.obj
 0002:0000dc80       __CT??_R0?AVlogic_error@std@@@8??0logic_error@std@@QAE@ABV01@@Z12 10048c80     libcpmt:xthrow.obj
 0002:0000dc9c       __TI3?AVlength_error@std@@ 10048c9c     libcpmt:xthrow.obj
 0002:0000dcac       __CTA3?AVlength_error@std@@ 10048cac     libcpmt:xthrow.obj
 0002:0000dcbc       __CT??_R0?AVlength_error@std@@@8??0length_error@std@@QAE@ABV01@@Z12 10048cbc     libcpmt:xthrow.obj
 0002:0000dcd8       __TI3?AVout_of_range@std@@ 10048cd8     libcpmt:xthrow.obj
 0002:0000dce8       __CTA3?AVout_of_range@std@@ 10048ce8     libcpmt:xthrow.obj
 0002:0000dcf8       __CT??_R0?AVout_of_range@std@@@8??0out_of_range@std@@QAE@ABV01@@Z12 10048cf8     libcpmt:xthrow.obj
 0002:0000e394       __TI2?AVbad_exception@std@@ 10049394     LIBCMT:frame.obj
 0002:0000e3a4       __CTA2?AVbad_exception@std@@ 100493a4     LIBCMT:frame.obj
 0002:0000e3b0       __CT??_R0?AVbad_exception@std@@@8??0bad_exception@std@@QAE@ABV01@@Z12 100493b0     LIBCMT:frame.obj
 0002:0000e4ac       __CT??_R0?AVexception@std@@@8??0exception@std@@QAE@ABV01@@Z12 100494ac     ContextSubmenu.obj
 0002:0000e4c8       __CT??_R0?AVbad_alloc@std@@@8??0bad_alloc@std@@QAE@ABV01@@Z12 100494c8     ContextSubmenu.obj
 0002:0000e4e4       __CTA2?AVbad_alloc@std@@   100494e4     ContextSubmenu.obj
 0002:0000e4f0       __TI2?AVbad_alloc@std@@    100494f0     ContextSubmenu.obj
 0002:0000ec48       __IMPORT_DESCRIPTOR_KERNEL32 10049c48     kernel32:KERNEL32.dll
 0002:0000ec5c       __IMPORT_DESCRIPTOR_USER32 10049c5c     user32:USER32.dll
 0002:0000ec70       __IMPORT_DESCRIPTOR_GDI32  10049c70     gdi32:GDI32.dll
 0002:0000ec84       __IMPORT_DESCRIPTOR_SHLWAPI 10049c84     WebCommonLib:SHLWAPI.dll
 0002:0000ec98       __IMPORT_DESCRIPTOR_ADVAPI32 10049c98     advapi32:ADVAPI32.dll
 0002:0000ecac       __IMPORT_DESCRIPTOR_WINMM  10049cac     winmm:WINMM.dll
 0002:0000ecc0       __IMPORT_DESCRIPTOR_SHELL32 10049cc0     shell32:SHELL32.dll
 0002:0000ecd4       __IMPORT_DESCRIPTOR_ole32  10049cd4     ole32:ole32.dll
 0002:0000ece8       __IMPORT_DESCRIPTOR_MSIMG32 10049ce8     MSImg32:MSIMG32.dll
 0002:0000ecfc       __IMPORT_DESCRIPTOR_VERSION 10049cfc     version:VERSION.dll
 0002:0000ed10       __NULL_IMPORT_DESCRIPTOR   10049d10     kernel32:KERNEL32.dll
 0003:00000000       ??_R0?AVlogic_error@std@@@8 1004c000     libcpmt:xthrow.obj
 0003:00000020       ??_R0?AVlength_error@std@@@8 1004c020     libcpmt:xthrow.obj
 0003:00000040       ??_R0?AVout_of_range@std@@@8 1004c040     libcpmt:xthrow.obj
 0003:00000060       ??_R0?AVtype_info@@@8      1004c060     LIBCMT:typinfo.obj
 0003:000001f0       ___abort_behavior          1004c1f0     LIBCMT:abort.obj
 0003:000001f8       ___initialmbcinfo          1004c1f8     LIBCMT:mbctype.obj
 0003:00000418       __mbctype                  1004c418     LIBCMT:mbctype.obj
 0003:00000520       __mbcasemap                1004c520     LIBCMT:mbctype.obj
 0003:00000620       ___ptmbcinfo               1004c620     LIBCMT:mbctype.obj
 0003:00000718       ___globallocalestatus      1004c718     LIBCMT:glstatus.obj
 0003:0000071c       ___clocalestr              1004c71c     LIBCMT:nlsdata2.obj
 0003:00000720       ___lc_time_c               1004c720     LIBCMT:nlsdata2.obj
 0003:00000888       ___initiallocinfo          1004c888     LIBCMT:nlsdata2.obj
 0003:00000960       ___ptlocinfo               1004c960     LIBCMT:nlsdata2.obj
 0003:00000964       ___initiallocalestructinfo 1004c964     LIBCMT:nlsdata2.obj
 0003:0000096c       ___flsindex                1004c96c     LIBCMT:tidtable.obj
 0003:00000970       ___getvalueindex           1004c970     LIBCMT:tidtable.obj
 0003:00000978       __iob                      1004c978     LIBCMT:_file.obj
 0003:00000bf8       ___nullstring              1004cbf8     LIBCMT:output.obj
 0003:00000bfc       ___wnullstring             1004cbfc     LIBCMT:output.obj
 0003:00000c00       ___security_cookie         1004cc00     LIBCMT:gs_cookie.obj
 0003:00000c04       ___security_cookie_complement 1004cc04     LIBCMT:gs_cookie.obj
 0003:00000c08       ___badioinfo               1004cc08     LIBCMT:ioinit.obj
 0003:00000d88       __timezone                 1004cd88     LIBCMT:timeset.obj
 0003:00000d8c       __daylight                 1004cd8c     LIBCMT:timeset.obj
 0003:00000d90       __dstbias                  1004cd90     LIBCMT:timeset.obj
 0003:00000e18       __tzname                   1004ce18     LIBCMT:timeset.obj
 0003:00000e20       __lookuptrailbytes         1004ce20     LIBCMT:read.obj
 0003:00000f20       __cfltcvt_tab              1004cf20     LIBCMT:cmiscdat.obj
 0003:00000f50       ___lconv_static_decimal    1004cf50     LIBCMT:lconv.obj
 0003:00000f54       ___lconv_static_W_decimal  1004cf54     LIBCMT:lconv.obj
 0003:00000f58       ___lconv_c                 1004cf58     LIBCMT:lconv.obj
 0003:00000fa8       ___lconv                   1004cfa8     LIBCMT:lconv.obj
 0003:00000fac       __pctype                   1004cfac     LIBCMT:ctype.obj
 0003:00000fb0       __pwctype                  1004cfb0     LIBCMT:ctype.obj
 0003:00000fb4       ___mb_cur_max              1004cfb4     LIBCMT:nlsdata1.obj
 0003:00000fb8       ___decimal_point           1004cfb8     LIBCMT:nlsdata1.obj
 0003:00000fbc       ___decimal_point_length    1004cfbc     LIBCMT:nlsdata1.obj
 0003:00000fc0       __NLG_Destination          1004cfc0     LIBCMT:exsup.obj
 0003:00000fd0       __lpdays                   1004cfd0     LIBCMT:days.obj
 0003:00001004       __days                     1004d004     LIBCMT:days.obj
 0003:00001038       ??_R0?AVbad_exception@std@@@8 1004d038     LIBCMT:frame.obj
 0003:00001060       __confh                    1004d060     LIBCMT:initcon.obj
 0003:000010cc       __fltused                  1004d0cc     LIBCMT:_fpinit_.obj
 0003:000010d0       __ldused                   1004d0d0     LIBCMT:_fpinit_.obj
 0003:000010e0       __half                     1004d0e0     LIBCMT:_pow_.obj
 0003:000011d8       __d_inf                    1004d1d8     LIBCMT:_util_.obj
 0003:000011e0       __d_ind                    1004d1e0     LIBCMT:_util_.obj
 0003:000011e8       __d_max                    1004d1e8     LIBCMT:_util_.obj
 0003:000011f0       __d_min                    1004d1f0     LIBCMT:_util_.obj
 0003:000011f8       __d_mzero                  1004d1f8     LIBCMT:_util_.obj
 0003:00001220       __HUGE                     1004d220     LIBCMT:_huge_.obj
 0003:00001230       __matherr_flag             1004d230     LIBCMT:_matherr_.obj
 0003:00001268       __pow10pos                 1004d268     LIBCMT:_constpow_.obj
 0003:000013c8       __pow10neg                 1004d3c8     LIBCMT:_constpow_.obj
 0003:00001524       ??_R0?AVexception@std@@@8  1004d524     ContextSubmenu.obj
 0003:00001540       ??_R0?AVbad_alloc@std@@@8  1004d540     ContextSubmenu.obj
 0003:00001588       ?kRegistryPath@@3PBDB      1004d588     WebCommonLib:GlobalPreferences.obj
 0003:0000158c       ?kGlobalRevisionFile@@3PBDB 1004d58c     WebCommonLib:RevisionsQuery.obj
 0003:00001590       ?gAllowSettingAutodateURL@@3_NA 1004d590     WebCommonLib:RevisionsQuery.obj
 0003:00001594       ?kImageTags@progress@@3PAPBDA 1004d594     WebCommonLib:ProgressDisplay.obj
 0003:000015a4       ?kColorTags@progress@@3PAPBDA 1004d5a4     WebCommonLib:ProgressDisplay.obj
 0003:000015b4       ?kBundleIDToDownloadLookup@@3PAPBDA 1004d5b4     WebCommonLib:PluginManager.obj
 0003:000015c0       ?kApplyUpdateMutexName@@3PBDB 1004d5c0     WebCommonLib:PluginManager.obj
 0003:00001604       ?kProgressImageResourceIDs@@3PAHA 1004d604     UnityWebPlayerPlugin.obj
 0003:00001620       ?nothrow@std@@3Unothrow_t@1@B 1004d620     libcpmt:nothrow.obj
 0003:0000163c       __aenvptr                  1004d63c     LIBCMT:dllcrt0.obj
 0003:00001640       __wenvptr                  1004d640     LIBCMT:dllcrt0.obj
 0003:00001644       ___error_mode              1004d644     LIBCMT:dllcrt0.obj
 0003:00001648       ___app_type                1004d648     LIBCMT:dllcrt0.obj
 0003:0000164c       ?_pnhHeap@@3P6AHI@ZA       1004d64c     LIBCMT:handler.obj
 0003:00001650       __maxwait                  1004d650     LIBCMT:crtheap.obj
 0003:00001654       __umaskval                 1004d654     LIBCMT:crt0dat.obj
 0003:00001658       ___argc                    1004d658     LIBCMT:crt0dat.obj
 0003:0000165c       ___argv                    1004d65c     LIBCMT:crt0dat.obj
 0003:00001660       ___wargv                   1004d660     LIBCMT:crt0dat.obj
 0003:00001664       __environ                  1004d664     LIBCMT:crt0dat.obj
 0003:00001668       ___initenv                 1004d668     LIBCMT:crt0dat.obj
 0003:0000166c       __wenviron                 1004d66c     LIBCMT:crt0dat.obj
 0003:00001670       ___winitenv                1004d670     LIBCMT:crt0dat.obj
 0003:00001674       __pgmptr                   1004d674     LIBCMT:crt0dat.obj
 0003:00001678       __wpgmptr                  1004d678     LIBCMT:crt0dat.obj
 0003:0000167c       __exitflag                 1004d67c     LIBCMT:crt0dat.obj
 0003:00001680       __C_Termination_Done       1004d680     LIBCMT:crt0dat.obj
 0003:00001684       __C_Exit_Done              1004d684     LIBCMT:crt0dat.obj
 0003:00001690       ___pInvalidArgHandler      1004d690     LIBCMT:invarg.obj
 0003:00001cc0       ___pPurecall               1004dcc0     LIBCMT:inithelp.obj
 0003:00001cc8       ___mbulinfo                1004dcc8     LIBCMT:mbctype.obj
 0003:00001cd4       ___mbcodepage              1004dcd4     LIBCMT:mbctype.obj
 0003:00001cd8       ___ismbcodepage            1004dcd8     LIBCMT:mbctype.obj
 0003:00001cdc       ___mblcid                  1004dcdc     LIBCMT:mbctype.obj
 0003:00001ce0       _gpFlsAlloc                1004dce0     LIBCMT:tidtable.obj
 0003:00001ce4       _gpFlsGetValue             1004dce4     LIBCMT:tidtable.obj
 0003:00001ce8       _gpFlsSetValue             1004dce8     LIBCMT:tidtable.obj
 0003:00001cec       _gpFlsFree                 1004dcec     LIBCMT:tidtable.obj
 0003:00001cf0       ___locale_changed          1004dcf0     LIBCMT:setlocal.obj
 0003:00001cf4       __cflush                   1004dcf4     LIBCMT:_file.obj
 0003:00001cf8       __stdbuf                   1004dcf8     LIBCMT:_sftbuf.obj
 0003:00001e08       __crtheap                  1004de08     LIBCMT:heapinit.obj
 0003:00002018       __newmode                  1004e018     LIBCMT:_newmode.obj
 0003:0000201c       ?__pInconsistency@@3P6AXXZA 1004e01c     LIBCMT:hooks.obj
 0003:0000204c       ?pArgList@UnDecorator@@0PAVReplicator@@A 1004e04c     LIBCMT:undname.obj
 0003:00002050       ?pZNameList@UnDecorator@@0PAVReplicator@@A 1004e050     LIBCMT:undname.obj
 0003:00002054       ?pTemplateArgList@UnDecorator@@0PAVReplicator@@A 1004e054     LIBCMT:undname.obj
 0003:00002058       ?gName@UnDecorator@@0PBDB  1004e058     LIBCMT:undname.obj
 0003:0000205c       ?name@UnDecorator@@0PBDB   1004e05c     LIBCMT:undname.obj
 0003:00002060       ?outputString@UnDecorator@@0PADA 1004e060     LIBCMT:undname.obj
 0003:00002064       ?maxStringLength@UnDecorator@@0HA 1004e064     LIBCMT:undname.obj
 0003:00002068       ?disableFlags@UnDecorator@@0KA 1004e068     LIBCMT:undname.obj
 0003:0000206c       ?m_pGetParameter@UnDecorator@@0P6APADJ@ZA 1004e06c     LIBCMT:undname.obj
 0003:00002070       ?fExplicitTemplateParams@UnDecorator@@0_NA 1004e070     LIBCMT:undname.obj
 0003:00002071       ?fGetTemplateArgumentList@UnDecorator@@0_NA 1004e071     LIBCMT:undname.obj
 0003:00002088       ___lconv_static_null       1004e088     LIBCMT:lconv.obj
 0003:0000208c       ___lconv_static_W_null     1004e08c     LIBCMT:lconv.obj
 0003:00002090       __commode                  1004e090     LIBCMT:ncommode.obj
 0003:000023bc       __fmode                    1004e3bc     LIBCMT:txtmode.obj
 0003:000043cc       ___fastflag                100503cc     LIBCMT:_fpinit_.obj
 0003:00004458       __outputformat             10050458     LIBCMT:outputformat.obj
 0003:00004460       ___@@_PchSym_@00@UyfrowztvmgUdlipUHFDFwvExzCGxCGzxUkozgulinwvkvmwvmgUdrmdvykoftrmUyfrowUivovzhvUdrmDCUmvghxzkvUhgwzucOlyq@ 10050460     stdafx.obj
 0003:00004470       ?NPNFuncs@@3U_NPNetscapeFuncs@@A 10050470     np_entry.obj
 0003:00004550       ?dummy_@ReentrancyChecker@@0_NA 10050550     WebCommonLib:WebPluginUtility.obj
 0003:00004568       ?s_Frequency@?A0x7b9a98a1@@3_JA 10050568     WebCommonLib:WinWebUtils.obj
 0003:00004570       ?s_QueryUnbiasedInterruptTime@?A0x7b9a98a1@@3P6GHPA_K@ZA 10050570     WebCommonLib:WinWebUtils.obj
 0003:0000457a       ?m_Initialized@CPUInfo@@0_NA 1005057a     WebCommonLib:CPUInfo.obj
 0003:0000457b       ?m_IsSSESupported@CPUInfo@@0_NA 1005057b     WebCommonLib:CPUInfo.obj
 0003:00004580       ?m_SingleInstance@PluginManager@@0PAV1@A 10050580     WebCommonLib:PluginManager.obj
 0003:00004584       ?gLastRevsionQueryDuration@@3MA 10050584     WebCommonLib:RevisionsQuery.obj
 0003:00004588       _EZXML_NIL                 10050588     WebCommonLib:ezxml.obj
 0003:0000458c       ?m_IsSSE2Supported@CPUInfo@@0_NA 1005058c     WebCommonLib:CPUInfo.obj
 0003:00004590       ?m_CPUIDFeatures@CPUInfo@@0IA 10050590     WebCommonLib:CPUInfo.obj
 0003:00004594       ?ms_WindowClass@ContextMenu@@0VContextMenuWindowClass@@B 10050594     ContextMenu.obj
 0003:00004598       ?globals@@3UPluginGlobals@@A 10050598     UnityWebPlayerPlugin.obj
 0003:00004608       ?m_SingletonMutex@PluginManager@@0VMutex@@A 10050608     WebCommonLib:PluginManager.obj
 0003:00004620       ?s_Kernel32@?A0x7b9a98a1@@3V?$Handle@PAUHINSTANCE__@@$1?FreeLibrary@@YGHPAU1@@Z$0A@@win@@A 10050620     WebCommonLib:WinWebUtils.obj
 0003:00004624       ?s_GetTimeUS@?A0x7b9a98a1@@3P6A_KXZA 10050624     WebCommonLib:WinWebUtils.obj
 0003:00004628       ?g_cpuInfo@@3VCPUInfo@@A   10050628     WebCommonLib:CPUInfo.obj
 0003:0000462c       __pmatherr                 1005062c     <common>
 0003:00004630       ___use_sse2_mathfcns       10050630     <common>
 0003:00004634       __debugger_hook_dummy      10050634     <common>
 0003:00004638       __nhandle                  10050638     <common>
 0003:00004640       ___pioinfo                 10050640     <common>
 0003:00004740       ___piob                    10050740     <common>
 0003:00004760       __bufin                    10050760     <common>
 0003:00005760       __nstream                  10051760     <common>
 0003:00005764       ___sse2_available          10051764     <common>
 0003:00005768       ___env_initialized         10051768     <common>
 0003:0000576c       ___onexitend               1005176c     <common>
 0003:00005770       ___onexitbegin             10051770     <common>
 0003:00005774       ___mbctype_initialized     10051774     <common>
 0003:00005778       ___dyn_tls_init_callback   10051778     <common>
 0003:0000577c       __acmdln                   1005177c     <common>

 entry point at        0001:00016604

 Static symbols

 0001:00000d12       __catch$?reserve@?$vector@UItem@ContextSubmenu@@V?$allocator@UItem@ContextSubmenu@@@std@@@std@@QAEXI@Z$0 10001d12 f i  CIL library: CIL module
 0001:0000107d       __catch$?_Copy@?$basic_string@_WU?$char_traits@_W@std@@V?$allocator@_W@2@@std@@QAEXII@Z$0 1000207d f i  CIL library: CIL module
 0001:00001102       __catch$?_Copy@?$basic_string@_WU?$char_traits@_W@std@@V?$allocator@_W@2@@std@@QAEXII@Z$1 10002102 f i  CIL library: CIL module
 0001:000012ec       __catch$??$_Uninit_move@PAUItem@ContextSubmenu@@PAU12@V?$allocator@UItem@ContextSubmenu@@@std@@U12@@std@@YAPAUItem@ContextSubmenu@@PAU12@00AAV?$allocator@UItem@ContextSubmenu@@@0@0U_Nonscalar_ptr_iterator_tag@0@@Z$0 100022ec f i  CIL library: CIL module
 0001:00002e1d       __catch$??0?$_Tree@V?$_Tset_traits@V?$basic_string@DU?$char_traits@D@std@@V?$allocator@D@2@@std@@U?$less@V?$basic_string@DU?$char_traits@D@std@@V?$allocator@D@2@@std@@@2@V?$allocator@V?$basic_string@DU?$char_traits@D@std@@V?$allocator@D@2@@std@@@2@$0A@@std@@@std@@QAE@ABV01@@Z$0 10003e1d f i  CIL library: CIL module
 0001:00003001       __catch$?_Copy@?$basic_string@DU?$char_traits@D@std@@V?$allocator@D@2@@std@@QAEXII@Z$0 10004001 f i  CIL library: CIL module
 0001:00003081       __catch$?_Copy@?$basic_string@DU?$char_traits@D@std@@V?$allocator@D@2@@std@@QAEXII@Z$1 10004081 f i  CIL library: CIL module
 0001:00003116       __catch$?_Copy@?$_Tree@V?$_Tset_traits@V?$basic_string@DU?$char_traits@D@std@@V?$allocator@D@2@@std@@U?$less@V?$basic_string@DU?$char_traits@D@std@@V?$allocator@D@2@@std@@@2@V?$allocator@V?$basic_string@DU?$char_traits@D@std@@V?$allocator@D@2@@std@@@2@$0A@@std@@@std@@IAEPAU_Node@?$_Tree_nod@V?$_Tset_traits@V?$basic_string@DU?$char_traits@D@std@@V?$allocator@D@2@@std@@U?$less@V?$basic_string@DU?$char_traits@D@std@@V?$allocator@D@2@@std@@@2@V?$allocator@V?$basic_string@DU?$char_traits@D@std@@V?$allocator@D@2@@std@@@2@$0A@@std@@@2@PAU342@0@Z$0 10004116 f i  CIL library: CIL module
 0001:00003362       __catch$??$_Buynode@AAV?$basic_string@DU?$char_traits@D@std@@V?$allocator@D@2@@std@@@?$_Tree_val@V?$_Tset_traits@V?$basic_string@DU?$char_traits@D@std@@V?$allocator@D@2@@std@@U?$less@V?$basic_string@DU?$char_traits@D@std@@V?$allocator@D@2@@std@@@2@V?$allocator@V?$basic_string@DU?$char_traits@D@std@@V?$allocator@D@2@@std@@@2@$0A@@std@@@std@@QAEPAU_Node@?$_Tree_nod@V?$_Tset_traits@V?$basic_string@DU?$char_traits@D@std@@V?$allocator@D@2@@std@@U?$less@V?$basic_string@DU?$char_traits@D@std@@V?$allocator@D@2@@std@@@2@V?$allocator@V?$basic_string@DU?$char_traits@D@std@@V?$allocator@D@2@@std@@@2@$0A@@std@@@1@AAV?$basic_string@DU?$char_traits@D@std@@V?$allocator@D@2@@1@@Z$0 10004362 f i  CIL library: CIL module
 0001:00003865       ?fillPluginFunctionTable@@YAFPAU_NPPluginFuncs@@@Z 10004865 f    CIL library: CIL module
 0001:00003c87       ?FindDownloadByID@@YAPAVDownloaderNetscape@@I@Z 10004c87 f    CIL library: CIL module
 0001:00004fab       __catch$??$_Buynode@U?$pair@IPAVDownloaderNetscape@@@std@@@?$_Tree_val@V?$_Tmap_traits@IPAVDownloaderNetscape@@U?$less@I@std@@V?$allocator@U?$pair@$$CBIPAVDownloaderNetscape@@@std@@@3@$0A@@std@@@std@@QAEPAU_Node@?$_Tree_nod@V?$_Tmap_traits@IPAVDownloaderNetscape@@U?$less@I@std@@V?$allocator@U?$pair@$$CBIPAVDownloaderNetscape@@@std@@@3@$0A@@std@@@1@$$QAU?$pair@IPAVDownloaderNetscape@@@1@@Z$0 10005fab f i  CIL library: CIL module
 0001:00005021       __catch$??$_Buynode@U?$pair@PAVDownloaderNetscape@@PAU_NPStream@@@std@@@?$_Tree_val@V?$_Tmap_traits@PAVDownload@@PAU_NPStream@@U?$less@PAVDownload@@@std@@V?$allocator@U?$pair@QAVDownload@@PAU_NPStream@@@std@@@4@$0A@@std@@@std@@QAEPAU_Node@?$_Tree_nod@V?$_Tmap_traits@PAVDownload@@PAU_NPStream@@U?$less@PAVDownload@@@std@@V?$allocator@U?$pair@QAVDownload@@PAU_NPStream@@@std@@@4@$0A@@std@@@1@$$QAU?$pair@PAVDownloaderNetscape@@PAU_NPStream@@@1@@Z$0 10006021 f i  CIL library: CIL module
 0001:000050bd       ?ConvertVariant@@YA?AUVariantValue@@ABU_NPVariant@@AAVLogger@@PAU_NPP@@H@Z 100060bd f    CIL library: CIL module
 0001:0000560b       ?png_user_warning_fn@@YAXPAUpng_struct_def@@PBD@Z 1000660b f    CIL library: CIL module
 0001:00005ca9       __catch$?reserve@?$vector@UVariantValue@@V?$allocator@UVariantValue@@@std@@@std@@QAEXI@Z$0 10006ca9 f i  CIL library: CIL module
 0001:00005d7f       __catch$??$_Uninit_move@PAUVariantValue@@PAU1@V?$allocator@UVariantValue@@@std@@U1@@std@@YAPAUVariantValue@@PAU1@00AAV?$allocator@UVariantValue@@@0@0U_Nonscalar_ptr_iterator_tag@0@@Z$0 10006d7f f i  CIL library: CIL module
 0001:00005eb6       ?CheckMembership@@YAHW4MembershipType@@@Z 10006eb6 f    CIL library: CIL module
 0001:00007693       ?SetPluginUpdateError@@YAXAAVLogger@@AAUUpdateInfo@PluginManager@@ABV?$basic_string@DU?$char_traits@D@std@@V?$allocator@D@2@@std@@@Z 10008693 f    CIL library: CIL module
 0001:00008845       __catch$?reserve@?$vector@UUpdateInfo@PluginManager@@V?$allocator@UUpdateInfo@PluginManager@@@std@@@std@@QAEXI@Z$0 10009845 f i  CIL library: CIL module
 0001:00008e4e       __catch$??$_Buynode@U?$pair@$$CBIW4UpdateStatus@UpdaterProxy@@@std@@@?$_Tree_val@V?$_Tmap_traits@IW4UpdateStatus@UpdaterProxy@@U?$less@I@std@@V?$allocator@U?$pair@$$CBIW4UpdateStatus@UpdaterProxy@@@std@@@4@$0A@@std@@@std@@QAEPAU_Node@?$_Tree_nod@V?$_Tmap_traits@IW4UpdateStatus@UpdaterProxy@@U?$less@I@std@@V?$allocator@U?$pair@$$CBIW4UpdateStatus@UpdaterProxy@@@std@@@4@$0A@@std@@@1@$$QAU?$pair@$$CBIW4UpdateStatus@UpdaterProxy@@@1@@Z$0 10009e4e f i  CIL library: CIL module
 0001:00008e4e       __catch$??$_Buynode@U?$pair@KPAVTimer@?A0xa59a0aab@@@std@@@?$_Tree_val@V?$_Tmap_traits@KPAVTimer@?A0xa59a0aab@@U?$less@K@std@@V?$allocator@U?$pair@$$CBKPAVTimer@?A0xa59a0aab@@@std@@@4@$0A@@std@@@std@@QAEPAU_Node@?$_Tree_nod@V?$_Tmap_traits@KPAVTimer@?A0xa59a0aab@@U?$less@K@std@@V?$allocator@U?$pair@$$CBKPAVTimer@?A0xa59a0aab@@@std@@@4@$0A@@std@@@1@$$QAU?$pair@KPAVTimer@?A0xa59a0aab@@@1@@Z$0 10009e4e f i  CIL library: CIL module
 0001:000090f8       __catch$??$_Uninit_move@PAUUpdateInfo@PluginManager@@PAU12@V?$allocator@UUpdateInfo@PluginManager@@@std@@U12@@std@@YAPAUUpdateInfo@PluginManager@@PAU12@00AAV?$allocator@UUpdateInfo@PluginManager@@@0@0U_Nonscalar_ptr_iterator_tag@0@@Z$0 1000a0f8 f i  CIL library: CIL module
 0001:0000956e       ?png_user_read_func@@YAXPAUpng_struct_def@@PAEI@Z 1000a56e f    CIL library: CIL module
 0001:000095a1       ?png_decode@@YA_NPBXIAAPAEAAH2@Z 1000a5a1 f    CIL library: CIL module
 0001:000099e9       ?InitializeImages@@YAXAAVSetup@progress@@PAUHDC__@@@Z 1000a9e9 f    CIL library: CIL module
 0001:0000b0f7       __catch$?reserve@?$vector@UWebMessage@@V?$allocator@UWebMessage@@@std@@@std@@QAEXI@Z$0 1000c0f7 f i  CIL library: CIL module
 0001:0000b19d       __catch$?reserve@?$vector@PAVPluginInstance@@V?$allocator@PAVPluginInstance@@@std@@@std@@QAEXI@Z$0 1000c19d f i  CIL library: CIL module
 0001:0000b19d       __catch$?reserve@?$vector@PAVDownload@@V?$allocator@PAVDownload@@@std@@@std@@QAEXI@Z$0 1000c19d f i  CIL library: CIL module
 0001:0000b19d       __catch$?reserve@?$vector@PAVUnityWebPlayerPluginInstance@@V?$allocator@PAVUnityWebPlayerPluginInstance@@@std@@@std@@QAEXI@Z$0 1000c19d f i  CIL library: CIL module
 0001:0000b33d       __catch$??$_Uninit_move@PAUWebMessage@@PAU1@V?$allocator@UWebMessage@@@std@@U1@@std@@YAPAUWebMessage@@PAU1@00AAV?$allocator@UWebMessage@@@0@0U_Nonscalar_ptr_iterator_tag@0@@Z$0 1000c33d f i  CIL library: CIL module
 0001:0000e046       __catch$??$_Buynode@V?$basic_string@DU?$char_traits@D@std@@V?$allocator@D@2@@std@@@?$_Tree_val@V?$_Tset_traits@V?$basic_string@DU?$char_traits@D@std@@V?$allocator@D@2@@std@@U?$less@V?$basic_string@DU?$char_traits@D@std@@V?$allocator@D@2@@std@@@2@V?$allocator@V?$basic_string@DU?$char_traits@D@std@@V?$allocator@D@2@@std@@@2@$0A@@std@@@std@@QAEPAU_Node@?$_Tree_nod@V?$_Tset_traits@V?$basic_string@DU?$char_traits@D@std@@V?$allocator@D@2@@std@@U?$less@V?$basic_string@DU?$char_traits@D@std@@V?$allocator@D@2@@std@@@2@V?$allocator@V?$basic_string@DU?$char_traits@D@std@@V?$allocator@D@2@@std@@@2@$0A@@std@@@1@$$QAV?$basic_string@DU?$char_traits@D@std@@V?$allocator@D@2@@1@@Z$0 1000f046 f i  CIL library: CIL module
 0001:0000f447       __catch$?_Buynode@?$_List_val@V?$ResourcePtr@VUpdateOperation@UpdaterProxy@@@@V?$allocator@V?$ResourcePtr@VUpdateOperation@UpdaterProxy@@@@@std@@@std@@QAEPAU_Node@?$_List_nod@V?$ResourcePtr@VUpdateOperation@UpdaterProxy@@@@V?$allocator@V?$ResourcePtr@VUpdateOperation@UpdaterProxy@@@@@std@@@2@PAU342@0ABV?$ResourcePtr@VUpdateOperation@UpdaterProxy@@@@@Z$0 10010447 f i  CIL library: CIL module
 0001:0001034e       ?zipExtractCurrentFile@@YA_NPAXABV?$basic_string@DU?$char_traits@D@std@@V?$allocator@D@2@@std@@@Z 1001134e f    CIL library: CIL module
 0001:00010d83       ?AppendPathNameImpl@@YAXABV?$basic_string@DU?$char_traits@D@std@@V?$allocator@D@2@@std@@0DAAV12@@Z 10011d83 f    CIL library: CIL module
 0001:00010efd       ?ReadBigEndian@@YA_NAAPBEPBEAAJ@Z 10011efd f    CIL library: CIL module
 0001:00010f35       ?ReadString@@YA_NAAPBEPBEAAV?$basic_string@DU?$char_traits@D@std@@V?$allocator@D@2@@std@@@Z 10011f35 f    CIL library: CIL module
 0001:00011048       __catch$??$_Construct@PBE@?$basic_string@DU?$char_traits@D@std@@V?$allocator@D@2@@std@@QAEXPBE0Uforward_iterator_tag@1@@Z$0 10012048 f i  CIL library: CIL module
 0001:00013fbd       __onexit_nolock            10014fbd f   LIBCMT:onexit.obj
 0001:0001650e       ___DllMainCRTStartup       1001750e f   LIBCMT:dllcrt0.obj
 0001:00016dba       _flsall                    10017dba f   LIBCMT:fflush.obj
 0001:000181ae       ?strtoxl@@YAKPAUlocaleinfo_struct@@PBDPAPBDHH@Z 100191ae f   LIBCMT:strtol.obj
 0001:000189fd       _doexit                    100199fd f   LIBCMT:crt0dat.obj
 0001:00019480       ?CPtoLCID@@YAHH@Z          1001a480 f   LIBCMT:mbctype.obj
 0001:000194af       ?setSBCS@@YAXPAUthreadmbcinfostruct@@@Z 1001a4af f   LIBCMT:mbctype.obj
 0001:00019513       ?setSBUpLow@@YAXPAUthreadmbcinfostruct@@@Z 1001a513 f   LIBCMT:mbctype.obj
 0001:00019747       ?getSystemCP@@YAHH@Z       1001a747 f   LIBCMT:mbctype.obj
 0001:0001a604       _write_char                1001b604 f   LIBCMT:output.obj
 0001:0001a637       _write_string              1001b637 f   LIBCMT:output.obj
 0001:0001b615       _parse_cmdline             1001c615 f   LIBCMT:stdargv.obj
 0001:0001c106       __catch$??2@YAPAXIABUnothrow_t@std@@@Z$0 1001d106 f   LIBCMT:newopnt.obj
 0001:0001c1b2       ?__crtLCMapStringA_stat@@YAHPAUlocaleinfo_struct@@KKPBDHPADHHH@Z 1001d1b2 f   LIBCMT:a_map.obj
 0001:0001d230       __unwind_handler4          1001e230 f   LIBCMT:exsup4.obj
 0001:0001d2f2       __tzset_nolock             1001e2f2 f   LIBCMT:tzset.obj
 0001:0001d605       _cvtdate                   1001e605 f   LIBCMT:tzset.obj
 0001:0001d7fc       __isindst_nolock           1001e7fc f   LIBCMT:tzset.obj
 0001:0001eb86       _siglookup                 1001fb86 f   LIBCMT:winsig.obj
 0001:0001f416       ?__crtGetStringTypeA_stat@@YAHPAUlocaleinfo_struct@@KPBDHPAGHHH@Z 10020416 f   LIBCMT:a_str.obj
 0001:0001fd95       ?x_ismbbtype_l@@YAHPAUlocaleinfo_struct@@IHH@Z 10020d95 f   LIBCMT:ismbbyte.obj
 0001:0002003c       ?__crtCompareStringA_stat@@YAHPAUlocaleinfo_struct@@KKPBDH1HH@Z 1002103c f   LIBCMT:a_cmp.obj
 0001:000203d6       _findenv                   100213d6 f   LIBCMT:setenv.obj
 0001:00020428       _copy_environ              10021428 f   LIBCMT:setenv.obj
 0001:0002078d       ?CatchGuardHandler@@YA?AW4_EXCEPTION_DISPOSITION@@PAUEHExceptionRecord@@PAUCatchGuardRN@@PAX2@Z 1002178d f   LIBCMT:_trnsctrl_.obj
 0001:00020897       ?TranslatorGuardHandler@@YA?AW4_EXCEPTION_DISPOSITION@@PAUEHExceptionRecord@@PAUTranslatorGuardRN@@PAX2@Z 10021897 f   LIBCMT:_trnsctrl_.obj
 0001:00020f6a       __tsopen_nolock            10021f6a f   LIBCMT:wopen.obj
 0001:000217e0       __unwind_handler           100227e0 f   LIBCMT:exsup.obj
 0001:00021dde       ?ExFilterRethrow@@YAHPAU_EXCEPTION_POINTERS@@@Z 10022dde f   LIBCMT:frame.obj
 0001:00021ea1       ?IsInExceptionSpec@@YAEPAUEHExceptionRecord@@PBU_s_ESTypeList@@@Z 10022ea1 f   LIBCMT:frame.obj
 0001:00021f17       ?CallUnexpected@@YAXPBU_s_ESTypeList@@@Z 10022f17 f   LIBCMT:frame.obj
 0001:00021f48       __catch$?CallUnexpected@@YAXPBU_s_ESTypeList@@@Z$0 10022f48 f   LIBCMT:frame.obj
 0001:00021f60       ?CallCatchBlock@@YAPAXPAUEHExceptionRecord@@PAUEHRegistrationNode@@PAU_CONTEXT@@PBU_s_FuncInfo@@PAXHK@Z 10022f60 f   LIBCMT:frame.obj
 0001:0002230d       ?CatchIt@@YAXPAUEHExceptionRecord@@PAUEHRegistrationNode@@PAU_CONTEXT@@PAXPBU_s_FuncInfo@@PBU_s_HandlerType@@PBU_s_CatchableType@@PBU_s_TryBlockMapEntry@@H1E@Z 1002330d f   LIBCMT:frame.obj
 0001:0002237b       ?FindHandlerForForeignException@@YAXPAUEHExceptionRecord@@PAUEHRegistrationNode@@PAU_CONTEXT@@PAXPBU_s_FuncInfo@@HH1@Z 1002337b f   LIBCMT:frame.obj
 0001:00022482       ?FindHandler@@YAXPAUEHExceptionRecord@@PAUEHRegistrationNode@@PAU_CONTEXT@@PAXPBU_s_FuncInfo@@EH1@Z 10023482 f   LIBCMT:frame.obj
 0001:00027a72       _png_format_buffer         10028a72 f   pnglib:pngerror.obj
 0001:00027afc       _png_default_error         10028afc f   pnglib:pngerror.obj
 0001:00027b84       _png_default_warning       10028b84 f   pnglib:pngerror.obj
 0001:0002ba81       _update_keys               1002ca81 f   zlib:unzip.obj
 0001:0002bac6       _unzlocal_getByte          1002cac6 f   zlib:unzip.obj
 0001:0002baff       _unzlocal_getShort         1002caff f   zlib:unzip.obj
 0001:0002bb45       _unzlocal_getLong          1002cb45 f   zlib:unzip.obj
 0001:0002bbbd       _unzlocal_SearchCentralDir 1002cbbd f   zlib:unzip.obj
 0001:0002bce5       _unzlocal_GetCurrentFileInfoInternal 1002cce5 f   zlib:unzip.obj
 0001:0002c0f1       _unzlocal_CheckCurrentFileCoherencyHeader 1002d0f1 f   zlib:unzip.obj
 0001:0002cb9e       _updatewindow              1002db9e f   zlib:inflate.obj
 0001:0002def7       _crc32_little              1002eef7 f   zlib:crc32.obj
 0001:0002ecc2       ?FormatTime@@YAXPADU_FILETIME@@@Z 1002fcc2 f   CrashHandlerLib:CrashHandler.obj
 0001:0002ed35       _swprintf                  1002fd35 f   CrashHandlerLib:CrashHandler.obj
 0001:0002ed51       ?hprintf@@YAXPAXPBDZZ      1002fd51 f   CrashHandlerLib:CrashHandler.obj
 0001:0002eda3       ?DumpMiniDump@@YA_NPAXPAU_EXCEPTION_POINTERS@@@Z 1002fda3 f   CrashHandlerLib:CrashHandler.obj
 0001:0002ee39       ?DumpModuleInfo@@YA_NPAXPAUHINSTANCE__@@H@Z 1002fe39 f   CrashHandlerLib:CrashHandler.obj
 0001:0002f0d6       ?DumpModuleList@@YAXPAX@Z  100300d6 f   CrashHandlerLib:CrashHandler.obj
 0001:0002f16a       ?DumpSystemInformation@@YAXPAXQAD@Z 1003016a f   CrashHandlerLib:CrashHandler.obj
 0001:0002f2c2       ?GetExceptionDescription@@YAPBDK@Z 100302c2 f   CrashHandlerLib:CrashHandler.obj
 0001:0002f46f       ?DumpStack@@YAXPAXPAK@Z    1003046f f   CrashHandlerLib:CrashHandler.obj
 0001:0002f5d7       ?DumpRegisters@@YAXPAXPAU_CONTEXT@@@Z 100305d7 f   CrashHandlerLib:CrashHandler.obj
 0001:0002f6ca       ?InternalProcessCrash@@YA_NPAU_EXCEPTION_POINTERS@@PAVCrashHandlerImpl@@@Z 100306ca f   CrashHandlerLib:CrashHandler.obj
 0001:0002fd7a       ?CustomUnhandledExceptionFilter@@YGJPAU_EXCEPTION_POINTERS@@@Z 10030d7a f   CrashHandlerLib:CrashHandler.obj
 0001:00031c8b       __shift                    10032c8b f   LIBCMT:cvt.obj
 0001:00031cd0       __cftoe2_l                 10032cd0 f   LIBCMT:cvt.obj
 0001:0003228e       __cftof2_l                 1003328e f   LIBCMT:cvt.obj
 0001:000345de       _write_char                100355de f   LIBCMT:woutput.obj
 0001:0003460d       _write_string              1003560d f   LIBCMT:woutput.obj
 0001:00035280       _ValidateScopeTableHandlers 10036280 f   LIBCMT:eh3valid.obj
 0001:00037168       __tsopen_nolock            10038168 f   LIBCMT:open.obj
 0001:00038783       __hw_cw                    10039783 f   LIBCMT:_ieee87_.obj
 0001:00038811       ___hw_cw_sse2              10039811 f   LIBCMT:_ieee87_.obj
 0001:00038f2e       __ehhandler$??2@YAPAXIABUnothrow_t@std@@@Z 10039f2e f   LIBCMT:newopnt.obj
 0001:00038f49       __ehhandler$?CallUnexpected@@YAXPBU_s_ESTypeList@@@Z 10039f49 f   LIBCMT:frame.obj
 0001:00038f64       __ehhandler$?_Buynode@?$_List_val@V?$ResourcePtr@VUpdateOperation@UpdaterProxy@@@@V?$allocator@V?$ResourcePtr@VUpdateOperation@UpdaterProxy@@@@@std@@@std@@QAEPAU_Node@?$_List_nod@V?$ResourcePtr@VUpdateOperation@UpdaterProxy@@@@V?$allocator@V?$ResourcePtr@VUpdateOperation@UpdaterProxy@@@@@std@@@2@PAU342@0ABV?$ResourcePtr@VUpdateOperation@UpdaterProxy@@@@@Z 10039f64 f    CIL library: CIL module
 0001:00038f6e       __ehhandler$?reserve@?$vector@PAVDownload@@V?$allocator@PAVDownload@@@std@@@std@@QAEXI@Z 10039f6e f    CIL library: CIL module
 0001:00038f6e       __ehhandler$?reserve@?$vector@PAVUnityWebPlayerPluginInstance@@V?$allocator@PAVUnityWebPlayerPluginInstance@@@std@@@std@@QAEXI@Z 10039f6e f    CIL library: CIL module
 0001:00038f6e       __ehhandler$?reserve@?$vector@PAVPluginInstance@@V?$allocator@PAVPluginInstance@@@std@@@std@@QAEXI@Z 10039f6e f    CIL library: CIL module
 0001:00038f78       __ehhandler$?_Copy@?$basic_string@DU?$char_traits@D@std@@V?$allocator@D@2@@std@@QAEXII@Z 10039f78 f    CIL library: CIL module
 0001:00038f82       __ehhandler$??$_Buynode@U?$pair@$$CBIW4UpdateStatus@UpdaterProxy@@@std@@@?$_Tree_val@V?$_Tmap_traits@IW4UpdateStatus@UpdaterProxy@@U?$less@I@std@@V?$allocator@U?$pair@$$CBIW4UpdateStatus@UpdaterProxy@@@std@@@4@$0A@@std@@@std@@QAEPAU_Node@?$_Tree_nod@V?$_Tmap_traits@IW4UpdateStatus@UpdaterProxy@@U?$less@I@std@@V?$allocator@U?$pair@$$CBIW4UpdateStatus@UpdaterProxy@@@std@@@4@$0A@@std@@@1@$$QAU?$pair@$$CBIW4UpdateStatus@UpdaterProxy@@@1@@Z 10039f82 f    CIL library: CIL module
 0001:00038f82       __ehhandler$??$_Buynode@U?$pair@KPAVTimer@?A0xa59a0aab@@@std@@@?$_Tree_val@V?$_Tmap_traits@KPAVTimer@?A0xa59a0aab@@U?$less@K@std@@V?$allocator@U?$pair@$$CBKPAVTimer@?A0xa59a0aab@@@std@@@4@$0A@@std@@@std@@QAEPAU_Node@?$_Tree_nod@V?$_Tmap_traits@KPAVTimer@?A0xa59a0aab@@U?$less@K@std@@V?$allocator@U?$pair@$$CBKPAVTimer@?A0xa59a0aab@@@std@@@4@$0A@@std@@@1@$$QAU?$pair@KPAVTimer@?A0xa59a0aab@@@1@@Z 10039f82 f    CIL library: CIL module
 0001:00038f8c       __ehhandler$??$_Buynode@U?$pair@PAVDownloaderNetscape@@PAU_NPStream@@@std@@@?$_Tree_val@V?$_Tmap_traits@PAVDownload@@PAU_NPStream@@U?$less@PAVDownload@@@std@@V?$allocator@U?$pair@QAVDownload@@PAU_NPStream@@@std@@@4@$0A@@std@@@std@@QAEPAU_Node@?$_Tree_nod@V?$_Tmap_traits@PAVDownload@@PAU_NPStream@@U?$less@PAVDownload@@@std@@V?$allocator@U?$pair@QAVDownload@@PAU_NPStream@@@std@@@4@$0A@@std@@@1@$$QAU?$pair@PAVDownloaderNetscape@@PAU_NPStream@@@1@@Z 10039f8c f    CIL library: CIL module
 0001:00038f96       __ehhandler$??$_Buynode@U?$pair@IPAVDownloaderNetscape@@@std@@@?$_Tree_val@V?$_Tmap_traits@IPAVDownloaderNetscape@@U?$less@I@std@@V?$allocator@U?$pair@$$CBIPAVDownloaderNetscape@@@std@@@3@$0A@@std@@@std@@QAEPAU_Node@?$_Tree_nod@V?$_Tmap_traits@IPAVDownloaderNetscape@@U?$less@I@std@@V?$allocator@U?$pair@$$CBIPAVDownloaderNetscape@@@std@@@3@$0A@@std@@@1@$$QAU?$pair@IPAVDownloaderNetscape@@@1@@Z 10039f96 f    CIL library: CIL module
 0001:00038fa0       __ehhandler$??$_Buynode@AAV?$basic_string@DU?$char_traits@D@std@@V?$allocator@D@2@@std@@@?$_Tree_val@V?$_Tset_traits@V?$basic_string@DU?$char_traits@D@std@@V?$allocator@D@2@@std@@U?$less@V?$basic_string@DU?$char_traits@D@std@@V?$allocator@D@2@@std@@@2@V?$allocator@V?$basic_string@DU?$char_traits@D@std@@V?$allocator@D@2@@std@@@2@$0A@@std@@@std@@QAEPAU_Node@?$_Tree_nod@V?$_Tset_traits@V?$basic_string@DU?$char_traits@D@std@@V?$allocator@D@2@@std@@U?$less@V?$basic_string@DU?$char_traits@D@std@@V?$allocator@D@2@@std@@@2@V?$allocator@V?$basic_string@DU?$char_traits@D@std@@V?$allocator@D@2@@std@@@2@$0A@@std@@@1@AAV?$basic_string@DU?$char_traits@D@std@@V?$allocator@D@2@@1@@Z 10039fa0 f    CIL library: CIL module
 0001:00038faa       __ehhandler$?_Copy@?$_Tree@V?$_Tset_traits@V?$basic_string@DU?$char_traits@D@std@@V?$allocator@D@2@@std@@U?$less@V?$basic_string@DU?$char_traits@D@std@@V?$allocator@D@2@@std@@@2@V?$allocator@V?$basic_string@DU?$char_traits@D@std@@V?$allocator@D@2@@std@@@2@$0A@@std@@@std@@IAEPAU_Node@?$_Tree_nod@V?$_Tset_traits@V?$basic_string@DU?$char_traits@D@std@@V?$allocator@D@2@@std@@U?$less@V?$basic_string@DU?$char_traits@D@std@@V?$allocator@D@2@@std@@@2@V?$allocator@V?$basic_string@DU?$char_traits@D@std@@V?$allocator@D@2@@std@@@2@$0A@@std@@@2@PAU342@0@Z 10039faa f    CIL library: CIL module
 0001:00038fb4       __ehhandler$?_Copy@?$basic_string@_WU?$char_traits@_W@std@@V?$allocator@_W@2@@std@@QAEXII@Z 10039fb4 f    CIL library: CIL module
 0001:00038fbe       __ehhandler$??$_Construct@PBE@?$basic_string@DU?$char_traits@D@std@@V?$allocator@D@2@@std@@QAEXPBE0Uforward_iterator_tag@1@@Z 10039fbe f    CIL library: CIL module
 0001:00038fc8       __ehhandler$??$_Buynode@V?$basic_string@DU?$char_traits@D@std@@V?$allocator@D@2@@std@@@?$_Tree_val@V?$_Tset_traits@V?$basic_string@DU?$char_traits@D@std@@V?$allocator@D@2@@std@@U?$less@V?$basic_string@DU?$char_traits@D@std@@V?$allocator@D@2@@std@@@2@V?$allocator@V?$basic_string@DU?$char_traits@D@std@@V?$allocator@D@2@@std@@@2@$0A@@std@@@std@@QAEPAU_Node@?$_Tree_nod@V?$_Tset_traits@V?$basic_string@DU?$char_traits@D@std@@V?$allocator@D@2@@std@@U?$less@V?$basic_string@DU?$char_traits@D@std@@V?$allocator@D@2@@std@@@2@V?$allocator@V?$basic_string@DU?$char_traits@D@std@@V?$allocator@D@2@@std@@@2@$0A@@std@@@1@$$QAV?$basic_string@DU?$char_traits@D@std@@V?$allocator@D@2@@1@@Z 10039fc8 f    CIL library: CIL module
 0001:00038fd2       __ehhandler$??$_Uninit_move@PAUUpdateInfo@PluginManager@@PAU12@V?$allocator@UUpdateInfo@PluginManager@@@std@@U12@@std@@YAPAUUpdateInfo@PluginManager@@PAU12@00AAV?$allocator@UUpdateInfo@PluginManager@@@0@0U_Nonscalar_ptr_iterator_tag@0@@Z 10039fd2 f    CIL library: CIL module
 0001:00038fdc       __ehhandler$?reserve@?$vector@UUpdateInfo@PluginManager@@V?$allocator@UUpdateInfo@PluginManager@@@std@@@std@@QAEXI@Z 10039fdc f    CIL library: CIL module
 0001:00038fe6       __ehhandler$??0?$_Tree@V?$_Tset_traits@V?$basic_string@DU?$char_traits@D@std@@V?$allocator@D@2@@std@@U?$less@V?$basic_string@DU?$char_traits@D@std@@V?$allocator@D@2@@std@@@2@V?$allocator@V?$basic_string@DU?$char_traits@D@std@@V?$allocator@D@2@@std@@@2@$0A@@std@@@std@@QAE@ABV01@@Z 10039fe6 f    CIL library: CIL module
 0001:00038ff0       __ehhandler$??$_Uninit_move@PAUItem@ContextSubmenu@@PAU12@V?$allocator@UItem@ContextSubmenu@@@std@@U12@@std@@YAPAUItem@ContextSubmenu@@PAU12@00AAV?$allocator@UItem@ContextSubmenu@@@0@0U_Nonscalar_ptr_iterator_tag@0@@Z 10039ff0 f    CIL library: CIL module
 0001:00038ffa       __ehhandler$?reserve@?$vector@UItem@ContextSubmenu@@V?$allocator@UItem@ContextSubmenu@@@std@@@std@@QAEXI@Z 10039ffa f    CIL library: CIL module
 0001:00039004       __ehhandler$??$_Uninit_move@PAUWebMessage@@PAU1@V?$allocator@UWebMessage@@@std@@U1@@std@@YAPAUWebMessage@@PAU1@00AAV?$allocator@UWebMessage@@@0@0U_Nonscalar_ptr_iterator_tag@0@@Z 1003a004 f    CIL library: CIL module
 0001:0003900e       __ehhandler$?reserve@?$vector@UWebMessage@@V?$allocator@UWebMessage@@@std@@@std@@QAEXI@Z 1003a00e f    CIL library: CIL module
 0001:00039018       __ehhandler$??$_Uninit_move@PAUVariantValue@@PAU1@V?$allocator@UVariantValue@@@std@@U1@@std@@YAPAUVariantValue@@PAU1@00AAV?$allocator@UVariantValue@@@0@0U_Nonscalar_ptr_iterator_tag@0@@Z 1003a018 f    CIL library: CIL module
 0001:00039022       __ehhandler$?reserve@?$vector@UVariantValue@@V?$allocator@UVariantValue@@@std@@@std@@QAEXI@Z 1003a022 f    CIL library: CIL module
 0001:0003902c       ??__E?ms_WindowClass@ContextMenu@@0VContextMenuWindowClass@@B@@YAXXZ 1003a02c f    CIL library: CIL module
 0001:0003903d       ??__Eglobals@@YAXXZ        1003a03d f    CIL library: CIL module
 0001:00039054       ??__Eg_InstanceCountMutex@@YAXXZ 1003a054 f    CIL library: CIL module
 0001:0003906b       ??__Eg_Downloads@@YAXXZ    1003a06b f    CIL library: CIL module
 0001:000390a5       ??__Eg_DownloaderToStream@@YAXXZ 1003a0a5 f    CIL library: CIL module
 0001:000390df       ??__Eg_DownloadsMutex@@YAXXZ 1003a0df f    CIL library: CIL module
 0001:000390f6       ??__E?m_SingletonMutex@PluginManager@@0VMutex@@A@@YAXXZ 1003a0f6 f    CIL library: CIL module
 0001:0003910d       ??__Es_Kernel32@?A0x7b9a98a1@@YAXXZ 1003a10d f    CIL library: CIL module
 0001:00039119       ??__Es_GetTimeUS@?A0x7b9a98a1@@YAXXZ 1003a119 f    CIL library: CIL module
 0001:00039124       ??__Eg_cpuInfo@@YAXXZ      1003a124 f    CIL library: CIL module
 0001:0003912f       ??__F?ms_WindowClass@ContextMenu@@0VContextMenuWindowClass@@B@@YAXXZ 1003a12f f    CIL library: CIL module
 0001:0003914b       ??__Fglobals@@YAXXZ        1003a14b f    CIL library: CIL module
 0001:00039157       ??__Fg_InstanceCountMutex@@YAXXZ 1003a157 f    CIL library: CIL module
 0001:00039163       ??__Fg_Downloads@@YAXXZ    1003a163 f    CIL library: CIL module
 0001:00039188       ??__Fg_DownloaderToStream@@YAXXZ 1003a188 f    CIL library: CIL module
 0001:000391ad       ??__Fg_DownloadsMutex@@YAXXZ 1003a1ad f    CIL library: CIL module
 0001:000391b9       ??__F?m_SingletonMutex@PluginManager@@0VMutex@@A@@YAXXZ 1003a1b9 f    CIL library: CIL module
 0001:000391c5       ??__Fs_Kernel32@?A0x7b9a98a1@@YAXXZ 1003a1c5 f    CIL library: CIL module
 0001:000391d6       ??__Fnomem@?5???2@YAPAXI@Z@YAXXZ 1003a1d6 f   LIBCMT:new.obj
